 SQLite.Interop

 Timestamp is 5224e612 (Mon Sep 02 23:25:06 2013)

 Preferred load address is 10000000

 Start         Length     Name                   Class
 0001:00000000 000a8f40H .text                   CODE
 0002:00000000 000001dcH .idata$5                DATA
 0002:000001dc 00000004H .CRT$XCA                DATA
 0002:000001e0 00000004H .CRT$XCZ                DATA
 0002:000001e4 00000004H .CRT$XIA                DATA
 0002:000001e8 00000014H .CRT$XIC                DATA
 0002:000001fc 00000004H .CRT$XIZ                DATA
 0002:00000200 00000004H .CRT$XPA                DATA
 0002:00000204 00000004H .CRT$XPX                DATA
 0002:00000208 00000004H .CRT$XPXA               DATA
 0002:0000020c 00000004H .CRT$XPZ                DATA
 0002:00000210 00000004H .CRT$XTA                DATA
 0002:00000214 00000004H .CRT$XTZ                DATA
 0002:00000220 000189d8H .rdata                  DATA
 0002:00018bf8 00000086H .rdata$debug            DATA
 0002:00018c80 0000000cH .rdata$sxdata           DATA
 0002:00018c8c 00000004H .rtc$IAA                DATA
 0002:00018c90 00000004H .rtc$IZZ                DATA
 0002:00018c94 00000004H .rtc$TAA                DATA
 0002:00018c98 00000004H .rtc$TZZ                DATA
 0002:00018ca0 00000314H .xdata$x                DATA
 0002:00018fb4 00000028H .idata$2                DATA
 0002:00018fdc 00000014H .idata$3                DATA
 0002:00018ff0 000001dcH .idata$4                DATA
 0002:000191cc 0000087eH .idata$6                DATA
 0002:00019a50 000023adH .edata                  DATA
 0003:00000000 00014900H .data                   DATA
 0003:00014900 000022e4H .bss                    DATA
 0004:00000000 00000058H .rsrc$01                DATA
 0004:00000060 00000520H .rsrc$02                DATA

  Address         Publics by Value              Rva+Base       Lib:Object

 0000:00000000       __except_list              00000000     <absolute>
 0000:00000003       ___safe_se_handler_count   00000003     <absolute>
 0000:00000000       ___ImageBase               10000000     <linker-defined>
 0001:00000000       _GetFullPathNameW@16       10001000 f   kernel32:KERNEL32.dll
 0001:00000006       _GetFullPathNameA@16       10001006 f   kernel32:KERNEL32.dll
 0001:0000000c       _HeapReAlloc@16            1000100c f   kernel32:KERNEL32.dll
 0001:00000012       _CreateFileA@28            10001012 f   kernel32:KERNEL32.dll
 0001:00000018       _GetFileSize@8             10001018 f   kernel32:KERNEL32.dll
 0001:0000001e       _CreateMutexW@12           1000101e f   kernel32:KERNEL32.dll
 0001:00000024       _SetFilePointer@16         10001024 f   kernel32:KERNEL32.dll
 0001:0000002a       _MapViewOfFile@20          1000102a f   kernel32:KERNEL32.dll
 0001:00000030       _UnmapViewOfFile@4         10001030 f   kernel32:KERNEL32.dll
 0001:00000036       _SetEndOfFile@4            10001036 f   kernel32:KERNEL32.dll
 0001:0000003c       _FreeLibrary@4             1000103c f   kernel32:KERNEL32.dll
 0001:00000042       _HeapAlloc@12              10001042 f   kernel32:KERNEL32.dll
 0001:00000048       _SystemTimeToFileTime@8    10001048 f   kernel32:KERNEL32.dll
 0001:0000004e       _QueryPerformanceCounter@4 1000104e f   kernel32:KERNEL32.dll
 0001:00000054       _HeapFree@12               10001054 f   kernel32:KERNEL32.dll
 0001:0000005a       _WaitForSingleObject@8     1000105a f   kernel32:KERNEL32.dll
 0001:00000060       _UnlockFile@20             10001060 f   kernel32:KERNEL32.dll
 0001:00000066       _LockFile@20               10001066 f   kernel32:KERNEL32.dll
 0001:0000006c       _OutputDebugStringW@4      1000106c f   kernel32:KERNEL32.dll
 0001:00000072       _GetTickCount@0            10001072 f   kernel32:KERNEL32.dll
 0001:00000078       _UnlockFileEx@20           10001078 f   kernel32:KERNEL32.dll
 0001:0000007e       _GetProcessHeap@0          1000107e f   kernel32:KERNEL32.dll
 0001:00000084       _GetSystemTimeAsFileTime@4 10001084 f   kernel32:KERNEL32.dll
 0001:0000008a       _FormatMessageA@28         1000108a f   kernel32:KERNEL32.dll
 0001:00000090       _WriteFile@20              10001090 f   kernel32:KERNEL32.dll
 0001:00000096       _WideCharToMultiByte@32    10001096 f   kernel32:KERNEL32.dll
 0001:0000009c       _LoadLibraryW@4            1000109c f   kernel32:KERNEL32.dll
 0001:000000a2       _Sleep@4                   100010a2 f   kernel32:KERNEL32.dll
 0001:000000a8       _FormatMessageW@28         100010a8 f   kernel32:KERNEL32.dll
 0001:000000ae       _HeapDestroy@4             100010ae f   kernel32:KERNEL32.dll
 0001:000000b4       _GetFileAttributesA@4      100010b4 f   kernel32:KERNEL32.dll
 0001:000000ba       _HeapCreate@12             100010ba f   kernel32:KERNEL32.dll
 0001:000000c0       _HeapValidate@12           100010c0 f   kernel32:KERNEL32.dll
 0001:000000c6       _GetFileAttributesW@4      100010c6 f   kernel32:KERNEL32.dll
 0001:000000cc       _ReadFile@20               100010cc f   kernel32:KERNEL32.dll
 0001:000000d2       _CreateFileW@28            100010d2 f   kernel32:KERNEL32.dll
 0001:000000d8       _MultiByteToWideChar@24    100010d8 f   kernel32:KERNEL32.dll
 0001:000000de       _FlushFileBuffers@4        100010de f   kernel32:KERNEL32.dll
 0001:000000e4       _GetTempPathW@8            100010e4 f   kernel32:KERNEL32.dll
 0001:000000ea       _GetLastError@0            100010ea f   kernel32:KERNEL32.dll
 0001:000000f0       _GetProcAddress@8          100010f0 f   kernel32:KERNEL32.dll
 0001:000000f6       _HeapSize@12               100010f6 f   kernel32:KERNEL32.dll
 0001:000000fc       _LockFileEx@24             100010fc f   kernel32:KERNEL32.dll
 0001:00000102       _GetDiskFreeSpaceW@20      10001102 f   kernel32:KERNEL32.dll
 0001:00000108       _LoadLibraryA@4            10001108 f   kernel32:KERNEL32.dll
 0001:0000010e       _CreateFileMappingA@24     1000110e f   kernel32:KERNEL32.dll
 0001:00000114       _CreateFileMappingW@24     10001114 f   kernel32:KERNEL32.dll
 0001:0000011a       _GetDiskFreeSpaceA@20      1000111a f   kernel32:KERNEL32.dll
 0001:00000120       _GetSystemInfo@4           10001120 f   kernel32:KERNEL32.dll
 0001:00000126       _GetFileAttributesExW@12   10001126 f   kernel32:KERNEL32.dll
 0001:0000012c       _OutputDebugStringA@4      1000112c f   kernel32:KERNEL32.dll
 0001:00000132       _GetVersionExA@4           10001132 f   kernel32:KERNEL32.dll
 0001:00000138       _CloseHandle@4             10001138 f   kernel32:KERNEL32.dll
 0001:0000013e       _DeleteFileW@4             1000113e f   kernel32:KERNEL32.dll
 0001:00000144       _GetCurrentProcessId@0     10001144 f   kernel32:KERNEL32.dll
 0001:0000014a       _GetTempPathA@8            1000114a f   kernel32:KERNEL32.dll
 0001:00000150       _LocalFree@4               10001150 f   kernel32:KERNEL32.dll
 0001:00000156       _GetSystemTime@4           10001156 f   kernel32:KERNEL32.dll
 0001:0000015c       _AreFileApisANSI@0         1000115c f   kernel32:KERNEL32.dll
 0001:00000162       _DeleteFileA@4             10001162 f   kernel32:KERNEL32.dll
 0001:00000168       @__security_check_cookie@4 10001168 f   LIBCMT:secchk.obj
 0001:00000180       _memmove                   10001180 f   LIBCMT:memmove.obj
 0001:000004e1       _strncmp                   100014e1 f   LIBCMT:strncmp.obj
 0001:000005b0       _ceil                      100015b0 f   LIBCMT:_ceil_pentium4_.obj
 0001:000005f0       __ceil_pentium4            100015f0 f   LIBCMT:_ceil_pentium4_.obj
 0001:000006cd       _free                      100016cd f   LIBCMT:free.obj
 0001:00000707       _calloc                    10001707 f   LIBCMT:calloc.obj
 0001:000007e0       _qsort                     100017e0 f   LIBCMT:qsort.obj
 0001:00000a6b       __localtime64_s            10001a6b f   LIBCMT:loctim64.obj
 0001:00000cf3       __get_sys_err_msg          10001cf3 f i LIBCMT:strerror.obj
 0001:00000d1b       _strerror                  10001d1b f   LIBCMT:strerror.obj
 0001:00000d85       __get_errno_from_oserr     10001d85 f   LIBCMT:dosmap.obj
 0001:00000dc7       __errno                    10001dc7 f   LIBCMT:dosmap.obj
 0001:00000dda       ___doserrno                10001dda f   LIBCMT:dosmap.obj
 0001:00000ded       __dosmaperr                10001ded f   LIBCMT:dosmap.obj
 0001:00000e10       ??0_LocaleUpdate@@QAE@PAUlocaleinfo_struct@@@Z 10001e10 f i LIBCMT:tolower.obj
 0001:00000e97       __tolower_l                10001e97 f   LIBCMT:tolower.obj
 0001:00000fac       _tolower                   10001fac f   LIBCMT:tolower.obj
 0001:00000fe0       _strncpy                   10001fe0 f   LIBCMT:strncpy.obj
 0001:00001104       __isalpha_l                10002104 f i LIBCMT:_ctype.obj
 0001:0000115a       _isalpha                   1000215a f i LIBCMT:_ctype.obj
 0001:0000118a       __isdigit_l                1000218a f i LIBCMT:_ctype.obj
 0001:000011db       _isdigit                   100021db f i LIBCMT:_ctype.obj
 0001:00001209       __toupper_l                10002209 f   LIBCMT:toupper.obj
 0001:0000131f       _toupper                   1000231f f   LIBCMT:toupper.obj
 0001:0000134b       __CRT_INIT@12              1000234b f   LIBCMT:dllcrt0.obj
 0001:000015a5       __DllMainCRTStartup@12     100025a5 f   LIBCMT:dllcrt0.obj
 0001:000015c8       ___report_gsfailure        100025c8 f   LIBCMT:gs_report.obj
 0001:000016ce       __VEC_memcpy               100026ce f   LIBCMT:p4_memcpy.obj
 0001:000017d1       ___sse2_available_init     100027d1 f   LIBCMT:cpu_disp.obj
 0001:000017e1       ___libm_error_support      100027e1 f   LIBCMT:_libm_error_.obj
 0001:00001aad       __sse2_mathfcns_init       10002aad f   LIBCMT:_mathfcns_.obj
 0001:00001abd       __ceil_default             10002abd f   LIBCMT:_ceil_.obj
 0001:00001b95       __heap_init                10002b95 f   LIBCMT:heapinit.obj
 0001:00001bb3       __heap_term                10002bb3 f   LIBCMT:heapinit.obj
 0001:00001bc7       __calloc_impl              10002bc7 f   LIBCMT:calloc_impl.obj
 0001:00001c49       __initp_misc_invarg        10002c49 f   LIBCMT:invarg.obj
 0001:00001c58       __call_reportfault         10002c58 f   LIBCMT:invarg.obj
 0001:00001d81       __invoke_watson            10002d81 f   LIBCMT:invarg.obj
 0001:00001da6       __invalid_parameter        10002da6 f   LIBCMT:invarg.obj
 0001:00001dd3       __invalid_parameter_noinfo 10002dd3 f   LIBCMT:invarg.obj
 0001:000024c4       ___tzset                   100034c4 f   LIBCMT:tzset.obj
 0001:00002513       __isindst                  10003513 f   LIBCMT:tzset.obj
 0001:00002554       __gmtime64_s               10003554 f   LIBCMT:gmtime64.obj
 0001:0000278d       __get_daylight             1000378d f   LIBCMT:timeset.obj
 0001:000027ba       __get_dstbias              100037ba f   LIBCMT:timeset.obj
 0001:000027e7       __get_timezone             100037e7 f   LIBCMT:timeset.obj
 0001:00002814       ___daylight                10003814 f   LIBCMT:timeset.obj
 0001:0000281a       ___dstbias                 1000381a f   LIBCMT:timeset.obj
 0001:00002820       ___timezone                10003820 f   LIBCMT:timeset.obj
 0001:00002826       ___tzname                  10003826 f   LIBCMT:timeset.obj
 0001:00002830       _memset                    10003830 f   LIBCMT:memset.obj
 0001:000028b0       __alldiv                   100038b0 f   LIBCMT:lldiv.obj
 0001:00002960       __allrem                   10003960 f   LIBCMT:llrem.obj
 0001:00002a12       ___sys_nerr                10003a12 f   LIBCMT:syserr.obj
 0001:00002a18       ___sys_errlist             10003a18 f   LIBCMT:syserr.obj
 0001:00002a1e       _strcpy_s                  10003a1e f   LIBCMT:strcpy_s.obj
 0001:00002a7d       __malloc_crt               10003a7d f   LIBCMT:crtheap.obj
 0001:00002ac2       __calloc_crt               10003ac2 f   LIBCMT:crtheap.obj
 0001:00002b0e       __realloc_crt              10003b0e f   LIBCMT:crtheap.obj
 0001:00002b5c       __recalloc_crt             10003b5c f   LIBCMT:crtheap.obj
 0001:00002bae       __encoded_null             10003bae f   LIBCMT:tidtable.obj
 0001:00002bb7       ___crtTlsAlloc@4           10003bb7 f   LIBCMT:tidtable.obj
 0001:00002bc0       ___set_flsgetvalue         10003bc0 f   LIBCMT:tidtable.obj
 0001:00002bf4       __mtterm                   10003bf4 f   LIBCMT:tidtable.obj
 0001:00002c31       __initptd                  10003c31 f   LIBCMT:tidtable.obj
 0001:00002ce5       __getptd_noexit            10003ce5 f   LIBCMT:tidtable.obj
 0001:00002d5e       __getptd                   10003d5e f   LIBCMT:tidtable.obj
 0001:00002d78       __freefls@4                10003d78 f   LIBCMT:tidtable.obj
 0001:00002ea7       __freeptd                  10003ea7 f   LIBCMT:tidtable.obj
 0001:00002f18       __mtinit                   10003f18 f   LIBCMT:tidtable.obj
 0001:00003093       _strncpy_s                 10004093 f   LIBCMT:strncpy_s.obj
 0001:0000336b       ___updatetmbcinfo          1000436b f   LIBCMT:mbctype.obj
 0001:0000348b       __setmbcp_nolock           1000448b f   LIBCMT:mbctype.obj
 0001:00003674       __setmbcp                  10004674 f   LIBCMT:mbctype.obj
 0001:0000380e       ___initmbctable            1000480e f   LIBCMT:mbctype.obj
 0001:0000382c       ___addlocaleref            1000482c f   LIBCMT:localref.obj
 0001:000038bb       ___removelocaleref         100048bb f   LIBCMT:localref.obj
 0001:00003954       ___freetlocinfo            10004954 f   LIBCMT:localref.obj
 0001:00003a9f       __updatetlocinfoEx_nolock  10004a9f f   LIBCMT:localref.obj
 0001:00003aec       ___updatetlocinfo          10004aec f   LIBCMT:localref.obj
 0001:00003b65       __freea                    10004b65 f i LIBCMT:a_map.obj
 0001:00003d6c       ___crtLCMapStringA         10004d6c f   LIBCMT:a_map.obj
 0001:00003db2       __isleadbyte_l             10004db2 f i LIBCMT:_wctype.obj
 0001:00003dea       _isleadbyte                10004dea f i LIBCMT:_wctype.obj
 0001:00003dfd       __isctype_l                10004dfd f   LIBCMT:isctype.obj
 0001:00003eb5       ___initstdio               10004eb5 f   LIBCMT:_file.obj
 0001:00003f66       ___endstdio                10004f66 f   LIBCMT:_file.obj
 0001:00003f86       __lock_file                10004f86 f   LIBCMT:_file.obj
 0001:00003fc7       __lock_file2               10004fc7 f   LIBCMT:_file.obj
 0001:00003ff9       __unlock_file              10004ff9 f   LIBCMT:_file.obj
 0001:00004035       __unlock_file2             10005035 f   LIBCMT:_file.obj
 0001:00004070       __SEH_prolog4              10005070 f   LIBCMT:sehprolg4.obj
 0001:000040b5       __SEH_epilog4              100050b5 f   LIBCMT:sehprolg4.obj
 0001:000040d0       __except_handler4          100050d0 f   LIBCMT:chandler4.obj
 0001:0000425f       ___crtCorExitProcess       1000525f f   LIBCMT:crt0dat.obj
 0001:0000428a       ___crtExitProcess          1000528a f   LIBCMT:crt0dat.obj
 0001:000042a2       __lockexit                 100052a2 f   LIBCMT:crt0dat.obj
 0001:000042ab       __unlockexit               100052ab f   LIBCMT:crt0dat.obj
 0001:000042b4       __init_pointers            100052b4 f   LIBCMT:crt0dat.obj
 0001:000042e7       __initterm_e               100052e7 f   LIBCMT:crt0dat.obj
 0001:0000430b       __cinit                    1000530b f   LIBCMT:crt0dat.obj
 0001:000044e2       __exit                     100054e2 f   LIBCMT:crt0dat.obj
 0001:000044f8       __cexit                    100054f8 f   LIBCMT:crt0dat.obj
 0001:00004507       __amsg_exit                10005507 f   LIBCMT:crt0dat.obj
 0001:00004525       __ioinit                   10005525 f   LIBCMT:ioinit.obj
 0001:0000476a       __ioterm                   1000576a f   LIBCMT:ioinit.obj
 0001:000047bd       __setenvp                  100057bd f   LIBCMT:stdenvp.obj
 0001:00004a33       __setargv                  10005a33 f   LIBCMT:stdargv.obj
 0001:00004aee       ___crtGetEnvironmentStringsA 10005aee f   LIBCMT:a_env.obj
 0001:00004b85       __RTC_Initialize           10005b85 f   LIBCMT:_initsect_.obj
 0001:00004bab       __RTC_Terminate            10005bab f   LIBCMT:_initsect_.obj
 0001:00004bd1       __XcptFilter               10005bd1 f   LIBCMT:winxfltr.obj
 0001:00004d1b       ___CppXcptFilter           10005d1b f   LIBCMT:winxfltr.obj
 0001:00004d3b       ___security_init_cookie    10005d3b f   LIBCMT:gs_support.obj
 0001:00004dd6       __crt_debugger_hook        10005dd6 f   LIBCMT:dbghook.obj
 0001:00004dde       __matherr                  10005dde f   LIBCMT:_matherr_.obj
 0001:00004de1       __cfltcvt_init             10005de1 f   LIBCMT:_fpinit_.obj
 0001:00004e41       __fpmath                   10005e41 f   LIBCMT:_fpinit_.obj
 0001:00004e5a       __raise_exc_ex             10005e5a f   LIBCMT:_fpexcept_.obj
 0001:00005136       __raise_exc                10006136 f   LIBCMT:_fpexcept_.obj
 0001:00005159       __handle_exc               10006159 f   LIBCMT:_fpexcept_.obj
 0001:0000533d       __set_errno_from_matherr   1000633d f   LIBCMT:_fpexcept_.obj
 0001:0000536a       __errcode                  1000636a f   LIBCMT:_fpexcept_.obj
 0001:0000539e       __umatherr                 1000639e f   LIBCMT:_fpexcept_.obj
 0001:0000543e       __handle_qnan1             1000643e f   LIBCMT:_fpexcept_.obj
 0001:00005493       __except1                  10006493 f   LIBCMT:_fpexcept_.obj
 0001:0000555d       __frnd                     1000655d f   LIBCMT:_frnd_.obj
 0001:00005571       __set_exp                  10006571 f   LIBCMT:_util_.obj
 0001:0000559e       __sptype                   1000659e f   LIBCMT:_util_.obj
 0001:00005604       __decomp                   10006604 f   LIBCMT:_util_.obj
 0001:000056c7       __statfp                   100066c7 f   LIBCMT:_fpctrl_.obj
 0001:000056d7       __clrfp                    100066d7 f   LIBCMT:_fpctrl_.obj
 0001:000056e8       __ctrlfp                   100066e8 f   LIBCMT:_fpctrl_.obj
 0001:00005713       __set_statfp               10006713 f   LIBCMT:_fpctrl_.obj
 0001:0000576b       ___set_fpsr_sse2           1000676b f   LIBCMT:_fpctrl_.obj
 0001:000057dd       __initp_heap_handler       100067dd f   LIBCMT:handler.obj
 0001:000057ec       __callnewh                 100067ec f   LIBCMT:handler.obj
 0001:00005814       __mtinitlocks              10006814 f   LIBCMT:mlock.obj
 0001:0000585e       __mtdeletelocks            1000685e f   LIBCMT:mlock.obj
 0001:000058b5       __unlock                   100068b5 f   LIBCMT:mlock.obj
 0001:000058cc       __mtinitlocknum            100068cc f   LIBCMT:mlock.obj
 0001:0000598e       __lock                     1000698e f   LIBCMT:mlock.obj
 0001:000059c1       _atol                      100069c1 f   LIBCMT:atox.obj
 0001:000059e0       _strlen                    100069e0 f   LIBCMT:strlen.obj
 0001:00005a70       _strcmp                    10006a70 f   LIBCMT:strcmp.obj
 0001:00005af8       __getenv_helper_nolock     10006af8 f   LIBCMT:getenv.obj
 0001:00005b7f       ____lc_codepage_func       10006b7f f   LIBCMT:initctyp.obj
 0001:00005bb0       __allmul                   10006bb0 f   LIBCMT:llmul.obj
 0001:00005be4       __VEC_memzero              10006be4 f   LIBCMT:p4_memset.obj
 0001:00005c9e       _malloc                    10006c9e f   LIBCMT:malloc.obj
 0001:00005d32       _realloc                   10006d32 f   LIBCMT:realloc.obj
 0001:00005ddf       __recalloc                 10006ddf f   LIBCMT:recalloc.obj
 0001:00005f34       ___crtGetStringTypeA       10006f34 f   LIBCMT:a_str.obj
 0001:00005f74       ___free_lc_time            10006f74 f   LIBCMT:inittime.obj
 0001:000062eb       ___free_lconv_num          100072eb f   LIBCMT:initnum.obj
 0001:00006354       ___free_lconv_mon          10007354 f   LIBCMT:initmon.obj
 0001:00006460       __alloca_probe_16          10007460 f   LIBCMT:alloca16.obj
 0001:00006476       __alloca_probe_8           10007476     LIBCMT:alloca16.obj
 0001:00006490       _strcspn                   10007490 f   LIBCMT:strcspn.obj
 0001:000064e0       _memcpy                    100074e0 f   LIBCMT:memcpy.obj
 0001:00006850       _strpbrk                   10007850 f   LIBCMT:strpbrk.obj
 0001:00006890       __fcloseall                10007890 f   LIBCMT:closeall.obj
 0001:0000692c       __flush                    1000792c f   LIBCMT:fflush.obj
 0001:00006994       __fflush_nolock            10007994 f   LIBCMT:fflush.obj
 0001:00006ab6       __flushall                 10007ab6 f   LIBCMT:fflush.obj
 0001:00006abf       __isatty                   10007abf f   LIBCMT:isatty.obj
 0001:00006b15       __fileno                   10007b15 f   LIBCMT:fileno.obj
 0001:00006b3b       __initp_misc_cfltcvt_tab   10007b3b f   LIBCMT:cmiscdat.obj
 0001:00006b60       __aulldvrm                 10007b60 f   LIBCMT:ulldvrm.obj
 0001:00006c00       __local_unwind4            10007c00 f   LIBCMT:exsup4.obj
 0001:00006cd6       __seh_longjmp_unwind4@4    10007cd6 f   LIBCMT:exsup4.obj
 0001:00006cf2       @_EH4_CallFilterFunc@8     10007cf2 f   LIBCMT:exsup4.obj
 0001:00006d09       @_EH4_TransferToHandler@8  10007d09 f   LIBCMT:exsup4.obj
 0001:00006d22       @_EH4_GlobalUnwind2@8      10007d22 f   LIBCMT:exsup4.obj
 0001:00006d3b       @_EH4_LocalUnwind@16       10007d3b f   LIBCMT:exsup4.obj
 0001:00006d60       __ValidateImageBase        10007d60 f   LIBCMT:pesect.obj
 0001:00006da0       __FindPESection            10007da0 f   LIBCMT:pesect.obj
 0001:00006df0       __IsNonwritableInCurrentImage 10007df0 f   LIBCMT:pesect.obj
 0001:00006eac       ?terminate@@YAXXZ          10007eac f   LIBCMT:hooks.obj
 0001:00006ee5       __initp_eh_hooks           10007ee5 f   LIBCMT:hooks.obj
 0001:00006ef6       __initp_misc_winsig        10007ef6 f   LIBCMT:winsig.obj
 0001:00006f4b       ___get_sigabrt             10007f4b f   LIBCMT:winsig.obj
 0001:00006f5a       _raise                     10007f5a f   LIBCMT:winsig.obj
 0001:000070fd       __initp_misc_rand_s        100080fd f   LIBCMT:rand_s.obj
 0001:0000710c       __initp_misc_purevirt      1000810c f   LIBCMT:inithelp.obj
 0001:000071d1       ___onexitinit              100081d1 f   LIBCMT:onexit.obj
 0001:00007202       __onexit                   10008202 f   LIBCMT:onexit.obj
 0001:0000723e       _atexit                    1000823e f   LIBCMT:onexit.obj
 0001:00007255       __GET_RTERRMSG             10008255 f   LIBCMT:crt0msg.obj
 0001:0000727b       __NMSG_WRITE               1000827b f   LIBCMT:crt0msg.obj
 0001:0000742a       __FF_MSGBANNER             1000842a f   LIBCMT:crt0msg.obj
 0001:000074b6       __ismbblead                100084b6 f   LIBCMT:ismbbyte.obj
 0001:000074ce       __forcdecpt_l              100084ce f   LIBCMT:cvt.obj
 0001:00007542       __cropzeros_l              10008542 f   LIBCMT:cvt.obj
 0001:000075c4       __positive                 100085c4 f   LIBCMT:cvt.obj
 0001:000075e0       __fassign_l                100085e0 f   LIBCMT:cvt.obj
 0001:00007622       __fassign                  10008622 f   LIBCMT:cvt.obj
 0001:0000765b       __forcdecpt                1000865b f   LIBCMT:cvt.obj
 0001:0000766e       __cropzeros                1000866e f   LIBCMT:cvt.obj
 0001:000077e2       __cftoe_l                  100087e2 f   LIBCMT:cvt.obj
 0001:000078a9       __cftoe                    100088a9 f   LIBCMT:cvt.obj
 0001:000078c9       __cftoa_l                  100088c9 f   LIBCMT:cvt.obj
 0001:00007d42       __cftof_l                  10008d42 f   LIBCMT:cvt.obj
 0001:00007e03       __cftog_l                  10008e03 f   LIBCMT:cvt.obj
 0001:00007ef0       __cfltcvt_l                10008ef0 f   LIBCMT:cvt.obj
 0001:00007f78       __cfltcvt                  10008f78 f   LIBCMT:cvt.obj
 0001:00007f9b       __setdefaultprecision      10008f9b f   LIBCMT:fp8.obj
 0001:000081ee       _strtol                    100091ee f   LIBCMT:strtol.obj
 0001:00008219       __mbsnbicoll_l             10009219 f   LIBCMT:mbsnbico.obj
 0001:000082f7       __mbsnbicoll               100092f7 f   LIBCMT:mbsnbico.obj
 0001:00008311       ___wtomb_environ           10009311 f   LIBCMT:wtombenv.obj
 0001:000083a8       __msize                    100093a8 f   LIBCMT:msize.obj
 0001:000083e0       __chkstk                   100093e0 f   LIBCMT:chkstk.obj
 0001:000083e0       __alloca_probe             100093e0     LIBCMT:chkstk.obj
 0001:0000840b       __strnicmp_l               1000940b f   LIBCMT:strnicmp.obj
 0001:000084ed       __fclose_nolock            100094ed f   LIBCMT:fclose.obj
 0001:0000855a       _fclose                    1000955a f   LIBCMT:fclose.obj
 0001:000085ce       __write_nolock             100095ce f   LIBCMT:write.obj
 0001:00008ccb       __write                    10009ccb f   LIBCMT:write.obj
 0001:00008d9f       __commit                   10009d9f f   LIBCMT:commit.obj
 0001:00008e78       __lseeki64_nolock          10009e78 f   LIBCMT:lseeki64.obj
 0001:00008efd       __fptrap                   10009efd f   LIBCMT:crt0fp.obj
 0001:00008f10       __global_unwind2           10009f10 f   LIBCMT:exsup.obj
 0001:00008f75       __local_unwind2            10009f75 f   LIBCMT:exsup.obj
 0001:00008ff9       __abnormal_termination     10009ff9 f   LIBCMT:exsup.obj
 0001:0000901c       __NLG_Notify1              1000a01c f   LIBCMT:exsup.obj
 0001:00009025       __NLG_Notify               1000a025 f   LIBCMT:exsup.obj
 0001:0000903c       __NLG_Dispatch             1000a03c     LIBCMT:exsup.obj
 0001:0000903c       __NLG_Dispatch2            1000a03c     LIBCMT:exsup.obj
 0001:00009044       __NLG_Call                 1000a044 f   LIBCMT:exsup.obj
 0001:00009046       __NLG_Return2              1000a046     LIBCMT:exsup.obj
 0001:00009047       _abort                     1000a047 f   LIBCMT:abort.obj
 0001:0000907a       ___crtMessageBoxW          1000a07a f   LIBCMT:crtmboxw.obj
 0001:000091e6       _wcscat_s                  1000a1e6 f   LIBCMT:wcscat_s.obj
 0001:0000925b       _wcsncpy_s                 1000a25b f   LIBCMT:wcsncpy_s.obj
 0001:00009328       _wcslen                    1000a328 f   LIBCMT:wcslen.obj
 0001:00009343       _wcscpy_s                  1000a343 f   LIBCMT:wcscpy_s.obj
 0001:000093a6       __set_error_mode           1000a3a6 f   LIBCMT:errmode.obj
 0001:000093f0       _strrchr                   1000a3f0 f   LIBCMT:strrchr.obj
 0001:0000941d       __atodbl_l                 1000a41d f   LIBCMT:atodbl.obj
 0001:000094c5       __atoflt_l                 1000a4c5 f   LIBCMT:atodbl.obj
 0001:0000956d       __fptostr                  1000a56d f   LIBCMT:_fptostr.obj
 0001:00009620       ___dtold                   1000a620 f   LIBCMT:_cfout_.obj
 0001:000096d3       __fltout2                  1000a6d3 f   LIBCMT:_cfout_.obj
 0001:00009770       __alldvrm                  1000a770 f   LIBCMT:lldvrm.obj
 0001:00009850       __aullshr                  1000a850 f   LIBCMT:ullshr.obj
 0001:0000986f       __controlfp_s              1000a86f f   LIBCMT:_contrlfp_.obj
 0001:00009b3c       ___crtCompareStringA       1000ab3c f   LIBCMT:a_cmp.obj
 0001:00009b7e       __strnicoll_l              1000ab7e f   LIBCMT:strnicol.obj
 0001:00009d1a       ___crtsetenv               1000ad1a f   LIBCMT:setenv.obj
 0001:00009f60       ___ascii_strnicmp          1000af60 f   LIBCMT:_strnicm.obj
 0001:00009fc1       __close_nolock             1000afc1 f   LIBCMT:close.obj
 0001:0000a05d       __close                    1000b05d f   LIBCMT:close.obj
 0001:0000a121       __freebuf                  1000b121 f   LIBCMT:_freebuf.obj
 0001:0000a152       __putwch_nolock            1000b152 f   LIBCMT:putwch.obj
 0001:0000a194       __mbtowc_l                 1000b194 f   LIBCMT:mbtowc.obj
 0001:0000a2aa       _mbtowc                    1000b2aa f   LIBCMT:mbtowc.obj
 0001:0000a2c4       __free_osfhnd              1000b2c4 f   LIBCMT:osfinfo.obj
 0001:0000a34a       __get_osfhandle            1000b34a f   LIBCMT:osfinfo.obj
 0001:0000a3b3       ___lock_fhandle            1000b3b3 f   LIBCMT:osfinfo.obj
 0001:0000a452       __unlock_fhandle           1000b452 f   LIBCMT:osfinfo.obj
 0001:0000a479       __ld12tod                  1000b479 f   LIBCMT:_intrncvt_.obj
 0001:0000a9ca       __ld12tof                  1000b9ca f   LIBCMT:_intrncvt_.obj
 0001:0000af1b       ___strgtold12_l            1000bf1b f   LIBCMT:_strgtold_.obj
 0001:0000b5f7       _$I10_OUTPUT               1000c5f7 f   LIBCMT:_x10fout_.obj
 0001:0000c01d       __control87                1000d01d f i LIBCMT:_ieee87_.obj
 0001:0000c32f       __strdup                   1000d32f f   LIBCMT:strdup.obj
 0001:0000c381       __mbschr_l                 1000d381 f   LIBCMT:mbschr.obj
 0001:0000c431       __mbschr                   1000d431 f   LIBCMT:mbschr.obj
 0001:0000c448       ___initconout              1000d448 f   LIBCMT:initcon.obj
 0001:0000c467       ___termconout              1000d467 f   LIBCMT:initcon.obj
 0001:0000c47e       ___mtold12                 1000d47e f   LIBCMT:_mantold_.obj
 0001:0000c680       _strchr                    1000d680 f   LIBCMT:strchr.obj
 0001:0000c686       ___from_strstr_to_strchr   1000d686     LIBCMT:strchr.obj
 0001:0000c73e       _RtlUnwind@16              1000d73e f   kernel32:KERNEL32.dll
 0001:0000c790       _sqlite3_context_collseq_interop@16 1000d790 f   interop.obj
 0001:0000c800       _sqlite3_context_collcompare_interop@20 1000d800 f   interop.obj
 0001:0000c840       _sqlite3Codec              1000d840 f   interop.obj
 0001:0000c9a0       _sqlite3_activate_see      1000d9a0 f   interop.obj
 0001:0000c9d0       _double_cmp                1000d9d0 f   interop.obj
 0001:0000ca10       _int_cmp                   1000da10 f   interop.obj
 0001:0000ca60       _node_iterate              1000da60 f   interop.obj
 0001:0000cab0       _xfree                     1000dab0 f   interop.obj
 0001:0000cac0       _xcalloc                   1000dac0 f   interop.obj
 0001:0000cad0       _map_make                  1000dad0 f   interop.obj
 0001:0000cd00       _isblank                   1000dd00 f   interop.obj
 0001:0000ce80       _sqlite3_vtshim_init       1000de80 f   interop.obj
 0001:0000ce90       _sqlite3_dispose_module    1000de90 f   interop.obj
 0001:0000e8a0       _sqlite3_thread_cleanup    1000f8a0 f   interop.obj
 0001:0000e8b0       _sqlite3_get_autocommit    1000f8b0 f   interop.obj
 0001:0000e8c0       _sqlite3_global_recover    1000f8c0 f   interop.obj
 0001:0000e8d0       _sqlite3_limit             1000f8d0 f   interop.obj
 0001:0000e920       _sqlite3_interrupt         1000f920 f   interop.obj
 0001:0000e990       _sqlite3_total_changes     1000f990 f   interop.obj
 0001:0000e9a0       _sqlite3_changes           1000f9a0 f   interop.obj
 0001:0000e9b0       _sqlite3_last_insert_rowid 1000f9b0 f   interop.obj
 0001:0000e9e0       _sqlite3_db_mutex          1000f9e0 f   interop.obj
 0001:0000e9f0       _sqlite3_threadsafe        1000f9f0 f   interop.obj
 0001:0000ea00       _sqlite3_libversion_number 1000fa00 f   interop.obj
 0001:0000ea10       _sqlite3_sourceid          1000fa10 f   interop.obj
 0001:0000ea20       _sqlite3_libversion        1000fa20 f   interop.obj
 0001:0000ef10       _sqlite3_vtab_on_conflict  1000ff10 f   interop.obj
 0001:00010570       _sqlite3_blob_bytes        10011570 f   interop.obj
 0001:000105c0       _sqlite3_stmt_status       100115c0 f   interop.obj
 0001:000105e0       _sqlite3_stmt_busy         100115e0 f   interop.obj
 0001:00010610       _sqlite3_stmt_readonly     10011610 f   interop.obj
 0001:00010630       _sqlite3_db_handle         10011630 f   interop.obj
 0001:000106b0       _sqlite3_bind_parameter_name 100116b0 f   interop.obj
 0001:000106e0       _sqlite3_bind_parameter_count 100116e0 f   interop.obj
 0001:00010700       _sqlite3_data_count        10011700 f   interop.obj
 0001:00010720       _sqlite3_column_count      10011720 f   interop.obj
 0001:00010740       _sqlite3_aggregate_count   10011740 f   interop.obj
 0001:00010750       _sqlite3_get_auxdata       10011750 f   interop.obj
 0001:00010780       _sqlite3_context_db_handle 10011780 f   interop.obj
 0001:00010790       _sqlite3_user_data         10011790 f   interop.obj
 0001:000107a0       _sqlite3_value_type        100117a0 f   interop.obj
 0001:000107b0       _sqlite3_value_text        100117b0 f   interop.obj
 0001:000107d0       _sqlite3_expired           100117d0 f   interop.obj
 0001:00010c00       _sqlite3_sql               10011c00 f   interop.obj
 0001:00010d60       _sqlite3_backup_pagecount  10011d60 f   interop.obj
 0001:00010d70       _sqlite3_backup_remaining  10011d70 f   interop.obj
 0001:00011130       _sqlite3_enable_shared_cache 10012130 f   interop.obj
 0001:00011f50       _sqlite3_os_end            10012f50 f   interop.obj
 0001:00012190       _sqlite3_win32_sleep       10013190 f   interop.obj
 0001:000121a0       _sqlite3_win32_write_debug 100131a0 f   interop.obj
 0001:00012f10       _sqlite3_strnicmp          10013f10 f   interop.obj
 0001:00012f70       _sqlite3_stricmp           10013f70 f   interop.obj
 0001:00013380       _sqlite3_release_memory    10014380 f   interop.obj
 0001:000134e0       _sqlite3_mutex_leave       100144e0 f   interop.obj
 0001:00013500       _sqlite3_mutex_try         10014500 f   interop.obj
 0001:00013520       _sqlite3_mutex_enter       10014520 f   interop.obj
 0001:00013540       _sqlite3_mutex_free        10014540 f   interop.obj
 0001:00013580       _sqlite3_mutex_alloc       10014580 f   interop.obj
 0001:00013630       _sqlite3_vfs_find          10014630 f   interop.obj
 0001:00013da0       _sqlite3_compileoption_get 10014da0 f   interop.obj
 0001:00013dc0       _sqlite3_compileoption_used 10014dc0 f   interop.obj
 0001:00013ee0       _sqlite3_table_cursor_interop@12 10014ee0 f   interop.obj
 0001:00013f70       _sqlite3_last_insert_rowid_interop@8 10014f70 f   interop.obj
 0001:00013f90       _sqlite3_bind_parameter_name_interop@12 10014f90 f   interop.obj
 0001:00013fe0       _sqlite3_changes_interop@4 10014fe0 f   interop.obj
 0001:00013ff0       _sqlite3_malloc_size_interop@4 10014ff0 f   interop.obj
 0001:00014010       _sqlite3CodecGetKey        10015010 f   interop.obj
 0001:000140d0       _node_destroy              100150d0 f   interop.obj
 0001:00014120       _map_iterate               10015120 f   interop.obj
 0001:00014130       _node_insert               10015130 f   interop.obj
 0001:000153d0       _sqlite3_uri_parameter     100163d0 f   interop.obj
 0001:00015480       _sqlite3_extended_result_codes 10016480 f   interop.obj
 0001:000154d0       _sqlite3_sleep             100164d0 f   interop.obj
 0001:00015510       _sqlite3_collation_needed16 10016510 f   interop.obj
 0001:00015560       _sqlite3_collation_needed  10016560 f   interop.obj
 0001:000155b0       _sqlite3_errstr            100165b0 f   interop.obj
 0001:000155f0       _sqlite3_wal_hook          100165f0 f   interop.obj
 0001:00015640       _sqlite3_rollback_hook     10016640 f   interop.obj
 0001:00015690       _sqlite3_update_hook       10016690 f   interop.obj
 0001:000156e0       _sqlite3_commit_hook       100166e0 f   interop.obj
 0001:00015730       _sqlite3_profile           10016730 f   interop.obj
 0001:00015780       _sqlite3_trace             10016780 f   interop.obj
 0001:000157d0       _sqlite3_progress_handler  100167d0 f   interop.obj
 0001:00015840       _sqlite3_busy_handler      10016840 f   interop.obj
 0001:00015a60       _sqlite3_complete          10016a60 f   interop.obj
 0001:000164f0       _sqlite3_enable_load_extension 100174f0 f   interop.obj
 0001:00016a90       _sqlite3_set_authorizer    10017a90 f   interop.obj
 0001:00017550       _sqlite3_next_stmt         10018550 f   interop.obj
 0001:00017590       _sqlite3_bind_parameter_index 10018590 f   interop.obj
 0001:000176b0       _sqlite3_value_bytes16     100186b0 f   interop.obj
 0001:000176f0       _sqlite3_value_bytes       100186f0 f   interop.obj
 0001:00017730       _sqlite3_value_blob        10018730 f   interop.obj
 0001:00019e30       _sqlite3_free              1001ae30 f   interop.obj
 0001:0001a160       _sqlite3_vfs_unregister    1001b160 f   interop.obj
 0001:0001a1f0       _sqlite3_vfs_register      1001b1f0 f   interop.obj
 0001:0001a460       _sqlite3_value_text_interop@8 1001b460 f   interop.obj
 0001:0001a5f0       _map_destroy               1001b5f0 f   interop.obj
 0001:0001a630       _map_insert                1001b630 f   interop.obj
 0001:0001b870       _sqlite3_db_readonly       1001c870 f   interop.obj
 0001:0001b8a0       _sqlite3_db_filename       1001c8a0 f   interop.obj
 0001:0001b8e0       _sqlite3_uri_int64         1001c8e0 f   interop.obj
 0001:0001b940       _sqlite3_busy_timeout      1001c940 f   interop.obj
 0001:0001c270       _sqlite3_free_table        1001d270 f   interop.obj
 0001:0001c5e0       _sqlite3_strglob           1001d5e0 f   interop.obj
 0001:0001cd00       _sqlite3_column_origin_name 1001dd00 f   interop.obj
 0001:0001cd70       _sqlite3_column_table_name 1001dd70 f   interop.obj
 0001:0001cde0       _sqlite3_column_database_name 1001dde0 f   interop.obj
 0001:0001ce50       _sqlite3_column_decltype   1001de50 f   interop.obj
 0001:0001cec0       _sqlite3_column_name       1001dec0 f   interop.obj
 0001:0001cf30       _sqlite3_value_double      1001df30 f   interop.obj
 0001:0001ec40       _sqlite3_randomness        1001fc40 f   interop.obj
 0001:0001edf0       _sqlite3_memory_alarm      1001fdf0 f   interop.obj
 0001:0001ef30       _sqlite3_column_origin_name_interop@12 1001ff30 f   interop.obj
 0001:0001efd0       _sqlite3_column_table_name_interop@12 1001ffd0 f   interop.obj
 0001:0001f070       _sqlite3_column_database_name_interop@12 10020070 f   interop.obj
 0001:0001f110       _sqlite3_value_double_interop@8 10020110 f   interop.obj
 0001:0001f180       _sqlite3_column_decltype_interop@12 10020180 f   interop.obj
 0001:0001f220       _sqlite3_column_name_interop@12 10020220 f   interop.obj
 0001:00020bc0       _sqlite3_file_control      10021bc0 f   interop.obj
 0001:00021ae0       _sqlite3_value_numeric_type 10022ae0 f   interop.obj
 0001:00021b40       _sqlite3_value_int64       10022b40 f   interop.obj
 0001:00021b50       _sqlite3_value_int         10022b50 f   interop.obj
 0001:00023380       _sqlite3_index_column_info_interop@32 10024380 f   interop.obj
 0001:000234a0       _sqlite3_value_int64_interop@8 100244a0 f   interop.obj
 0001:00023b50       _sqlite3_uri_boolean       10024b50 f   interop.obj
 0001:00023b90       _sqlite3_db_release_memory 10024b90 f   interop.obj
 0001:000262b0       _sqlite3_malloc            100272b0 f   interop.obj
 0001:00027ca0       _sqlite3_db_config         10028ca0 f   interop.obj
 0001:00028620       _sqlite3_aggregate_context 10029620 f   interop.obj
 0001:000286a0       _sqlite3_result_error_nomem 100296a0 f   interop.obj
 0001:00028700       _sqlite3_result_null       10029700 f   interop.obj
 0001:00029e80       _sqlite3CodecSizeChange    1002ae80 f   interop.obj
 0001:0002bb20       _sqlite3_result_value      1002cb20 f   interop.obj
 0001:0002bb90       _sqlite3_clear_bindings    1002cb90 f   interop.obj
 0001:0002d1d0       _sqlite3_win32_utf8_to_mbcs 1002e1d0 f   interop.obj
 0001:0002d210       _sqlite3_win32_mbcs_to_utf8 1002e210 f   interop.obj
 0001:0002d2f0       _sqlite3_vsnprintf         1002e2f0 f   interop.obj
 0001:0002d350       _sqlite3_vmprintf          1002e350 f   interop.obj
 0001:0002e6a0       _sqlite3_result_error_toobig 1002f6a0 f   interop.obj
 0001:0002e760       _sqlite3_result_error_code 1002f760 f   interop.obj
 0001:0002e7c0       _sqlite3_result_zeroblob   1002f7c0 f   interop.obj
 0001:0002e830       _sqlite3_result_int64      1002f830 f   interop.obj
 0001:0002e890       _sqlite3_result_int        1002f890 f   interop.obj
 0001:0002e8e0       _sqlite3_result_error16    1002f8e0 f   interop.obj
 0001:0002e910       _sqlite3_result_error      1002f910 f   interop.obj
 0001:0002e940       _sqlite3_result_double     1002f940 f   interop.obj
 0001:0002f4f0       _sqlite3_log               100304f0 f   interop.obj
 0001:0002f510       _sqlite3_snprintf          10030510 f   interop.obj
 0001:0002f570       _sqlite3_mprintf           10030570 f   interop.obj
 0001:0002f900       _sqlite3_result_int64_interop@8 10030900 f   interop.obj
 0001:0002f960       _sqlite3_result_double_interop@8 10030960 f   interop.obj
 0001:0002f990       _sqlite3CodecAttach        10030990 f   interop.obj
 0001:00033700       _sqlite3_test_control      10034700 f   interop.obj
 0001:00034670       _sqlite3_vtab_config       10035670 f   interop.obj
 0001:00037b90       _sqlite3_transfer_bindings 10038b90 f   interop.obj
 0001:00037dc0       _sqlite3_result_text16le   10038dc0 f   interop.obj
 0001:00037df0       _sqlite3_result_text16be   10038df0 f   interop.obj
 0001:00037e20       _sqlite3_result_text16     10038e20 f   interop.obj
 0001:00037e50       _sqlite3_result_text       10038e50 f   interop.obj
 0001:00037e90       _sqlite3_result_blob       10038e90 f   interop.obj
 0001:00039bf0       _sqlite3_status            1003abf0 f   interop.obj
 0001:00039c50       _sqlite3_key_v2            1003ac50 f   interop.obj
 0001:0003c000       _sqlite3_create_collation_v2 1003d000 f   interop.obj
 0001:0003c080       _sqlite3_create_collation  1003d080 f   interop.obj
 0001:0003c100       _sqlite3_overload_function 1003d100 f   interop.obj
 0001:0003c1c0       _sqlite3_create_function_v2 1003d1c0 f   interop.obj
 0001:0003c2b0       _sqlite3_create_function   1003d2b0 f   interop.obj
 0001:0003c510       _sqlite3_create_module_v2  1003d510 f   interop.obj
 0001:0003c520       _sqlite3_create_module     1003d520 f   interop.obj
 0001:0003c990       _sqlite3_load_extension    1003d990 f   interop.obj
 0001:0003f8c0       _sqlite3_column_type       100408c0 f   interop.obj
 0001:0003f940       _sqlite3_column_value      10040940 f   interop.obj
 0001:0003f9d0       _sqlite3_column_text       100409d0 f   interop.obj
 0001:0003fa50       _sqlite3_column_int64      10040a50 f   interop.obj
 0001:0003fae0       _sqlite3_column_int        10040ae0 f   interop.obj
 0001:0003fb60       _sqlite3_column_double     10040b60 f   interop.obj
 0001:0003fc20       _sqlite3_column_bytes16    10040c20 f   interop.obj
 0001:0003fcc0       _sqlite3_column_bytes      10040cc0 f   interop.obj
 0001:0003fd60       _sqlite3_column_blob       10040d60 f   interop.obj
 0001:00040c30       _sqlite3_memory_highwater  10041c30 f   interop.obj
 0001:00040c60       _sqlite3_memory_used       10041c60 f   interop.obj
 0001:00040dc0       _sqlite3_db_status         10041dc0 f   interop.obj
 0001:00041110       _sqlite3_create_function_interop@36 10042110 f   interop.obj
 0001:00041190       _sqlite3_column_text_interop@12 10042190 f   interop.obj
 0001:000411c0       _sqlite3_memory_highwater_interop@8 100421c0 f   interop.obj
 0001:000411f0       _sqlite3_memory_used_interop@4 100421f0 f   interop.obj
 0001:00041210       _sqlite3_column_int64_interop@12 10042210 f   interop.obj
 0001:00041230       _sqlite3_column_double_interop@12 10042230 f   interop.obj
 0001:00041250       _sqlite3_key               10042250 f   interop.obj
 0001:00041270       _RegisterExtensionFunctions 10042270 f   interop.obj
 0001:00041440       _sqlite3_create_disposable_module 10042440 f   interop.obj
 0001:00041690       _sqlite3_rtree_geometry_callback 10042690 f   interop.obj
 0001:00041870       _sqlite3_extended_errcode  10042870 f   interop.obj
 0001:000418e0       _sqlite3_errcode           100428e0 f   interop.obj
 0001:00041950       _sqlite3_errmsg            10042950 f   interop.obj
 0001:00044e80       _sqlite3_create_disposable_module_interop@112 10045e80 f   interop.obj
 0001:00044f40       _sqlite3_errmsg_interop@8  10045f40 f   interop.obj
 0001:00044f80       _sqlite3_config            10045f80 f   interop.obj
 0001:000459c0       _sqlite3_bind_zeroblob     100469c0 f   interop.obj
 0001:00045a50       _sqlite3_bind_null         10046a50 f   interop.obj
 0001:00045a80       _sqlite3_bind_int64        10046a80 f   interop.obj
 0001:00045b10       _sqlite3_bind_int          10046b10 f   interop.obj
 0001:00045b30       _sqlite3_bind_double       10046b30 f   interop.obj
 0001:00045fa0       _sqlite3_os_init           10046fa0 f   interop.obj
 0001:000466c0       _sqlite3_bind_int64_interop@12 100476c0 f   interop.obj
 0001:000466f0       _sqlite3_bind_double_interop@12 100476f0 f   interop.obj
 0001:00048010       _sqlite3_initialize        10049010 f   interop.obj
 0001:000481e0       _sqlite3_reset_auto_extension 100491e0 f   interop.obj
 0001:000485e0       _sqlite3_win32_set_directory 100495e0 f   interop.obj
 0001:00048650       _sqlite3_realloc           10049650 f   interop.obj
 0001:00048680       _sqlite3_soft_heap_limit64 10049680 f   interop.obj
 0001:000495c0       _sqlite3_shutdown          1004a5c0 f   interop.obj
 0001:00049900       _sqlite3_auto_extension    1004a900 f   interop.obj
 0001:00049e40       _sqlite3_soft_heap_limit   1004ae40 f   interop.obj
 0001:0004b000       _sqlite3_set_auxdata       1004c000 f   interop.obj
 0001:00053e30       _sqlite3_create_collation16 10054e30 f   interop.obj
 0001:00053ed0       _sqlite3_create_function16 10054ed0 f   interop.obj
 0001:00056b50       _sqlite3_bind_text16       10057b50 f   interop.obj
 0001:00056b80       _sqlite3_bind_text         10057b80 f   interop.obj
 0001:00056bb0       _sqlite3_bind_blob         10057bb0 f   interop.obj
 0001:00057820       _sqlite3_complete16        10058820 f   interop.obj
 0001:00057a90       _sqlite3_bind_value        10058a90 f   interop.obj
 0001:00057c20       _sqlite3_value_text16le    10058c20 f   interop.obj
 0001:00057c40       _sqlite3_value_text16be    10058c40 f   interop.obj
 0001:00057c60       _sqlite3_value_text16      10058c60 f   interop.obj
 0001:00058ce0       _sqlite3_value_text16_interop@8 10059ce0 f   interop.obj
 0001:00058d50       _sqlite3_errmsg16          10059d50 f   interop.obj
 0001:00058f70       _sqlite3_wal_checkpoint_v2 10059f70 f   interop.obj
 0001:00059af0       _sqlite3_column_origin_name16 1005aaf0 f   interop.obj
 0001:00059b60       _sqlite3_column_table_name16 1005ab60 f   interop.obj
 0001:00059bd0       _sqlite3_column_database_name16 1005abd0 f   interop.obj
 0001:00059c40       _sqlite3_column_decltype16 1005ac40 f   interop.obj
 0001:00059cb0       _sqlite3_column_name16     1005acb0 f   interop.obj
 0001:00059d20       _sqlite3_column_text16     1005ad20 f   interop.obj
 0001:0005aae0       _sqlite3_column_origin_name16_interop@12 1005bae0 f   interop.obj
 0001:0005ab80       _sqlite3_column_table_name16_interop@12 1005bb80 f   interop.obj
 0001:0005ac20       _sqlite3_column_database_name16_interop@12 1005bc20 f   interop.obj
 0001:0005acc0       _sqlite3_column_text16_interop@12 1005bcc0 f   interop.obj
 0001:0005acf0       _sqlite3_column_decltype16_interop@12 1005bcf0 f   interop.obj
 0001:0005ad90       _sqlite3_column_name16_interop@12 1005bd90 f   interop.obj
 0001:0005ae30       _sqlite3_wal_checkpoint    1005be30 f   interop.obj
 0001:0005eeb0       _sqlite3_wal_autocheckpoint 1005feb0 f   interop.obj
 0001:0006bce0       _sqlite3_backup_init       1006cce0 f   interop.obj
 0001:000704e0       _sqlite3_backup_finish     100714e0 f   interop.obj
 0001:00071050       _sqlite3_backup_finish_interop@4 10072050 f   interop.obj
 0001:00071070       _sqlite3_close_v2          10072070 f   interop.obj
 0001:00071090       _sqlite3_close             10072090 f   interop.obj
 0001:000734c0       _sqlite3_backup_step       100744c0 f   interop.obj
 0001:000742b0       _sqlite3_cursor_rowid_interop@12 100752b0 f   interop.obj
 0001:00074360       _sqlite3_close_interop@4   10075360 f   interop.obj
 0001:00074380       _sqlite3_rekey_v2          10075380 f   interop.obj
 0001:00077a10       _sqlite3_rekey             10078a10 f   interop.obj
 0001:0007bbb0       _sqlite3_reset             1007cbb0 f   interop.obj
 0001:0007bcd0       _sqlite3_reset_interop@4   1007ccd0 f   interop.obj
 0001:0007d350       _sqlite3_finalize          1007e350 f   interop.obj
 0001:0007d3f0       _sqlite3_finalize_interop@4 1007e3f0 f   interop.obj
 0001:000809c0       _sqlite3_blob_write        100819c0 f   interop.obj
 0001:000809f0       _sqlite3_blob_read         100819f0 f   interop.obj
 0001:00080a20       _sqlite3_blob_close        10081a20 f   interop.obj
 0001:0008ac10       _sqlite3_declare_vtab      1008bc10 f   interop.obj
 0001:0008b740       _sqlite3_prepare_v2        1008c740 f   interop.obj
 0001:0008b770       _sqlite3_prepare           1008c770 f   interop.obj
 0001:0008bdd0       _sqlite3_prepare_interop@24 1008cdd0 f   interop.obj
 0001:0008c490       _sqlite3_prepare16_v2      1008d490 f   interop.obj
 0001:0008c4c0       _sqlite3_prepare16         1008d4c0 f   interop.obj
 0001:0008c630       _sqlite3_prepare16_interop@24 1008d630 f   interop.obj
 0001:000927d0       _sqlite3_step              100937d0 f   interop.obj
 0001:00094310       _sqlite3_exec              10095310 f   interop.obj
 0001:00095f60       _sqlite3_get_table         10096f60 f   interop.obj
 0001:00096610       _sqlite3_blob_reopen       10097610 f   interop.obj
 0001:000966f0       _sqlite3_blob_open         100976f0 f   interop.obj
 0001:0009aef0       _sqlite3_table_column_metadata 1009bef0 f   interop.obj
 0001:0009b130       _sqlite3_table_column_metadata_interop@44 1009c130 f   interop.obj
 0001:0009fb10       _sqlite3_open16            100a0b10 f   interop.obj
 0001:0009fc10       _sqlite3_open_v2           100a0c10 f   interop.obj
 0001:0009fc20       _sqlite3_open              100a0c20 f   interop.obj
 0001:0009fc40       _sqlite3_open_interop@12   100a0c40 f   interop.obj
 0001:000a0680       _sqlite3_open16_interop@12 100a1680 f   interop.obj
 0001:000a3760       _sqlite3_unicode_unacc     100a4760 f   sqlite3_unicode.obj
 0001:000a3800       _sqlite3_unicode_title     100a4800 f   sqlite3_unicode.obj
 0001:000a3860       _sqlite3_unicode_upper     100a4860 f   sqlite3_unicode.obj
 0001:000a38c0       _sqlite3_unicode_lower     100a48c0 f   sqlite3_unicode.obj
 0001:000a3920       _sqlite3_unicode_fold      100a4920 f   sqlite3_unicode.obj
 0001:000a45b0       _sqlite3_unicode_collate   100a55b0 f   sqlite3_unicode.obj
 0001:000a4710       _sqlite3_unicode_init      100a5710 f   sqlite3_unicode.obj
 0001:000a48b0       _sqlite3_extension_init    100a58b0 f   sqlite3_unicode.obj
 0001:000a48d0       _sqlite3_unicode_free      100a58d0 f   sqlite3_unicode.obj
 0001:000a48e0       _sqlite3_unicode_load      100a58e0 f   sqlite3_unicode.obj
 0001:000a48f0       _DllMain@12                100a58f0 f   sqlite3_unicode.obj
 0001:000a4930       _sinh                      100a5930 f   LIBCMT:_87ctrigh_.obj
 0001:000a493a       _cosh                      100a593a f   LIBCMT:_87ctrigh_.obj
 0001:000a4941       _tanh                      100a5941 f   LIBCMT:_87ctrigh_.obj
 0001:000a4948       __CIsinh                   100a5948 f   LIBCMT:_87ctrigh_.obj
 0001:000a4952       __CIcosh                   100a5952 f   LIBCMT:_87ctrigh_.obj
 0001:000a4959       __CItanh                   100a5959 f   LIBCMT:_87ctrigh_.obj
 0001:000a4960       _tan                       100a5960 f   LIBCMT:_tan_.obj
 0001:000a49a0       __CItan                    100a59a0 f   LIBCMT:_tan_.obj
 0001:000a49db       __CItan_default            100a59db f   LIBCMT:_tan_.obj
 0001:000a49ef       __tan_default              100a59ef     LIBCMT:_tan_.obj
 0001:000a4a90       _log                       100a5a90 f   LIBCMT:_log_.obj
 0001:000a4ad0       __CIlog                    100a5ad0 f   LIBCMT:_log_.obj
 0001:000a4b0b       __CIlog_default            100a5b0b f   LIBCMT:_log_.obj
 0001:000a4b1f       __log_default              100a5b1f     LIBCMT:_log_.obj
 0001:000a4be0       __CIsqrt                   100a5be0 f   LIBCMT:_sqrt_.obj
 0001:000a4bf4       _sqrt                      100a5bf4     LIBCMT:_sqrt_.obj
 0001:000a4ca0       __allshl                   100a5ca0 f   LIBCMT:llshl.obj
 0001:000a4cc0       __ftol2_sse                100a5cc0 f   LIBCMT:ftol2.obj
 0001:000a4cc9       __ftol2_pentium4           100a5cc9 f   LIBCMT:ftol2.obj
 0001:000a4cdc       __ftol2_sse_excpt          100a5cdc f   LIBCMT:ftol2.obj
 0001:000a4cf6       __ftol2                    100a5cf6 f   LIBCMT:ftol2.obj
 0001:000a4d70       __aullrem                  100a5d70 f   LIBCMT:ullrem.obj
 0001:000a4df0       __aulldiv                  100a5df0 f   LIBCMT:ulldiv.obj
 0001:000a4e60       _floor                     100a5e60 f   LIBCMT:_floor_pentium4_.obj
 0001:000a4ea0       __floor_pentium4           100a5ea0 f   LIBCMT:_floor_pentium4_.obj
 0001:000a4f90       _atan2                     100a5f90 f   LIBCMT:_87ctriga_.obj
 0001:000a4f9a       __CIatan2                  100a5f9a f   LIBCMT:_87ctriga_.obj
 0001:000a4fb0       _pow                       100a5fb0 f   LIBCMT:_pow_.obj
 0001:000a4ff0       __CIpow                    100a5ff0 f   LIBCMT:_pow_.obj
 0001:000a502b       __CIpow_default            100a602b f   LIBCMT:_pow_.obj
 0001:000a5044       __pow_default              100a6044     LIBCMT:_pow_.obj
 0001:000a5240       _exp                       100a6240 f   LIBCMT:_87ctran_.obj
 0001:000a527c       __CIexp                    100a627c f   LIBCMT:_87ctran_.obj
 0001:000a52b7       __exp_default              100a62b7 f   LIBCMT:_87ctran_.obj
 0001:000a52c1       __CIexp_default            100a62c1 f   LIBCMT:_87ctran_.obj
 0001:000a52d0       _log10                     100a62d0 f   LIBCMT:_log10_.obj
 0001:000a5310       __CIlog10                  100a6310 f   LIBCMT:_log10_.obj
 0001:000a534b       __CIlog10_default          100a634b f   LIBCMT:_log10_.obj
 0001:000a535f       __log10_default            100a635f     LIBCMT:_log10_.obj
 0001:000a5420       _cos                       100a6420 f   LIBCMT:_cos_.obj
 0001:000a5460       __CIcos                    100a6460 f   LIBCMT:_cos_.obj
 0001:000a549b       __CIcos_default            100a649b f   LIBCMT:_cos_.obj
 0001:000a54af       __cos_default              100a64af     LIBCMT:_cos_.obj
 0001:000a5550       _sin                       100a6550 f   LIBCMT:_sin_.obj
 0001:000a5590       __CIsin                    100a6590 f   LIBCMT:_sin_.obj
 0001:000a55cb       __CIsin_default            100a65cb f   LIBCMT:_sin_.obj
 0001:000a55df       __sin_default              100a65df     LIBCMT:_sin_.obj
 0001:000a5680       _atan                      100a6680 f   LIBCMT:_atan_.obj
 0001:000a56c0       __CIatan                   100a66c0 f   LIBCMT:_atan_.obj
 0001:000a56fb       __CIatan_default           100a66fb f   LIBCMT:_atan_.obj
 0001:000a570f       __atan_default             100a670f     LIBCMT:_atan_.obj
 0001:000a57a0       _asin                      100a67a0 f   LIBCMT:_asin_.obj
 0001:000a57e0       __CIasin                   100a67e0 f   LIBCMT:_asin_.obj
 0001:000a581b       __CIasin_default           100a681b f   LIBCMT:_asin_.obj
 0001:000a582f       __asin_default             100a682f     LIBCMT:_asin_.obj
 0001:000a58f0       _acos                      100a68f0 f   LIBCMT:_acos_.obj
 0001:000a5930       __CIacos                   100a6930 f   LIBCMT:_acos_.obj
 0001:000a596b       __CIacos_default           100a696b f   LIBCMT:_acos_.obj
 0001:000a597f       __acos_default             100a697f     LIBCMT:_acos_.obj
 0001:000a5a40       __fFSINH                   100a6a40     LIBCMT:_87trigh_.obj
 0001:000a5a92       __fFCOSH                   100a6a92     LIBCMT:_87trigh_.obj
 0001:000a5b40       __cintrindisp2             100a6b40 f   LIBCMT:_87cdisp_.obj
 0001:000a5b7e       __cintrindisp1             100a6b7e f   LIBCMT:_87cdisp_.obj
 0001:000a5bbb       __ctrandisp2               100a6bbb f   LIBCMT:_87cdisp_.obj
 0001:000a5d4a       __ctrandisp1               100a6d4a f   LIBCMT:_87cdisp_.obj
 0001:000a5d7d       __fload                    100a6d7d f   LIBCMT:_87cdisp_.obj
 0001:000a5dc0       __CItan_pentium4           100a6dc0 f   LIBCMT:_tan_pentium4_.obj
 0001:000a5dd8       __tan_pentium4             100a6dd8     LIBCMT:_tan_pentium4_.obj
 0001:000a6020       __trandisp1                100a7020 f   LIBCMT:_87disp_.obj
 0001:000a6087       __trandisp2                100a7087 f   LIBCMT:_87disp_.obj
 0001:000a6113       __rttospopde               100a7113     LIBCMT:_87disp_.obj
 0001:000a6118       __rttospop                 100a7118     LIBCMT:_87disp_.obj
 0001:000a611a       __rtnospop                 100a711a     LIBCMT:_87disp_.obj
 0001:000a611c       __rttosnpop                100a711c     LIBCMT:_87disp_.obj
 0001:000a611d       __rtnospopde               100a711d     LIBCMT:_87disp_.obj
 0001:000a6124       __rtzeropop                100a7124     LIBCMT:_87disp_.obj
 0001:000a6126       __rtzeronpop               100a7126     LIBCMT:_87disp_.obj
 0001:000a612b       __rtonepop                 100a712b     LIBCMT:_87disp_.obj
 0001:000a612d       __rtonenpop                100a712d     LIBCMT:_87disp_.obj
 0001:000a6132       __tosnan1                  100a7132     LIBCMT:_87disp_.obj
 0001:000a615d       __nosnan2                  100a715d     LIBCMT:_87disp_.obj
 0001:000a615f       __tosnan2                  100a715f     LIBCMT:_87disp_.obj
 0001:000a6187       __nan2                     100a7187     LIBCMT:_87disp_.obj
 0001:000a61c6       __rtindfpop                100a71c6     LIBCMT:_87disp_.obj
 0001:000a61c8       __rtindfnpop               100a71c8     LIBCMT:_87disp_.obj
 0001:000a61d9       __rttosnpopde              100a71d9     LIBCMT:_87disp_.obj
 0001:000a61e3       __rtchsifneg               100a71e3     LIBCMT:_87disp_.obj
 0001:000a61f0       __twoToTOS                 100a71f0 f   LIBCMT:_common_.obj
 0001:000a6205       __load_CW                  100a7205 f   LIBCMT:_common_.obj
 0001:000a621c       __convertTOStoQNaN         100a721c f   LIBCMT:_common_.obj
 0001:000a6235       __fload_withFB             100a7235 f   LIBCMT:_common_.obj
 0001:000a6278       __checkTOS_withFB          100a7278 f   LIBCMT:_common_.obj
 0001:000a628e       __fast_exit                100a728e f   LIBCMT:_common_.obj
 0001:000a629b       __math_exit                100a729b f   LIBCMT:_common_.obj
 0001:000a62c5       __check_overflow_exit      100a72c5 f   LIBCMT:_common_.obj
 0001:000a62d9       __check_range_exit         100a72d9 f   LIBCMT:_common_.obj
 0001:000a6380       __startTwoArgErrorHandling 100a7380 f   LIBCMT:_genexcep_.obj
 0001:000a6397       __startOneArgErrorHandling 100a7397 f   LIBCMT:_genexcep_.obj
 0001:000a63e0       __CIlog_pentium4           100a73e0 f   LIBCMT:_log_pentium4_.obj
 0001:000a63f8       __log_pentium4             100a73f8     LIBCMT:_log_pentium4_.obj
 0001:000a6661       __fFEXP                    100a7661     LIBCMT:_87tran_.obj
 0001:000a66b8       __rtinfpopse               100a76b8     LIBCMT:_87tran_.obj
 0001:000a66ba       __rtinfnpopse              100a76ba     LIBCMT:_87tran_.obj
 0001:000a66ca       __fFLN                     100a76ca     LIBCMT:_87tran_.obj
 0001:000a677f       __rtinfpop                 100a777f     LIBCMT:_87tran_.obj
 0001:000a6781       __rtinfnpop                100a7781     LIBCMT:_87tran_.obj
 0001:000a679e       __ffexpm1                  100a779e     LIBCMT:_87tran_.obj
 0001:000a6847       __floor_default            100a7847 f   LIBCMT:_floor_.obj
 0001:000a693c       __fFATN2                   100a793c     LIBCMT:_87triga_.obj
 0001:000a698c       __rtpiby2                  100a798c     LIBCMT:_87triga_.obj
 0001:000a69d0       __CIpow_pentium4           100a79d0 f   LIBCMT:_pow_pentium4_.obj
 0001:000a69e9       __pow_pentium4             100a79e9     LIBCMT:_pow_pentium4_.obj
 0001:000a7530       __d_inttype                100a8530 f   LIBCMT:_powhlp_.obj
 0001:000a759a       __powhlp                   100a859a f   LIBCMT:_powhlp_.obj
 0001:000a76d0       __CIexp_pentium4           100a86d0 f   LIBCMT:_exp_pentium4_.obj
 0001:000a76e8       __exp_pentium4             100a86e8     LIBCMT:_exp_pentium4_.obj
 0001:000a7990       __CIlog10_pentium4         100a8990 f   LIBCMT:_log10_pentium4_.obj
 0001:000a79a8       __log10_pentium4           100a89a8     LIBCMT:_log10_pentium4_.obj
 0001:000a7c20       __CIcos_pentium4           100a8c20 f   LIBCMT:_cos_pentium4_.obj
 0001:000a7c38       __cos_pentium4             100a8c38     LIBCMT:_cos_pentium4_.obj
 0001:000a7dd0       __CIsin_pentium4           100a8dd0 f   LIBCMT:_sin_pentium4_.obj
 0001:000a7de8       __sin_pentium4             100a8de8     LIBCMT:_sin_pentium4_.obj
 0001:000a7fa0       __CIatan_pentium4          100a8fa0 f   LIBCMT:_atan_pentium4_.obj
 0001:000a7fb8       __atan_pentium4            100a8fb8     LIBCMT:_atan_pentium4_.obj
 0001:000a8290       __CIasin_pentium4          100a9290 f   LIBCMT:_asin_pentium4_.obj
 0001:000a82a8       __asin_pentium4            100a92a8     LIBCMT:_asin_pentium4_.obj
 0001:000a8810       __CIacos_pentium4          100a9810 f   LIBCMT:_acos_pentium4_.obj
 0001:000a8828       __acos_pentium4            100a9828     LIBCMT:_acos_pentium4_.obj
 0001:000a8d64       __87except                 100a9d64 f   LIBCMT:_87except_.obj
 0001:000a8ea3       __fpclass                  100a9ea3 f   LIBCMT:_ieeemisc_.obj
 0002:00000000       __imp__CryptDestroyHash@4  100aa000     advapi32:ADVAPI32.dll
 0002:00000004       __imp__CryptDecrypt@24     100aa004     advapi32:ADVAPI32.dll
 0002:00000008       __imp__CryptDestroyKey@4   100aa008     advapi32:ADVAPI32.dll
 0002:0000000c       __imp__CryptCreateHash@20  100aa00c     advapi32:ADVAPI32.dll
 0002:00000010       __imp__CryptEncrypt@28     100aa010     advapi32:ADVAPI32.dll
 0002:00000014       __imp__CryptDuplicateKey@16 100aa014     advapi32:ADVAPI32.dll
 0002:00000018       __imp__CryptDeriveKey@20   100aa018     advapi32:ADVAPI32.dll
 0002:0000001c       __imp__CryptAcquireContextW@20 100aa01c     advapi32:ADVAPI32.dll
 0002:00000020       __imp__CryptHashData@16    100aa020     advapi32:ADVAPI32.dll
 0002:00000024       \177ADVAPI32_NULL_THUNK_DATA 100aa024     advapi32:ADVAPI32.dll
 0002:00000028       __imp__FreeLibrary@4       100aa028     kernel32:KERNEL32.dll
 0002:0000002c       __imp__HeapAlloc@12        100aa02c     kernel32:KERNEL32.dll
 0002:00000030       __imp__SystemTimeToFileTime@8 100aa030     kernel32:KERNEL32.dll
 0002:00000034       __imp__QueryPerformanceCounter@4 100aa034     kernel32:KERNEL32.dll
 0002:00000038       __imp__HeapFree@12         100aa038     kernel32:KERNEL32.dll
 0002:0000003c       __imp__WaitForSingleObject@8 100aa03c     kernel32:KERNEL32.dll
 0002:00000040       __imp__InterlockedCompareExchange@12 100aa040     kernel32:KERNEL32.dll
 0002:00000044       __imp__UnlockFile@20       100aa044     kernel32:KERNEL32.dll
 0002:00000048       __imp__LockFile@20         100aa048     kernel32:KERNEL32.dll
 0002:0000004c       __imp__OutputDebugStringW@4 100aa04c     kernel32:KERNEL32.dll
 0002:00000050       __imp__GetTickCount@0      100aa050     kernel32:KERNEL32.dll
 0002:00000054       __imp__UnlockFileEx@20     100aa054     kernel32:KERNEL32.dll
 0002:00000058       __imp__GetProcessHeap@0    100aa058     kernel32:KERNEL32.dll
 0002:0000005c       __imp__GetSystemTimeAsFileTime@4 100aa05c     kernel32:KERNEL32.dll
 0002:00000060       __imp__FormatMessageA@28   100aa060     kernel32:KERNEL32.dll
 0002:00000064       __imp__WriteFile@20        100aa064     kernel32:KERNEL32.dll
 0002:00000068       __imp__InitializeCriticalSection@4 100aa068     kernel32:KERNEL32.dll
 0002:0000006c       __imp__WideCharToMultiByte@32 100aa06c     kernel32:KERNEL32.dll
 0002:00000070       __imp__LoadLibraryW@4      100aa070     kernel32:KERNEL32.dll
 0002:00000074       __imp__Sleep@4             100aa074     kernel32:KERNEL32.dll
 0002:00000078       __imp__FormatMessageW@28   100aa078     kernel32:KERNEL32.dll
 0002:0000007c       __imp__HeapDestroy@4       100aa07c     kernel32:KERNEL32.dll
 0002:00000080       __imp__LeaveCriticalSection@4 100aa080     kernel32:KERNEL32.dll
 0002:00000084       __imp__GetFileAttributesA@4 100aa084     kernel32:KERNEL32.dll
 0002:00000088       __imp__HeapCreate@12       100aa088     kernel32:KERNEL32.dll
 0002:0000008c       __imp__HeapValidate@12     100aa08c     kernel32:KERNEL32.dll
 0002:00000090       __imp__GetFileAttributesW@4 100aa090     kernel32:KERNEL32.dll
 0002:00000094       __imp__SetEndOfFile@4      100aa094     kernel32:KERNEL32.dll
 0002:00000098       __imp__CreateFileW@28      100aa098     kernel32:KERNEL32.dll
 0002:0000009c       __imp__MultiByteToWideChar@24 100aa09c     kernel32:KERNEL32.dll
 0002:000000a0       __imp__FlushFileBuffers@4  100aa0a0     kernel32:KERNEL32.dll
 0002:000000a4       __imp__GetTempPathW@8      100aa0a4     kernel32:KERNEL32.dll
 0002:000000a8       __imp__GetLastError@0      100aa0a8     kernel32:KERNEL32.dll
 0002:000000ac       __imp__GetProcAddress@8    100aa0ac     kernel32:KERNEL32.dll
 0002:000000b0       __imp__HeapSize@12         100aa0b0     kernel32:KERNEL32.dll
 0002:000000b4       __imp__LockFileEx@24       100aa0b4     kernel32:KERNEL32.dll
 0002:000000b8       __imp__EnterCriticalSection@4 100aa0b8     kernel32:KERNEL32.dll
 0002:000000bc       __imp__GetDiskFreeSpaceW@20 100aa0bc     kernel32:KERNEL32.dll
 0002:000000c0       __imp__LoadLibraryA@4      100aa0c0     kernel32:KERNEL32.dll
 0002:000000c4       __imp__CreateFileMappingA@24 100aa0c4     kernel32:KERNEL32.dll
 0002:000000c8       __imp__CreateFileMappingW@24 100aa0c8     kernel32:KERNEL32.dll
 0002:000000cc       __imp__GetDiskFreeSpaceA@20 100aa0cc     kernel32:KERNEL32.dll
 0002:000000d0       __imp__GetSystemInfo@4     100aa0d0     kernel32:KERNEL32.dll
 0002:000000d4       __imp__GetFileAttributesExW@12 100aa0d4     kernel32:KERNEL32.dll
 0002:000000d8       __imp__DeleteCriticalSection@4 100aa0d8     kernel32:KERNEL32.dll
 0002:000000dc       __imp__OutputDebugStringA@4 100aa0dc     kernel32:KERNEL32.dll
 0002:000000e0       __imp__GetVersionExA@4     100aa0e0     kernel32:KERNEL32.dll
 0002:000000e4       __imp__CloseHandle@4       100aa0e4     kernel32:KERNEL32.dll
 0002:000000e8       __imp__DeleteFileW@4       100aa0e8     kernel32:KERNEL32.dll
 0002:000000ec       __imp__GetCurrentProcessId@0 100aa0ec     kernel32:KERNEL32.dll
 0002:000000f0       __imp__GetTempPathA@8      100aa0f0     kernel32:KERNEL32.dll
 0002:000000f4       __imp__LocalFree@4         100aa0f4     kernel32:KERNEL32.dll
 0002:000000f8       __imp__GetSystemTime@4     100aa0f8     kernel32:KERNEL32.dll
 0002:000000fc       __imp__AreFileApisANSI@0   100aa0fc     kernel32:KERNEL32.dll
 0002:00000100       __imp__DeleteFileA@4       100aa100     kernel32:KERNEL32.dll
 0002:00000104       __imp__UnmapViewOfFile@4   100aa104     kernel32:KERNEL32.dll
 0002:00000108       __imp__MapViewOfFile@20    100aa108     kernel32:KERNEL32.dll
 0002:0000010c       __imp__SetFilePointer@16   100aa10c     kernel32:KERNEL32.dll
 0002:00000110       __imp__CreateMutexW@12     100aa110     kernel32:KERNEL32.dll
 0002:00000114       __imp__GetFileSize@8       100aa114     kernel32:KERNEL32.dll
 0002:00000118       __imp__CreateFileA@28      100aa118     kernel32:KERNEL32.dll
 0002:0000011c       __imp__HeapReAlloc@16      100aa11c     kernel32:KERNEL32.dll
 0002:00000120       __imp__GetFullPathNameA@16 100aa120     kernel32:KERNEL32.dll
 0002:00000124       __imp__ReadFile@20         100aa124     kernel32:KERNEL32.dll
 0002:00000128       __imp__GetFullPathNameW@16 100aa128     kernel32:KERNEL32.dll
 0002:0000012c       __imp__GetCurrentThreadId@0 100aa12c     kernel32:KERNEL32.dll
 0002:00000130       __imp__DecodePointer@4     100aa130     kernel32:KERNEL32.dll
 0002:00000134       __imp__GetCommandLineA@0   100aa134     kernel32:KERNEL32.dll
 0002:00000138       __imp__TerminateProcess@8  100aa138     kernel32:KERNEL32.dll
 0002:0000013c       __imp__GetCurrentProcess@0 100aa13c     kernel32:KERNEL32.dll
 0002:00000140       __imp__UnhandledExceptionFilter@4 100aa140     kernel32:KERNEL32.dll
 0002:00000144       __imp__SetUnhandledExceptionFilter@4 100aa144     kernel32:KERNEL32.dll
 0002:00000148       __imp__IsDebuggerPresent@0 100aa148     kernel32:KERNEL32.dll
 0002:0000014c       __imp__IsProcessorFeaturePresent@4 100aa14c     kernel32:KERNEL32.dll
 0002:00000150       __imp__EncodePointer@4     100aa150     kernel32:KERNEL32.dll
 0002:00000154       __imp__GetTimeZoneInformation@4 100aa154     kernel32:KERNEL32.dll
 0002:00000158       __imp__TlsAlloc@0          100aa158     kernel32:KERNEL32.dll
 0002:0000015c       __imp__TlsGetValue@4       100aa15c     kernel32:KERNEL32.dll
 0002:00000160       __imp__TlsSetValue@8       100aa160     kernel32:KERNEL32.dll
 0002:00000164       __imp__TlsFree@4           100aa164     kernel32:KERNEL32.dll
 0002:00000168       __imp__InterlockedIncrement@4 100aa168     kernel32:KERNEL32.dll
 0002:0000016c       __imp__GetModuleHandleW@4  100aa16c     kernel32:KERNEL32.dll
 0002:00000170       __imp__SetLastError@4      100aa170     kernel32:KERNEL32.dll
 0002:00000174       __imp__InterlockedDecrement@4 100aa174     kernel32:KERNEL32.dll
 0002:00000178       __imp__GetCPInfo@8         100aa178     kernel32:KERNEL32.dll
 0002:0000017c       __imp__GetACP@0            100aa17c     kernel32:KERNEL32.dll
 0002:00000180       __imp__GetOEMCP@0          100aa180     kernel32:KERNEL32.dll
 0002:00000184       __imp__IsValidCodePage@4   100aa184     kernel32:KERNEL32.dll
 0002:00000188       __imp__LCMapStringW@24     100aa188     kernel32:KERNEL32.dll
 0002:0000018c       __imp__ExitProcess@4       100aa18c     kernel32:KERNEL32.dll
 0002:00000190       __imp__SetHandleCount@4    100aa190     kernel32:KERNEL32.dll
 0002:00000194       __imp__GetStdHandle@4      100aa194     kernel32:KERNEL32.dll
 0002:00000198       __imp__InitializeCriticalSectionAndSpinCount@8 100aa198     kernel32:KERNEL32.dll
 0002:0000019c       __imp__GetFileType@4       100aa19c     kernel32:KERNEL32.dll
 0002:000001a0       __imp__GetStartupInfoW@4   100aa1a0     kernel32:KERNEL32.dll
 0002:000001a4       __imp__GetModuleFileNameA@12 100aa1a4     kernel32:KERNEL32.dll
 0002:000001a8       __imp__FreeEnvironmentStringsW@4 100aa1a8     kernel32:KERNEL32.dll
 0002:000001ac       __imp__GetEnvironmentStringsW@0 100aa1ac     kernel32:KERNEL32.dll
 0002:000001b0       __imp__RaiseException@16   100aa1b0     kernel32:KERNEL32.dll
 0002:000001b4       __imp__GetStringTypeW@16   100aa1b4     kernel32:KERNEL32.dll
 0002:000001b8       __imp__RtlUnwind@16        100aa1b8     kernel32:KERNEL32.dll
 0002:000001bc       __imp__GetModuleFileNameW@12 100aa1bc     kernel32:KERNEL32.dll
 0002:000001c0       __imp__GetConsoleCP@0      100aa1c0     kernel32:KERNEL32.dll
 0002:000001c4       __imp__GetConsoleMode@8    100aa1c4     kernel32:KERNEL32.dll
 0002:000001c8       __imp__CompareStringW@24   100aa1c8     kernel32:KERNEL32.dll
 0002:000001cc       __imp__SetEnvironmentVariableA@8 100aa1cc     kernel32:KERNEL32.dll
 0002:000001d0       __imp__WriteConsoleW@20    100aa1d0     kernel32:KERNEL32.dll
 0002:000001d4       __imp__SetStdHandle@8      100aa1d4     kernel32:KERNEL32.dll
 0002:000001d8       \177KERNEL32_NULL_THUNK_DATA 100aa1d8     kernel32:KERNEL32.dll
 0002:000001dc       ___xc_a                    100aa1dc     LIBCMT:crt0init.obj
 0002:000001e0       ___xc_z                    100aa1e0     LIBCMT:crt0init.obj
 0002:000001e4       ___xi_a                    100aa1e4     LIBCMT:crt0init.obj
 0002:000001fc       ___xi_z                    100aa1fc     LIBCMT:crt0init.obj
 0002:00000200       ___xp_a                    100aa200     LIBCMT:crt0init.obj
 0002:0000020c       ___xp_z                    100aa20c     LIBCMT:crt0init.obj
 0002:00000210       ___xt_a                    100aa210     LIBCMT:crt0init.obj
 0002:00000214       ___xt_z                    100aa214     LIBCMT:crt0init.obj
 0002:00000288       ??_C@_0EA@FCLIIPNN@Visual?5C?$CL?$CL?5CRT?3?5Not?5enough?5memor@ 100aa288     LIBCMT:strerror.obj
 0002:000002c8       __pDefaultRawDllMain       100aa2c8     LIBCMT:dllcrt0.obj
 0002:000002c8       __pRawDllMain              100aa2c8     LIBCMT:dllcrt0.obj
 0002:00000340       ??_C@_04EHEDPDJG@modf?$AA@ 100aa340     LIBCMT:_libm_error_.obj
 0002:00000348       ??_C@_05EOHGHCHD@exp10?$AA@ 100aa348     LIBCMT:_libm_error_.obj
 0002:00000350       ??_C@_03JGHBODFD@pow?$AA@  100aa350     LIBCMT:_libm_error_.obj
 0002:00000354       ??_C@_02CLFPBFFP@TZ?$AA@   100aa354     LIBCMT:tzset.obj
 0002:00000358       ___dnames                  100aa358     LIBCMT:timeset.obj
 0002:00000370       ___mnames                  100aa370     LIBCMT:timeset.obj
 0002:00000398       ??_C@_0BG@KLEAJEFJ@Illegal?5byte?5sequence?$AA@ 100aa398     LIBCMT:syserr.obj
 0002:000003b0       ??_C@_0BE@ICMCHPHH@Directory?5not?5empty?$AA@ 100aa3b0     LIBCMT:syserr.obj
 0002:000003c4       ??_C@_0BJ@IHEHINLI@Function?5not?5implemented?$AA@ 100aa3c4     LIBCMT:syserr.obj
 0002:000003e0       ??_C@_0BD@CLHBCGPB@No?5locks?5available?$AA@ 100aa3e0     LIBCMT:syserr.obj
 0002:000003f4       ??_C@_0BC@BEDIHIDK@Filename?5too?5long?$AA@ 100aa3f4     LIBCMT:syserr.obj
 0002:00000408       ??_C@_0BK@JAEBMJJM@Resource?5deadlock?5avoided?$AA@ 100aa408     LIBCMT:syserr.obj
 0002:00000424       ??_C@_0BB@FCBJFCAJ@Result?5too?5large?$AA@ 100aa424     LIBCMT:syserr.obj
 0002:00000438       ??_C@_0N@MMJPGLJK@Domain?5error?$AA@ 100aa438     LIBCMT:syserr.obj
 0002:00000448       ??_C@_0M@LHEPIIOM@Broken?5pipe?$AA@ 100aa448     LIBCMT:syserr.obj
 0002:00000454       ??_C@_0P@PKCJJLLM@Too?5many?5links?$AA@ 100aa454     LIBCMT:syserr.obj
 0002:00000464       ??_C@_0BG@DDBFNKBH@Read?9only?5file?5system?$AA@ 100aa464     LIBCMT:syserr.obj
 0002:0000047c       ??_C@_0N@FEHLOILP@Invalid?5seek?$AA@ 100aa47c     LIBCMT:syserr.obj
 0002:0000048c       ??_C@_0BI@FEALHKLD@No?5space?5left?5on?5device?$AA@ 100aa48c     LIBCMT:syserr.obj
 0002:000004a4       ??_C@_0P@LFMMIPAE@File?5too?5large?$AA@ 100aa4a4     LIBCMT:syserr.obj
 0002:000004b4       ??_C@_0CE@ONOKNLPF@Inappropriate?5I?1O?5control?5operat@ 100aa4b4     LIBCMT:syserr.obj
 0002:000004d8       ??_C@_0BE@INBJMKGG@Too?5many?5open?5files?$AA@ 100aa4d8     LIBCMT:syserr.obj
 0002:000004ec       ??_C@_0BO@IIFBODJE@Too?5many?5open?5files?5in?5system?$AA@ 100aa4ec     LIBCMT:syserr.obj
 0002:0000050c       ??_C@_0BB@HMGGCEBG@Invalid?5argument?$AA@ 100aa50c     LIBCMT:syserr.obj
 0002:00000520       ??_C@_0P@NDHGCGKE@Is?5a?5directory?$AA@ 100aa520     LIBCMT:syserr.obj
 0002:00000530       ??_C@_0BA@CJBACOOL@Not?5a?5directory?$AA@ 100aa530     LIBCMT:syserr.obj
 0002:00000540       ??_C@_0P@NLEIANHE@No?5such?5device?$AA@ 100aa540     LIBCMT:syserr.obj
 0002:00000550       ??_C@_0O@OAMDNOCP@Improper?5link?$AA@ 100aa550     LIBCMT:syserr.obj
 0002:00000560       ??_C@_0M@NAAJNNGH@File?5exists?$AA@ 100aa560     LIBCMT:syserr.obj
 0002:0000056c       ??_C@_0BA@BIBLIOEK@Resource?5device?$AA@ 100aa56c     LIBCMT:syserr.obj
 0002:0000057c       ??_C@_0O@NIPGCINC@Unknown?5error?$AA@ 100aa57c     LIBCMT:syserr.obj
 0002:0000058c       ??_C@_0M@LOEHLCJD@Bad?5address?$AA@ 100aa58c     LIBCMT:syserr.obj
 0002:00000598       ??_C@_0BC@HFNFNKAI@Permission?5denied?$AA@ 100aa598     LIBCMT:syserr.obj
 0002:000005ac       ??_C@_0BB@IMDKMPFB@Not?5enough?5space?$AA@ 100aa5ac     LIBCMT:syserr.obj
 0002:000005c0       ??_C@_0CB@EPFKGNAK@Resource?5temporarily?5unavailable@ 100aa5c0     LIBCMT:syserr.obj
 0002:000005e4       ??_C@_0BD@LOHELEP@No?5child?5processes?$AA@ 100aa5e4     LIBCMT:syserr.obj
 0002:000005f8       ??_C@_0BE@NFGDDCEF@Bad?5file?5descriptor?$AA@ 100aa5f8     LIBCMT:syserr.obj
 0002:0000060c       ??_C@_0BC@HKPNECK@Exec?5format?5error?$AA@ 100aa60c     LIBCMT:syserr.obj
 0002:00000620       ??_C@_0BC@MFFGCDFL@Arg?5list?5too?5long?$AA@ 100aa620     LIBCMT:syserr.obj
 0002:00000634       ??_C@_0BK@DPKMCKJ@No?5such?5device?5or?5address?$AA@ 100aa634     LIBCMT:syserr.obj
 0002:00000650       ??_C@_0BD@KKNFOBBD@Input?1output?5error?$AA@ 100aa650     LIBCMT:syserr.obj
 0002:00000664       ??_C@_0BK@FJBOAFDK@Interrupted?5function?5call?$AA@ 100aa664     LIBCMT:syserr.obj
 0002:00000680       ??_C@_0BA@FKIAIBGA@No?5such?5process?$AA@ 100aa680     LIBCMT:syserr.obj
 0002:00000690       ??_C@_0BK@FMDHKPNF@No?5such?5file?5or?5directory?$AA@ 100aa690     LIBCMT:syserr.obj
 0002:000006ac       ??_C@_0BI@BJFCGOHL@Operation?5not?5permitted?$AA@ 100aa6ac     LIBCMT:syserr.obj
 0002:000006c4       ??_C@_08INEPGKHH@No?5error?$AA@ 100aa6c4     LIBCMT:syserr.obj
 0002:000006d0       ??_C@_1BK@DBDEIDLH@?$AAK?$AAE?$AAR?$AAN?$AAE?$AAL?$AA3?$AA2?$AA?4?$AAD?$AAL?$AAL?$AA?$AA@ 100aa6d0     LIBCMT:tidtable.obj
 0002:000006ec       ??_C@_07PEJMOBNF@FlsFree?$AA@ 100aa6ec     LIBCMT:tidtable.obj
 0002:000006f4       ??_C@_0M@JCPCPOEF@FlsSetValue?$AA@ 100aa6f4     LIBCMT:tidtable.obj
 0002:00000700       ??_C@_0M@GDNOONDI@FlsGetValue?$AA@ 100aa700     LIBCMT:tidtable.obj
 0002:0000070c       ??_C@_08KNHFBNJ@FlsAlloc?$AA@ 100aa70c     LIBCMT:tidtable.obj
 0002:00000718       ??_C@_1BC@GDGBMEMK@?$AAH?$AAH?$AA?3?$AAm?$AAm?$AA?3?$AAs?$AAs?$AA?$AA@ 100aa718     LIBCMT:nlsdata2.obj
 0002:0000072c       ??_C@_1CI@KNAKOEBC@?$AAd?$AAd?$AAd?$AAd?$AA?0?$AA?5?$AAM?$AAM?$AAM?$AAM?$AA?5?$AAd?$AAd?$AA?0?$AA?5?$AAy?$AAy?$AAy?$AAy?$AA?$AA@ 100aa72c     LIBCMT:nlsdata2.obj
 0002:00000754       ??_C@_1BC@IEBCMHCM@?$AAM?$AAM?$AA?1?$AAd?$AAd?$AA?1?$AAy?$AAy?$AA?$AA@ 100aa754     LIBCMT:nlsdata2.obj
 0002:00000768       ??_C@_15CLMNNGEL@?$AAP?$AAM?$AA?$AA@ 100aa768     LIBCMT:nlsdata2.obj
 0002:00000770       ??_C@_15ODEHAHHF@?$AAA?$AAM?$AA?$AA@ 100aa770     LIBCMT:nlsdata2.obj
 0002:00000778       ??_C@_1BC@FEMKIFH@?$AAD?$AAe?$AAc?$AAe?$AAm?$AAb?$AAe?$AAr?$AA?$AA@ 100aa778     LIBCMT:nlsdata2.obj
 0002:0000078c       ??_C@_1BC@BGLIFPF@?$AAN?$AAo?$AAv?$AAe?$AAm?$AAb?$AAe?$AAr?$AA?$AA@ 100aa78c     LIBCMT:nlsdata2.obj
 0002:000007a0       ??_C@_1BA@EPANDLNG@?$AAO?$AAc?$AAt?$AAo?$AAb?$AAe?$AAr?$AA?$AA@ 100aa7a0     LIBCMT:nlsdata2.obj
 0002:000007b0       ??_C@_1BE@DKAAMBJL@?$AAS?$AAe?$AAp?$AAt?$AAe?$AAm?$AAb?$AAe?$AAr?$AA?$AA@ 100aa7b0     LIBCMT:nlsdata2.obj
 0002:000007c4       ??_C@_1O@PAHLKOAC@?$AAA?$AAu?$AAg?$AAu?$AAs?$AAt?$AA?$AA@ 100aa7c4     LIBCMT:nlsdata2.obj
 0002:000007d4       ??_C@_19BIFMLPCD@?$AAJ?$AAu?$AAl?$AAy?$AA?$AA@ 100aa7d4     LIBCMT:nlsdata2.obj
 0002:000007e0       ??_C@_19EPFLPGAP@?$AAJ?$AAu?$AAn?$AAe?$AA?$AA@ 100aa7e0     LIBCMT:nlsdata2.obj
 0002:000007ec       ??_C@_1M@GJNLMHFD@?$AAA?$AAp?$AAr?$AAi?$AAl?$AA?$AA@ 100aa7ec     LIBCMT:nlsdata2.obj
 0002:000007f8       ??_C@_1M@IKEENEDF@?$AAM?$AAa?$AAr?$AAc?$AAh?$AA?$AA@ 100aa7f8     LIBCMT:nlsdata2.obj
 0002:00000804       ??_C@_1BC@JGDDFFAM@?$AAF?$AAe?$AAb?$AAr?$AAu?$AAa?$AAr?$AAy?$AA?$AA@ 100aa804     LIBCMT:nlsdata2.obj
 0002:00000818       ??_C@_1BA@EFMEIEBA@?$AAJ?$AAa?$AAn?$AAu?$AAa?$AAr?$AAy?$AA?$AA@ 100aa818     LIBCMT:nlsdata2.obj
 0002:00000828       ??_C@_17EGKACKIF@?$AAD?$AAe?$AAc?$AA?$AA@ 100aa828     LIBCMT:nlsdata2.obj
 0002:00000830       ??_C@_17BBDMLCIG@?$AAN?$AAo?$AAv?$AA?$AA@ 100aa830     LIBCMT:nlsdata2.obj
 0002:00000838       ??_C@_17FNLKOI@?$AAO?$AAc?$AAt?$AA?$AA@ 100aa838     LIBCMT:nlsdata2.obj
 0002:00000840       ??_C@_17HCHCOKMG@?$AAS?$AAe?$AAp?$AA?$AA@ 100aa840     LIBCMT:nlsdata2.obj
 0002:00000848       ??_C@_17ICPELBCN@?$AAA?$AAu?$AAg?$AA?$AA@ 100aa848     LIBCMT:nlsdata2.obj
 0002:00000850       ??_C@_17IJPCKHK@?$AAJ?$AAu?$AAl?$AA?$AA@ 100aa850     LIBCMT:nlsdata2.obj
 0002:00000858       ??_C@_17KCJGOCPB@?$AAJ?$AAu?$AAn?$AA?$AA@ 100aa858     LIBCMT:nlsdata2.obj
 0002:00000860       ??_C@_17PNNKMEED@?$AAM?$AAa?$AAy?$AA?$AA@ 100aa860     LIBCMT:nlsdata2.obj
 0002:00000868       ??_C@_17LFPOIHDD@?$AAA?$AAp?$AAr?$AA?$AA@ 100aa868     LIBCMT:nlsdata2.obj
 0002:00000870       ??_C@_17CKNLEDEC@?$AAM?$AAa?$AAr?$AA?$AA@ 100aa870     LIBCMT:nlsdata2.obj
 0002:00000878       ??_C@_17LMDJEKJN@?$AAF?$AAe?$AAb?$AA?$AA@ 100aa878     LIBCMT:nlsdata2.obj
 0002:00000880       ??_C@_17DKNBKCHM@?$AAJ?$AAa?$AAn?$AA?$AA@ 100aa880     LIBCMT:nlsdata2.obj
 0002:00000888       ??_C@_1BC@ENMNNPAJ@?$AAS?$AAa?$AAt?$AAu?$AAr?$AAd?$AAa?$AAy?$AA?$AA@ 100aa888     LIBCMT:nlsdata2.obj
 0002:0000089c       ??_C@_1O@PDICJHAG@?$AAF?$AAr?$AAi?$AAd?$AAa?$AAy?$AA?$AA@ 100aa89c     LIBCMT:nlsdata2.obj
 0002:000008ac       ??_C@_1BC@HHMNLIHE@?$AAT?$AAh?$AAu?$AAr?$AAs?$AAd?$AAa?$AAy?$AA?$AA@ 100aa8ac     LIBCMT:nlsdata2.obj
 0002:000008c0       ??_C@_1BE@EBOGMDOH@?$AAW?$AAe?$AAd?$AAn?$AAe?$AAs?$AAd?$AAa?$AAy?$AA?$AA@ 100aa8c0     LIBCMT:nlsdata2.obj
 0002:000008d4       ??_C@_1BA@ENFBFFEK@?$AAT?$AAu?$AAe?$AAs?$AAd?$AAa?$AAy?$AA?$AA@ 100aa8d4     LIBCMT:nlsdata2.obj
 0002:000008e4       ??_C@_1O@MMNBFLIA@?$AAM?$AAo?$AAn?$AAd?$AAa?$AAy?$AA?$AA@ 100aa8e4     LIBCMT:nlsdata2.obj
 0002:000008f4       ??_C@_1O@IHNHDHPB@?$AAS?$AAu?$AAn?$AAd?$AAa?$AAy?$AA?$AA@ 100aa8f4     LIBCMT:nlsdata2.obj
 0002:00000904       ??_C@_17GGIBDPIH@?$AAS?$AAa?$AAt?$AA?$AA@ 100aa904     LIBCMT:nlsdata2.obj
 0002:0000090c       ??_C@_17HFOLPPLP@?$AAF?$AAr?$AAi?$AA?$AA@ 100aa90c     LIBCMT:nlsdata2.obj
 0002:00000914       ??_C@_17PDPHAADD@?$AAT?$AAh?$AAu?$AA?$AA@ 100aa914     LIBCMT:nlsdata2.obj
 0002:0000091c       ??_C@_17CJEDCEPE@?$AAW?$AAe?$AAd?$AA?$AA@ 100aa91c     LIBCMT:nlsdata2.obj
 0002:00000924       ??_C@_17BMKGEGOJ@?$AAT?$AAu?$AAe?$AA?$AA@ 100aa924     LIBCMT:nlsdata2.obj
 0002:0000092c       ??_C@_17KBOMKBF@?$AAM?$AAo?$AAn?$AA?$AA@ 100aa92c     LIBCMT:nlsdata2.obj
 0002:00000934       ??_C@_17MBGCMIPB@?$AAS?$AAu?$AAn?$AA?$AA@ 100aa934     LIBCMT:nlsdata2.obj
 0002:0000093c       ??_C@_08JCCMCCIL@HH?3mm?3ss?$AA@ 100aa93c     LIBCMT:nlsdata2.obj
 0002:00000948       ??_C@_0BE@CKGJFCPC@dddd?0?5MMMM?5dd?0?5yyyy?$AA@ 100aa948     LIBCMT:nlsdata2.obj
 0002:0000095c       ??_C@_08BPBNCDIB@MM?1dd?1yy?$AA@ 100aa95c     LIBCMT:nlsdata2.obj
 0002:00000968       ??_C@_02CJNFDJBF@PM?$AA@   100aa968     LIBCMT:nlsdata2.obj
 0002:0000096c       ??_C@_02DEDBPAFC@AM?$AA@   100aa96c     LIBCMT:nlsdata2.obj
 0002:00000970       ??_C@_08EDHMEBNP@December?$AA@ 100aa970     LIBCMT:nlsdata2.obj
 0002:0000097c       ??_C@_08HCHEGEOA@November?$AA@ 100aa97c     LIBCMT:nlsdata2.obj
 0002:00000988       ??_C@_07JJNFCEND@October?$AA@ 100aa988     LIBCMT:nlsdata2.obj
 0002:00000990       ??_C@_09BHHEALKD@September?$AA@ 100aa990     LIBCMT:nlsdata2.obj
 0002:0000099c       ??_C@_06LBBHFDDG@August?$AA@ 100aa99c     LIBCMT:nlsdata2.obj
 0002:000009a4       ??_C@_04MIEPOIFP@July?$AA@ 100aa9a4     LIBCMT:nlsdata2.obj
 0002:000009ac       ??_C@_04CNLMGBGM@June?$AA@ 100aa9ac     LIBCMT:nlsdata2.obj
 0002:000009b4       ??_C@_05DMJDNLEJ@April?$AA@ 100aa9b4     LIBCMT:nlsdata2.obj
 0002:000009bc       ??_C@_05HPCKOFNC@March?$AA@ 100aa9bc     LIBCMT:nlsdata2.obj
 0002:000009c4       ??_C@_08GNJGEPFN@February?$AA@ 100aa9c4     LIBCMT:nlsdata2.obj
 0002:000009d0       ??_C@_07CGJPFGJA@January?$AA@ 100aa9d0     LIBCMT:nlsdata2.obj
 0002:000009d8       ??_C@_03MKABNOCG@Dec?$AA@  100aa9d8     LIBCMT:nlsdata2.obj
 0002:000009dc       ??_C@_03JPJOFNIA@Nov?$AA@  100aa9dc     LIBCMT:nlsdata2.obj
 0002:000009e0       ??_C@_03BMAOKBAD@Oct?$AA@  100aa9e0     LIBCMT:nlsdata2.obj
 0002:000009e4       ??_C@_03GGCAPAJC@Sep?$AA@  100aa9e4     LIBCMT:nlsdata2.obj
 0002:000009e8       ??_C@_03IFJFEIGA@Aug?$AA@  100aa9e8     LIBCMT:nlsdata2.obj
 0002:000009ec       ??_C@_03LBGABGKK@Jul?$AA@  100aa9ec     LIBCMT:nlsdata2.obj
 0002:000009f0       ??_C@_03IDFGHECI@Jun?$AA@  100aa9f0     LIBCMT:nlsdata2.obj
 0002:000009f4       ??_C@_03CNMDKL@May?$AA@    100aa9f4     LIBCMT:nlsdata2.obj
 0002:000009f8       ??_C@_03LEOLGMJP@Apr?$AA@  100aa9f8     LIBCMT:nlsdata2.obj
 0002:000009fc       ??_C@_03ODNJBKGA@Mar?$AA@  100aa9fc     LIBCMT:nlsdata2.obj
 0002:00000a00       ??_C@_03HJBDCHOM@Feb?$AA@  100aaa00     LIBCMT:nlsdata2.obj
 0002:00000a04       ??_C@_03JIHJHPIE@Jan?$AA@  100aaa04     LIBCMT:nlsdata2.obj
 0002:00000a08       ??_C@_08INBOOONO@Saturday?$AA@ 100aaa08     LIBCMT:nlsdata2.obj
 0002:00000a14       ??_C@_06JECMNKMI@Friday?$AA@ 100aaa14     LIBCMT:nlsdata2.obj
 0002:00000a1c       ??_C@_08HACCIKIA@Thursday?$AA@ 100aaa1c     LIBCMT:nlsdata2.obj
 0002:00000a28       ??_C@_09DLIGFAKA@Wednesday?$AA@ 100aaa28     LIBCMT:nlsdata2.obj
 0002:00000a34       ??_C@_07BAAGCFCM@Tuesday?$AA@ 100aaa34     LIBCMT:nlsdata2.obj
 0002:00000a3c       ??_C@_06JLEDEDGH@Monday?$AA@ 100aaa3c     LIBCMT:nlsdata2.obj
 0002:00000a44       ??_C@_06OOPIFAJ@Sunday?$AA@ 100aaa44     LIBCMT:nlsdata2.obj
 0002:00000a4c       ??_C@_03FEFJNEK@Sat?$AA@   100aaa4c     LIBCMT:nlsdata2.obj
 0002:00000a50       ??_C@_03IDIOELNC@Fri?$AA@  100aaa50     LIBCMT:nlsdata2.obj
 0002:00000a54       ??_C@_03IOFIKPDN@Thu?$AA@  100aaa54     LIBCMT:nlsdata2.obj
 0002:00000a58       ??_C@_03MHOMLAJA@Wed?$AA@  100aaa58     LIBCMT:nlsdata2.obj
 0002:00000a5c       ??_C@_03NAGEINEP@Tue?$AA@  100aaa5c     LIBCMT:nlsdata2.obj
 0002:00000a60       ??_C@_03PDAGKDH@Mon?$AA@   100aaa60     LIBCMT:nlsdata2.obj
 0002:00000a64       ??_C@_03KOEHGMDN@Sun?$AA@  100aaa64     LIBCMT:nlsdata2.obj
 0002:00000ae8       ??_C@_1O@CEDCILHN@?$AA?$CI?$AAn?$AAu?$AAl?$AAl?$AA?$CJ?$AA?$AA@ 100aaae8     LIBCMT:output.obj
 0002:00000af8       ??_C@_06OJHGLDPL@?$CInull?$CJ?$AA@ 100aaaf8     LIBCMT:output.obj
 0002:00000b00       ___lookuptable             100aab00     LIBCMT:output.obj
 0002:00000b5c       ??_C@_0P@MIGLKIOC@CorExitProcess?$AA@ 100aab5c     LIBCMT:crt0dat.obj
 0002:00000b6c       ??_C@_1BI@BGOHAHKC@?$AAm?$AAs?$AAc?$AAo?$AAr?$AAe?$AAe?$AA?4?$AAd?$AAl?$AAl?$AA?$AA@ 100aab6c     LIBCMT:crt0dat.obj
 0002:00000b88       __XcptActTab               100aab88     LIBCMT:winxfltr.obj
 0002:00000c18       __First_FPE_Indx           100aac18     LIBCMT:winxfltr.obj
 0002:00000c1c       __Num_FPE                  100aac1c     LIBCMT:winxfltr.obj
 0002:00000c20       __XcptActTabSize           100aac20     LIBCMT:winxfltr.obj
 0002:00000c24       __XcptActTabCount          100aac24     LIBCMT:winxfltr.obj
 0002:00000c28       __FPinit                   100aac28     LIBCMT:_fpinit_.obj
 0002:00000c2c       ??_C@_0L@KDOEJCKC@_nextafter?$AA@ 100aac2c     LIBCMT:_fpexcept_.obj
 0002:00000c38       ??_C@_05JGDBENOH@_logb?$AA@ 100aac38     LIBCMT:_fpexcept_.obj
 0002:00000c40       ??_C@_03ONILCKOB@_yn?$AA@  100aac40     LIBCMT:_fpexcept_.obj
 0002:00000c44       ??_C@_03NAKIGLHK@_y1?$AA@  100aac44     LIBCMT:_fpexcept_.obj
 0002:00000c48       ??_C@_03MJLDFKDL@_y0?$AA@  100aac48     LIBCMT:_fpexcept_.obj
 0002:00000c4c       ??_C@_05GKKHEGJL@frexp?$AA@ 100aac4c     LIBCMT:_fpexcept_.obj
 0002:00000c54       ??_C@_04KEPJIHGP@fmod?$AA@ 100aac54     LIBCMT:_fpexcept_.obj
 0002:00000c5c       ??_C@_06MEIMCGCF@_hypot?$AA@ 100aac5c     LIBCMT:_fpexcept_.obj
 0002:00000c64       ??_C@_05KBKMEMPO@_cabs?$AA@ 100aac64     LIBCMT:_fpexcept_.obj
 0002:00000c6c       ??_C@_05CEJMAHNP@ldexp?$AA@ 100aac6c     LIBCMT:_fpexcept_.obj
 0002:00000c74       ??_C@_04ODHECPBC@fabs?$AA@ 100aac74     LIBCMT:_fpexcept_.obj
 0002:00000c80       ___newctype                100aac80     LIBCMT:ctype.obj
 0002:00000f80       __wctype                   100aaf80     LIBCMT:ctype.obj
 0002:00001188       ___newclmap                100ab188     LIBCMT:ctype.obj
 0002:00001308       ___newcumap                100ab308     LIBCMT:ctype.obj
 0002:00001488       ___lookuptable_s           100ab488     LIBCMT:outputs.obj
 0002:000014e4       ??_C@_1BO@BKOMIGKJ@?$AAr?$AAu?$AAn?$AAt?$AAi?$AAm?$AAe?$AA?5?$AAe?$AAr?$AAr?$AAo?$AAr?$AA?5?$AA?$AA@ 100ab4e4     LIBCMT:crt0msg.obj
 0002:00001504       ??_C@_15JNBOKNOG@?$AA?$AN?$AA?6?$AA?$AA@ 100ab504     LIBCMT:crt0msg.obj
 0002:0000150c       ??_C@_1BM@JBBEPPHI@?$AAT?$AAL?$AAO?$AAS?$AAS?$AA?5?$AAe?$AAr?$AAr?$AAo?$AAr?$AA?$AN?$AA?6?$AA?$AA@ 100ab50c     LIBCMT:crt0msg.obj
 0002:00001528       ??_C@_1BK@KMOMNAAI@?$AAS?$AAI?$AAN?$AAG?$AA?5?$AAe?$AAr?$AAr?$AAo?$AAr?$AA?$AN?$AA?6?$AA?$AA@ 100ab528     LIBCMT:crt0msg.obj
 0002:00001544       ??_C@_1BO@BFCDCGC@?$AAD?$AAO?$AAM?$AAA?$AAI?$AAN?$AA?5?$AAe?$AAr?$AAr?$AAo?$AAr?$AA?$AN?$AA?6?$AA?$AA@ 100ab544     LIBCMT:crt0msg.obj
 0002:00001568       ??_C@_1BOO@KGEDBGAJ@?$AAR?$AA6?$AA0?$AA3?$AA3?$AA?$AN?$AA?6?$AA?9?$AA?5?$AAA?$AAt?$AAt?$AAe?$AAm?$AAp?$AAt?$AA?5?$AAt?$AAo?$AA?5?$AAu?$AAs?$AAe?$AA?5?$AAM?$AAS?$AAI?$AAL?$AA?5?$AAc?$AAo?$AAd@ 100ab568     LIBCMT:crt0msg.obj
 0002:00001758       ??_C@_1GG@GOPILAJP@?$AAR?$AA6?$AA0?$AA3?$AA2?$AA?$AN?$AA?6?$AA?9?$AA?5?$AAn?$AAo?$AAt?$AA?5?$AAe?$AAn?$AAo?$AAu?$AAg?$AAh?$AA?5?$AAs?$AAp?$AAa?$AAc?$AAe?$AA?5?$AAf?$AAo?$AAr?$AA?5?$AAl?$AAo@ 100ab758     LIBCMT:crt0msg.obj
 0002:000017c0       ??_C@_1MG@ENCOOIDF@?$AAR?$AA6?$AA0?$AA3?$AA1?$AA?$AN?$AA?6?$AA?9?$AA?5?$AAA?$AAt?$AAt?$AAe?$AAm?$AAp?$AAt?$AA?5?$AAt?$AAo?$AA?5?$AAi?$AAn?$AAi?$AAt?$AAi?$AAa?$AAl?$AAi?$AAz?$AAe?$AA?5?$AAt@ 100ab7c0     LIBCMT:crt0msg.obj
 0002:00001888       ??_C@_1DO@BMFCDCD@?$AAR?$AA6?$AA0?$AA3?$AA0?$AA?$AN?$AA?6?$AA?9?$AA?5?$AAC?$AAR?$AAT?$AA?5?$AAn?$AAo?$AAt?$AA?5?$AAi?$AAn?$AAi?$AAt?$AAi?$AAa?$AAl?$AAi?$AAz?$AAe?$AAd?$AA?$AN?$AA?6?$AA?$AA@ 100ab888     LIBCMT:crt0msg.obj
 0002:000018c8       ??_C@_1EK@HHFLMAOL@?$AAR?$AA6?$AA0?$AA2?$AA8?$AA?$AN?$AA?6?$AA?9?$AA?5?$AAu?$AAn?$AAa?$AAb?$AAl?$AAe?$AA?5?$AAt?$AAo?$AA?5?$AAi?$AAn?$AAi?$AAt?$AAi?$AAa?$AAl?$AAi?$AAz?$AAe?$AA?5?$AAh?$AAe@ 100ab8c8     LIBCMT:crt0msg.obj
 0002:00001918       ??_C@_1GK@MFGOKLAG@?$AAR?$AA6?$AA0?$AA2?$AA7?$AA?$AN?$AA?6?$AA?9?$AA?5?$AAn?$AAo?$AAt?$AA?5?$AAe?$AAn?$AAo?$AAu?$AAg?$AAh?$AA?5?$AAs?$AAp?$AAa?$AAc?$AAe?$AA?5?$AAf?$AAo?$AAr?$AA?5?$AAl?$AAo@ 100ab918     LIBCMT:crt0msg.obj
 0002:00001988       ??_C@_1GK@MCAAGJMO@?$AAR?$AA6?$AA0?$AA2?$AA6?$AA?$AN?$AA?6?$AA?9?$AA?5?$AAn?$AAo?$AAt?$AA?5?$AAe?$AAn?$AAo?$AAu?$AAg?$AAh?$AA?5?$AAs?$AAp?$AAa?$AAc?$AAe?$AA?5?$AAf?$AAo?$AAr?$AA?5?$AAs?$AAt@ 100ab988     LIBCMT:crt0msg.obj
 0002:000019f8       ??_C@_1EM@MAADIHMB@?$AAR?$AA6?$AA0?$AA2?$AA5?$AA?$AN?$AA?6?$AA?9?$AA?5?$AAp?$AAu?$AAr?$AAe?$AA?5?$AAv?$AAi?$AAr?$AAt?$AAu?$AAa?$AAl?$AA?5?$AAf?$AAu?$AAn?$AAc?$AAt?$AAi?$AAo?$AAn?$AA?5?$AAc@ 100ab9f8     LIBCMT:crt0msg.obj
 0002:00001a48       ??_C@_1GK@FHCKBEFA@?$AAR?$AA6?$AA0?$AA2?$AA4?$AA?$AN?$AA?6?$AA?9?$AA?5?$AAn?$AAo?$AAt?$AA?5?$AAe?$AAn?$AAo?$AAu?$AAg?$AAh?$AA?5?$AAs?$AAp?$AAa?$AAc?$AAe?$AA?5?$AAf?$AAo?$AAr?$AA?5?$AA_?$AAo@ 100aba48     LIBCMT:crt0msg.obj
 0002:00001ab8       ??_C@_1FC@ECHBIFBC@?$AAR?$AA6?$AA0?$AA1?$AA9?$AA?$AN?$AA?6?$AA?9?$AA?5?$AAu?$AAn?$AAa?$AAb?$AAl?$AAe?$AA?5?$AAt?$AAo?$AA?5?$AAo?$AAp?$AAe?$AAn?$AA?5?$AAc?$AAo?$AAn?$AAs?$AAo?$AAl?$AAe?$AA?5@ 100abab8     LIBCMT:crt0msg.obj
 0002:00001b10       ??_C@_1EC@JIBHAOPH@?$AAR?$AA6?$AA0?$AA1?$AA8?$AA?$AN?$AA?6?$AA?9?$AA?5?$AAu?$AAn?$AAe?$AAx?$AAp?$AAe?$AAc?$AAt?$AAe?$AAd?$AA?5?$AAh?$AAe?$AAa?$AAp?$AA?5?$AAe?$AAr?$AAr?$AAo?$AAr?$AA?$AN?$AA?6@ 100abb10     LIBCMT:crt0msg.obj
 0002:00001b58       ??_C@_1FK@BEOGODMC@?$AAR?$AA6?$AA0?$AA1?$AA7?$AA?$AN?$AA?6?$AA?9?$AA?5?$AAu?$AAn?$AAe?$AAx?$AAp?$AAe?$AAc?$AAt?$AAe?$AAd?$AA?5?$AAm?$AAu?$AAl?$AAt?$AAi?$AAt?$AAh?$AAr?$AAe?$AAa?$AAd?$AA?5@ 100abb58     LIBCMT:crt0msg.obj
 0002:00001bb8       ??_C@_1FI@LOGNIKDM@?$AAR?$AA6?$AA0?$AA1?$AA6?$AA?$AN?$AA?6?$AA?9?$AA?5?$AAn?$AAo?$AAt?$AA?5?$AAe?$AAn?$AAo?$AAu?$AAg?$AAh?$AA?5?$AAs?$AAp?$AAa?$AAc?$AAe?$AA?5?$AAf?$AAo?$AAr?$AA?5?$AAt?$AAh@ 100abbb8     LIBCMT:crt0msg.obj
 0002:00001c10       ??_C@_1EG@BEHAGFJD@?$AAR?$AA6?$AA0?$AA1?$AA0?$AA?$AN?$AA?6?$AA?9?$AA?5?$AAa?$AAb?$AAo?$AAr?$AAt?$AA?$CI?$AA?$CJ?$AA?5?$AAh?$AAa?$AAs?$AA?5?$AAb?$AAe?$AAe?$AAn?$AA?5?$AAc?$AAa?$AAl?$AAl?$AAe?$AAd@ 100abc10     LIBCMT:crt0msg.obj
 0002:00001c58       ??_C@_1FI@HONFMGBI@?$AAR?$AA6?$AA0?$AA0?$AA9?$AA?$AN?$AA?6?$AA?9?$AA?5?$AAn?$AAo?$AAt?$AA?5?$AAe?$AAn?$AAo?$AAu?$AAg?$AAh?$AA?5?$AAs?$AAp?$AAa?$AAc?$AAe?$AA?5?$AAf?$AAo?$AAr?$AA?5?$AAe?$AAn@ 100abc58     LIBCMT:crt0msg.obj
 0002:00001cb0       ??_C@_1FE@LLNEDJMD@?$AAR?$AA6?$AA0?$AA0?$AA8?$AA?$AN?$AA?6?$AA?9?$AA?5?$AAn?$AAo?$AAt?$AA?5?$AAe?$AAn?$AAo?$AAu?$AAg?$AAh?$AA?5?$AAs?$AAp?$AAa?$AAc?$AAe?$AA?5?$AAf?$AAo?$AAr?$AA?5?$AAa?$AAr@ 100abcb0     LIBCMT:crt0msg.obj
 0002:00001d08       ??_C@_1FK@PGACCAFB@?$AAR?$AA6?$AA0?$AA0?$AA2?$AA?$AN?$AA?6?$AA?9?$AA?5?$AAf?$AAl?$AAo?$AAa?$AAt?$AAi?$AAn?$AAg?$AA?5?$AAp?$AAo?$AAi?$AAn?$AAt?$AA?5?$AAs?$AAu?$AAp?$AAp?$AAo?$AAr?$AAt?$AA?5@ 100abd08     LIBCMT:crt0msg.obj
 0002:00001e18       ??_C@_1EK@MBDPDCGA@?$AAM?$AAi?$AAc?$AAr?$AAo?$AAs?$AAo?$AAf?$AAt?$AA?5?$AAV?$AAi?$AAs?$AAu?$AAa?$AAl?$AA?5?$AAC?$AA?$CL?$AA?$CL?$AA?5?$AAR?$AAu?$AAn?$AAt?$AAi?$AAm?$AAe?$AA?5?$AAL?$AAi?$AAb@ 100abe18     LIBCMT:crt0msg.obj
 0002:00001e64       ??_C@_15IABLJNFO@?$AA?6?$AA?6?$AA?$AA@ 100abe64     LIBCMT:crt0msg.obj
 0002:00001e6c       ??_C@_17LGKOMLJ@?$AA?4?$AA?4?$AA?4?$AA?$AA@ 100abe6c     LIBCMT:crt0msg.obj
 0002:00001e74       ??_C@_1CO@EAEJAADC@?$AA?$DM?$AAp?$AAr?$AAo?$AAg?$AAr?$AAa?$AAm?$AA?5?$AAn?$AAa?$AAm?$AAe?$AA?5?$AAu?$AAn?$AAk?$AAn?$AAo?$AAw?$AAn?$AA?$DO?$AA?$AA@ 100abe74     LIBCMT:crt0msg.obj
 0002:00001ea4       ??_C@_1DE@JNGNBFGO@?$AAR?$AAu?$AAn?$AAt?$AAi?$AAm?$AAe?$AA?5?$AAE?$AAr?$AAr?$AAo?$AAr?$AA?$CB?$AA?6?$AA?6?$AAP?$AAr?$AAo?$AAg?$AAr?$AAa?$AAm?$AA?3?$AA?5?$AA?$AA@ 100abea4     LIBCMT:crt0msg.obj
 0002:00001ed8       ??_C@_05KLBDPFGC@e?$CL000?$AA@ 100abed8     LIBCMT:cvt.obj
 0002:00001ee0       ??_C@_0BI@DFKBFLJE@GetProcessWindowStation?$AA@ 100abee0     LIBCMT:crtmboxw.obj
 0002:00001ef8       ??_C@_0BK@DEKFELLI@GetUserObjectInformationW?$AA@ 100abef8     LIBCMT:crtmboxw.obj
 0002:00001f14       ??_C@_0BD@HHGDFDBJ@GetLastActivePopup?$AA@ 100abf14     LIBCMT:crtmboxw.obj
 0002:00001f28       ??_C@_0BA@HNOPNCHB@GetActiveWindow?$AA@ 100abf28     LIBCMT:crtmboxw.obj
 0002:00001f38       ??_C@_0M@DLDCCGNP@MessageBoxW?$AA@ 100abf38     LIBCMT:crtmboxw.obj
 0002:00001f44       ??_C@_1BG@GOEBHBDC@?$AAU?$AAS?$AAE?$AAR?$AA3?$AA2?$AA?4?$AAD?$AAL?$AAL?$AA?$AA@ 100abf44     LIBCMT:crtmboxw.obj
 0002:00001f5c       ??_C@_06IMKFLFPG@1?$CDQNAN?$AA@ 100abf5c     LIBCMT:_x10fout_.obj
 0002:00001f64       ??_C@_05DNEBIAHO@1?$CDINF?$AA@ 100abf64     LIBCMT:_x10fout_.obj
 0002:00001f6c       ??_C@_05PHHOCPM@1?$CDIND?$AA@ 100abf6c     LIBCMT:_x10fout_.obj
 0002:00001f74       ??_C@_06PGGFOGJG@1?$CDSNAN?$AA@ 100abf74     LIBCMT:_x10fout_.obj
 0002:00001f7c       ??_C@_1BA@BALFACEM@?$AAC?$AAO?$AAN?$AAO?$AAU?$AAT?$AA$?$AA?$AA@ 100abf7c     LIBCMT:initcon.obj
 0002:00001f90       _sqlite3_version           100abf90     interop.obj
 0002:00005da8       ??_C@_0CB@LFIMBCA@LIKE?5or?5GLOB?5pattern?5too?5complex@ 100afda8     sqlite3_unicode.obj
 0002:00005dcc       ??_C@_0CN@PAMOLCDH@ESCAPE?5expression?5must?5be?5a?5sing@ 100afdcc     sqlite3_unicode.obj
 0002:00005dfc       ??_C@_08ILALGPFF@5?41?40?412?$AA@ 100afdfc     sqlite3_unicode.obj
 0002:00005e08       ??_C@_0BA@BNJIKJKH@unicode_version?$AA@ 100afe08     sqlite3_unicode.obj
 0002:00005e18       ??_C@_04HPDJJBAE@like?$AA@ 100afe18     sqlite3_unicode.obj
 0002:00005e20       ??_C@_04MLGPBLN@fold?$AA@  100afe20     sqlite3_unicode.obj
 0002:00005e28       ??_C@_05IPJEPLHL@lower?$AA@ 100afe28     sqlite3_unicode.obj
 0002:00005e30       ??_C@_05NECKJAMC@upper?$AA@ 100afe30     sqlite3_unicode.obj
 0002:00005e38       ??_C@_05PHLGJONK@title?$AA@ 100afe38     sqlite3_unicode.obj
 0002:00005e40       ??_C@_08BOHCLFJD@unaccent?$AA@ 100afe40     sqlite3_unicode.obj
 0002:00005e4c       ??_C@_06FHKGKAHE@NOCASE?$AA@ 100afe4c     sqlite3_unicode.obj
 0002:00005e54       ??_C@_0P@GILEIKMI@upper_quartile?$AA@ 100afe54     interop.obj
 0002:00005e64       ??_C@_0P@BHPBIMCK@lower_quartile?$AA@ 100afe64     interop.obj
 0002:00005e74       ??_C@_06EIDMBNHH@median?$AA@ 100afe74     interop.obj
 0002:00005e7c       ??_C@_08PPLCFKON@variance?$AA@ 100afe7c     interop.obj
 0002:00005e88       ??_C@_05EMOENAND@stdev?$AA@ 100afe88     interop.obj
 0002:00005e90       ??_C@_09GOCGDFFD@strfilter?$AA@ 100afe90     interop.obj
 0002:00005e9c       ??_C@_04ECJLCDND@padc?$AA@ 100afe9c     interop.obj
 0002:00005ea4       ??_C@_04BBECAAMD@padr?$AA@ 100afea4     interop.obj
 0002:00005eac       ??_C@_04MFADDPBM@padl?$AA@ 100afeac     interop.obj
 0002:00005eb4       ??_C@_06OLFJAONP@proper?$AA@ 100afeb4     interop.obj
 0002:00005ebc       ??_C@_07KOIEOCCE@reverse?$AA@ 100afebc     interop.obj
 0002:00005ec4       ??_C@_08JJJINGEL@rightstr?$AA@ 100afec4     interop.obj
 0002:00005ed0       ??_C@_07CBJDIIOC@leftstr?$AA@ 100afed0     interop.obj
 0002:00005ed8       ??_C@_09LCOPGHLO@charindex?$AA@ 100afed8     interop.obj
 0002:00005ee4       ??_C@_09CBPKCNMB@replicate?$AA@ 100afee4     interop.obj
 0002:00005ef0       ??_C@_0BD@IFENDAKA@last_rows_affected?$AA@ 100afef0     interop.obj
 0002:00005f04       ??_C@_02OAHAJOFD@pi?$AA@   100aff04     interop.obj
 0002:00005f08       ??_C@_05PBJFFIGL@floor?$AA@ 100aff08     interop.obj
 0002:00005f10       ??_C@_07EANFIDJB@ceiling?$AA@ 100aff10     interop.obj
 0002:00005f18       ??_C@_04GFPJNGEK@ceil?$AA@ 100aff18     interop.obj
 0002:00005f20       ??_C@_06ICDKOIFG@square?$AA@ 100aff20     interop.obj
 0002:00005f28       ??_C@_04EIAKFFMI@sqrt?$AA@ 100aff28     interop.obj
 0002:00005f30       ??_C@_04HHGHLBPI@sign?$AA@ 100aff30     interop.obj
 0002:00005f38       ??_C@_05PLIADJJL@power?$AA@ 100aff38     interop.obj
 0002:00005f40       ??_C@_05HGHHAHAP@log10?$AA@ 100aff40     interop.obj
 0002:00005f48       ??_C@_03KHJOGHMM@exp?$AA@  100aff48     interop.obj
 0002:00005f4c       ??_C@_04HKNGMDAJ@coth?$AA@ 100aff4c     interop.obj
 0002:00005f54       ??_C@_04FJHINJAO@tanh?$AA@ 100aff54     interop.obj
 0002:00005f5c       ??_C@_04COOMCNPB@sinh?$AA@ 100aff5c     interop.obj
 0002:00005f64       ??_C@_04HPJJNFIM@cosh?$AA@ 100aff64     interop.obj
 0002:00005f6c       ??_C@_03PPPAEIOB@cot?$AA@  100aff6c     interop.obj
 0002:00005f70       ??_C@_03IIINPABG@tan?$AA@  100aff70     interop.obj
 0002:00005f74       ??_C@_03BLEJJJBH@sin?$AA@  100aff74     interop.obj
 0002:00005f78       ??_C@_03LALBNOCG@cos?$AA@  100aff78     interop.obj
 0002:00005f7c       ??_C@_07JLOPPFCD@radians?$AA@ 100aff7c     interop.obj
 0002:00005f84       ??_C@_07MHOHEFBH@degrees?$AA@ 100aff84     interop.obj
 0002:00005f8c       ??_C@_0L@CHCOIIBP@difference?$AA@ 100aff8c     interop.obj
 0002:00005f98       ??_C@_05ONDAFDEP@atanh?$AA@ 100aff98     interop.obj
 0002:00005fa0       ??_C@_05JKKEKHLA@asinh?$AA@ 100affa0     interop.obj
 0002:00005fa8       ??_C@_05MLNBFPMN@acosh?$AA@ 100affa8     interop.obj
 0002:00005fb0       ??_C@_05KNGEOGJB@atan2?$AA@ 100affb0     interop.obj
 0002:00005fb8       ??_C@_04NGOLNDIP@atn2?$AA@ 100affb8     interop.obj
 0002:00005fc0       ??_C@_04MLLJIGOK@atan?$AA@ 100affc0     interop.obj
 0002:00005fc8       ??_C@_04FIHNOPOL@asin?$AA@ 100affc8     interop.obj
 0002:00005fd0       ??_C@_04PDIFKINK@acos?$AA@ 100affd0     interop.obj
 0002:00005fd8       ??_C@_0CP@DMLOGJAI@DELETE?5FROM?5?8?$CFq?8?4?8?$CFq_parent?8?5WHE@ 100affd8     interop.obj
 0002:00006008       ??_C@_0DH@IPNBEOMK@INSERT?5OR?5REPLACE?5INTO?5?8?$CFq?8?4?8?$CFq_@ 100b0008     interop.obj
 0002:00006040       ??_C@_0DK@LBKGHCLI@SELECT?5parentnode?5FROM?5?8?$CFq?8?4?8?$CFq_@ 100b0040     interop.obj
 0002:0000607c       ??_C@_0CN@JLLIJKKP@DELETE?5FROM?5?8?$CFq?8?4?8?$CFq_rowid?8?5WHER@ 100b007c     interop.obj
 0002:000060ac       ??_C@_0DG@OPBLMGLD@INSERT?5OR?5REPLACE?5INTO?5?8?$CFq?8?4?8?$CFq_@ 100b00ac     interop.obj
 0002:000060e4       ??_C@_0DE@NMCAHMCK@SELECT?5nodeno?5FROM?5?8?$CFq?8?4?8?$CFq_rowi@ 100b00e4     interop.obj
 0002:00006118       ??_C@_0CN@NJAIPDIA@DELETE?5FROM?5?8?$CFq?8?4?8?$CFq_node?8?5WHERE@ 100b0118     interop.obj
 0002:00006148       ??_C@_0DF@HGBHOIBO@INSERT?5OR?5REPLACE?5INTO?5?8?$CFq?8?4?8?$CFq_@ 100b0148     interop.obj
 0002:00006180       ??_C@_0DC@LADEDDNO@SELECT?5data?5FROM?5?8?$CFq?8?4?8?$CFq_node?8?5@ 100b0180     interop.obj
 0002:000061b4       ??_C@_04ILABJOOE@NEAR?$AA@ 100b01b4     interop.obj
 0002:000061bc       ??_C@_03GBFNEA@NOT?$AA@    100b01bc     interop.obj
 0002:000061c0       ??_C@_03BDACDFHA@AND?$AA@  100b01c0     interop.obj
 0002:000061c4       ??_C@_02PDPFNDMG@OR?$AA@   100b01c4     interop.obj
 0002:000061c8       ??_C@_03ODAOEF@rwc?$AA@    100b01c8     interop.obj
 0002:000061cc       ??_C@_02DHLFHFOC@rw?$AA@   100b01cc     interop.obj
 0002:000061d0       ??_C@_02LFKOONLL@ro?$AA@   100b01d0     interop.obj
 0002:000061d4       ??_C@_07NMPLPEPB@private?$AA@ 100b01d4     interop.obj
 0002:000061dc       ??_C@_06HBFNPGIC@shared?$AA@ 100b01dc     interop.obj
 0002:000061e4       ??_C@_0CH@JKOMOHHH@file?5is?5encrypted?5or?5is?5not?5a?5da@ 100b01e4     interop.obj
 0002:0000620c       ??_C@_0CC@OHMKLHEA@bind?5or?5column?5index?5out?5of?5rang@ 100b020c     interop.obj
 0002:00006230       ??_C@_0CA@DBBJFBEG@auxiliary?5database?5format?5error?$AA@ 100b0230     interop.obj
 0002:00006250       ??_C@_0BF@LMCDAPDN@authorization?5denied?$AA@ 100b0250     interop.obj
 0002:00006268       ??_C@_0BP@GMDPJID@large?5file?5support?5is?5disabled?$AA@ 100b0268     interop.obj
 0002:00006288       ??_C@_0CH@GCDGLLPA@library?5routine?5called?5out?5of?5se@ 100b0288     interop.obj
 0002:000062b0       ??_C@_0BC@FILINGOB@datatype?5mismatch?$AA@ 100b02b0     interop.obj
 0002:000062c4       ??_C@_0BC@IFKPGMGK@constraint?5failed?$AA@ 100b02c4     interop.obj
 0002:000062d8       ??_C@_0BH@OCNELEJF@table?5contains?5no?5data?$AA@ 100b02d8     interop.obj
 0002:000062f0       ??_C@_0BB@MCPOJJBB@locking?5protocol?$AA@ 100b02f0     interop.obj
 0002:00006304       ??_C@_0BN@JLONMGIA@unable?5to?5open?5database?5file?$AA@ 100b0304     interop.obj
 0002:00006324       ??_C@_0BJ@GDNBBAEL@database?5or?5disk?5is?5full?$AA@ 100b0324     interop.obj
 0002:00006340       ??_C@_0BC@BDMDPLFD@unknown?5operation?$AA@ 100b0340     interop.obj
 0002:00006354       ??_C@_0CB@ONDDCPGK@database?5disk?5image?5is?5malformed@ 100b0354     interop.obj
 0002:00006378       ??_C@_0P@FOPPKBJH@disk?5I?1O?5error?$AA@ 100b0378     interop.obj
 0002:00006388       ??_C@_0M@EGEKIIMP@interrupted?$AA@ 100b0388     interop.obj
 0002:00006394       ??_C@_0CF@JBLJEMGC@attempt?5to?5write?5a?5readonly?5data@ 100b0394     interop.obj
 0002:000063bc       ??_C@_0BJ@DNPONIEG@database?5table?5is?5locked?$AA@ 100b03bc     interop.obj
 0002:000063d8       ??_C@_0BD@DAAAMHOI@database?5is?5locked?$AA@ 100b03d8     interop.obj
 0002:000063ec       ??_C@_0BP@BFMDEDKN@callback?5requested?5query?5abort?$AA@ 100b03ec     interop.obj
 0002:0000640c       ??_C@_0BJ@OFHFLJKH@access?5permission?5denied?$AA@ 100b040c     interop.obj
 0002:00006428       ??_C@_0CE@BCMAPMOL@SQL?5logic?5error?5or?5missing?5datab@ 100b0428     interop.obj
 0002:0000644c       ??_C@_0N@FKKFHCIB@not?5an?5error?$AA@ 100b044c     interop.obj
 0002:0000645c       ??_C@_06EENFNEPD@detail?$AA@ 100b045c     interop.obj
 0002:00006464       ??_C@_05NDNMCCJH@order?$AA@ 100b0464     interop.obj
 0002:0000646c       ??_C@_08CAKEGGLM@selectid?$AA@ 100b046c     interop.obj
 0002:00006478       ??_C@_07GJGNEJFD@comment?$AA@ 100b0478     interop.obj
 0002:00006480       ??_C@_02PGHOIMAL@p5?$AA@   100b0480     interop.obj
 0002:00006484       ??_C@_02OPGFLNEK@p4?$AA@   100b0484     interop.obj
 0002:00006488       ??_C@_02KACECLIN@p3?$AA@   100b0488     interop.obj
 0002:0000648c       ??_C@_02LJDPBKMM@p2?$AA@   100b048c     interop.obj
 0002:00006490       ??_C@_02JCBCEJAP@p1?$AA@   100b0490     interop.obj
 0002:00006494       ??_C@_06POMMAHJK@opcode?$AA@ 100b0494     interop.obj
 0002:0000649c       ??_C@_04HLBMEOMD@addr?$AA@ 100b049c     interop.obj
 0002:000064a4       ??_C@_05MNCHLHCA@UTF16?$AA@ 100b04a4     interop.obj
 0002:000064ac       ??_C@_06KNDPGIKI@UTF?916?$AA@ 100b04ac     interop.obj
 0002:000064b4       ??_C@_07JDFIEPAG@UTF16be?$AA@ 100b04b4     interop.obj
 0002:000064bc       ??_C@_07JJMGGCAM@UTF16le?$AA@ 100b04bc     interop.obj
 0002:000064c4       ??_C@_08HGGOPCBI@UTF?916be?$AA@ 100b04c4     interop.obj
 0002:000064d0       ??_C@_08HMPANPBC@UTF?916le?$AA@ 100b04d0     interop.obj
 0002:000064dc       ??_C@_05EGJIMALK@UTF?98?$AA@ 100b04dc     interop.obj
 0002:000064e4       ??_C@_04OOMJJNCF@UTF8?$AA@ 100b04e4     interop.obj
 0002:000064ec       ??_C@_03KIAODNHK@wal?$AA@  100b04ec     interop.obj
 0002:000064f0       ??_C@_08MABILMFG@truncate?$AA@ 100b04f0     interop.obj
 0002:000064fc       ??_C@_03MCADLMAF@off?$AA@  100b04fc     interop.obj
 0002:00006500       ??_C@_07EMFBDGOD@persist?$AA@ 100b0500     interop.obj
 0002:00006508       ??_C@_06FOBLBEIN@delete?$AA@ 100b0508     interop.obj
 0002:00006510       ??_C@_0N@CEEMEAMB@foreign_keys?$AA@ 100b0510     interop.obj
 0002:00006520       ??_C@_0BD@IAMNLMFM@recursive_triggers?$AA@ 100b0520     interop.obj
 0002:00006534       ??_C@_0BB@KLHJNGLH@read_uncommitted?$AA@ 100b0534     interop.obj
 0002:00006548       ??_C@_0BA@OHBCLCAL@writable_schema?$AA@ 100b0548     interop.obj
 0002:00006558       ??_C@_0BJ@KLIMENGM@ignore_check_constraints?$AA@ 100b0558     interop.obj
 0002:00006574       ??_C@_0BA@NMINPKHE@automatic_index?$AA@ 100b0574     interop.obj
 0002:00006584       ??_C@_0BK@ECMFJINF@reverse_unordered_selects?$AA@ 100b0584     interop.obj
 0002:000065a0       ??_C@_0BF@IOJNJBPA@checkpoint_fullfsync?$AA@ 100b05a0     interop.obj
 0002:000065b8       ??_C@_09MLJLLBEB@fullfsync?$AA@ 100b05b8     interop.obj
 0002:000065c4       ??_C@_0BD@LEFOEGBK@legacy_file_format?$AA@ 100b05c4     interop.obj
 0002:000065d8       ??_C@_0BH@CMLDBHJP@empty_result_callbacks?$AA@ 100b05d8     interop.obj
 0002:000065f0       ??_C@_0O@PEBBJPHD@count_changes?$AA@ 100b05f0     interop.obj
 0002:00006600       ??_C@_0BD@BFIEDLEP@short_column_names?$AA@ 100b0600     interop.obj
 0002:00006614       ??_C@_0BC@CBBNFKC@full_column_names?$AA@ 100b0614     interop.obj
 0002:00006628       ??_C@_03OCHKFGFI@dll?$AA@  100b0628     interop.obj
 0002:0000662c       ??_C@_0N@KKLIBDFO@group_concat?$AA@ 100b062c     interop.obj
 0002:0000663c       ??_C@_05IOMEMJEC@count?$AA@ 100b063c     interop.obj
 0002:00006644       ??_C@_03CHOBFJAH@avg?$AA@  100b0644     interop.obj
 0002:00006648       ??_C@_05KBOMEDGA@total?$AA@ 100b0648     interop.obj
 0002:00006650       ??_C@_03CFFIJAMA@sum?$AA@  100b0650     interop.obj
 0002:00006654       ??_C@_0P@BJKPICNH@load_extension?$AA@ 100b0654     interop.obj
 0002:00006664       ??_C@_07KFKPEFNG@soundex?$AA@ 100b0664     interop.obj
 0002:0000666c       ??_C@_08OAGHJJOG@zeroblob?$AA@ 100b066c     interop.obj
 0002:00006678       ??_C@_07CLEHDIEJ@replace?$AA@ 100b0678     interop.obj
 0002:00006680       ??_C@_0O@MLEKHAGK@total_changes?$AA@ 100b0680     interop.obj
 0002:00006690       ??_C@_07HFLFHMNL@changes?$AA@ 100b0690     interop.obj
 0002:00006698       ??_C@_0BC@EKKKCJJE@last_insert_rowid?$AA@ 100b0698     interop.obj
 0002:000066ac       ??_C@_05JHEGFHLM@quote?$AA@ 100b06ac     interop.obj
 0002:000066b4       ??_C@_0BJ@BHKPGCCL@sqlite_compileoption_get?$AA@ 100b06b4     interop.obj
 0002:000066d0       ??_C@_0BK@NPIMPNGH@sqlite_compileoption_used?$AA@ 100b06d0     interop.obj
 0002:000066ec       ??_C@_0L@HNFKFGGK@sqlite_log?$AA@ 100b06ec     interop.obj
 0002:000066f8       ??_C@_0BB@HPCCOLJC@sqlite_source_id?$AA@ 100b06f8     interop.obj
 0002:0000670c       ??_C@_0P@IPDPEBN@sqlite_version?$AA@ 100b070c     interop.obj
 0002:0000671c       ??_C@_06LLGGGFDC@nullif?$AA@ 100b071c     interop.obj
 0002:00006724       ??_C@_0L@IDMFPHDO@randomblob?$AA@ 100b0724     interop.obj
 0002:00006730       ??_C@_06NLFCANPD@random?$AA@ 100b0730     interop.obj
 0002:00006738       ??_C@_06FAHGEKJN@ifnull?$AA@ 100b0738     interop.obj
 0002:00006740       ??_C@_03IJNDAFDK@hex?$AA@  100b0740     interop.obj
 0002:00006744       ??_C@_08FNGHHBID@coalesce?$AA@ 100b0744     interop.obj
 0002:00006750       ??_C@_05MIMAKCN@round?$AA@ 100b0750     interop.obj
 0002:00006758       ??_C@_03BCGAIFPO@abs?$AA@  100b0758     interop.obj
 0002:0000675c       ??_C@_04ENMBGAPA@char?$AA@ 100b075c     interop.obj
 0002:00006764       ??_C@_07GAJMMAJO@unicode?$AA@ 100b0764     interop.obj
 0002:0000676c       ??_C@_06DAHFIGOC@substr?$AA@ 100b076c     interop.obj
 0002:00006774       ??_C@_05HALPBNGI@instr?$AA@ 100b0774     interop.obj
 0002:0000677c       ??_C@_06IJDLPEM@length?$AA@ 100b077c     interop.obj
 0002:00006784       ??_C@_06NDJPCPHC@typeof?$AA@ 100b0784     interop.obj
 0002:0000678c       ??_C@_03LJAEFNNE@max?$AA@  100b078c     interop.obj
 0002:00006790       ??_C@_03KLIPLJLL@min?$AA@  100b0790     interop.obj
 0002:00006794       ??_C@_04GDOMMDLP@trim?$AA@ 100b0794     interop.obj
 0002:0000679c       ??_C@_05FCOGDJML@rtrim?$AA@ 100b079c     interop.obj
 0002:000067a4       ??_C@_05GLDKFKCA@ltrim?$AA@ 100b07a4     interop.obj
 0002:000067ac       ??_C@_07LDDIIHCM@RELEASE?$AA@ 100b07ac     interop.obj
 0002:000067b4       ??_C@_05IKBMIIDA@?5REAL?$AA@ 100b07b4     interop.obj
 0002:000067bc       ??_C@_04LKNDAIML@?5INT?$AA@ 100b07bc     interop.obj
 0002:000067c4       ??_C@_04KMHHNFPL@?5NUM?$AA@ 100b07c4     interop.obj
 0002:000067cc       ??_C@_05JELAHNDG@?5TEXT?$AA@ 100b07cc     interop.obj
 0002:000067d4       ??_C@_0O@GJLGHGMJ@sqlite_attach?$AA@ 100b07d4     interop.obj
 0002:000067e4       ??_C@_0O@PDAEIIFA@sqlite_detach?$AA@ 100b07e4     interop.obj
 0002:000067f4       ??_C@_09DDDBDIEM@stat3_get?$AA@ 100b07f4     interop.obj
 0002:00006800       ??_C@_0L@FFOLNHKE@stat3_push?$AA@ 100b0800     interop.obj
 0002:0000680c       ??_C@_0L@EIMFIJDC@stat3_init?$AA@ 100b080c     interop.obj
 0002:00006818       ??_C@_0BM@EJONBLKK@tbl?0idx?0neq?0nlt?0ndlt?0sample?$AA@ 100b0818     interop.obj
 0002:00006834       ??_C@_0N@HKFCOGAL@sqlite_stat3?$AA@ 100b0834     interop.obj
 0002:00006844       ??_C@_0N@BCOBMINH@tbl?0idx?0stat?$AA@ 100b0844     interop.obj
 0002:00006854       ??_C@_0N@EIGEIEIJ@sqlite_stat1?$AA@ 100b0854     interop.obj
 0002:00006864       ??_C@_0BF@CIKMGNA@sqlite_rename_parent?$AA@ 100b0864     interop.obj
 0002:0000687c       ??_C@_0BG@DKJJOMDK@sqlite_rename_trigger?$AA@ 100b087c     interop.obj
 0002:00006894       ??_C@_0BE@JHJAJICL@sqlite_rename_table?$AA@ 100b0894     interop.obj
 0002:000068a8       ??_C@_0BJ@EKFPCGJA@CreateFileMappingFromApp?$AA@ 100b08a8     interop.obj
 0002:000068c4       ??_C@_0P@BOLOPLNF@GetProcessHeap?$AA@ 100b08c4     interop.obj
 0002:000068d4       ??_C@_0BD@JHPCPJIF@OutputDebugStringW?$AA@ 100b08d4     interop.obj
 0002:000068e8       ??_C@_0BD@ILGKEMFC@OutputDebugStringA?$AA@ 100b08e8     interop.obj
 0002:000068fc       ??_C@_0BE@HLKFLAJF@GetNativeSystemInfo?$AA@ 100b08fc     interop.obj
 0002:00006910       ??_C@_0P@CDHHOHKP@GetTickCount64?$AA@ 100b0910     interop.obj
 0002:00006920       ??_C@_0BE@GMOAPDKA@LoadPackagedLibrary?$AA@ 100b0920     interop.obj
 0002:00006934       ??_C@_0M@HHGEPIBF@CreateFile2?$AA@ 100b0934     interop.obj
 0002:00006940       ??_C@_0BF@ECJCKDGL@MapViewOfFileFromApp?$AA@ 100b0940     interop.obj
 0002:00006958       ??_C@_0BN@NEEHBBPO@GetFileInformationByHandleEx?$AA@ 100b0958     interop.obj
 0002:00006978       ??_C@_0BB@GDGABGCO@SetFilePointerEx?$AA@ 100b0978     interop.obj
 0002:0000698c       ??_C@_0BG@IFNJHLEG@WaitForSingleObjectEx?$AA@ 100b098c     interop.obj
 0002:000069a4       ??_C@_0BE@CLKLPNNG@WaitForSingleObject?$AA@ 100b09a4     interop.obj
 0002:000069b8       ??_C@_0P@DLHPPCNH@CreateEventExW?$AA@ 100b09b8     interop.obj
 0002:000069c8       ??_C@_09NOIIIIGM@WriteFile?$AA@ 100b09c8     interop.obj
 0002:000069d4       ??_C@_0BE@LJADKLBD@WideCharToMultiByte?$AA@ 100b09d4     interop.obj
 0002:000069e8       ??_C@_0BA@GLKNLELN@UnmapViewOfFile?$AA@ 100b09e8     interop.obj
 0002:000069f8       ??_C@_0N@HOKNOHPO@UnlockFileEx?$AA@ 100b09f8     interop.obj
 0002:00006a08       ??_C@_0L@PBJENKDG@UnlockFile?$AA@ 100b0a08     interop.obj
 0002:00006a14       ??_C@_0BF@HBHGIPOG@SystemTimeToFileTime?$AA@ 100b0a14     interop.obj
 0002:00006a2c       ??_C@_05PFDOMJEF@Sleep?$AA@ 100b0a2c     interop.obj
 0002:00006a34       ??_C@_0P@HKHKGCLN@SetFilePointer?$AA@ 100b0a34     interop.obj
 0002:00006a44       ??_C@_0N@KGGGLBCJ@SetEndOfFile?$AA@ 100b0a44     interop.obj
 0002:00006a54       ??_C@_08KLCHJOKF@ReadFile?$AA@ 100b0a54     interop.obj
 0002:00006a60       ??_C@_0BI@LFICGGHO@QueryPerformanceCounter?$AA@ 100b0a60     interop.obj
 0002:00006a78       ??_C@_0BE@HCIKGJGE@MultiByteToWideChar?$AA@ 100b0a78     interop.obj
 0002:00006a8c       ??_C@_0O@IGIELGBD@MapViewOfFile?$AA@ 100b0a8c     interop.obj
 0002:00006a9c       ??_C@_0L@EJAEKEDD@LockFileEx?$AA@ 100b0a9c     interop.obj
 0002:00006aa8       ??_C@_08DICMLIHC@LockFile?$AA@ 100b0aa8     interop.obj
 0002:00006ab4       ??_C@_09FHKJECCN@LocalFree?$AA@ 100b0ab4     interop.obj
 0002:00006ac0       ??_C@_0N@KCFDJLIF@LoadLibraryW?$AA@ 100b0ac0     interop.obj
 0002:00006ad0       ??_C@_0N@LOMLCOFC@LoadLibraryA?$AA@ 100b0ad0     interop.obj
 0002:00006ae0       ??_C@_0N@BKFJNCJM@HeapValidate?$AA@ 100b0ae0     interop.obj
 0002:00006af0       ??_C@_08LKCFNBPH@HeapSize?$AA@ 100b0af0     interop.obj
 0002:00006afc       ??_C@_0M@HHKAEGMB@HeapReAlloc?$AA@ 100b0afc     interop.obj
 0002:00006b08       ??_C@_08ICEHPNNG@HeapFree?$AA@ 100b0b08     interop.obj
 0002:00006b14       ??_C@_0M@NELNNOPP@HeapDestroy?$AA@ 100b0b14     interop.obj
 0002:00006b20       ??_C@_0L@ICEGIJOB@HeapCreate?$AA@ 100b0b20     interop.obj
 0002:00006b2c       ??_C@_09JDKINLHP@HeapAlloc?$AA@ 100b0b2c     interop.obj
 0002:00006b38       ??_C@_0O@LLCLDPIK@GetVersionExA?$AA@ 100b0b38     interop.obj
 0002:00006b48       ??_C@_0N@JOMACIEF@GetTickCount?$AA@ 100b0b48     interop.obj
 0002:00006b58       ??_C@_0N@DAENKDLF@GetTempPathW?$AA@ 100b0b58     interop.obj
 0002:00006b68       ??_C@_0N@CMNFBGGC@GetTempPathA?$AA@ 100b0b68     interop.obj
 0002:00006b78       ??_C@_0BI@ENMDHCMK@GetSystemTimeAsFileTime?$AA@ 100b0b78     interop.obj
 0002:00006b90       ??_C@_0O@IKEIBEBH@GetSystemTime?$AA@ 100b0b90     interop.obj
 0002:00006ba0       ??_C@_0O@HJFFHIPG@GetSystemInfo?$AA@ 100b0ba0     interop.obj
 0002:00006bb0       ??_C@_0BA@EJGIKKLP@GetProcAddressA?$AA@ 100b0bb0     interop.obj
 0002:00006bc0       ??_C@_0N@HICKNDGL@GetLastError?$AA@ 100b0bc0     interop.obj
 0002:00006bd0       ??_C@_0BB@GMCPPICF@GetFullPathNameW?$AA@ 100b0bd0     interop.obj
 0002:00006be4       ??_C@_0BB@HALHENPC@GetFullPathNameA?$AA@ 100b0be4     interop.obj
 0002:00006bf8       ??_C@_0M@BAICHOOE@GetFileSize?$AA@ 100b0bf8     interop.obj
 0002:00006c04       ??_C@_0BF@JODNCFOA@GetFileAttributesExW?$AA@ 100b0c04     interop.obj
 0002:00006c1c       ??_C@_0BD@CFFEJJPG@GetFileAttributesW?$AA@ 100b0c1c     interop.obj
 0002:00006c30       ??_C@_0BD@DJMMCMCB@GetFileAttributesA?$AA@ 100b0c30     interop.obj
 0002:00006c44       ??_C@_0BC@BOCPGOAP@GetDiskFreeSpaceW?$AA@ 100b0c44     interop.obj
 0002:00006c58       ??_C@_0BC@CLHNLNI@GetDiskFreeSpaceA?$AA@ 100b0c58     interop.obj
 0002:00006c6c       ??_C@_0BE@BEODBHKD@GetCurrentProcessId?$AA@ 100b0c6c     interop.obj
 0002:00006c80       ??_C@_0M@FACAOGOA@FreeLibrary?$AA@ 100b0c80     interop.obj
 0002:00006c8c       ??_C@_0P@EGGMAMDC@FormatMessageW?$AA@ 100b0c8c     interop.obj
 0002:00006c9c       ??_C@_0P@FKPELJOF@FormatMessageA?$AA@ 100b0c9c     interop.obj
 0002:00006cac       ??_C@_0BB@MOGECGEP@FlushFileBuffers?$AA@ 100b0cac     interop.obj
 0002:00006cc0       ??_C@_0BF@KPJNHALE@FileTimeToSystemTime?$AA@ 100b0cc0     interop.obj
 0002:00006cd8       ??_C@_0BI@EKFDIGHI@FileTimeToLocalFileTime?$AA@ 100b0cd8     interop.obj
 0002:00006cf0       ??_C@_0M@DNECCFPG@DeleteFileW?$AA@ 100b0cf0     interop.obj
 0002:00006cfc       ??_C@_0M@CBNKJACB@DeleteFileA?$AA@ 100b0cfc     interop.obj
 0002:00006d08       ??_C@_0N@MDNOAJMP@CreateMutexW?$AA@ 100b0d08     interop.obj
 0002:00006d18       ??_C@_0BD@HFNFJDEE@CreateFileMappingW?$AA@ 100b0d18     interop.obj
 0002:00006d2c       ??_C@_0BD@GJENCGJD@CreateFileMappingA?$AA@ 100b0d2c     interop.obj
 0002:00006d40       ??_C@_0M@GPOOGHPH@CreateFileW?$AA@ 100b0d40     interop.obj
 0002:00006d4c       ??_C@_0M@HDHGNCCA@CreateFileA?$AA@ 100b0d4c     interop.obj
 0002:00006d58       ??_C@_0M@JHJNLFGC@CloseHandle?$AA@ 100b0d58     interop.obj
 0002:00006d64       ??_C@_0L@JBOFCNPB@CharUpperW?$AA@ 100b0d64     interop.obj
 0002:00006d70       ??_C@_0L@CDADJILC@CharLowerW?$AA@ 100b0d70     interop.obj
 0002:00006d7c       ??_C@_0BA@FHFNEAED@AreFileApisANSI?$AA@ 100b0d7c     interop.obj
 0002:00006d8c       ??_C@_07EMCFMDDO@Explain?$AA@ 100b0d8c     interop.obj
 0002:00006d94       ??_C@_04NBOPPMHE@Noop?$AA@ 100b0d94     interop.obj
 0002:00006d9c       ??_C@_05ILLBNNOP@Trace?$AA@ 100b0d9c     interop.obj
 0002:00006da4       ??_C@_08PCPIJAPH@MaxPgcnt?$AA@ 100b0da4     interop.obj
 0002:00006db0       ??_C@_09CNCANJNI@Pagecount?$AA@ 100b0db0     interop.obj
 0002:00006dbc       ??_C@_06ICNNEOIM@ToReal?$AA@ 100b0dbc     interop.obj
 0002:00006dc4       ??_C@_05CNEGLJEO@ToInt?$AA@ 100b0dc4     interop.obj
 0002:00006dcc       ??_C@_09IAEPJEPI@ToNumeric?$AA@ 100b0dcc     interop.obj
 0002:00006dd8       ??_C@_06LCIJGAA@ToBlob?$AA@ 100b0dd8     interop.obj
 0002:00006de0       ??_C@_06JMHBLLIK@ToText?$AA@ 100b0de0     interop.obj
 0002:00006de8       ??_C@_07NHABAPID@VUpdate?$AA@ 100b0de8     interop.obj
 0002:00006df0       ??_C@_07BIPKCCHL@VRename?$AA@ 100b0df0     interop.obj
 0002:00006df8       ??_C@_05GOGANBLF@VNext?$AA@ 100b0df8     interop.obj
 0002:00006e00       ??_C@_07DOIHNMAE@VColumn?$AA@ 100b0e00     interop.obj
 0002:00006e08       ??_C@_07OKDOHLDO@VFilter?$AA@ 100b0e08     interop.obj
 0002:00006e10       ??_C@_05JABEJFFA@VOpen?$AA@ 100b0e10     interop.obj
 0002:00006e18       ??_C@_08JBEDGDCN@VDestroy?$AA@ 100b0e18     interop.obj
 0002:00006e24       ??_C@_07KDKHCOMM@VCreate?$AA@ 100b0e24     interop.obj
 0002:00006e2c       ??_C@_06CLFNNGGK@VBegin?$AA@ 100b0e2c     interop.obj
 0002:00006e34       ??_C@_09FDKNKOOK@TableLock?$AA@ 100b0e34     interop.obj
 0002:00006e40       ??_C@_04PHKLBGME@Real?$AA@ 100b0e40     interop.obj
 0002:00006e48       ??_C@_06GDNCIOGJ@Expire?$AA@ 100b0e48     interop.obj
 0002:00006e50       ??_C@_0L@POHPJECG@IncrVacuum?$AA@ 100b0e50     interop.obj
 0002:00006e5c       ??_C@_06OBCEMCJB@Vacuum?$AA@ 100b0e5c     interop.obj
 0002:00006e64       ??_C@_0M@FAIDBMDK@JournalMode?$AA@ 100b0e64     interop.obj
 0002:00006e70       ??_C@_0L@IHLHABNJ@Checkpoint?$AA@ 100b0e70     interop.obj
 0002:00006e7c       ??_C@_08FCKHNOBN@AggFinal?$AA@ 100b0e7c     interop.obj
 0002:00006e88       ??_C@_07NOMHFNIB@AggStep?$AA@ 100b0e88     interop.obj
 0002:00006e90       ??_C@_06KGOGOHGB@IfZero?$AA@ 100b0e90     interop.obj
 0002:00006e98       ??_C@_05GPHDFMLA@IfNeg?$AA@ 100b0e98     interop.obj
 0002:00006ea0       ??_C@_05PMIMCOJP@IfPos?$AA@ 100b0ea0     interop.obj
 0002:00006ea8       ??_C@_06LJFJMLCE@MemMax?$AA@ 100b0ea8     interop.obj
 0002:00006eb0       ??_C@_08PNIKOKNB@FkIfZero?$AA@ 100b0eb0     interop.obj
 0002:00006ebc       ??_C@_09EBKOHGDP@FkCounter?$AA@ 100b0ebc     interop.obj
 0002:00006ec8       ??_C@_05LOJBNELM@Param?$AA@ 100b0ec8     interop.obj
 0002:00006ed0       ??_C@_07DOMMNIGK@Program?$AA@ 100b0ed0     interop.obj
 0002:00006ed8       ??_C@_0L@EOJPAHGG@RowSetTest?$AA@ 100b0ed8     interop.obj
 0002:00006ee4       ??_C@_0L@JELPJHIJ@RowSetRead?$AA@ 100b0ee4     interop.obj
 0002:00006ef0       ??_C@_09KPGKMOML@RowSetAdd?$AA@ 100b0ef0     interop.obj
 0002:00006efc       ??_C@_0M@KCIGPGBI@IntegrityCk?$AA@ 100b0efc     interop.obj
 0002:00006f08       ??_C@_0M@JKNINGPB@DropTrigger?$AA@ 100b0f08     interop.obj
 0002:00006f14       ??_C@_09KDDJLBNF@DropIndex?$AA@ 100b0f14     interop.obj
 0002:00006f20       ??_C@_09ELPHDPAO@DropTable?$AA@ 100b0f20     interop.obj
 0002:00006f2c       ??_C@_0N@FEAPPFEN@LoadAnalysis?$AA@ 100b0f2c     interop.obj
 0002:00006f3c       ??_C@_0M@IPJMJJPI@ParseSchema?$AA@ 100b0f3c     interop.obj
 0002:00006f48       ??_C@_0M@BDPOJHGL@CreateTable?$AA@ 100b0f48     interop.obj
 0002:00006f54       ??_C@_0M@PLDABJLA@CreateIndex?$AA@ 100b0f54     interop.obj
 0002:00006f60       ??_C@_05MDNHABIA@Clear?$AA@ 100b0f60     interop.obj
 0002:00006f68       ??_C@_07BDCAJABG@Destroy?$AA@ 100b0f68     interop.obj
 0002:00006f70       ??_C@_05FMIIHMAD@IdxGE?$AA@ 100b0f70     interop.obj
 0002:00006f78       ??_C@_05DAELAPC@IdxLT?$AA@ 100b0f78     interop.obj
 0002:00006f80       ??_C@_08KLKOBEJ@IdxRowid?$AA@ 100b0f80     interop.obj
 0002:00006f8c       ??_C@_09PDNFOMPO@IdxDelete?$AA@ 100b0f8c     interop.obj
 0002:00006f98       ??_C@_09ENCBCCAM@IdxInsert?$AA@ 100b0f98     interop.obj
 0002:00006fa4       ??_C@_0N@PCKBEOAP@SorterInsert?$AA@ 100b0fa4     interop.obj
 0002:00006fb4       ??_C@_04MDFHGMOB@Next?$AA@ 100b0fb4     interop.obj
 0002:00006fbc       ??_C@_07KGFHIBD@String8?$AA@ 100b0fbc     interop.obj
 0002:00006fc4       ??_C@_06OBLNEDKN@BitNot?$AA@ 100b0fc4     interop.obj
 0002:00006fcc       ??_C@_04PHIBHIIF@Prev?$AA@ 100b0fcc     interop.obj
 0002:00006fd4       ??_C@_06ODAFHOMO@Concat?$AA@ 100b0fd4     interop.obj
 0002:00006fdc       ??_C@_09DPOHBCHJ@Remainder?$AA@ 100b0fdc     interop.obj
 0002:00006fe8       ??_C@_06JKMEHOIB@Divide?$AA@ 100b0fe8     interop.obj
 0002:00006ff0       ??_C@_08EOBDLMOI@Multiply?$AA@ 100b0ff0     interop.obj
 0002:00006ffc       ??_C@_08DLEJPBEP@Subtract?$AA@ 100b0ffc     interop.obj
 0002:00007008       ??_C@_03LDFMNCOE@Add?$AA@  100b1008     interop.obj
 0002:0000700c       ??_C@_0L@DHHFIOFJ@ShiftRight?$AA@ 100b100c     interop.obj
 0002:00007018       ??_C@_09IIGOLNPP@ShiftLeft?$AA@ 100b1018     interop.obj
 0002:00007024       ??_C@_05BKBNAGEF@BitOr?$AA@ 100b1024     interop.obj
 0002:0000702c       ??_C@_06PCNOCLJN@BitAnd?$AA@ 100b102c     interop.obj
 0002:00007034       ??_C@_0L@MGGJHFHJ@SorterNext?$AA@ 100b1034     interop.obj
 0002:00007040       ??_C@_02GNOBCCEK@Ge?$AA@   100b1040     interop.obj
 0002:00007044       ??_C@_02DCGNOOLL@Lt?$AA@   100b1044     interop.obj
 0002:00007048       ??_C@_02GBLEMNKL@Le?$AA@   100b1048     interop.obj
 0002:0000704c       ??_C@_02DODIABFK@Gt?$AA@   100b104c     interop.obj
 0002:00007050       ??_C@_02EAMLCBHB@Eq?$AA@   100b1050     interop.obj
 0002:00007054       ??_C@_02GCDABJMF@Ne?$AA@   100b1054     interop.obj
 0002:00007058       ??_C@_07HICACDPL@NotNull?$AA@ 100b1058     interop.obj
 0002:00007060       ??_C@_06NBBMPCN@IsNull?$AA@ 100b1060     interop.obj
 0002:00007068       ??_C@_06MAOEIKCJ@Rewind?$AA@ 100b1068     interop.obj
 0002:00007070       ??_C@_04DJANFKGA@Sort?$AA@ 100b1070     interop.obj
 0002:00007078       ??_C@_0L@DMDDEDPI@SorterSort?$AA@ 100b1078     interop.obj
 0002:00007084       ??_C@_03LOMLFHDC@And?$AA@  100b1084     interop.obj
 0002:00007088       ??_C@_02GGHBPHGE@Or?$AA@   100b1088     interop.obj
 0002:0000708c       ??_C@_04DKKAEHDH@Last?$AA@ 100b108c     interop.obj
 0002:00007094       ??_C@_07HJJPPOKN@NullRow?$AA@ 100b1094     interop.obj
 0002:0000709c       ??_C@_05KEGGNBBF@Rowid?$AA@ 100b109c     interop.obj
 0002:000070a4       ??_C@_07OHPACBNN@RowData?$AA@ 100b10a4     interop.obj
 0002:000070ac       ??_C@_06JIHNENAH@RowKey?$AA@ 100b10ac     interop.obj
 0002:000070b4       ??_C@_0L@DNBEOFPP@SorterData?$AA@ 100b10b4     interop.obj
 0002:000070c0       ??_C@_0O@GIINMLJL@SorterCompare?$AA@ 100b10c0     interop.obj
 0002:000070d0       ??_C@_0L@NDDNCBN@ResetCount?$AA@ 100b10d0     interop.obj
 0002:000070dc       ??_C@_06JBKGCNBB@Delete?$AA@ 100b10dc     interop.obj
 0002:000070e4       ??_C@_09LEJELDEO@InsertInt?$AA@ 100b10e4     interop.obj
 0002:000070f0       ??_C@_06CPFCODOD@Insert?$AA@ 100b10f0     interop.obj
 0002:000070f8       ??_C@_08FEDJPMPH@NewRowid?$AA@ 100b10f8     interop.obj
 0002:00007104       ??_C@_08DOCONEG@Sequence?$AA@ 100b1104     interop.obj
 0002:00007110       ??_C@_09HMMGFEAA@NotExists?$AA@ 100b1110     interop.obj
 0002:0000711c       ??_C@_08HBKIHNI@IsUnique?$AA@ 100b111c     interop.obj
 0002:00007128       ??_C@_05JDGHEPJG@Found?$AA@ 100b1128     interop.obj
 0002:00007130       ??_C@_08MDBAGECB@NotFound?$AA@ 100b1130     interop.obj
 0002:0000713c       ??_C@_04ICIDABGP@Seek?$AA@ 100b113c     interop.obj
 0002:00007144       ??_C@_06KLOEOCMK@SeekGt?$AA@ 100b1144     interop.obj
 0002:0000714c       ??_C@_06PIDNMBNK@SeekGe?$AA@ 100b114c     interop.obj
 0002:00007154       ??_C@_06PEGICODL@SeekLe?$AA@ 100b1154     interop.obj
 0002:0000715c       ??_C@_06KHLBANCL@SeekLt?$AA@ 100b115c     interop.obj
 0002:00007164       ??_C@_05LGELBCGM@Close?$AA@ 100b1164     interop.obj
 0002:0000716c       ??_C@_0L@PKPPHKBP@OpenPseudo?$AA@ 100b116c     interop.obj
 0002:00007178       ??_C@_0L@DIBNDBJM@SorterOpen?$AA@ 100b1178     interop.obj
 0002:00007184       ??_C@_0O@MHKNMBPC@OpenEphemeral?$AA@ 100b1184     interop.obj
 0002:00007194       ??_C@_0O@LLCBFLCA@OpenAutoindex?$AA@ 100b1194     interop.obj
 0002:000071a4       ??_C@_09FPCAPNBB@OpenWrite?$AA@ 100b11a4     interop.obj
 0002:000071b0       ??_C@_08FJFCCPFB@OpenRead?$AA@ 100b11b0     interop.obj
 0002:000071bc       ??_C@_0N@NKEHNBGM@VerifyCookie?$AA@ 100b11bc     interop.obj
 0002:000071cc       ??_C@_09FEDANMPL@SetCookie?$AA@ 100b11cc     interop.obj
 0002:000071d8       ??_C@_0L@LIFFPDNM@ReadCookie?$AA@ 100b11d8     interop.obj
 0002:000071e4       ??_C@_0M@MEGKBOMN@Transaction?$AA@ 100b11e4     interop.obj
 0002:000071f0       ??_C@_0L@BPKAOEDK@AutoCommit?$AA@ 100b11f0     interop.obj
 0002:000071fc       ??_C@_09OJILMLHM@Savepoint?$AA@ 100b11fc     interop.obj
 0002:00007208       ??_C@_05IJGIMMHE@Count?$AA@ 100b1208     interop.obj
 0002:00007210       ??_C@_0L@PGPMFKDB@MakeRecord?$AA@ 100b1210     interop.obj
 0002:0000721c       ??_C@_08MMCPABPC@Affinity?$AA@ 100b121c     interop.obj
 0002:00007228       ??_C@_06FFIACGFC@Column?$AA@ 100b1228     interop.obj
 0002:00007230       ??_C@_05DALJIPE@IfNot?$AA@ 100b1230     interop.obj
 0002:00007238       ??_C@_02EMFCFMID@If?$AA@   100b1238     interop.obj
 0002:0000723c       ??_C@_04GKJMKNNB@Once?$AA@ 100b123c     interop.obj
 0002:00007244       ??_C@_04BIEPDJCB@Jump?$AA@ 100b1244     interop.obj
 0002:0000724c       ??_C@_07MBOMJGGF@Compare?$AA@ 100b124c     interop.obj
 0002:00007254       ??_C@_0M@LPEOJDB@Permutation?$AA@ 100b1254     interop.obj
 0002:00007260       ??_C@_0N@KGPEGHPK@RealAffinity?$AA@ 100b1260     interop.obj
 0002:00007270       ??_C@_09LLJOBHN@MustBeInt?$AA@ 100b1270     interop.obj
 0002:0000727c       ??_C@_06JHIJIKD@AddImm?$AA@ 100b127c     interop.obj
 0002:00007284       ??_C@_03KNKIDPAC@Not?$AA@  100b1284     interop.obj
 0002:00007288       ??_C@_08PHKOHANG@Function?$AA@ 100b1288     interop.obj
 0002:00007294       ??_C@_07MCEFGNMJ@CollSeq?$AA@ 100b1294     interop.obj
 0002:0000729c       ??_C@_09BKHKEBMD@ResultRow?$AA@ 100b129c     interop.obj
 0002:000072a8       ??_C@_05BCDNELCG@SCopy?$AA@ 100b12a8     interop.obj
 0002:000072b0       ??_C@_04OPMHGHMB@Copy?$AA@ 100b12b0     interop.obj
 0002:000072b8       ??_C@_04LCANPIEP@Move?$AA@ 100b12b8     interop.obj
 0002:000072c0       ??_C@_08DMMJCAML@Variable?$AA@ 100b12c0     interop.obj
 0002:000072cc       ??_C@_04HOFOMOEI@Blob?$AA@ 100b12cc     interop.obj
 0002:000072d4       ??_C@_04KHKKIIL@Null?$AA@  100b12d4     interop.obj
 0002:000072dc       ??_C@_06ENNEIMBA@String?$AA@ 100b12dc     interop.obj
 0002:000072e4       ??_C@_05DPPJJBMK@Int64?$AA@ 100b12e4     interop.obj
 0002:000072ec       ??_C@_07EDADKEAH@Integer?$AA@ 100b12ec     interop.obj
 0002:000072f4       ??_C@_04NIFKAFLK@Halt?$AA@ 100b12f4     interop.obj
 0002:000072fc       ??_C@_0L@GIACEIKJ@HaltIfNull?$AA@ 100b12fc     interop.obj
 0002:00007308       ??_C@_05LNDKIJIJ@Yield?$AA@ 100b1308     interop.obj
 0002:00007310       ??_C@_06HCFIKKEA@Return?$AA@ 100b1310     interop.obj
 0002:00007318       ??_C@_05DLHJCIPI@Gosub?$AA@ 100b1318     interop.obj
 0002:00007320       ??_C@_04BNGNMAK@Goto?$AA@  100b1320     interop.obj
 0002:00007328       ??_C@_01OGPIMHDM@?$DP?$AA@ 100b1328     interop.obj
 0002:0000732c       ??_C@_0N@DJJJGBGD@current_date?$AA@ 100b132c     interop.obj
 0002:0000733c       ??_C@_0BC@DDICBCEN@current_timestamp?$AA@ 100b133c     interop.obj
 0002:00007350       ??_C@_0N@IPDKEGPB@current_time?$AA@ 100b1350     interop.obj
 0002:00007360       ??_C@_08EPGBJPHJ@strftime?$AA@ 100b1360     interop.obj
 0002:0000736c       ??_C@_08FGNPMIBK@datetime?$AA@ 100b136c     interop.obj
 0002:00007378       ??_C@_04CLCEDBPF@time?$AA@ 100b1378     interop.obj
 0002:00007380       ??_C@_04JNIHBGGH@date?$AA@ 100b1380     interop.obj
 0002:00007388       ??_C@_09BPOICPEH@julianday?$AA@ 100b1388     interop.obj
 0002:00007394       ??_C@_0N@HEAGAILC@THREADSAFE?$DN1?$AA@ 100b1394     interop.obj
 0002:000073a4       ??_C@_07FIPCPJFC@SOUNDEX?$AA@ 100b13a4     interop.obj
 0002:000073ac       ??_C@_09LMNJIBDP@HAS_CODEC?$AA@ 100b13ac     interop.obj
 0002:000073b8       ??_C@_0N@HDELIEAL@ENABLE_STAT3?$AA@ 100b13b8     interop.obj
 0002:000073c8       ??_C@_0N@JODKLIOI@ENABLE_RTREE?$AA@ 100b13c8     interop.obj
 0002:000073d8       ??_C@_0BG@DOKPBAOP@ENABLE_LOAD_EXTENSION?$AA@ 100b13d8     interop.obj
 0002:000073f0       ??_C@_0M@LFFMHLBN@ENABLE_FTS3?$AA@ 100b13f0     interop.obj
 0002:000073fc       ??_C@_0BH@CMJLKIMD@ENABLE_COLUMN_METADATA?$AA@ 100b13fc     interop.obj
 0002:00007414       ??_C@_01HIHLOKLC@1?$AA@    100b1414     interop.obj
 0002:00007418       ??_C@_01GBGANLPD@0?$AA@    100b1418     interop.obj
 0002:0000741c       ??_C@_07OGLCFANK@SQLITE_?$AA@ 100b141c     interop.obj
 0002:00007424       ??_C@_03CGLHMDPP@now?$AA@  100b1424     interop.obj
 0002:00007428       ??_C@_0BH@HEILFFIJ@local?5time?5unavailable?$AA@ 100b1428     interop.obj
 0002:00007440       ??_C@_09EKBOCLDN@localtime?$AA@ 100b1440     interop.obj
 0002:0000744c       ??_C@_09KNIMKLBK@unixepoch?$AA@ 100b144c     interop.obj
 0002:00007458       ??_C@_03JPHCIIKF@utc?$AA@  100b1458     interop.obj
 0002:0000745c       ??_C@_08IPAOEBNP@weekday?5?$AA@ 100b145c     interop.obj
 0002:00007468       ??_C@_09CABLEOFK@start?5of?5?$AA@ 100b1468     interop.obj
 0002:00007474       ??_C@_05MEBAADFH@month?$AA@ 100b1474     interop.obj
 0002:0000747c       ??_C@_04JFPLDHAO@year?$AA@ 100b147c     interop.obj
 0002:00007484       ??_C@_03NNBHCDBP@day?$AA@  100b1484     interop.obj
 0002:00007488       ??_C@_04LMOJGCPE@hour?$AA@ 100b1488     interop.obj
 0002:00007490       ??_C@_06JGJIJFNK@minute?$AA@ 100b1490     interop.obj
 0002:00007498       ??_C@_06BJCFNGJP@second?$AA@ 100b1498     interop.obj
 0002:000074a0       ??_C@_0BO@NGNOHJIK@?$CF04d?9?$CF02d?9?$CF02d?5?$CF02d?3?$CF02d?3?$CF02d?$AA@ 100b14a0     interop.obj
 0002:000074c0       ??_C@_0P@PLMNPDMB@?$CF02d?3?$CF02d?3?$CF02d?$AA@ 100b14c0     interop.obj
 0002:000074d0       ??_C@_0P@MCDGMPHH@?$CF04d?9?$CF02d?9?$CF02d?$AA@ 100b14d0     interop.obj
 0002:000074e0       ??_C@_04OGKJMPGK@?$CF02d?$AA@ 100b14e0     interop.obj
 0002:000074e8       ??_C@_06IAGKDDNE@?$CF06?43f?$AA@ 100b14e8     interop.obj
 0002:000074f0       ??_C@_04OHGLKFFN@?$CF03d?$AA@ 100b14f0     interop.obj
 0002:000074f8       ??_C@_05CFGAKADK@?$CF?416g?$AA@ 100b14f8     interop.obj
 0002:00007500       ??_C@_04BFAHMMK@?$CFlld?$AA@ 100b1500     interop.obj
 0002:00007508       ??_C@_04OCCELDNI@?$CF04d?$AA@ 100b1508     interop.obj
 0002:00007510       ??_C@_01FGNFDNOH@?$CF?$AA@ 100b1510     interop.obj
 0002:00007514       ??_C@_03ICJPMMHB@NaN?$AA@  100b1514     interop.obj
 0002:00007518       ??_C@_04JHHONOOL@?9Inf?$AA@ 100b1518     interop.obj
 0002:00007520       ??_C@_04BIDOCLEL@?$CLInf?$AA@ 100b1520     interop.obj
 0002:00007528       ??_C@_03EJEJBNFP@Inf?$AA@  100b1528     interop.obj
 0002:0000752c       ??_C@_00CNPNBAHC@?$AA@     100b152c     interop.obj
 0002:00007530       ??_C@_04HIBGFPH@NULL?$AA@  100b1530     interop.obj
 0002:00007538       ??_C@_06LHGEHABH@?$CINULL?$CJ?$AA@ 100b1538     interop.obj
 0002:00007540       ??_C@_01LFCBOECM@?4?$AA@   100b1540     interop.obj
 0002:00007544       ??_C@_0BD@FKIFACO@922337203685477580?$AA@ 100b1544     interop.obj
 0002:00007558       ??_C@_0CN@EOKIBNLJ@API?5call?5with?5?$CFs?5database?5connec@ 100b1558     interop.obj
 0002:00007588       ??_C@_08NFNJDBOK@unopened?$AA@ 100b1588     interop.obj
 0002:00007594       ??_C@_07MALOAKCI@invalid?$AA@ 100b1594     interop.obj
 0002:0000759c       ??_C@_0CL@BNLKJAJL@failed?5to?5HeapAlloc?5?$CFu?5bytes?5?$CI?$CFd@ 100b159c     interop.obj
 0002:000075c8       ??_C@_0CK@MKEMOJHF@failed?5to?5HeapFree?5block?5?$CFp?5?$CI?$CFd?$CJ@ 100b15c8     interop.obj
 0002:000075f4       ??_C@_0CE@OGBCNCMD@failed?5to?5?$CFs?5?$CFu?5bytes?5?$CI?$CFd?$CJ?0?5heap@ 100b15f4     interop.obj
 0002:00007618       ??_C@_0CK@NOKLGMDC@failed?5to?5HeapSize?5block?5?$CFp?5?$CI?$CFd?$CJ@ 100b1618     interop.obj
 0002:00007644       ??_C@_0DN@FJJLINBJ@failed?5to?5HeapCreate?5?$CI?$CFd?$CJ?0?5flags@ 100b1644     interop.obj
 0002:00007684       ??_C@_0CE@LPELHPP@failed?5to?5HeapDestroy?5?$CI?$CFd?$CJ?0?5heap@ 100b1684     interop.obj
 0002:000076a8       ??_C@_0BE@MJECGBL@OsError?50x?$CFlx?5?$CI?$CFlu?$CJ?$AA@ 100b16a8     interop.obj
 0002:000076bc       ??_C@_02DKCKIIND@?$CFs?$AA@ 100b16bc     interop.obj
 0002:000076c0       ??_C@_0BP@JDJJJHMH@os_win?4c?3?$CFd?3?5?$CI?$CFlu?$CJ?5?$CFs?$CI?$CFs?$CJ?5?9?5?$CFs?$AA@ 100b16c0     interop.obj
 0002:000076e0       ??_C@_0CH@IOAFGIGM@delayed?5?$CFdms?5for?5lock?1sharing?5co@ 100b16e0     interop.obj
 0002:00007708       ??_C@_0M@KEGMKFKG@seekWinFile?$AA@ 100b1708     interop.obj
 0002:00007714       ??_C@_08GBGPIFFF@winClose?$AA@ 100b1714     interop.obj
 0002:00007720       ??_C@_07BGDHELCN@winRead?$AA@ 100b1720     interop.obj
 0002:00007728       ??_C@_08GNMKFGC@winWrite?$AA@ 100b1728     interop.obj
 0002:00007734       ??_C@_0N@JHOIFHJA@winTruncate1?$AA@ 100b1734     interop.obj
 0002:00007744       ??_C@_0N@LMMFAEFD@winTruncate2?$AA@ 100b1744     interop.obj
 0002:00007754       ??_C@_07HFIFFLEA@winSync?$AA@ 100b1754     interop.obj
 0002:0000775c       ??_C@_0M@DODNMLAG@winFileSize?$AA@ 100b175c     interop.obj
 0002:00007768       ??_C@_0P@DMNKIFMO@unlockReadLock?$AA@ 100b1768     interop.obj
 0002:00007778       ??_C@_09INENJOCI@winUnlock?$AA@ 100b1778     interop.obj
 0002:00007784       ??_C@_05NMJMPJJB@win32?$AA@ 100b1784     interop.obj
 0002:0000778c       ??_C@_06KEOMCCGA@?$CFs?9shm?$AA@ 100b178c     interop.obj
 0002:00007794       ??_C@_0L@NHPDAEHO@winOpenShm?$AA@ 100b1794     interop.obj
 0002:000077a0       ??_C@_0L@JMPNPFLA@winShmMap1?$AA@ 100b17a0     interop.obj
 0002:000077ac       ??_C@_0L@LHNAKGHD@winShmMap2?$AA@ 100b17ac     interop.obj
 0002:000077b8       ??_C@_0L@KOMLJHDC@winShmMap3?$AA@ 100b17b8     interop.obj
 0002:000077c4       ??_C@_09OMGGIFM@winUnmap1?$AA@ 100b17c4     interop.obj
 0002:000077d0       ??_C@_09CFOLDLJP@winUnmap2?$AA@ 100b17d0     interop.obj
 0002:000077dc       ??_C@_0L@GHFCHGIB@winMapfile?$AA@ 100b17dc     interop.obj
 0002:000077e8       ??_C@_07NBNPOOME@etilqs_?$AA@ 100b17e8     interop.obj
 0002:000077f0       ??_C@_0L@KBKJCPCN@?$CFs?2etilqs_?$AA@ 100b17f0     interop.obj
 0002:000077fc       ??_C@_07BEGGPPOF@winOpen?$AA@ 100b17fc     interop.obj
 0002:00007804       ??_C@_04JKHAIEHD@psow?$AA@ 100b1804     interop.obj
 0002:0000780c       ??_C@_09MOHEIBIO@winDelete?$AA@ 100b180c     interop.obj
 0002:00007818       ??_C@_09NBJCHJLH@winAccess?$AA@ 100b1818     interop.obj
 0002:00007824       ??_C@_05BMGBEOOC@?$CFs?2?$CFs?$AA@ 100b1824     interop.obj
 0002:0000782c       ??_C@_0BC@INDFPMAN@GetFullPathNameW1?$AA@ 100b182c     interop.obj
 0002:00007840       ??_C@_0BC@KGBIKPMO@GetFullPathNameW2?$AA@ 100b1840     interop.obj
 0002:00007854       ??_C@_0BC@JFJOCDMP@GetFullPathNameA1?$AA@ 100b1854     interop.obj
 0002:00007868       ??_C@_0BC@LOLDHAAM@GetFullPathNameA2?$AA@ 100b1868     interop.obj
 0002:0000787c       ??_C@_0BL@FJPGAHP@recovered?5?$CFd?5pages?5from?5?$CFs?$AA@ 100b187c     interop.obj
 0002:00007898       ??_C@_09HKLPJOIM@?9journal?$AA?$AA@ 100b1898     interop.obj
 0002:000078a4       ??_C@_05HMKKNGEJ@?9wal?$AA?$AA@ 100b18a4     interop.obj
 0002:000078ac       ??_C@_0CF@EDMDCOFB@recovered?5?$CFd?5frames?5from?5WAL?5fil@ 100b18ac     interop.obj
 0002:000078d4       ??_C@_0BK@NCCCKLLJ@cannot?5limit?5WAL?5size?3?5?$CFs?$AA@ 100b18d4     interop.obj
 0002:000078f0       ??_C@_08CADOGOJM@?3memory?3?$AA@ 100b18f0     interop.obj
 0002:000078fc       ??_C@_01EEMJAFIK@?6?$AA@   100b18fc     interop.obj
 0002:00007900       ??_C@_0BH@LLKFEBHC@invalid?5page?5number?5?$CFd?$AA@ 100b1900     interop.obj
 0002:00007918       ??_C@_0BJ@HHKCLCDH@2nd?5reference?5to?5page?5?$CFd?$AA@ 100b1918     interop.obj
 0002:00007934       ??_C@_0BN@NJCBBLIO@Failed?5to?5read?5ptrmap?5key?$DN?$CFd?$AA@ 100b1934     interop.obj
 0002:00007954       ??_C@_0DG@EAEHHDPC@Bad?5ptr?5map?5entry?5key?$DN?$CFd?5expecte@ 100b1954     interop.obj
 0002:0000798c       ??_C@_0DJ@PBFEOOMP@?$CFd?5of?5?$CFd?5pages?5missing?5from?5over@ 100b198c     interop.obj
 0002:000079c8       ??_C@_0BG@GMIBDIEE@failed?5to?5get?5page?5?$CFd?$AA@ 100b19c8     interop.obj
 0002:000079e0       ??_C@_0CH@LNHECGJJ@freelist?5leaf?5count?5too?5big?5on?5p@ 100b19e0     interop.obj
 0002:00007a08       ??_C@_09OLGIMPDE@Page?5?$CFd?3?5?$AA@ 100b1a08     interop.obj
 0002:00007a14       ??_C@_0CG@ILLDAEJM@unable?5to?5get?5the?5page?4?5error?5co@ 100b1a14     interop.obj
 0002:00007a3c       ??_C@_0CG@FFKEALPN@btreeInitPage?$CI?$CJ?5returns?5error?5co@ 100b1a3c     interop.obj
 0002:00007a64       ??_C@_0BK@DEBKKJM@On?5tree?5page?5?$CFd?5cell?5?$CFd?3?5?$AA@ 100b1a64     interop.obj
 0002:00007a80       ??_C@_0CM@NFGNKDIE@Rowid?5?$CFlld?5out?5of?5order?5?$CIpreviou@ 100b1a80     interop.obj
 0002:00007aac       ??_C@_0BJ@FLOCKNJL@Child?5page?5depth?5differs?$AA@ 100b1aac     interop.obj
 0002:00007ac8       ??_C@_0BM@FMPLCKPB@On?5page?5?$CFd?5at?5right?5child?3?5?$AA@ 100b1ac8     interop.obj
 0002:00007ae4       ??_C@_0DN@FNPJJAIO@Rowid?5?$CFlld?5out?5of?5order?5?$CImax?5lar@ 100b1ae4     interop.obj
 0002:00007b24       ??_C@_0DL@JMELIBGM@Rowid?5?$CFlld?5out?5of?5order?5?$CImin?5les@ 100b1b24     interop.obj
 0002:00007b60       ??_C@_0DN@BNLGOIPI@Rowid?5?$CFlld?5out?5of?5order?5?$CImax?5lar@ 100b1b60     interop.obj
 0002:00007ba0       ??_C@_0DL@NMAEPJBK@Rowid?5?$CFlld?5out?5of?5order?5?$CImin?5les@ 100b1ba0     interop.obj
 0002:00007bdc       ??_C@_0CK@JLHLDHFB@Corruption?5detected?5in?5cell?5?$CFd?5o@ 100b1bdc     interop.obj
 0002:00007c08       ??_C@_0CF@DKGAOHID@Multiple?5uses?5for?5byte?5?$CFd?5of?5pag@ 100b1c08     interop.obj
 0002:00007c30       ??_C@_0DE@NONOJPEC@Fragmentation?5of?5?$CFd?5bytes?5report@ 100b1c30     interop.obj
 0002:00007c64       ??_C@_0BA@EAICBBKE@Main?5freelist?3?5?$AA@ 100b1c64     interop.obj
 0002:00007c74       ??_C@_0BF@CFAFGJN@List?5of?5tree?5roots?3?5?$AA@ 100b1c74     interop.obj
 0002:00007c8c       ??_C@_0BG@NJBAMKDO@Page?5?$CFd?5is?5never?5used?$AA@ 100b1c8c     interop.obj
 0002:00007ca4       ??_C@_0CC@IBCKHFBM@Pointer?5map?5page?5?$CFd?5is?5reference@ 100b1ca4     interop.obj
 0002:00007cc8       ??_C@_0DP@PJBOOLEO@Outstanding?5page?5count?5goes?5from@ 100b1cc8     interop.obj
 0002:00007d08       ??_C@_0O@BNNCBLEN@out?5of?5memory?$AA@ 100b1d08     interop.obj
 0002:00007d18       ??_C@_0BE@OKPJBBEB@unknown?5database?5?$CFs?$AA@ 100b1d18     interop.obj
 0002:00007d2c       ??_C@_0CI@IHDDPHMP@source?5and?5destination?5must?5be?5d@ 100b1d2c     interop.obj
 0002:00007d54       ??_C@_06NJMDEJD@?$CF?$CB?415g?$AA@ 100b1d54     interop.obj
 0002:00007d5c       ??_C@_01JOAMLHOP@?9?$AA@   100b1d5c     interop.obj
 0002:00007d60       ??_C@_04HDOCAJNK@?$CFs?$CFs?$AA@ 100b1d60     interop.obj
 0002:00007d68       ??_C@_0L@HDAMIFP@keyinfo?$CI?$CFd?$AA@ 100b1d68     interop.obj
 0002:00007d74       ??_C@_03ILAMHENH@nil?$AA@  100b1d74     interop.obj
 0002:00007d78       ??_C@_0P@BMGKNHBK@collseq?$CI?$CF?420s?$CJ?$AA@ 100b1d78     interop.obj
 0002:00007d88       ??_C@_06BPGFIOAL@?$CFs?$CI?$CFd?$CJ?$AA@ 100b1d88     interop.obj
 0002:00007d90       ??_C@_02DPKJAMEF@?$CFd?$AA@ 100b1d90     interop.obj
 0002:00007d94       ??_C@_06OLGPAEJH@?$CIblob?$CJ?$AA@ 100b1d94     interop.obj
 0002:00007d9c       ??_C@_0L@IIBEKKAO@vtab?3?$CFp?3?$CFp?$AA@ 100b1d9c     interop.obj
 0002:00007da8       ??_C@_08CBEPOPA@intarray?$AA@ 100b1da8     interop.obj
 0002:00007db4       ??_C@_07MHLKLKDM@program?$AA@ 100b1db4     interop.obj
 0002:00007dbc       ??_C@_04LABILCJL@?$CF?42x?$AA@ 100b1dbc     interop.obj
 0002:00007dc4       ??_C@_0BA@FKMAFLJK@?$CFs?9mjXXXXXX9XXz?$AA@ 100b1dc4     interop.obj
 0002:00007dd4       ??_C@_0O@IDFCBAPA@MJ?5delete?3?5?$CFs?$AA@ 100b1dd4     interop.obj
 0002:00007de4       ??_C@_0P@EKBGDFBG@MJ?5collide?3?5?$CFs?$AA@ 100b1de4     interop.obj
 0002:00007df4       ??_C@_0N@FLHACMNC@?9mj?$CF06X9?$CF02X?$AA@ 100b1df4     interop.obj
 0002:00007e04       ??_C@_0BO@IFNOPDMA@foreign?5key?5constraint?5failed?$AA@ 100b1e04     interop.obj
 0002:00007e24       ??_C@_0CN@JCKHFJMJ@API?5called?5with?5finalized?5prepar@ 100b1e24     interop.obj
 0002:00007e54       ??_C@_0CI@DGDEMKDJ@API?5called?5with?5NULL?5prepared?5st@ 100b1e54     interop.obj
 0002:00007e7c       ??_C@_0BH@BEFJIDGM@string?5or?5blob?5too?5big?$AA@ 100b1e7c     interop.obj
 0002:00007e94       ??_C@_0DD@BOPMNMAO@unable?5to?5use?5function?5?$CFs?5in?5the@ 100b1e94     interop.obj
 0002:00007ec8       ??_C@_0CI@NKIMDBDG@bind?5on?5a?5busy?5prepared?5statemen@ 100b1ec8     interop.obj
 0002:00007ef0       ??_C@_03CJPCKGBB@?9?9?5?$AA@ 100b1ef0     interop.obj
 0002:00007ef4       ??_C@_06BGANNCL@?8?$CF?4?$CKq?8?$AA@ 100b1ef4     interop.obj
 0002:00007efc       ??_C@_0N@OGKFEFFN@zeroblob?$CI?$CFd?$CJ?$AA@ 100b1efc     interop.obj
 0002:00007f0c       ??_C@_02IAJJKNGA@x?8?$AA@  100b1f0c     interop.obj
 0002:00007f10       ??_C@_04NOJCDH@?$CF02x?$AA@ 100b1f10     interop.obj
 0002:00007f18       ??_C@_01GEODFPGF@?8?$AA@   100b1f18     interop.obj
 0002:00007f1c       ??_C@_0BI@CKCEIKAL@abort?5at?5?$CFd?5in?5?$FL?$CFs?$FN?3?5?$CFs?$AA@ 100b1f1c     interop.obj
 0002:00007f34       ??_C@_0CA@CCGMBGM@constraint?5failed?5at?5?$CFd?5in?5?$FL?$CFs?$FN?$AA@ 100b1f34     interop.obj
 0002:00007f54       ??_C@_0DD@EHMCJFDN@cannot?5open?5savepoint?5?9?5SQL?5stat@ 100b1f54     interop.obj
 0002:00007f88       ??_C@_0BG@NADCOEGF@no?5such?5savepoint?3?5?$CFs?$AA@ 100b1f88     interop.obj
 0002:00007fa0       ??_C@_0DG@JCGPCDM@cannot?5release?5savepoint?5?9?5SQL?5s@ 100b1fa0     interop.obj
 0002:00007fd8       ??_C@_0DH@EPKPHENF@cannot?5commit?5transaction?5?9?5SQL?5@ 100b1fd8     interop.obj
 0002:00008010       ??_C@_0DA@CKKHGBEC@cannot?5start?5a?5transaction?5withi@ 100b2010     interop.obj
 0002:00008040       ??_C@_0CL@DIEDEFLK@cannot?5rollback?5?9?5no?5transaction@ 100b2040     interop.obj
 0002:0000806c       ??_C@_0CJ@LALCBGBP@cannot?5commit?5?9?5no?5transaction?5i@ 100b206c     interop.obj
 0002:00008098       ??_C@_0BM@FKBOKANJ@database?5schema?5has?5changed?$AA@ 100b2098     interop.obj
 0002:000080b4       ??_C@_0BD@OLGFAFA@sqlite_temp_master?$AA@ 100b20b4     interop.obj
 0002:000080c8       ??_C@_0O@JMEKHCEB@sqlite_master?$AA@ 100b20c8     interop.obj
 0002:000080d8       ??_C@_0EA@GFNDAJBJ@SELECT?5name?0?5rootpage?0?5sql?5FROM?5@ 100b20d8     interop.obj
 0002:00008118       ??_C@_0CF@DBNDEPJP@too?5many?5levels?5of?5trigger?5recur@ 100b2118     interop.obj
 0002:00008140       ??_C@_04MHJLCKAK@into?$AA@ 100b2140     interop.obj
 0002:00008148       ??_C@_06JIMOCJPC@out?5of?$AA@ 100b2148     interop.obj
 0002:00008150       ??_C@_0DE@KIPNAMAA@cannot?5change?5?$CFs?5wal?5mode?5from?5w@ 100b2150     interop.obj
 0002:00008184       ??_C@_0BN@JOIFECGM@database?5table?5is?5locked?3?5?$CFs?$AA@ 100b2184     interop.obj
 0002:000081a4       ??_C@_0CA@JGFGBIFL@statement?5aborts?5at?5?$CFd?3?5?$FL?$CFs?$FN?5?$CFs?$AA@ 100b21a4     interop.obj
 0002:000081c4       ??_C@_04MLLLIHIP@null?$AA@ 100b21c4     interop.obj
 0002:000081cc       ??_C@_04DGGKDJMA@real?$AA@ 100b21cc     interop.obj
 0002:000081d4       ??_C@_07LKHFMGFB@integer?$AA@ 100b21d4     interop.obj
 0002:000081dc       ??_C@_0BN@OFFACDFM@cannot?5open?5value?5of?5type?5?$CFs?$AA@ 100b21dc     interop.obj
 0002:000081fc       ??_C@_0BE@PGLAJEIK@no?5such?5rowid?3?5?$CFlld?$AA@ 100b21fc     interop.obj
 0002:00008210       ??_C@_0BO@BCBGJJEM@cannot?5open?5virtual?5table?3?5?$CFs?$AA@ 100b2210     interop.obj
 0002:00008230       ??_C@_0BF@LEHNPEDD@cannot?5open?5view?3?5?$CFs?$AA@ 100b2230     interop.obj
 0002:00008248       ??_C@_0BF@IFOHJMAC@no?5such?5column?3?5?$CC?$CFs?$CC?$AA@ 100b2248     interop.obj
 0002:00008260       ??_C@_0M@EKGNDAGL@foreign?5key?$AA@ 100b2260     interop.obj
 0002:0000826c       ??_C@_07KNEBDGNE@indexed?$AA@ 100b226c     interop.obj
 0002:00008274       ??_C@_0CC@PCDMPIAA@cannot?5open?5?$CFs?5column?5for?5writin@ 100b2274     interop.obj
 0002:00008298       ??_C@_03CLCAEGCJ@new?$AA@  100b2298     interop.obj
 0002:0000829c       ??_C@_03PNKCFLFB@old?$AA@  100b229c     interop.obj
 0002:000082a0       ??_C@_0BP@LIGNHLP@misuse?5of?5aliased?5aggregate?5?$CFs?$AA@ 100b22a0     interop.obj
 0002:000082c0       ??_C@_0P@OOEELNMH@no?5such?5column?$AA@ 100b22c0     interop.obj
 0002:000082d0       ??_C@_0BG@CPPEOILG@ambiguous?5column?5name?$AA@ 100b22d0     interop.obj
 0002:000082e8       ??_C@_0N@GOMHGJCA@?$CFs?3?5?$CFs?4?$CFs?4?$CFs?$AA@ 100b22e8     interop.obj
 0002:000082f8       ??_C@_09DEPFKOIN@?$CFs?3?5?$CFs?4?$CFs?$AA@ 100b22f8     interop.obj
 0002:00008304       ??_C@_06DJHOIPC@?$CFs?3?5?$CFs?$AA@ 100b2304     interop.obj
 0002:0000830c       ??_C@_0CD@CLOCOINF@not?5authorized?5to?5use?5function?3?5@ 100b230c     interop.obj
 0002:00008330       ??_C@_0CE@JOMBDPK@misuse?5of?5aggregate?5function?5?$CF?4?$CK@ 100b2330     interop.obj
 0002:00008354       ??_C@_0BH@DEPAIHDK@no?5such?5function?3?5?$CF?4?$CKs?$AA@ 100b2354     interop.obj
 0002:0000836c       ??_C@_0CN@GBOJIJCC@wrong?5number?5of?5arguments?5to?5fun@ 100b236c     interop.obj
 0002:0000839c       ??_C@_0CL@HPCDGFPK@subqueries?5prohibited?5in?5CHECK?5c@ 100b239c     interop.obj
 0002:000083c8       ??_C@_0CL@HIKOHDBA@parameters?5prohibited?5in?5CHECK?5c@ 100b23c8     interop.obj
 0002:000083f4       ??_C@_0DI@IJOLPLNO@?$CFr?5?$CFs?5BY?5term?5out?5of?5range?5?9?5sho@ 100b23f4     interop.obj
 0002:0000842c       ??_C@_0CC@GEJJPDIE@too?5many?5terms?5in?5ORDER?5BY?5claus@ 100b242c     interop.obj
 0002:00008450       ??_C@_05BIEKMFNJ@ORDER?$AA@ 100b2450     interop.obj
 0002:00008458       ??_C@_0DN@KHANHMIL@?$CFr?5ORDER?5BY?5term?5does?5not?5match?5@ 100b2458     interop.obj
 0002:00008498       ??_C@_0BP@OLNMGBH@too?5many?5terms?5in?5?$CFs?5BY?5clause?$AA@ 100b2498     interop.obj
 0002:000084b8       ??_C@_0CM@CFGBPLAG@a?5GROUP?5BY?5clause?5is?5required?5be@ 100b24b8     interop.obj
 0002:000084e4       ??_C@_05NAIABEH@GROUP?$AA@ 100b24e4     interop.obj
 0002:000084ec       ??_C@_0DL@LDIIFJFH@aggregate?5functions?5are?5not?5allo@ 100b24ec     interop.obj
 0002:00008528       ??_C@_0DA@HPOBBFJP@Expression?5tree?5is?5too?5large?5?$CIma@ 100b2528     interop.obj
 0002:00008558       ??_C@_0CL@MAPAMFMM@variable?5number?5must?5be?5between?5@ 100b2558     interop.obj
 0002:00008584       ??_C@_0BH@KLMBLGJH@too?5many?5SQL?5variables?$AA@ 100b2584     interop.obj
 0002:0000859c       ??_C@_0BH@HJGFDJPB@too?5many?5columns?5in?5?$CFs?$AA@ 100b259c     interop.obj
 0002:000085b4       ??_C@_07HKAAOBDA@_ROWID_?$AA@ 100b25b4     interop.obj
 0002:000085bc       ??_C@_05GIFMDDGN@ROWID?$AA@ 100b25bc     interop.obj
 0002:000085c4       ??_C@_03PGJCFEMG@OID?$AA@  100b25c4     interop.obj
 0002:000085c8       ??_C@_04PCOPKCKE@LIST?$AA@ 100b25c8     interop.obj
 0002:000085d0       ??_C@_06LEOGOFDE@SCALAR?$AA@ 100b25d0     interop.obj
 0002:000085d8       ??_C@_0M@MCLOEEML@CORRELATED?5?$AA@ 100b25d8     interop.obj
 0002:000085e4       ??_C@_0BJ@HNBNONDH@EXECUTE?5?$CFs?$CFs?5SUBQUERY?5?$CFd?$AA@ 100b25e4     interop.obj
 0002:00008600       ??_C@_0BK@BMEAFNCN@misuse?5of?5aggregate?3?5?$CFs?$CI?$CJ?$AA@ 100b2600     interop.obj
 0002:0000861c       ??_C@_0BJ@HFDHLKDG@unknown?5function?3?5?$CF?4?$CKs?$CI?$CJ?$AA@ 100b261c     interop.obj
 0002:00008638       ??_C@_0DC@JGGJAPOJ@RAISE?$CI?$CJ?5may?5only?5be?5used?5within?5@ 100b2638     interop.obj
 0002:0000866c       ??_C@_0L@HDDJIJMP@?$CF?4?$CKs?$CC?$CFw?$CC?$CFs?$AA@ 100b266c     interop.obj
 0002:00008678       ??_C@_0L@GGMNOGLF@?$CFs?$CF?4?$CKs?$CC?$CFw?$CC?$AA@ 100b2678     interop.obj
 0002:00008684       ??_C@_07IKCPJJF@name?$DN?$CFQ?$AA@ 100b2684     interop.obj
 0002:0000868c       ??_C@_0O@JAFDLLMD@?$CFs?5OR?5name?$DN?$CFQ?$AA@ 100b268c     interop.obj
 0002:0000869c       ??_C@_0BI@IBIDABAM@type?$DN?8trigger?8?5AND?5?$CI?$CFs?$CJ?$AA@ 100b269c     interop.obj
 0002:000086b4       ??_C@_0M@FPJBBPLI@tbl_name?$DN?$CFQ?$AA@ 100b26b4     interop.obj
 0002:000086c0       ??_C@_07IOGLMIPM@sqlite_?$AA@ 100b26c0     interop.obj
 0002:000086c8       ??_C@_0BM@IAHFHDLE@table?5?$CFs?5may?5not?5be?5altered?$AA@ 100b26c8     interop.obj
 0002:000086e4       ??_C@_0DL@DAEIJKNC@there?5is?5already?5another?5table?5o@ 100b26e4     interop.obj
 0002:00008720       ??_C@_0BL@FIDIAKLG@view?5?$CFs?5may?5not?5be?5altered?$AA@ 100b2720     interop.obj
 0002:00008740       ??_C@_0EF@LBDFNLNO@UPDATE?5?$CC?$CFw?$CC?4?$CFs?5SET?5sql?5?$DN?5sqlite_@ 100b2740     interop.obj
 0002:00008788       ??_C@_0BIA@DMFFJHNO@UPDATE?5?$CFQ?4?$CFs?5SET?5sql?5?$DN?5CASE?5WHEN@ 100b2788     interop.obj
 0002:00008908       ??_C@_0BA@KDDGKFDH@sqlite_sequence?$AA@ 100b2908     interop.obj
 0002:00008918       ??_C@_0DK@NPMGFNPC@UPDATE?5?$CC?$CFw?$CC?4sqlite_sequence?5set?5@ 100b2918     interop.obj
 0002:00008958       ??_C@_0FM@GJOILOPP@UPDATE?5sqlite_temp_master?5SET?5sq@ 100b2958     interop.obj
 0002:000089b4       ??_C@_0CA@KEHKHMLG@Cannot?5add?5a?5PRIMARY?5KEY?5column?$AA@ 100b29b4     interop.obj
 0002:000089d4       ??_C@_0BL@NAFLCLKF@Cannot?5add?5a?5UNIQUE?5column?$AA@ 100b29d4     interop.obj
 0002:000089f0       ??_C@_0DL@KNFPANHI@Cannot?5add?5a?5REFERENCES?5column?5w@ 100b29f0     interop.obj
 0002:00008a2c       ??_C@_0DF@JACFJFPO@Cannot?5add?5a?5NOT?5NULL?5column?5wit@ 100b2a2c     interop.obj
 0002:00008a64       ??_C@_0CO@DPKGGDEF@Cannot?5add?5a?5column?5with?5non?9con@ 100b2a64     interop.obj
 0002:00008a98       ??_C@_0GN@GPPLIGGM@UPDATE?5?$CC?$CFw?$CC?4?$CFs?5SET?5sql?5?$DN?5substr?$CI@ 100b2a98     interop.obj
 0002:00008b08       ??_C@_0CC@HCCMFAJP@virtual?5tables?5may?5not?5be?5altere@ 100b2b08     interop.obj
 0002:00008b2c       ??_C@_0BO@IKHDEECD@Cannot?5add?5a?5column?5to?5a?5view?$AA@ 100b2b2c     interop.obj
 0002:00008b4c       ??_C@_0BD@PKLNNDD@sqlite_altertab_?$CFs?$AA@ 100b2b4c     interop.obj
 0002:00008b60       ??_C@_0BH@NPNIHFHO@CREATE?5TABLE?5?$CFQ?4?$CFs?$CI?$CFs?$CJ?$AA@ 100b2b60     interop.obj
 0002:00008b78       ??_C@_0BO@HNIAJBGG@DELETE?5FROM?5?$CFQ?4?$CFs?5WHERE?5?$CFs?$DN?$CFQ?$AA@ 100b2b78     interop.obj
 0002:00008b98       ??_C@_06FFMDNONC@bbbbbb?$AA@ 100b2b98     interop.obj
 0002:00008ba0       ??_C@_01CLKCMJKC@?5?$AA@   100b2ba0     interop.obj
 0002:00008ba4       ??_C@_03GINCELHE@aaa?$AA@  100b2ba4     interop.obj
 0002:00008ba8       ??_C@_03DAKNAIGI@idx?$AA@  100b2ba8     interop.obj
 0002:00008bac       ??_C@_03LIPNCMMN@tbl?$AA@  100b2bac     interop.obj
 0002:00008bb0       ??_C@_09KGIEIKHI@unordered?$AA@ 100b2bb0     interop.obj
 0002:00008bbc       ??_C@_0DG@KHFPEBKH@SELECT?5idx?0count?$CI?$CK?$CJ?5FROM?5?$CFQ?4sqli@ 100b2bbc     interop.obj
 0002:00008bf4       ??_C@_0DE@GKJIFEOA@SELECT?5idx?0neq?0nlt?0ndlt?0sample?5F@ 100b2bf4     interop.obj
 0002:00008c28       ??_C@_0CJ@CJKDHBGL@SELECT?5tbl?0idx?0stat?5FROM?5?$CFQ?4sqli@ 100b2c28     interop.obj
 0002:00008c54       ??_C@_0BD@BGLLCPKM@invalid?5name?3?5?$CC?$CFs?$CC?$AA@ 100b2c54     interop.obj
 0002:00008c68       ??_C@_0CF@FLFLBLIN@too?5many?5attached?5databases?5?9?5ma@ 100b2c68     interop.obj
 0002:00008c90       ??_C@_0CK@JEFPBLHB@cannot?5ATTACH?5database?5within?5tr@ 100b2c90     interop.obj
 0002:00008cbc       ??_C@_0BO@FOBANNIG@database?5?$CFs?5is?5already?5in?5use?$AA@ 100b2cbc     interop.obj
 0002:00008cdc       ??_C@_0BN@IAAPNCPC@database?5is?5already?5attached?$AA@ 100b2cdc     interop.obj
 0002:00008d00       ??_C@_0EE@MLIDCBJA@attached?5databases?5must?5use?5the?5@ 100b2d00     interop.obj
 0002:00008d44       ??_C@_0BC@BMCHOAML@Invalid?5key?5value?$AA@ 100b2d44     interop.obj
 0002:00008d58       ??_C@_0BM@JECJFHOP@unable?5to?5open?5database?3?5?$CFs?$AA@ 100b2d58     interop.obj
 0002:00008d74       ??_C@_0BF@PJFCJDG@no?5such?5database?3?5?$CFs?$AA@ 100b2d74     interop.obj
 0002:00008d8c       ??_C@_0BK@KGABJE@cannot?5detach?5database?5?$CFs?$AA@ 100b2d8c     interop.obj
 0002:00008da8       ??_C@_0CK@NCGPBHIO@cannot?5DETACH?5database?5within?5tr@ 100b2da8     interop.obj
 0002:00008dd4       ??_C@_0BG@HKAEEBEM@database?5?$CFs?5is?5locked?$AA@ 100b2dd4     interop.obj
 0002:00008dec       ??_C@_0CO@IGOBCPDP@?$CFs?5?$CFT?5cannot?5reference?5objects?5i@ 100b2dec     interop.obj
 0002:00008e1c       ??_C@_0BH@KNHNEHPN@authorizer?5malfunction?$AA@ 100b2e1c     interop.obj
 0002:00008e34       ??_C@_0CB@NCPGIDCD@access?5to?5?$CFs?4?$CFs?4?$CFs?5is?5prohibited@ 100b2e34     interop.obj
 0002:00008e58       ??_C@_0BO@CMCIGPCH@access?5to?5?$CFs?4?$CFs?5is?5prohibited?$AA@ 100b2e58     interop.obj
 0002:00008e78       ??_C@_0P@PEBGBLCC@not?5authorized?$AA@ 100b2e78     interop.obj
 0002:00008e88       ??_C@_0N@IAMBEAMM@no?5such?5view?$AA@ 100b2e88     interop.obj
 0002:00008e98       ??_C@_0O@HKMEEONL@no?5such?5table?$AA@ 100b2e98     interop.obj
 0002:00008ea8       ??_C@_0BB@GODMDNII@corrupt?5database?$AA@ 100b2ea8     interop.obj
 0002:00008ebc       ??_C@_0BE@DADMKDCE@unknown?5database?5?$CFT?$AA@ 100b2ebc     interop.obj
 0002:00008ed0       ??_C@_0CK@DHAAGEMP@object?5name?5reserved?5for?5interna@ 100b2ed0     interop.obj
 0002:00008efc       ??_C@_0CJ@GGBIBJLH@temporary?5table?5name?5must?5be?5unq@ 100b2efc     interop.obj
 0002:00008f28       ??_C@_0BI@NMBJKJHP@table?5?$CFT?5already?5exists?$AA@ 100b2f28     interop.obj
 0002:00008f40       ??_C@_0CD@FJHICPML@there?5is?5already?5an?5index?5named?5@ 100b2f40     interop.obj
 0002:00008f64       ??_C@_0BH@KPDMNKOM@too?5many?5columns?5on?5?$CFs?$AA@ 100b2f64     interop.obj
 0002:00008f7c       ??_C@_0BK@CJJKBEHE@duplicate?5column?5name?3?5?$CFs?$AA@ 100b2f7c     interop.obj
 0002:00008f98       ??_C@_0CN@MLPCOIJO@default?5value?5of?5column?5?$FL?$CFs?$FN?5is?5@ 100b2f98     interop.obj
 0002:00008fc8       ??_C@_0CJ@LEOOFHMA@table?5?$CC?$CFs?$CC?5has?5more?5than?5one?5pri@ 100b2fc8     interop.obj
 0002:00008ff4       ??_C@_07EHCIHKNF@INTEGER?$AA@ 100b2ff4     interop.obj
 0002:00008ffc       ??_C@_0DI@IAIBDBA@AUTOINCREMENT?5is?5only?5allowed?5on@ 100b2ffc     interop.obj
 0002:00009034       ??_C@_01IHBHIGKO@?0?$AA@   100b3034     interop.obj
 0002:00009038       ??_C@_01PKGAHCOL@?$CJ?$AA@ 100b3038     interop.obj
 0002:0000903c       ??_C@_03BMMPKCMF@?6?5?5?$AA@ 100b303c     interop.obj
 0002:00009040       ??_C@_04PPJIEIMB@?0?6?5?5?$AA@ 100b3040     interop.obj
 0002:00009048       ??_C@_02EJGPDMNA@?6?$CJ?$AA@ 100b3048     interop.obj
 0002:0000904c       ??_C@_0O@BLHKEBID@CREATE?5TABLE?5?$AA@ 100b304c     interop.obj
 0002:0000905c       ??_C@_05LCLENNFI@table?$AA@ 100b305c     interop.obj
 0002:00009064       ??_C@_05HJCCDKBG@TABLE?$AA@ 100b3064     interop.obj
 0002:0000906c       ??_C@_04CHADEDPO@view?$AA@ 100b306c     interop.obj
 0002:00009074       ??_C@_04OLDJKBIG@VIEW?$AA@ 100b3074     interop.obj
 0002:0000907c       ??_C@_0P@BPBAOJCC@CREATE?5?$CFs?5?$CF?4?$CKs?$AA@ 100b307c     interop.obj
 0002:00009090       ??_C@_0FH@BLIGLCKI@UPDATE?5?$CFQ?4?$CFs?5SET?5type?$DN?8?$CFs?8?0?5name@ 100b3090     interop.obj
 0002:000090e8       ??_C@_0CK@BLJIJAMD@CREATE?5TABLE?5?$CFQ?4sqlite_sequence?$CI@ 100b30e8     interop.obj
 0002:00009114       ??_C@_0O@LAHPKCHN@tbl_name?$DN?8?$CFq?8?$AA@ 100b3114     interop.obj
 0002:00009124       ??_C@_0CE@HIMMFEMD@parameters?5are?5not?5allowed?5in?5vi@ 100b3124     interop.obj
 0002:00009148       ??_C@_0BO@BLAOKNKN@view?5?$CFs?5is?5circularly?5defined?$AA@ 100b3148     interop.obj
 0002:00009168       ??_C@_0DI@GKCMDFKF@UPDATE?5?$CFQ?4?$CFs?5SET?5rootpage?$DN?$CFd?5WHE@ 100b3168     interop.obj
 0002:000091a0       ??_C@_0O@IOJCPKAP@sqlite_stat?$CFd?$AA@ 100b31a0     interop.obj
 0002:000091b0       ??_C@_0CN@DKDOKGOO@DELETE?5FROM?5?$CFQ?4sqlite_sequence?5W@ 100b31b0     interop.obj
 0002:000091e0       ??_C@_0DI@FOLLFOLB@DELETE?5FROM?5?$CFQ?4?$CFs?5WHERE?5tbl_name@ 100b31e0     interop.obj
 0002:00009218       ??_C@_0M@IHGMMCJN@sqlite_stat?$AA@ 100b3218     interop.obj
 0002:00009224       ??_C@_0BM@JEGMLIGC@table?5?$CFs?5may?5not?5be?5dropped?$AA@ 100b3224     interop.obj
 0002:00009240       ??_C@_0CC@HNNEDPB@use?5DROP?5TABLE?5to?5delete?5table?5?$CF@ 100b3240     interop.obj
 0002:00009264       ??_C@_0CA@FJIHAAAA@use?5DROP?5VIEW?5to?5delete?5view?5?$CFs?$AA@ 100b3264     interop.obj
 0002:00009284       ??_C@_0DP@HFDIOLMB@foreign?5key?5on?5?$CFs?5should?5referen@ 100b3284     interop.obj
 0002:000092c8       ??_C@_0FO@BDBBNOLJ@number?5of?5columns?5in?5foreign?5key@ 100b32c8     interop.obj
 0002:00009328       ??_C@_0CO@ECJPGOGF@unknown?5column?5?$CC?$CFs?$CC?5in?5foreign?5k@ 100b3328     interop.obj
 0002:00009358       ??_C@_0BP@NPACMCHA@indexed?5columns?5are?5not?5unique?$AA@ 100b3358     interop.obj
 0002:00009378       ??_C@_05FKHKFDID@index?$AA@ 100b3378     interop.obj
 0002:00009380       ??_C@_09NGMBFCCJ@altertab_?$AA@ 100b3380     interop.obj
 0002:0000938c       ??_C@_0BM@KIGEJLNH@table?5?$CFs?5may?5not?5be?5indexed?$AA@ 100b338c     interop.obj
 0002:000093a8       ??_C@_0BJ@CFGNJLOC@views?5may?5not?5be?5indexed?$AA@ 100b33a8     interop.obj
 0002:000093c4       ??_C@_0CC@FKDNLIPM@virtual?5tables?5may?5not?5be?5indexe@ 100b33c4     interop.obj
 0002:000093e8       ??_C@_0CC@CKJEJGLG@there?5is?5already?5a?5table?5named?5?$CF@ 100b33e8     interop.obj
 0002:0000940c       ??_C@_0BI@HPCDPJFN@index?5?$CFs?5already?5exists?$AA@ 100b340c     interop.obj
 0002:00009424       ??_C@_0BH@HCCALECK@sqlite_autoindex_?$CFs_?$CFd?$AA@ 100b3424     interop.obj
 0002:0000943c       ??_C@_0CA@MKEFOFFD@table?5?$CFs?5has?5no?5column?5named?5?$CFs?$AA@ 100b343c     interop.obj
 0002:0000945c       ??_C@_06FJHKNKMG@BINARY?$AA@ 100b345c     interop.obj
 0002:00009464       ??_C@_0CK@BPKJMBLB@conflicting?5ON?5CONFLICT?5clauses?5@ 100b3464     interop.obj
 0002:00009490       ??_C@_07OGDPOKCI@?5UNIQUE?$AA@ 100b3490     interop.obj
 0002:00009498       ??_C@_0BE@NHCJMGDI@CREATE?$CFs?5INDEX?5?$CF?4?$CKs?$AA@ 100b3498     interop.obj
 0002:000094ac       ??_C@_0DA@DLDDDEKN@INSERT?5INTO?5?$CFQ?4?$CFs?5VALUES?$CI?8index?8@ 100b34ac     interop.obj
 0002:000094dc       ??_C@_0BL@CHCJOOMG@name?$DN?8?$CFq?8?5AND?5type?$DN?8index?8?$AA@ 100b34dc     interop.obj
 0002:000094f8       ??_C@_0BC@JBPCAJCH@no?5such?5index?3?5?$CFS?$AA@ 100b34f8     interop.obj
 0002:00009510       ??_C@_0EJ@MFMNFJHB@index?5associated?5with?5UNIQUE?5or?5@ 100b3510     interop.obj
 0002:0000955c       ??_C@_0DB@DNHAJCKG@DELETE?5FROM?5?$CFQ?4?$CFs?5WHERE?5name?$DN?$CFQ?5@ 100b355c     interop.obj
 0002:00009590       ??_C@_02BFICIOJL@ON?$AA@   100b3590     interop.obj
 0002:00009594       ??_C@_05EOONBMLM@USING?$AA@ 100b3594     interop.obj
 0002:0000959c       ??_C@_0CE@GFPKLECD@a?5JOIN?5clause?5is?5required?5before@ 100b359c     interop.obj
 0002:000095c0       ??_C@_05ILMMJGEC@BEGIN?$AA@ 100b35c0     interop.obj
 0002:000095c8       ??_C@_06IBPPMFNL@COMMIT?$AA@ 100b35c8     interop.obj
 0002:000095d0       ??_C@_08COBEBGNM@ROLLBACK?$AA@ 100b35d0     interop.obj
 0002:000095e0       ??_C@_0EG@GIEOJFED@unable?5to?5open?5a?5temporary?5datab@ 100b35e0     interop.obj
 0002:00009628       ??_C@_0CO@PMBDNHDC@unable?5to?5identify?5the?5object?5to@ 100b3628     interop.obj
 0002:00009658       ??_C@_0BP@CGLMEPGG@no?5such?5collation?5sequence?3?5?$CFs?$AA@ 100b3658     interop.obj
 0002:00009678       ??_C@_0BN@GLMOOAMK@table?5?$CFs?5may?5not?5be?5modified?$AA@ 100b3678     interop.obj
 0002:00009698       ??_C@_0CG@CNPJIJGN@cannot?5modify?5?$CFs?5because?5it?5is?5a@ 100b3698     interop.obj
 0002:000096c0       ??_C@_0N@DAGIBCDP@rows?5deleted?$AA@ 100b36c0     interop.obj
 0002:000096d0       ??_C@_04CIMGMMMG@text?$AA@ 100b36d0     interop.obj
 0002:000096d8       ??_C@_04LPJPOBEM@blob?$AA@ 100b36d8     interop.obj
 0002:000096e0       ??_C@_0BB@KBEKGHFK@integer?5overflow?$AA@ 100b36e0     interop.obj
 0002:000096f4       ??_C@_04HGGMHPIM@?$CF?4?$CKf?$AA@ 100b36f4     interop.obj
 0002:000096fc       ??_C@_06CLNEDLBE@?$CF?$CB?420e?$AA@ 100b36fc     interop.obj
 0002:00009704       ??_C@_04BBKKAMHH@?$DP000?$AA@ 100b3704     interop.obj
 0002:0000970c       ??_C@_05JGHLFIHG@MATCH?$AA@ 100b370c     interop.obj
 0002:00009714       ??_C@_04HHHPGODM@glob?$AA@ 100b3714     interop.obj
 0002:0000971c       ??_C@_0CN@NOKHDNFH@foreign?5key?5mismatch?5?9?5?$CC?$CFw?$CC?5refe@ 100b371c     interop.obj
 0002:0000974c       ??_C@_03PLGJJJLK@oid?$AA@  100b374c     interop.obj
 0002:00009750       ??_C@_0DE@HLHNLKJ@table?5?$CFS?5has?5?$CFd?5columns?5but?5?$CFd?5v@ 100b3750     interop.obj
 0002:00009784       ??_C@_0BJ@IABIHKKK@?$CFd?5values?5for?5?$CFd?5columns?$AA@ 100b3784     interop.obj
 0002:000097a0       ??_C@_0CA@HKGLKLIP@table?5?$CFS?5has?5no?5column?5named?5?$CFs?$AA@ 100b37a0     interop.obj
 0002:000097c0       ??_C@_0O@OMFDFDMH@rows?5inserted?$AA@ 100b37c0     interop.obj
 0002:000097d0       ??_C@_0BG@OAHBMIAD@?$CFs?4?$CFs?5may?5not?5be?5NULL?$AA@ 100b37d0     interop.obj
 0002:000097e8       ??_C@_0BF@PCAEONAJ@constraint?5?$CFs?5failed?$AA@ 100b37e8     interop.obj
 0002:00009800       ??_C@_0BL@MIGFAHKG@PRIMARY?5KEY?5must?5be?5unique?$AA@ 100b3800     interop.obj
 0002:0000981c       ??_C@_08BLECJPKD@columns?5?$AA@ 100b381c     interop.obj
 0002:00009828       ??_C@_07OJMCPGAK@column?5?$AA@ 100b3828     interop.obj
 0002:00009830       ??_C@_02KEGNLNML@?0?5?$AA@ 100b3830     interop.obj
 0002:00009834       ??_C@_0BA@IJKPAPH@?5are?5not?5unique?$AA@ 100b3834     interop.obj
 0002:00009844       ??_C@_0P@GKKFBNCL@?5is?5not?5unique?$AA@ 100b3844     interop.obj
 0002:00009854       ??_C@_0BH@NNAEMFED@sqlite3_extension_init?$AA@ 100b3854     interop.obj
 0002:0000986c       ??_C@_05NNFHCGPF@?$CFs?4?$CFs?$AA@ 100b386c     interop.obj
 0002:00009874       ??_C@_0CD@FENJJFPL@unable?5to?5open?5shared?5library?5?$FL?$CF@ 100b3874     interop.obj
 0002:00009898       ??_C@_08MIGLKGCA@sqlite3_?$AA@ 100b3898     interop.obj
 0002:000098a4       ??_C@_03LPIGJBNC@lib?$AA@  100b38a4     interop.obj
 0002:000098a8       ??_C@_05PAGLDNCP@_init?$AA@ 100b38a8     interop.obj
 0002:000098b0       ??_C@_0CL@IHPFGADB@no?5entry?5point?5?$FL?$CFs?$FN?5in?5shared?5li@ 100b38b0     interop.obj
 0002:000098dc       ??_C@_0CA@BPLHPOIJ@error?5during?5initialization?3?5?$CFs?$AA@ 100b38dc     interop.obj
 0002:000098fc       ??_C@_0CH@EKKEGGML@automatic?5extension?5loading?5fail@ 100b38fc     interop.obj
 0002:00009924       ??_C@_09JJPHINFN@exclusive?$AA@ 100b3924     interop.obj
 0002:00009930       ??_C@_06IKLLLDHL@normal?$AA@ 100b3930     interop.obj
 0002:00009938       ??_C@_04CGFJFPFD@none?$AA@ 100b3938     interop.obj
 0002:00009940       ??_C@_04PLMLMMEO@full?$AA@ 100b3940     interop.obj
 0002:00009948       ??_C@_0M@LPKHOAFP@incremental?$AA@ 100b3948     interop.obj
 0002:00009954       ??_C@_04DAMGJPCA@file?$AA@ 100b3954     interop.obj
 0002:0000995c       ??_C@_06HLKELJGF@memory?$AA@ 100b395c     interop.obj
 0002:00009964       ??_C@_0DO@MAKCDDCJ@temporary?5storage?5cannot?5be?5chan@ 100b3964     interop.obj
 0002:000099a4       ??_C@_08NNDOPPOM@SET?5NULL?$AA@ 100b39a4     interop.obj
 0002:000099b0       ??_C@_0M@GCMLNHF@SET?5DEFAULT?$AA@ 100b39b0     interop.obj
 0002:000099bc       ??_C@_07JDMPGCJB@CASCADE?$AA@ 100b39bc     interop.obj
 0002:000099c4       ??_C@_08KJMJNHDG@RESTRICT?$AA@ 100b39c4     interop.obj
 0002:000099d0       ??_C@_09DBFINONP@NO?5ACTION?$AA@ 100b39d0     interop.obj
 0002:000099dc       ??_C@_03GMLCELFL@?9?$CFT?$AA@ 100b39dc     interop.obj
 0002:000099e0       ??_C@_06KJFADLGN@result?$AA@ 100b39e0     interop.obj
 0002:000099e8       ??_C@_0BD@EMJOENCP@default_cache_size?$AA@ 100b39e8     interop.obj
 0002:000099fc       ??_C@_0L@JIGNFOJJ@cache_size?$AA@ 100b39fc     interop.obj
 0002:00009a08       ??_C@_09OGOMKHMG@page_size?$AA@ 100b3a08     interop.obj
 0002:00009a14       ??_C@_0O@CPOJHNIK@secure_delete?$AA@ 100b3a14     interop.obj
 0002:00009a24       ??_C@_0L@OBBCDPFM@page_count?$AA@ 100b3a24     interop.obj
 0002:00009a30       ??_C@_0P@FMLMLOHD@max_page_count?$AA@ 100b3a30     interop.obj
 0002:00009a40       ??_C@_0N@NOOMDJH@locking_mode?$AA@ 100b3a40     interop.obj
 0002:00009a50       ??_C@_0N@IPLFJDHP@journal_mode?$AA@ 100b3a50     interop.obj
 0002:00009a60       ??_C@_0BD@MCBLCGGI@journal_size_limit?$AA@ 100b3a60     interop.obj
 0002:00009a74       ??_C@_0M@ENMLGDH@auto_vacuum?$AA@ 100b3a74     interop.obj
 0002:00009a80       ??_C@_0BD@IEMDKFHA@incremental_vacuum?$AA@ 100b3a80     interop.obj
 0002:00009a94       ??_C@_09CBABOEGE@mmap_size?$AA@ 100b3a94     interop.obj
 0002:00009aa0       ??_C@_0L@JEPCDDIC@temp_store?$AA@ 100b3aa0     interop.obj
 0002:00009aac       ??_C@_0BF@OPALIJKE@temp_store_directory?$AA@ 100b3aac     interop.obj
 0002:00009ac4       ??_C@_0BJ@INLPNACB@not?5a?5writable?5directory?$AA@ 100b3ac4     interop.obj
 0002:00009ae0       ??_C@_0BF@OGPCDMDP@data_store_directory?$AA@ 100b3ae0     interop.obj
 0002:00009af8       ??_C@_0M@GKGFOGDE@synchronous?$AA@ 100b3af8     interop.obj
 0002:00009b04       ??_C@_0DF@GMDBDCKL@Safety?5level?5may?5not?5be?5changed?5@ 100b3b04     interop.obj
 0002:00009b3c       ??_C@_0L@NEMFJAGM@table_info?$AA@ 100b3b3c     interop.obj
 0002:00009b48       ??_C@_03LBLPCGAC@cid?$AA@  100b3b48     interop.obj
 0002:00009b4c       ??_C@_04MEMAJGDJ@name?$AA@ 100b3b4c     interop.obj
 0002:00009b54       ??_C@_04GPMDFGEJ@type?$AA@ 100b3b54     interop.obj
 0002:00009b5c       ??_C@_07EAJHGOKJ@notnull?$AA@ 100b3b5c     interop.obj
 0002:00009b64       ??_C@_0L@KNDFGGNJ@dflt_value?$AA@ 100b3b64     interop.obj
 0002:00009b70       ??_C@_02NCEGPMNB@pk?$AA@   100b3b70     interop.obj
 0002:00009b74       ??_C@_0L@CKPANNIC@index_info?$AA@ 100b3b74     interop.obj
 0002:00009b80       ??_C@_05OBPGIPLF@seqno?$AA@ 100b3b80     interop.obj
 0002:00009b88       ??_C@_0L@MMBMMAEK@index_list?$AA@ 100b3b88     interop.obj
 0002:00009b94       ??_C@_03NPAJGOON@seq?$AA@  100b3b94     interop.obj
 0002:00009b98       ??_C@_06ODCMFGLL@unique?$AA@ 100b3b98     interop.obj
 0002:00009ba0       ??_C@_0O@EBMNDACF@database_list?$AA@ 100b3ba0     interop.obj
 0002:00009bb0       ??_C@_0P@KOJNIGCH@collation_list?$AA@ 100b3bb0     interop.obj
 0002:00009bc0       ??_C@_0BB@KJMCGNAI@foreign_key_list?$AA@ 100b3bc0     interop.obj
 0002:00009bd4       ??_C@_02EGCJHIOB@id?$AA@   100b3bd4     interop.obj
 0002:00009bd8       ??_C@_04HNEBHLOP@from?$AA@ 100b3bd8     interop.obj
 0002:00009be0       ??_C@_02LBCDJBAJ@to?$AA@   100b3be0     interop.obj
 0002:00009be4       ??_C@_09DFBGJPOA@on_update?$AA@ 100b3be4     interop.obj
 0002:00009bf0       ??_C@_09BILGEHCE@on_delete?$AA@ 100b3bf0     interop.obj
 0002:00009bfc       ??_C@_05FNONLPDI@match?$AA@ 100b3bfc     interop.obj
 0002:00009c04       ??_C@_04OKGDLNCL@NONE?$AA@ 100b3c04     interop.obj
 0002:00009c0c       ??_C@_0BC@CIFGNOOA@foreign_key_check?$AA@ 100b3c0c     interop.obj
 0002:00009c20       ??_C@_05KDMKNECD@rowid?$AA@ 100b3c20     interop.obj
 0002:00009c28       ??_C@_06MLKDMCBD@parent?$AA@ 100b3c28     interop.obj
 0002:00009c30       ??_C@_04IFBPKEAB@fkid?$AA@ 100b3c30     interop.obj
 0002:00009c38       ??_C@_0BE@LKBHCIHN@case_sensitive_like?$AA@ 100b3c38     interop.obj
 0002:00009c4c       ??_C@_0BA@EDNFHOBJ@integrity_check?$AA@ 100b3c4c     interop.obj
 0002:00009c5c       ??_C@_0M@EDPCDMIO@quick_check?$AA@ 100b3c5c     interop.obj
 0002:00009c68       ??_C@_0BI@FOLPKNAK@?$CK?$CK?$CK?5in?5database?5?$CFs?5?$CK?$CK?$CK?6?$AA@ 100b3c68     interop.obj
 0002:00009c80       ??_C@_06DHEAJPAE@rowid?5?$AA@ 100b3c80     interop.obj
 0002:00009c88       ??_C@_0BF@JGBLFHJL@?5missing?5from?5index?5?$AA@ 100b3c88     interop.obj
 0002:00009ca0       ??_C@_0BN@JKHLHJNK@wrong?5?$CD?5of?5entries?5in?5index?5?$AA@ 100b3ca0     interop.obj
 0002:00009cc0       ??_C@_02MFDMBIJM@ok?$AA@   100b3cc0     interop.obj
 0002:00009cc4       ??_C@_08MLPGAEIK@encoding?$AA@ 100b3cc4     interop.obj
 0002:00009cd0       ??_C@_0BJ@GJBMJNNI@unsupported?5encoding?3?5?$CFs?$AA@ 100b3cd0     interop.obj
 0002:00009cec       ??_C@_0P@JGMMHBPP@schema_version?$AA@ 100b3cec     interop.obj
 0002:00009cfc       ??_C@_0N@MPKCHLKL@user_version?$AA@ 100b3cfc     interop.obj
 0002:00009d0c       ??_C@_0P@GDKICNML@freelist_count?$AA@ 100b3d0c     interop.obj
 0002:00009d1c       ??_C@_0P@MIBGKNHF@application_id?$AA@ 100b3d1c     interop.obj
 0002:00009d2c       ??_C@_0BA@CFJEIIDP@compile_options?$AA@ 100b3d2c     interop.obj
 0002:00009d3c       ??_C@_0P@DCFGLPDE@compile_option?$AA@ 100b3d3c     interop.obj
 0002:00009d4c       ??_C@_0P@OLFGCBDE@wal_checkpoint?$AA@ 100b3d4c     interop.obj
 0002:00009d5c       ??_C@_07LDHOHMPD@restart?$AA@ 100b3d5c     interop.obj
 0002:00009d64       ??_C@_04COIEGINH@busy?$AA@ 100b3d64     interop.obj
 0002:00009d6c       ??_C@_03MGHMBJCF@log?$AA@  100b3d6c     interop.obj
 0002:00009d70       ??_C@_0N@NLAOCFOK@checkpointed?$AA@ 100b3d70     interop.obj
 0002:00009d80       ??_C@_0BD@JPABJEAI@wal_autocheckpoint?$AA@ 100b3d80     interop.obj
 0002:00009d94       ??_C@_0O@ILHLPNHH@shrink_memory?$AA@ 100b3d94     interop.obj
 0002:00009da4       ??_C@_0N@ELBKLHHC@busy_timeout?$AA@ 100b3da4     interop.obj
 0002:00009db4       ??_C@_07DDHNKDGP@timeout?$AA@ 100b3db4     interop.obj
 0002:00009dbc       ??_C@_03ICHNJLJF@key?$AA@  100b3dbc     interop.obj
 0002:00009dc0       ??_C@_05FMDLBNN@rekey?$AA@ 100b3dc0     interop.obj
 0002:00009dc8       ??_C@_06BHJHKMJC@hexkey?$AA@ 100b3dc8     interop.obj
 0002:00009dd0       ??_C@_08PCDPBHPP@hexrekey?$AA@ 100b3dd0     interop.obj
 0002:00009ddc       ??_C@_0BP@EHGGIFII@malformed?5database?5schema?5?$CI?$CFs?$CJ?$AA@ 100b3ddc     interop.obj
 0002:00009dfc       ??_C@_07FCJAGJJB@?$CFs?5?9?5?$CFs?$AA@ 100b3dfc     interop.obj
 0002:00009e04       ??_C@_0BB@JDJPANJL@invalid?5rootpage?$AA@ 100b3e04     interop.obj
 0002:00009e18       ??_C@_0BI@FFDCNLCF@unsupported?5file?5format?$AA@ 100b3e18     interop.obj
 0002:00009e30       ??_C@_0DH@EMHOBABL@SELECT?5name?0?5rootpage?0?5sql?5FROM?5@ 100b3e30     interop.obj
 0002:00009e68       ??_C@_0BO@EBFEALBC@database?5schema?5is?5locked?3?5?$CFs?$AA@ 100b3e68     interop.obj
 0002:00009e88       ??_C@_0BD@NDJILONF@statement?5too?5long?$AA@ 100b3e88     interop.obj
 0002:00009e9c       ??_C@_0CM@LOMFMKCH@unknown?5or?5unsupported?5join?5type@ 100b3e9c     interop.obj
 0002:00009ec8       ??_C@_0DH@LJEHIDDA@RIGHT?5and?5FULL?5OUTER?5JOINs?5are?5n@ 100b3ec8     interop.obj
 0002:00009f00       ??_C@_0DC@NBGJANJH@a?5NATURAL?5join?5may?5not?5have?5an?5O@ 100b3f00     interop.obj
 0002:00009f34       ??_C@_0DH@DHMOHNCE@cannot?5have?5both?5ON?5and?5USING?5cl@ 100b3f34     interop.obj
 0002:00009f70       ??_C@_0EA@LFCKDDII@cannot?5join?5using?5column?5?$CFs?5?9?5co@ 100b3f70     interop.obj
 0002:00009fb0       ??_C@_0EI@FMCKEHHB@only?5a?5single?5result?5allowed?5for@ 100b3fb0     interop.obj
 0002:00009ff8       ??_C@_09CDPONBKL@UNION?5ALL?$AA@ 100b3ff8     interop.obj
 0002:0000a004       ??_C@_09JBOBNLLF@INTERSECT?$AA@ 100b4004     interop.obj
 0002:0000a010       ??_C@_06JFIPMMLD@EXCEPT?$AA@ 100b4010     interop.obj
 0002:0000a018       ??_C@_05GJNJOPB@UNION?$AA@ 100b4018     interop.obj
 0002:0000a020       ??_C@_0BH@JCGMDKCI@USE?5TEMP?5B?9TREE?5FOR?5?$CFs?$AA@ 100b4020     interop.obj
 0002:0000a038       ??_C@_0BD@INMGDFNB@USING?5TEMP?5B?9TREE?5?$AA@ 100b4038     interop.obj
 0002:0000a04c       ??_C@_0CF@IFPCHLOK@COMPOUND?5SUBQUERIES?5?$CFd?5AND?5?$CFd?5?$CFs@ 100b404c     interop.obj
 0002:0000a074       ??_C@_05HKPGCKL@?$CFs?3?$CFd?$AA@ 100b4074     interop.obj
 0002:0000a07c       ??_C@_0DA@GPNKNMMI@ORDER?5BY?5clause?5should?5come?5afte@ 100b407c     interop.obj
 0002:0000a0ac       ??_C@_0CN@DDIHOHHL@LIMIT?5clause?5should?5come?5after?5?$CF@ 100b40ac     interop.obj
 0002:0000a0dc       ??_C@_0CO@DAHFDIDO@all?5VALUES?5must?5have?5the?5same?5nu@ 100b40dc     interop.obj
 0002:0000a110       ??_C@_0FC@CMDCIIHA@SELECTs?5to?5the?5left?5and?5right?5of@ 100b4110     interop.obj
 0002:0000a164       ??_C@_0BC@EHGCNIF@no?5such?5index?3?5?$CFs?$AA@ 100b4164     interop.obj
 0002:0000a178       ??_C@_0BE@EGABPGJI@sqlite_subquery_?$CFp_?$AA@ 100b4178     interop.obj
 0002:0000a18c       ??_C@_0CH@HMBFCKPN@too?5many?5references?5to?5?$CC?$CFs?$CC?3?5max@ 100b418c     interop.obj
 0002:0000a1b4       ??_C@_01NBENCBCI@?$CK?$AA@ 100b41b4     interop.obj
 0002:0000a1b8       ??_C@_08PPKHIAKG@?$CFs?4?$CFs?4?$CFs?$AA@ 100b41b8     interop.obj
 0002:0000a1c4       ??_C@_0BC@OFCALFBN@no?5such?5table?3?5?$CFs?$AA@ 100b41c4     interop.obj
 0002:0000a1d8       ??_C@_0BE@EGLAAHPP@no?5tables?5specified?$AA@ 100b41d8     interop.obj
 0002:0000a1ec       ??_C@_0BP@JFMLENOH@too?5many?5columns?5in?5result?5set?$AA@ 100b41ec     interop.obj
 0002:0000a20c       ??_C@_0DD@MKKFPBAF@DISTINCT?5aggregates?5must?5have?5ex@ 100b420c     interop.obj
 0002:0000a240       ??_C@_0BG@JAICCEJG@USING?5COVERING?5INDEX?5?$AA@ 100b4240     interop.obj
 0002:0000a258       ??_C@_0BN@NKANBDNO@SCAN?5TABLE?5?$CFs?5?$CFs?$CFs?$CI?$HO?$CFd?5rows?$CJ?$AA@ 100b4258     interop.obj
 0002:0000a278       ??_C@_0CC@DHLFNDIF@too?5many?5terms?5in?5compound?5SELEC@ 100b4278     interop.obj
 0002:0000a29c       ??_C@_08KLFLGHKI@DISTINCT?$AA@ 100b429c     interop.obj
 0002:0000a2a8       ??_C@_08NKEADCLG@GROUP?5BY?$AA@ 100b42a8     interop.obj
 0002:0000a2b4       ??_C@_08BKIJJFKP@ORDER?5BY?$AA@ 100b42b4     interop.obj
 0002:0000a2c0       ??_C@_0EB@PHGCKHIG@sqlite3_get_table?$CI?$CJ?5called?5with?5@ 100b42c0     interop.obj
 0002:0000a304       ??_C@_0CO@CGGBEMGD@temporary?5trigger?5may?5not?5have?5q@ 100b4304     interop.obj
 0002:0000a334       ??_C@_07DIDNFGDE@trigger?$AA@ 100b4334     interop.obj
 0002:0000a33c       ??_C@_0CJ@KLDCMPKB@cannot?5create?5triggers?5on?5virtua@ 100b433c     interop.obj
 0002:0000a368       ??_C@_0BK@IACDKJFA@trigger?5?$CFT?5already?5exists?$AA@ 100b4368     interop.obj
 0002:0000a384       ??_C@_0CG@JAGCNIHD@cannot?5create?5trigger?5on?5system?5@ 100b4384     interop.obj
 0002:0000a3ac       ??_C@_06BIGAHLBC@BEFORE?$AA@ 100b43ac     interop.obj
 0002:0000a3b4       ??_C@_05OHDJMCHE@AFTER?$AA@ 100b43b4     interop.obj
 0002:0000a3bc       ??_C@_0CF@CNPIEMED@cannot?5create?5?$CFs?5trigger?5on?5view@ 100b43bc     interop.obj
 0002:0000a3e4       ??_C@_0CO@GJNALGCE@cannot?5create?5INSTEAD?5OF?5trigger@ 100b43e4     interop.obj
 0002:0000a418       ??_C@_0EA@IJNEMIHP@INSERT?5INTO?5?$CFQ?4?$CFs?5VALUES?$CI?8trigge@ 100b4418     interop.obj
 0002:0000a458       ??_C@_0BN@JFPIJHCG@type?$DN?8trigger?8?5AND?5name?$DN?8?$CFq?8?$AA@ 100b4458     interop.obj
 0002:0000a478       ??_C@_0BE@ELCABEID@no?5such?5trigger?3?5?$CFS?$AA@ 100b4478     interop.obj
 0002:0000a48c       ??_C@_0O@JKBKLFDA@?9?9?5TRIGGER?5?$CFs?$AA@ 100b448c     interop.obj
 0002:0000a49c       ??_C@_0BD@IEIMFPKF@no?5such?5column?3?5?$CFs?$AA@ 100b449c     interop.obj
 0002:0000a4b0       ??_C@_0N@KMEMLEEO@rows?5updated?$AA@ 100b44b0     interop.obj
 0002:0000a4c0       ??_C@_07OLKPBLEA@_rowid_?$AA@ 100b44c0     interop.obj
 0002:0000a4c8       ??_C@_0CI@CPMJIPOI@cannot?5VACUUM?5from?5within?5a?5tran@ 100b44c8     interop.obj
 0002:0000a4f0       ??_C@_0CL@HKLPPLKM@cannot?5VACUUM?5?9?5SQL?5statements?5i@ 100b44f0     interop.obj
 0002:0000a51c       ??_C@_0CA@LDLCFKGD@ATTACH?5?8?3memory?3?8?5AS?5vacuum_db?$DL?$AA@ 100b451c     interop.obj
 0002:0000a53c       ??_C@_0BI@OOHLJPLG@ATTACH?5?8?8?5AS?5vacuum_db?$DL?$AA@ 100b453c     interop.obj
 0002:0000a554       ??_C@_0CB@NBNOHMDI@PRAGMA?5vacuum_db?4synchronous?$DNOFF@ 100b4554     interop.obj
 0002:0000a578       ??_C@_06KEOLADBC@BEGIN?$DL?$AA@ 100b4578     interop.obj
 0002:0000a580       ??_C@_0II@FEBAKHNN@SELECT?5?8CREATE?5TABLE?5vacuum_db?4?8@ 100b4580     interop.obj
 0002:0000a608       ??_C@_0GI@FEDHFMIE@SELECT?5?8CREATE?5INDEX?5vacuum_db?4?8@ 100b4608     interop.obj
 0002:0000a670       ??_C@_0HG@GKDDPPFI@SELECT?5?8CREATE?5UNIQUE?5INDEX?5vacu@ 100b4670     interop.obj
 0002:0000a6e8       ??_C@_0LI@KDJAMIMI@SELECT?5?8INSERT?5INTO?5vacuum_db?4?8?5@ 100b46e8     interop.obj
 0002:0000a7a0       ??_C@_0HB@CJENIKHO@SELECT?5?8DELETE?5FROM?5vacuum_db?4?8?5@ 100b47a0     interop.obj
 0002:0000a818       ??_C@_0JL@BNIMKHIL@SELECT?5?8INSERT?5INTO?5vacuum_db?4?8?5@ 100b4818     interop.obj
 0002:0000a8b8       ??_C@_0LI@DFGNFIOM@INSERT?5INTO?5vacuum_db?4sqlite_mas@ 100b48b8     interop.obj
 0002:0000a970       ??_C@_0BI@PDMEEOA@CREATE?5VIRTUAL?5TABLE?5?$CFT?$AA@ 100b4970     interop.obj
 0002:0000a988       ??_C@_0FI@IFIJAFLJ@UPDATE?5?$CFQ?4?$CFs?5SET?5type?$DN?8table?8?0?5n@ 100b4988     interop.obj
 0002:0000a9e0       ??_C@_0BL@DGMACLBE@name?$DN?8?$CFq?8?5AND?5type?$DN?8table?8?$AA@ 100b49e0     interop.obj
 0002:0000a9fc       ??_C@_0BO@DEKEKMPI@vtable?5constructor?5failed?3?5?$CFs?$AA@ 100b49fc     interop.obj
 0002:0000aa1c       ??_C@_0CO@NAIIFAKI@vtable?5constructor?5did?5not?5decla@ 100b4a1c     interop.obj
 0002:0000aa4c       ??_C@_06JIKFICKK@hidden?$AA@ 100b4a4c     interop.obj
 0002:0000aa54       ??_C@_07JJJNOAOL@?5hidden?$AA@ 100b4a54     interop.obj
 0002:0000aa5c       ??_C@_0BD@KBJCCNMM@no?5such?5module?3?5?$CFs?$AA@ 100b4a5c     interop.obj
 0002:0000aa70       ??_C@_0L@LOLDMHK@auto?9index?$AA@ 100b4a70     interop.obj
 0002:0000aa7c       ??_C@_0CO@KDPCLLKJ@table?5?$CFs?3?5xBestIndex?5returned?5an@ 100b4a7c     interop.obj
 0002:0000aaac       ??_C@_05LFNOAECD@?5AND?5?$AA@ 100b4aac     interop.obj
 0002:0000aab4       ??_C@_02GFKOMOKH@?5?$CI?$AA@ 100b4ab4     interop.obj
 0002:0000aab8       ??_C@_01NEMOKFLO@?$DN?$AA@ 100b4ab8     interop.obj
 0002:0000aabc       ??_C@_01PPODPGHN@?$DO?$AA@ 100b4abc     interop.obj
 0002:0000aac0       ??_C@_01MNNFJEPP@?$DM?$AA@ 100b4ac0     interop.obj
 0002:0000aac4       ??_C@_06GBNAAIDA@SEARCH?$AA@ 100b4ac4     interop.obj
 0002:0000aacc       ??_C@_04NAGNMPFG@SCAN?$AA@ 100b4acc     interop.obj
 0002:0000aad4       ??_C@_0P@OLOBPMPI@?$CFs?5SUBQUERY?5?$CFd?$AA@ 100b4ad4     interop.obj
 0002:0000aae4       ??_C@_0M@EHBHAICN@?$CFs?5TABLE?5?$CFs?$AA@ 100b4ae4     interop.obj
 0002:0000aaf0       ??_C@_08BNODOOIA@?$CFs?5AS?5?$CFs?$AA@ 100b4af0     interop.obj
 0002:0000aafc       ??_C@_09GCJGEEEO@COVERING?5?$AA@ 100b4afc     interop.obj
 0002:0000ab08       ??_C@_0L@COIPKBPM@AUTOMATIC?5?$AA@ 100b4b08     interop.obj
 0002:0000ab14       ??_C@_0BJ@EKHJMJEF@?$CFs?5USING?5?$CFs?$CFsINDEX?$CFs?$CFs?$CFs?$AA@ 100b4b14     interop.obj
 0002:0000ab30       ??_C@_0BN@POCKMKPK@?$CFs?5USING?5INTEGER?5PRIMARY?5KEY?$AA@ 100b4b30     interop.obj
 0002:0000ab50       ??_C@_0N@DDAPLKI@?$CFs?5?$CIrowid?$DN?$DP?$CJ?$AA@ 100b4b50     interop.obj
 0002:0000ab60       ??_C@_0BJ@POOJNAFN@?$CFs?5?$CIrowid?$DO?$DP?5AND?5rowid?$DM?$DP?$CJ?$AA@ 100b4b60     interop.obj
 0002:0000ab7c       ??_C@_0N@BBIFFEEG@?$CFs?5?$CIrowid?$DO?$DP?$CJ?$AA@ 100b4b7c     interop.obj
 0002:0000ab8c       ??_C@_0N@LLIMJMMN@?$CFs?5?$CIrowid?$DM?$DP?$CJ?$AA@ 100b4b8c     interop.obj
 0002:0000ab9c       ??_C@_0BN@GEIFLGHO@?$CFs?5VIRTUAL?5TABLE?5INDEX?5?$CFd?3?$CFs?$AA@ 100b4b9c     interop.obj
 0002:0000abbc       ??_C@_0BA@CEKLKPCJ@?$CFs?5?$CI?$HO?$CFlld?5rows?$CJ?$AA@ 100b4bbc     interop.obj
 0002:0000abcc       ??_C@_0BM@BLDEAGOK@at?5most?5?$CFd?5tables?5in?5a?5join?$AA@ 100b4bcc     interop.obj
 0002:0000abe8       ??_C@_0BF@CGOICHOE@cannot?5use?5index?3?5?$CFs?$AA@ 100b4be8     interop.obj
 0002:0000ac00       ??_C@_0BG@FMAEELCM@parser?5stack?5overflow?$AA@ 100b4c00     interop.obj
 0002:0000ac18       ??_C@_08FAFAADKO@set?5list?$AA@ 100b4c18     interop.obj
 0002:0000ac24       ??_C@_0BI@CBJKLAIG@near?5?$CC?$CFT?$CC?3?5syntax?5error?$AA@ 100b4c24     interop.obj
 0002:0000ac3c       ??_C@_0CC@BHLMPGNH@too?5many?5arguments?5on?5function?5?$CF@ 100b4c3c     interop.obj
 0002:0000ac60       ??_C@_0FP@BDHEAEAL@qualified?5table?5names?5are?5not?5al@ 100b4c60     interop.obj
 0002:0000acc0       ??_C@_0FE@ONDNFGPP@the?5INDEXED?5BY?5clause?5is?5not?5all@ 100b4cc0     interop.obj
 0002:0000ad18       ??_C@_0FF@IPEGLKPG@the?5NOT?5INDEXED?5clause?5is?5not?5al@ 100b4d18     interop.obj
 0002:0000ad70       ??_C@_09NCAJIFEE@interrupt?$AA@ 100b4d70     interop.obj
 0002:0000ad7c       ??_C@_0BJ@EMNEDDKJ@unrecognized?5token?3?5?$CC?$CFT?$CC?$AA@ 100b4d7c     interop.obj
 0002:0000ad98       ??_C@_06HBNONAG@create?$AA@ 100b4d98     interop.obj
 0002:0000ada0       ??_C@_04FGEHGIFJ@temp?$AA@ 100b4da0     interop.obj
 0002:0000ada8       ??_C@_09CAHPDAG@temporary?$AA@ 100b4da8     interop.obj
 0002:0000adb4       ??_C@_03JBJLGPFL@end?$AA@  100b4db4     interop.obj
 0002:0000adb8       ??_C@_07LFFDKBGI@explain?$AA@ 100b4db8     interop.obj
 0002:0000adc0       ??_C@_0DN@PGOGOMBM@2013?905?920?500?356?322?5118a3b35693b@ 100b4dc0     interop.obj
 0002:0000ae00       ??_C@_0EE@DHFGJPIC@unable?5to?5close?5due?5to?5unfinaliz@ 100b4e00     interop.obj
 0002:0000ae44       ??_C@_0O@BFJCFAAK@unknown?5error?$AA@ 100b4e44     interop.obj
 0002:0000ae54       ??_C@_0BG@MJDEINHO@abort?5due?5to?5ROLLBACK?$AA@ 100b4e54     interop.obj
 0002:0000ae6c       ??_C@_0DP@BDIELDAF@unable?5to?5delete?1modify?5user?9fun@ 100b4e6c     interop.obj
 0002:0000aeac       ??_C@_0BF@HAJMIPDB@unknown?5database?3?5?$CFs?$AA@ 100b4eac     interop.obj
 0002:0000aec8       ??_C@_0EE@IKACNBHK@unable?5to?5delete?1modify?5collatio@ 100b4ec8     interop.obj
 0002:0000af0c       ??_C@_09IPAEKDAI@localhost?$AA@ 100b4f0c     interop.obj
 0002:0000af18       ??_C@_0BM@COJKMEBB@invalid?5uri?5authority?3?5?$CF?4?$CKs?$AA@ 100b4f18     interop.obj
 0002:0000af34       ??_C@_05BDNCCAMC@cache?$AA@ 100b4f34     interop.obj
 0002:0000af3c       ??_C@_04GMGOKAFF@mode?$AA@ 100b4f3c     interop.obj
 0002:0000af44       ??_C@_06EBPNOMLE@access?$AA@ 100b4f44     interop.obj
 0002:0000af4c       ??_C@_0BE@CEDEHNFE@no?5such?5?$CFs?5mode?3?5?$CFs?$AA@ 100b4f4c     interop.obj
 0002:0000af60       ??_C@_0BI@PGEAHBFI@?$CFs?5mode?5not?5allowed?3?5?$CFs?$AA@ 100b4f60     interop.obj
 0002:0000af78       ??_C@_0BA@JNKNNOBA@no?5such?5vfs?3?5?$CFs?$AA@ 100b4f78     interop.obj
 0002:0000af88       ??_C@_05JJHANOIF@RTRIM?$AA@ 100b4f88     interop.obj
 0002:0000af90       ??_C@_04GHJNJNPO@main?$AA@ 100b4f90     interop.obj
 0002:0000af98       ??_C@_0CK@EFFGEIFI@database?5corruption?5at?5line?5?$CFd?5o@ 100b4f98     interop.obj
 0002:0000afc4       ??_C@_0BN@JFEBGPPP@misuse?5at?5line?5?$CFd?5of?5?$FL?$CF?410s?$FN?$AA@ 100b4fc4     interop.obj
 0002:0000afe4       ??_C@_0CH@CFKHNID@cannot?5open?5file?5at?5line?5?$CFd?5of?5?$FL@ 100b4fe4     interop.obj
 0002:0000b00c       ??_C@_0BM@OILBPENI@no?5such?5table?5column?3?5?$CFs?4?$CFs?$AA@ 100b500c     interop.obj
 0002:0000b028       ??_C@_0CF@JMBAPJDM@DROP?5TABLE?5IF?5EXISTS?5?$CFQ?4?8?$CFq_cont@ 100b5028     interop.obj
 0002:0000b050       ??_C@_0CG@MBAKJBDH@DROP?5TABLE?5IF?5EXISTS?5?$CFQ?4?8?$CFq_segm@ 100b5050     interop.obj
 0002:0000b078       ??_C@_0CE@ONKNGDLL@DROP?5TABLE?5IF?5EXISTS?5?$CFQ?4?8?$CFq_segd@ 100b5078     interop.obj
 0002:0000b09c       ??_C@_0CF@IDMMCBAD@DROP?5TABLE?5IF?5EXISTS?5?$CFQ?4?8?$CFq_docs@ 100b509c     interop.obj
 0002:0000b0c4       ??_C@_0CC@IOIKPJHP@DROP?5TABLE?5IF?5EXISTS?5?$CFQ?4?8?$CFq_stat@ 100b50c4     interop.obj
 0002:0000b0e8       ??_C@_08HBMBCGGI@__langid?$AA@ 100b50e8     interop.obj
 0002:0000b0f4       ??_C@_04OHJOFLHH@?$CFQ?0?5?$AA@ 100b50f4     interop.obj
 0002:0000b0fc       ??_C@_06ILOMELII@?$CFz?$CFQ?0?5?$AA@ 100b50fc     interop.obj
 0002:0000b104       ??_C@_0DG@KNNCMIAK@CREATE?5TABLE?5x?$CI?$CFs?5?$CFQ?5HIDDEN?0?5doc@ 100b5104     interop.obj
 0002:0000b140       ??_C@_0EN@BNJDGKOP@CREATE?5TABLE?5IF?5NOT?5EXISTS?5?$CFQ?4?8?$CF@ 100b5140     interop.obj
 0002:0000b190       ??_C@_0BK@ILPNCKDD@docid?5INTEGER?5PRIMARY?5KEY?$AA@ 100b5190     interop.obj
 0002:0000b1ac       ??_C@_0M@KFIBGJMD@?$CFz?0?5?8c?$CFd?$CFq?8?$AA@ 100b51ac     interop.obj
 0002:0000b1b8       ??_C@_0L@FGLBMJMC@?$CFz?0?5langid?$AA@ 100b51b8     interop.obj
 0002:0000b1c4       ??_C@_0CB@GGGOGPJJ@CREATE?5TABLE?5?$CFQ?4?8?$CFq_content?8?$CI?$CFs?$CJ@ 100b51c4     interop.obj
 0002:0000b1e8       ??_C@_0EI@JJJNEMPK@CREATE?5TABLE?5?$CFQ?4?8?$CFq_segments?8?$CIbl@ 100b51e8     interop.obj
 0002:0000b230       ??_C@_0JJ@EINNGPFL@CREATE?5TABLE?5?$CFQ?4?8?$CFq_segdir?8?$CIleve@ 100b5230     interop.obj
 0002:0000b2d0       ??_C@_0EE@MDIIHKIJ@CREATE?5TABLE?5?$CFQ?4?8?$CFq_docsize?8?$CIdoc@ 100b52d0     interop.obj
 0002:0000b314       ??_C@_0BE@JJENHHFJ@PRAGMA?5?$CFQ?4page_size?$AA@ 100b5314     interop.obj
 0002:0000b328       ??_C@_05KJDOPFGN@docid?$AA@ 100b5328     interop.obj
 0002:0000b330       ??_C@_0P@LFFPPLAI@?0?$CFs?$CIx?4?8c?$CFd?$CFq?8?$CJ?$AA@ 100b5330     interop.obj
 0002:0000b340       ??_C@_06CLEJICHF@langid?$AA@ 100b5340     interop.obj
 0002:0000b348       ??_C@_06HJELONEC@?0?5x?4?$CFQ?$AA@ 100b5348     interop.obj
 0002:0000b350       ??_C@_08NJPBOKA@?0?5x?4?8?$CFq?8?$AA@ 100b5350     interop.obj
 0002:0000b35c       ??_C@_08KMMJILGO@_content?$AA@ 100b535c     interop.obj
 0002:0000b368       ??_C@_0BH@DJGBFAID@?5FROM?5?8?$CFq?8?4?8?$CFq?$CFs?8?5AS?5x?$AA@ 100b5368     interop.obj
 0002:0000b380       ??_C@_06INGKMHGE@?0?$CFs?$CI?$DP?$CJ?$AA@ 100b5380     interop.obj
 0002:0000b388       ??_C@_03FEMMFMLJ@?0?5?$DP?$AA@ 100b5388     interop.obj
 0002:0000b38c       ??_C@_0BE@NJEPGLOD@SELECT?5?$CK?5FROM?5?$CFQ?4?$CFQ?$AA@ 100b538c     interop.obj
 0002:0000b3a0       ??_C@_08ENDKEOKI@tokenize?$AA@ 100b53a0     interop.obj
 0002:0000b3ac       ??_C@_09OEHDJMHN@matchinfo?$AA@ 100b53ac     interop.obj
 0002:0000b3b8       ??_C@_06CHGOAPND@prefix?$AA@ 100b53b8     interop.obj
 0002:0000b3c0       ??_C@_08EJNPIMGB@compress?$AA@ 100b53c0     interop.obj
 0002:0000b3cc       ??_C@_0L@IEAKODFB@uncompress?$AA@ 100b53cc     interop.obj
 0002:0000b3d8       ??_C@_07ICAJMOAO@content?$AA@ 100b53d8     interop.obj
 0002:0000b3e0       ??_C@_0L@KCJJAHCF@languageid?$AA@ 100b53e0     interop.obj
 0002:0000b3ec       ??_C@_0BL@LDDPBJJP@unrecognized?5parameter?3?5?$CFs?$AA@ 100b53ec     interop.obj
 0002:0000b408       ??_C@_04GJCOAOPN@fts3?$AA@ 100b5408     interop.obj
 0002:0000b410       ??_C@_0BL@LGOAFHOC@unrecognized?5matchinfo?3?5?$CFs?$AA@ 100b5410     interop.obj
 0002:0000b42c       ??_C@_03EFEGFOOI@asc?$AA@  100b542c     interop.obj
 0002:0000b430       ??_C@_04EBPADADD@desc?$AA@ 100b5430     interop.obj
 0002:0000b438       ??_C@_0BH@DEFIELBN@unrecognized?5order?3?5?$CFs?$AA@ 100b5438     interop.obj
 0002:0000b450       ??_C@_06MDDCAKGD@simple?$AA@ 100b5450     interop.obj
 0002:0000b458       ??_C@_0CD@HIKDEBHJ@error?5parsing?5prefix?5parameter?3?5@ 100b5458     interop.obj
 0002:0000b47c       ??_C@_0CJ@LIAMDBLK@missing?5?$CFs?5parameter?5in?5fts4?5con@ 100b547c     interop.obj
 0002:0000b4a8       ??_C@_0CG@BMNJKDFD@SELECT?51?5FROM?5?$CFQ?4?8?$CFq_stat?8?5WHERE@ 100b54a8     interop.obj
 0002:0000b4d0       ??_C@_04INMKNCEL@DESC?$AA@ 100b54d0     interop.obj
 0002:0000b4d8       ??_C@_03EILNJDJE@ASC?$AA@  100b54d8     interop.obj
 0002:0000b4dc       ??_C@_0BK@DAHJKJOI@SELECT?5?$CFs?5WHERE?5rowid?5?$DN?5?$DP?$AA@ 100b54dc     interop.obj
 0002:0000b4f8       ??_C@_0BM@EFGHBBLP@SELECT?5?$CFs?5ORDER?5BY?5rowid?5?$CFs?$AA@ 100b54f8     interop.obj
 0002:0000b514       ??_C@_0BN@HNFGPPAE@illegal?5first?5argument?5to?5?$CFs?$AA@ 100b5514     interop.obj
 0002:0000b534       ??_C@_03GONAGDMJ@?$DMb?$DO?$AA@ 100b5534     interop.obj
 0002:0000b538       ??_C@_04KPMLOGDO@?$DM?1b?$DO?$AA@ 100b5538     interop.obj
 0002:0000b540       ??_C@_0L@FNCHOAPK@?$DMb?$DO?4?4?4?$DM?1b?$DO?$AA@ 100b5540     interop.obj
 0002:0000b54c       ??_C@_0DA@BPKHEBAA@wrong?5number?5of?5arguments?5to?5fun@ 100b554c     interop.obj
 0002:0000b57c       ??_C@_07NLNCCKKF@snippet?$AA@ 100b557c     interop.obj
 0002:0000b584       ??_C@_07EALNHAIO@offsets?$AA@ 100b5584     interop.obj
 0002:0000b58c       ??_C@_08GHMAOHAP@optimize?$AA@ 100b558c     interop.obj
 0002:0000b598       ??_C@_0BA@OAEHOEOG@Index?5optimized?$AA@ 100b5598     interop.obj
 0002:0000b5a8       ??_C@_0BG@LMCLNKNA@Index?5already?5optimal?$AA@ 100b55a8     interop.obj
 0002:0000b5c0       ??_C@_0DF@DCFHAMLC@ALTER?5TABLE?5?$CFQ?4?8?$CFq_content?8?5?5REN@ 100b55c0     interop.obj
 0002:0000b5f8       ??_C@_0DF@DCOLKKAO@ALTER?5TABLE?5?$CFQ?4?8?$CFq_docsize?8?5?5REN@ 100b55f8     interop.obj
 0002:0000b630       ??_C@_0CP@CGFDJKNC@ALTER?5TABLE?5?$CFQ?4?8?$CFq_stat?8?5?5RENAME@ 100b5630     interop.obj
 0002:0000b660       ??_C@_0DG@DAAAGDKF@ALTER?5TABLE?5?$CFQ?4?8?$CFq_segments?8?5REN@ 100b5660     interop.obj
 0002:0000b698       ??_C@_0DE@LHKMPNFJ@ALTER?5TABLE?5?$CFQ?4?8?$CFq_segdir?8?5?5?5REN@ 100b5698     interop.obj
 0002:0000b6cc       ??_C@_06EDADNLPO@porter?$AA@ 100b56cc     interop.obj
 0002:0000b6d4       ??_C@_0P@ONNIBBGC@fts3_tokenizer?$AA@ 100b56d4     interop.obj
 0002:0000b6e4       ??_C@_04CGGPJIDK@fts4?$AA@ 100b56e4     interop.obj
 0002:0000b6ec       ??_C@_0DC@EHKCEINM@CREATE?5TABLE?5x?$CIterm?0?5col?0?5docume@ 100b56ec     interop.obj
 0002:0000b720       ??_C@_0CJ@KNMGIKGK@invalid?5arguments?5to?5fts4aux?5con@ 100b5720     interop.obj
 0002:0000b74c       ??_C@_07HLCPNFJI@fts4aux?$AA@ 100b574c     interop.obj
 0002:0000b754       ??_C@_0DE@GLAEHGBM@FTS?5expression?5tree?5is?5too?5large@ 100b5754     interop.obj
 0002:0000b788       ??_C@_0CB@FOEJOLMC@malformed?5MATCH?5expression?3?5?$FL?$CFs?$FN@ 100b5788     interop.obj
 0002:0000b7ac       ??_C@_02FCBLNKNB@ss?$AA@   100b57ac     interop.obj
 0002:0000b7b0       ??_C@_04NJPCGJPA@sess?$AA@ 100b57b0     interop.obj
 0002:0000b7b8       ??_C@_01KBJDNOO@i?$AA@     100b57b8     interop.obj
 0002:0000b7bc       ??_C@_03FNBCPGLE@sei?$AA@  100b57bc     interop.obj
 0002:0000b7c0       ??_C@_02FGCILAME@ee?$AA@   100b57c0     interop.obj
 0002:0000b7c4       ??_C@_03DMGJNGJO@dee?$AA@  100b57c4     interop.obj
 0002:0000b7c8       ??_C@_03IODMNJJN@gni?$AA@  100b57c8     interop.obj
 0002:0000b7cc       ??_C@_02FHOKNKPD@de?$AA@   100b57cc     interop.obj
 0002:0000b7d0       ??_C@_03BGFDOPOL@ate?$AA@  100b57d0     interop.obj
 0002:0000b7d4       ??_C@_02CPKALMIH@ta?$AA@   100b57d4     interop.obj
 0002:0000b7d8       ??_C@_03BGNDLCMN@ble?$AA@  100b57d8     interop.obj
 0002:0000b7dc       ??_C@_02BGLIBNIM@lb?$AA@   100b57dc     interop.obj
 0002:0000b7e0       ??_C@_03NJHJOKAO@ize?$AA@  100b57e0     interop.obj
 0002:0000b7e4       ??_C@_02ONOHBLIF@zi?$AA@   100b57e4     interop.obj
 0002:0000b7e8       ??_C@_07HAPEHOGG@lanoita?$AA@ 100b57e8     interop.obj
 0002:0000b7f0       ??_C@_04MLFEDMFA@tion?$AA@ 100b57f0     interop.obj
 0002:0000b7f8       ??_C@_06KEDPLIML@lanoit?$AA@ 100b57f8     interop.obj
 0002:0000b800       ??_C@_04OBONJKHE@ence?$AA@ 100b5800     interop.obj
 0002:0000b808       ??_C@_04NOKPDMPL@icne?$AA@ 100b5808     interop.obj
 0002:0000b810       ??_C@_04BEGNDMLE@ance?$AA@ 100b5810     interop.obj
 0002:0000b818       ??_C@_04LKMDPJPP@icna?$AA@ 100b5818     interop.obj
 0002:0000b820       ??_C@_04FLGOIBBE@rezi?$AA@ 100b5820     interop.obj
 0002:0000b828       ??_C@_04IBMNHKNC@igol?$AA@ 100b5828     interop.obj
 0002:0000b830       ??_C@_03IOJDKDAL@ilb?$AA@  100b5830     interop.obj
 0002:0000b834       ??_C@_02IAODKDFB@al?$AA@   100b5834     interop.obj
 0002:0000b838       ??_C@_04OBCEDNMH@illa?$AA@ 100b5838     interop.obj
 0002:0000b840       ??_C@_03NLFJHNAK@ent?$AA@  100b5840     interop.obj
 0002:0000b844       ??_C@_05IDJKNEIB@iltne?$AA@ 100b5844     interop.obj
 0002:0000b84c       ??_C@_01KGKMHCOC@e?$AA@    100b584c     interop.obj
 0002:0000b850       ??_C@_03MBNCDFMM@ile?$AA@  100b5850     interop.obj
 0002:0000b854       ??_C@_03OLNGEHDI@ous?$AA@  100b5854     interop.obj
 0002:0000b858       ??_C@_05PENBEICD@ilsuo?$AA@ 100b5858     interop.obj
 0002:0000b860       ??_C@_07GPCIBLIA@noitazi?$AA@ 100b5860     interop.obj
 0002:0000b868       ??_C@_05OJBPCAJ@noita?$AA@ 100b5868     interop.obj
 0002:0000b870       ??_C@_04PGJEMGHC@rota?$AA@ 100b5870     interop.obj
 0002:0000b878       ??_C@_05DPCAAIOM@msila?$AA@ 100b5878     interop.obj
 0002:0000b880       ??_C@_03NAGDBDGK@ive?$AA@  100b5880     interop.obj
 0002:0000b884       ??_C@_07PDACOIKL@ssenevi?$AA@ 100b5884     interop.obj
 0002:0000b88c       ??_C@_03FLIEAGCM@ful?$AA@  100b588c     interop.obj
 0002:0000b890       ??_C@_07LNEAFLH@ssenluf?$AA@ 100b5890     interop.obj
 0002:0000b898       ??_C@_07NCGMPJDH@ssensuo?$AA@ 100b5898     interop.obj
 0002:0000b8a0       ??_C@_05BGJBJGOK@itila?$AA@ 100b58a0     interop.obj
 0002:0000b8a8       ??_C@_05MPPJDKEE@itivi?$AA@ 100b58a8     interop.obj
 0002:0000b8b0       ??_C@_06BJBBMCGN@itilib?$AA@ 100b58b0     interop.obj
 0002:0000b8b8       ??_C@_02JGIOOCG@ic?$AA@    100b58b8     interop.obj
 0002:0000b8bc       ??_C@_05GHGCLDEL@etaci?$AA@ 100b58bc     interop.obj
 0002:0000b8c4       ??_C@_05JKGPHDJ@evita?$AA@ 100b58c4     interop.obj
 0002:0000b8cc       ??_C@_05NOGDOIPA@ezila?$AA@ 100b58cc     interop.obj
 0002:0000b8d4       ??_C@_05NFBEFLNP@itici?$AA@ 100b58d4     interop.obj
 0002:0000b8dc       ??_C@_04BICLKHFP@laci?$AA@ 100b58dc     interop.obj
 0002:0000b8e4       ??_C@_03MONGAOMC@luf?$AA@  100b58e4     interop.obj
 0002:0000b8e8       ??_C@_04ELEHNCGN@ssen?$AA@ 100b58e8     interop.obj
 0002:0000b8f0       ??_C@_05KMPBBIAH@tneme?$AA@ 100b58f0     interop.obj
 0002:0000b8f8       ??_C@_04HADJNCPM@tnem?$AA@ 100b58f8     interop.obj
 0002:0000b900       ??_C@_03GACFGOOA@tne?$AA@  100b5900     interop.obj
 0002:0000b904       ??_C@_03PCPGPMCA@noi?$AA@  100b5904     interop.obj
 0002:0000b908       ??_C@_03PNFNLNLI@eta?$AA@  100b5908     interop.obj
 0002:0000b90c       ??_C@_03HPFCIIAI@iti?$AA@  100b590c     interop.obj
 0002:0000b910       ??_C@_0BH@PMNILKKF@argument?5type?5mismatch?$AA@ 100b5910     interop.obj
 0002:0000b928       ??_C@_0BG@CPKCHLPM@unknown?5tokenizer?3?5?$CFs?$AA@ 100b5928     interop.obj
 0002:0000b940       ??_C@_0BC@MIGNHNIC@unknown?5tokenizer?$AA@ 100b5940     interop.obj
 0002:0000b954       ??_C@_0DD@EDFEHGLO@CREATE?5TABLE?5x?$CIinput?0?5token?0?5sta@ 100b5954     interop.obj
 0002:0000b988       ??_C@_0N@MJBJKOEF@fts3tokenize?$AA@ 100b5988     interop.obj
 0002:0000b998       ??_C@_0CM@CCEIGCNK@DELETE?5FROM?5?$CFQ?4?8?$CFq_content?8?5WHER@ 100b5998     interop.obj
 0002:0000b9c8       ??_C@_0EE@NIHFGMMI@SELECT?5NOT?5EXISTS?$CISELECT?5docid?5F@ 100b59c8     interop.obj
 0002:0000ba0c       ??_C@_0BM@PEBOBMKF@DELETE?5FROM?5?$CFQ?4?8?$CFq_content?8?$AA@ 100b5a0c     interop.obj
 0002:0000ba28       ??_C@_0BN@EILBLEDC@DELETE?5FROM?5?$CFQ?4?8?$CFq_segments?8?$AA@ 100b5a28     interop.obj
 0002:0000ba48       ??_C@_0BL@DOPLACGJ@DELETE?5FROM?5?$CFQ?4?8?$CFq_segdir?8?$AA@ 100b5a48     interop.obj
 0002:0000ba64       ??_C@_0BM@OLMCMEJK@DELETE?5FROM?5?$CFQ?4?8?$CFq_docsize?8?$AA@ 100b5a64     interop.obj
 0002:0000ba80       ??_C@_0BJ@HOMEFFOK@DELETE?5FROM?5?$CFQ?4?8?$CFq_stat?8?$AA@ 100b5a80     interop.obj
 0002:0000ba9c       ??_C@_0BI@EHNAAIOC@SELECT?5?$CFs?5WHERE?5rowid?$DN?$DP?$AA@ 100b5a9c     interop.obj
 0002:0000bab8       ??_C@_0EB@JLFIAJAO@SELECT?5?$CISELECT?5max?$CIidx?$CJ?5FROM?5?$CFQ?4@ 100b5ab8     interop.obj
 0002:0000bafc       ??_C@_0DL@MFGEIOD@REPLACE?5INTO?5?$CFQ?4?8?$CFq_segments?8?$CIbl@ 100b5afc     interop.obj
 0002:0000bb38       ??_C@_0EE@PDNODLPC@SELECT?5coalesce?$CI?$CISELECT?5max?$CIbloc@ 100b5b38     interop.obj
 0002:0000bb7c       ??_C@_0DA@CMKKFBOL@REPLACE?5INTO?5?$CFQ?4?8?$CFq_segdir?8?5VALU@ 100b5b7c     interop.obj
 0002:0000bbb0       ??_C@_0HA@JJLMMHPL@SELECT?5idx?0?5start_block?0?5leaves_@ 100b5bb0     interop.obj
 0002:0000bc20       ??_C@_0IH@CHFFJLEM@SELECT?5idx?0?5start_block?0?5leaves_@ 100b5c20     interop.obj
 0002:0000bca8       ??_C@_0DE@JFBNLGCM@SELECT?5count?$CI?$CK?$CJ?5FROM?5?$CFQ?4?8?$CFq_segd@ 100b5ca8     interop.obj
 0002:0000bce0       ??_C@_0EC@NJOFEFNB@SELECT?5max?$CIlevel?$CJ?5FROM?5?$CFQ?4?8?$CFq_se@ 100b5ce0     interop.obj
 0002:0000bd24       ??_C@_0CL@LJFNCCFI@DELETE?5FROM?5?$CFQ?4?8?$CFq_segdir?8?5WHERE@ 100b5d24     interop.obj
 0002:0000bd50       ??_C@_0DL@FMDHOPDD@DELETE?5FROM?5?$CFQ?4?8?$CFq_segments?8?5WHE@ 100b5d50     interop.obj
 0002:0000bd8c       ??_C@_0CH@KOJCNEKB@INSERT?5INTO?5?$CFQ?4?8?$CFq_content?8?5VALU@ 100b5d8c     interop.obj
 0002:0000bdb4       ??_C@_0CM@JNJGJAMO@DELETE?5FROM?5?$CFQ?4?8?$CFq_docsize?8?5WHER@ 100b5db4     interop.obj
 0002:0000bde0       ??_C@_0CJ@LFPHJFLB@REPLACE?5INTO?5?$CFQ?4?8?$CFq_docsize?8?5VAL@ 100b5de0     interop.obj
 0002:0000be0c       ??_C@_0CP@OHAINFIB@SELECT?5size?5FROM?5?$CFQ?4?8?$CFq_docsize?8@ 100b5e0c     interop.obj
 0002:0000be3c       ??_C@_0CK@NBNCGFLN@SELECT?5value?5FROM?5?$CFQ?4?8?$CFq_stat?8?5W@ 100b5e3c     interop.obj
 0002:0000be68       ??_C@_0CG@FNKMPDFF@REPLACE?5INTO?5?$CFQ?4?8?$CFq_stat?8?5VALUES@ 100b5e68     interop.obj
 0002:0000be90       ??_C@_0DH@BCKMOPJL@DELETE?5FROM?5?$CFQ?4?8?$CFq_segdir?8?5WHERE@ 100b5e90     interop.obj
 0002:0000bec8       ??_C@_0DH@FMGMEHPE@SELECT?5DISTINCT?5level?5?1?5?$CI1024?5?$CK?5@ 100b5ec8     interop.obj
 0002:0000bf00       ??_C@_0GJ@LOLHDHAJ@SELECT?5level?5FROM?5?$CFQ?4?8?$CFq_segdir?8@ 100b5f00     interop.obj
 0002:0000bf70       ??_C@_0GH@DPJIHEGC@SELECT?52?5?$CK?5total?$CI1?5?$CL?5leaves_end_@ 100b5f70     interop.obj
 0002:0000bfd8       ??_C@_0DH@DBLDPJEO@DELETE?5FROM?5?$CFQ?4?8?$CFq_segdir?8?5WHERE@ 100b5fd8     interop.obj
 0002:0000c010       ??_C@_0DK@IIIPEDBM@UPDATE?5?$CFQ?4?8?$CFq_segdir?8?5SET?5idx?5?$DN?5@ 100b6010     interop.obj
 0002:0000c050       ??_C@_0GL@HMGCAOBI@SELECT?5idx?0?5start_block?0?5leaves_@ 100b6050     interop.obj
 0002:0000c0c0       ??_C@_0EP@DBFLEABP@UPDATE?5?$CFQ?4?8?$CFq_segdir?8?5SET?5start_@ 100b60c0     interop.obj
 0002:0000c110       ??_C@_0EB@INOOLLID@SELECT?51?5FROM?5?$CFQ?4?8?$CFq_segments?8?5W@ 100b6110     interop.obj
 0002:0000c154       ??_C@_0DM@EICDJEDC@SELECT?5idx?5FROM?5?$CFQ?4?8?$CFq_segdir?8?5W@ 100b6154     interop.obj
 0002:0000c190       ??_C@_0DA@ONAEGFD@SELECT?5max?$CI?5level?5?$CF?$CF?51024?5?$CJ?5FROM@ 100b6190     interop.obj
 0002:0000c1c0       ??_C@_0M@FNPINBNL@?$CFs_segments?$AA@ 100b61c0     interop.obj
 0002:0000c1cc       ??_C@_05PIBOEKAB@block?$AA@ 100b61cc     interop.obj
 0002:0000c1d4       ??_C@_09GMKLHBDP@SELECT?5?$CFs?$AA@ 100b61d4     interop.obj
 0002:0000c1e0       ??_C@_07NPFKDALJ@rebuild?$AA@ 100b61e0     interop.obj
 0002:0000c1e8       ??_C@_0BA@DICCLPBL@integrity?9check?$AA@ 100b61e8     interop.obj
 0002:0000c1f8       ??_C@_06NBNMKOCN@merge?$DN?$AA@ 100b61f8     interop.obj
 0002:0000c200       ??_C@_0L@CIJOHFF@automerge?$DN?$AA@ 100b6200     interop.obj
 0002:0000c20c       ??_C@_0P@LDDNGGJP@SAVEPOINT?5fts3?$AA@ 100b620c     interop.obj
 0002:0000c21c       ??_C@_0N@MGHAAGPN@RELEASE?5fts3?$AA@ 100b621c     interop.obj
 0002:0000c22c       ??_C@_0BB@FILGCGJ@ROLLBACK?5TO?5fts3?$AA@ 100b622c     interop.obj
 0002:0000c240       ??_C@_0CD@HGBIMAPM@unrecognized?5matchinfo?5request?3?5@ 100b6240     interop.obj
 0002:0000c264       ??_C@_0N@CAAIIPHA@?$CFd?5?$CFd?5?$CFd?5?$CFd?5?$AA@ 100b6264     interop.obj
 0002:0000c274       ??_C@_03BIPDAGPI@pcx?$AA@  100b6274     interop.obj
 0002:0000c278       ??_C@_0FC@PCOGINLL@DROP?5TABLE?5?8?$CFq?8?4?8?$CFq_node?8?$DLDROP?5T@ 100b6278     interop.obj
 0002:0000c2d0       ??_C@_0JB@OPIDJEFG@ALTER?5TABLE?5?$CFQ?4?8?$CFq_node?8?5?5?5RENAM@ 100b62d0     interop.obj
 0002:0000c368       ??_C@_0BAM@HLINMDBI@CREATE?5TABLE?5?$CC?$CFw?$CC?4?$CC?$CFw_node?$CC?$CInode@ 100b6368     interop.obj
 0002:0000c474       ??_C@_0DJ@FJHIAAMI@SELECT?5length?$CIdata?$CJ?5FROM?5?8?$CFq?8?4?8?$CF@ 100b6474     interop.obj
 0002:0000c4b0       ??_C@_0CL@JLGEGOKF@Wrong?5number?5of?5columns?5for?5an?5r@ 100b64b0     interop.obj
 0002:0000c4dc       ??_C@_0CD@LNBABDIB@Too?5few?5columns?5for?5an?5rtree?5tab@ 100b64dc     interop.obj
 0002:0000c500       ??_C@_0CE@OFDKEPLE@Too?5many?5columns?5for?5an?5rtree?5ta@ 100b6500     interop.obj
 0002:0000c524       ??_C@_0BC@EHLBCEFD@CREATE?5TABLE?5x?$CI?$CFs?$AA@ 100b6524     interop.obj
 0002:0000c538       ??_C@_06OMDHIKNA@?$CFs?0?5?$CFs?$AA@ 100b6538     interop.obj
 0002:0000c540       ??_C@_04ECFIDFLD@?$CFs?$CJ?$DL?$AA@ 100b6540     interop.obj
 0002:0000c548       ??_C@_03HDKIMHPH@?5?$CFf?$AA@ 100b6548     interop.obj
 0002:0000c54c       ??_C@_07CEKPNMEE@?$CFs?5?$HL?$CFs?$HN?$AA@ 100b654c     interop.obj
 0002:0000c554       ??_C@_04OMBFFHIC@?$HL?$CFs?$HN?$AA@ 100b6554     interop.obj
 0002:0000c55c       ??_C@_0CB@GBDNHMJO@Invalid?5argument?5to?5rtreedepth?$CI?$CJ@ 100b655c     interop.obj
 0002:0000c580       ??_C@_09DOFHOJNE@rtreenode?$AA@ 100b6580     interop.obj
 0002:0000c58c       ??_C@_0L@FBAJCMD@rtreedepth?$AA@ 100b658c     interop.obj
 0002:0000c598       ??_C@_05JDCFEKKH@rtree?$AA@ 100b6598     interop.obj
 0002:0000c5a0       ??_C@_09BLHENEJI@rtree_i32?$AA@ 100b65a0     interop.obj
 0002:0000c5ac       ??_C@_0CB@CGLCOOIM@virtual?5table?5was?5disposed?3?5?$CC?$CFs?$CC@ 100b65ac     interop.obj
 0002:0000c5d0       ??_C@_0N@HPOBCAGP@domain?5error?$AA@ 100b65d0     interop.obj
 0002:0000c5e0       ??_C@_1FO@GBKEFGLF@?$AAM?$AAi?$AAc?$AAr?$AAo?$AAs?$AAo?$AAf?$AAt?$AA?5?$AAE?$AAn?$AAh?$AAa?$AAn?$AAc?$AAe?$AAd?$AA?5?$AAC?$AAr?$AAy?$AAp?$AAt?$AAo?$AAg?$AAr?$AAa?$AAp?$AAh?$AAi?$AAc@ 100b65e0     interop.obj
 0002:0000c640       ??_C@_0CF@PDNGJJHH@Cryptographic?5provider?5not?5avail@ 100b6640     interop.obj
 0002:0000c668       __real@400921fb54442d18    100b6668      CIL library: CIL module
 0002:0000c670       __real@4066800000000000    100b6670      CIL library: CIL module
 0002:0000c678       __real@3ff0000000000000    100b6678      CIL library: CIL module
 0002:0000c680       __real@3fe0000000000000    100b6680      CIL library: CIL module
 0002:0000c688       __real@0000000000000000    100b6688      CIL library: CIL module
 0002:0000c690       __real@40d3880000000000    100b6690      CIL library: CIL module
 0002:0000c698       __real@4014000000000000    100b6698      CIL library: CIL module
 0002:0000c6a0       __real@4000000000000000    100b66a0      CIL library: CIL module
 0002:0000c6a8       __real@411e848000000000    100b66a8      CIL library: CIL module
 0002:0000c6b0       __real@4024000000000000    100b66b0      CIL library: CIL module
 0002:0000c6b8       __real@4480f0cf064dd592    100b66b8      CIL library: CIL module
 0002:0000c6c0       __real@7ff0000000000000    100b66c0      CIL library: CIL module
 0002:0000c6c8       __real@7fe1ccf385ebc8a0    100b66c8      CIL library: CIL module
 0002:0000c6d0       __real@8000000000000000    100b66d0      CIL library: CIL module
 0002:0000c6d8       __real@4194997000000000    100b66d8      CIL library: CIL module
 0002:0000c6e0       __real@403e99a027525461    100b66e0      CIL library: CIL module
 0002:0000c6e8       __real@4076d40000000000    100b66e8      CIL library: CIL module
 0002:0000c6f0       __real@405e866666666666    100b66f0      CIL library: CIL module
 0002:0000c6f8       __real@40e1d58800000000    100b66f8      CIL library: CIL module
 0002:0000c700       __real@413c7dd040000000    100b6700      CIL library: CIL module
 0002:0000c708       __real@c08f400000000000    100b6708      CIL library: CIL module
 0002:0000c710       __real@4097d20000000000    100b6710      CIL library: CIL module
 0002:0000c718       __real@408f400000000000    100b6718      CIL library: CIL module
 0002:0000c720       __real@4048000000000000    100b6720      CIL library: CIL module
 0002:0000c728       __real@3ff0000020000000    100b6728      CIL library: CIL module
 0002:0000c730       __real@3fefffffc0000000    100b6730      CIL library: CIL module
 0002:0000c738       __real@3e45798ee2308c3a    100b6738      CIL library: CIL module
 0002:0000c740       __real@4197d78400000000    100b6740      CIL library: CIL module
 0002:0000c748       __real@4d384f03e93ff9f5    100b6748      CIL library: CIL module
 0002:0000c750       __real@54b249ad2594c37d    100b6750      CIL library: CIL module
 0002:0000c758       __real@3fb999999999999a    100b6758      CIL library: CIL module
 0002:0000c760       __real@41f0000000000000    100b6760      CIL library: CIL module
 0002:0000c768       __real@413e848000000000    100b6768      CIL library: CIL module
 0002:0000c770       __real@43e0000000000000    100b6770      CIL library: CIL module
 0002:0000c778       __real@4076d00000000000    100b6778      CIL library: CIL module
 0002:0000c780       __real@403e000000000000    100b6780      CIL library: CIL module
 0002:0000c788       __real@40ed4c0000000000    100b6788      CIL library: CIL module
 0002:0000c790       __real@414b774000000000    100b6790      CIL library: CIL module
 0002:0000c798       __real@bfe0000000000000    100b6798      CIL library: CIL module
 0002:0000c7a0       __real@401c000000000000    100b67a0      CIL library: CIL module
 0002:0000c7a8       __real@3fd0000000000000    100b67a8      CIL library: CIL module
 0002:0000c7b0       __real@404dffdf3b645a1d    100b67b0      CIL library: CIL module
 0002:0000c7b8       __real@4010000000000000    100b67b8      CIL library: CIL module
 0002:0000c7c0       __real@4008000000000000    100b67c0      CIL library: CIL module
 0002:0000c7c8       __real@547d42aea2879f2e    100b67c8      CIL library: CIL module
 0002:0000c7d0       __real@546d42aea2879f2e    100b67d0      CIL library: CIL module
 0002:0000c7d8       __real@4059000000000000    100b67d8      CIL library: CIL module
 0002:0000c83a       __OP_SINHjmptab            100b683a     LIBCMT:_87trigh_.obj
 0002:0000c85a       __OP_COSHjmptab            100b685a     LIBCMT:_87trigh_.obj
 0002:0000c87a       __OP_TANHjmptab            100b687a     LIBCMT:_87trigh_.obj
 0002:0000df70       __indefinite               100b7f70     LIBCMT:_87disp_.obj
 0002:0000df7a       __piby2                    100b7f7a     LIBCMT:_87disp_.obj
 0002:0000dfa8       __DEFAULT_CW_in_mem        100b7fa8     LIBCMT:_common_.obj
 0002:0000dfaa       __pi_by_2_to_61            100b7faa     LIBCMT:_common_.obj
 0002:0000e8f0       __infinity                 100b88f0     LIBCMT:_87tran_.obj
 0002:0000e8fa       __minfinity                100b88fa     LIBCMT:_87tran_.obj
 0002:0000e904       __logemax                  100b8904     LIBCMT:_87tran_.obj
 0002:0000e92a       __OP_EXPjmptab             100b892a     LIBCMT:_87tran_.obj
 0002:0000e950       __OP_ATAN2jmptab           100b8950     LIBCMT:_87triga_.obj
 0002:000173a0       __atan_table               100c13a0     LIBCMT:_atan_table_.obj
 0002:00018bb0       __load_config_used         100c2bb0     LIBCMT:loadcfg.obj
 0002:00018c80       ___safe_se_handler_table   100c2c80     <linker-defined>
 0002:00018c8c       ___rtc_iaa                 100c2c8c     LIBCMT:_initsect_.obj
 0002:00018c90       ___rtc_izz                 100c2c90     LIBCMT:_initsect_.obj
 0002:00018c94       ___rtc_taa                 100c2c94     LIBCMT:_initsect_.obj
 0002:00018c98       ___rtc_tzz                 100c2c98     LIBCMT:_initsect_.obj
 0002:00018fb4       __IMPORT_DESCRIPTOR_KERNEL32 100c2fb4     kernel32:KERNEL32.dll
 0002:00018fc8       __IMPORT_DESCRIPTOR_ADVAPI32 100c2fc8     advapi32:ADVAPI32.dll
 0002:00018fdc       __NULL_IMPORT_DESCRIPTOR   100c2fdc     kernel32:KERNEL32.dll
 0003:00000170       ___security_cookie         100c6170     LIBCMT:gs_cookie.obj
 0003:00000174       ___security_cookie_complement 100c6174     LIBCMT:gs_cookie.obj
 0003:00000198       __timezone                 100c6198     LIBCMT:timeset.obj
 0003:0000019c       __daylight                 100c619c     LIBCMT:timeset.obj
 0003:000001a0       __dstbias                  100c61a0     LIBCMT:timeset.obj
 0003:00000228       __tzname                   100c6228     LIBCMT:timeset.obj
 0003:00000230       __sys_errlist              100c6230     LIBCMT:syserr.obj
 0003:000002e0       __sys_nerr                 100c62e0     LIBCMT:syserr.obj
 0003:000002e4       ___flsindex                100c62e4     LIBCMT:tidtable.obj
 0003:000002e8       ___getvalueindex           100c62e8     LIBCMT:tidtable.obj
 0003:000002f0       ___initialmbcinfo          100c62f0     LIBCMT:mbctype.obj
 0003:00000510       __mbctype                  100c6510     LIBCMT:mbctype.obj
 0003:00000618       __mbcasemap                100c6618     LIBCMT:mbctype.obj
 0003:00000718       ___ptmbcinfo               100c6718     LIBCMT:mbctype.obj
 0003:00000810       ___globallocalestatus      100c6810     LIBCMT:glstatus.obj
 0003:00000814       ___clocalestr              100c6814     LIBCMT:nlsdata2.obj
 0003:00000818       ___lc_time_c               100c6818     LIBCMT:nlsdata2.obj
 0003:00000980       ___initiallocinfo          100c6980     LIBCMT:nlsdata2.obj
 0003:00000a58       ___ptlocinfo               100c6a58     LIBCMT:nlsdata2.obj
 0003:00000a5c       ___initiallocalestructinfo 100c6a5c     LIBCMT:nlsdata2.obj
 0003:00000a68       __iob                      100c6a68     LIBCMT:_file.obj
 0003:00000ce8       ___nullstring              100c6ce8     LIBCMT:output.obj
 0003:00000cec       ___wnullstring             100c6cec     LIBCMT:output.obj
 0003:00000cf0       ___badioinfo               100c6cf0     LIBCMT:ioinit.obj
 0003:00000d30       __matherr_flag             100c6d30     LIBCMT:_matherr_.obj
 0003:00000d34       __fltused                  100c6d34     LIBCMT:_fpinit_.obj
 0003:00000d38       __ldused                   100c6d38     LIBCMT:_fpinit_.obj
 0003:00000e28       __d_inf                    100c6e28     LIBCMT:_util_.obj
 0003:00000e30       __d_ind                    100c6e30     LIBCMT:_util_.obj
 0003:00000e38       __d_max                    100c6e38     LIBCMT:_util_.obj
 0003:00000e40       __d_min                    100c6e40     LIBCMT:_util_.obj
 0003:00000e48       __d_mzero                  100c6e48     LIBCMT:_util_.obj
 0003:00000f90       __lpdays                   100c6f90     LIBCMT:days.obj
 0003:00000fc4       __days                     100c6fc4     LIBCMT:days.obj
 0003:00001000       ___lconv_static_decimal    100c7000     LIBCMT:lconv.obj
 0003:00001004       ___lconv_static_W_decimal  100c7004     LIBCMT:lconv.obj
 0003:00001008       ___lconv_c                 100c7008     LIBCMT:lconv.obj
 0003:00001058       ___lconv                   100c7058     LIBCMT:lconv.obj
 0003:0000105c       __pctype                   100c705c     LIBCMT:ctype.obj
 0003:00001060       __pwctype                  100c7060     LIBCMT:ctype.obj
 0003:00001070       ___mb_cur_max              100c7070     LIBCMT:nlsdata1.obj
 0003:00001074       ___decimal_point           100c7074     LIBCMT:nlsdata1.obj
 0003:00001078       ___decimal_point_length    100c7078     LIBCMT:nlsdata1.obj
 0003:00001080       __cfltcvt_tab              100c7080     LIBCMT:cmiscdat.obj
 0003:000010b0       __NLG_Destination          100c70b0     LIBCMT:exsup.obj
 0003:000010c0       ___abort_behavior          100c70c0     LIBCMT:abort.obj
 0003:00001100       __confh                    100c7100     LIBCMT:initcon.obj
 0003:00001108       __pow10pos                 100c7108     LIBCMT:_constpow_.obj
 0003:00001268       __pow10neg                 100c7268     LIBCMT:_constpow_.obj
 0003:00014880       __half                     100da880     LIBCMT:_pow_.obj
 0003:00014908       __aenvptr                  100da908     LIBCMT:dllcrt0.obj
 0003:0001490c       __wenvptr                  100da90c     LIBCMT:dllcrt0.obj
 0003:00014910       ___error_mode              100da910     LIBCMT:dllcrt0.obj
 0003:00014914       ___app_type                100da914     LIBCMT:dllcrt0.obj
 0003:00014c40       __crtheap                  100dac40     LIBCMT:heapinit.obj
 0003:00014c44       ___pInvalidArgHandler      100dac44     LIBCMT:invarg.obj
 0003:00014d00       __maxwait                  100dad00     LIBCMT:crtheap.obj
 0003:00014d04       _gpFlsAlloc                100dad04     LIBCMT:tidtable.obj
 0003:00014d08       _gpFlsGetValue             100dad08     LIBCMT:tidtable.obj
 0003:00014d0c       _gpFlsSetValue             100dad0c     LIBCMT:tidtable.obj
 0003:00014d10       _gpFlsFree                 100dad10     LIBCMT:tidtable.obj
 0003:00014d18       ___mbulinfo                100dad18     LIBCMT:mbctype.obj
 0003:00014d24       ___mbcodepage              100dad24     LIBCMT:mbctype.obj
 0003:00014d28       ___ismbcodepage            100dad28     LIBCMT:mbctype.obj
 0003:00014d2c       ___mblcid                  100dad2c     LIBCMT:mbctype.obj
 0003:00014d30       ___locale_changed          100dad30     LIBCMT:setlocal.obj
 0003:00014d34       __cflush                   100dad34     LIBCMT:_file.obj
 0003:00014d38       __stdbuf                   100dad38     LIBCMT:_sftbuf.obj
 0003:00014d40       __umaskval                 100dad40     LIBCMT:crt0dat.obj
 0003:00014d44       ___argc                    100dad44     LIBCMT:crt0dat.obj
 0003:00014d48       ___argv                    100dad48     LIBCMT:crt0dat.obj
 0003:00014d4c       ___wargv                   100dad4c     LIBCMT:crt0dat.obj
 0003:00014d50       __environ                  100dad50     LIBCMT:crt0dat.obj
 0003:00014d54       ___initenv                 100dad54     LIBCMT:crt0dat.obj
 0003:00014d58       __wenviron                 100dad58     LIBCMT:crt0dat.obj
 0003:00014d5c       ___winitenv                100dad5c     LIBCMT:crt0dat.obj
 0003:00014d60       __pgmptr                   100dad60     LIBCMT:crt0dat.obj
 0003:00014d64       __wpgmptr                  100dad64     LIBCMT:crt0dat.obj
 0003:00014d68       __exitflag                 100dad68     LIBCMT:crt0dat.obj
 0003:00014d6c       __C_Termination_Done       100dad6c     LIBCMT:crt0dat.obj
 0003:00014d70       __C_Exit_Done              100dad70     LIBCMT:crt0dat.obj
 0003:00014e80       ___fastflag                100dae80     LIBCMT:_fpinit_.obj
 0003:00014e84       ?_pnhHeap@@3P6AHI@ZA       100dae84     LIBCMT:handler.obj
 0003:00014e88       __newmode                  100dae88     LIBCMT:_newmode.obj
 0003:00014fe0       ___lconv_static_null       100dafe0     LIBCMT:lconv.obj
 0003:00014fe4       ___lconv_static_W_null     100dafe4     LIBCMT:lconv.obj
 0003:00014fe8       ?__pInconsistency@@3P6AXXZA 100dafe8     LIBCMT:hooks.obj
 0003:00015004       ___pPurecall               100db004     LIBCMT:inithelp.obj
 0003:00015644       __outputformat             100db644     LIBCMT:outputformat.obj
 0003:00015914       _sqlite3_api               100db914     sqlite3_unicode.obj
 0003:00015a68       _sqlite3_temp_directory    100dba68     interop.obj
 0003:00015a6c       _sqlite3_data_directory    100dba6c     interop.obj
 0003:00015a70       _g_hProvider               100dba70     interop.obj
 0003:00015a74       __debugger_hook_dummy      100dba74     <common>
 0003:00015a78       __nhandle                  100dba78     <common>
 0003:00015a80       ___pioinfo                 100dba80     <common>
 0003:00015b80       ___env_initialized         100dbb80     <common>
 0003:00015b84       ___onexitend               100dbb84     <common>
 0003:00015b88       ___onexitbegin             100dbb88     <common>
 0003:00015b8c       ___mbctype_initialized     100dbb8c     <common>
 0003:00015b90       ___dyn_tls_init_callback   100dbb90     <common>
 0003:00015b94       __pDestructExceptionObject 100dbb94     <common>
 0003:00015b98       ___piob                    100dbb98     <common>
 0003:00015ba0       __bufin                    100dbba0     <common>
 0003:00016ba0       __nstream                  100dcba0     <common>
 0003:00016ba4       ___use_sse2_mathfcns       100dcba4     <common>
 0003:00016ba8       __pmatherr                 100dcba8     <common>
 0003:00016bac       ___sse2_available          100dcbac     <common>
 0003:00016bb0       __acmdln                   100dcbb0     <common>
 0003:00016bc0       _winSysInfo                100dcbc0     <common>

 entry point at        0001:000015a5

 Static symbols

 0001:00000750       _shortsort                 10001750 f   LIBCMT:qsort.obj
 0001:000014af       ___DllMainCRTStartup       100024af f   LIBCMT:dllcrt0.obj
 0001:00001de3       __tzset_nolock             10002de3 f   LIBCMT:tzset.obj
 0001:000020f6       _cvtdate                   100030f6 f   LIBCMT:tzset.obj
 0001:000022ed       __isindst_nolock           100032ed f   LIBCMT:tzset.obj
 0001:00003148       ?CPtoLCID@@YAHH@Z          10004148 f   LIBCMT:mbctype.obj
 0001:00003177       ?setSBCS@@YAXPAUthreadmbcinfostruct@@@Z 10004177 f   LIBCMT:mbctype.obj
 0001:000031db       ?setSBUpLow@@YAXPAUthreadmbcinfostruct@@@Z 100041db f   LIBCMT:mbctype.obj
 0001:0000340f       ?getSystemCP@@YAHH@Z       1000440f f   LIBCMT:mbctype.obj
 0001:00003b85       ?__crtLCMapStringA_stat@@YAHPAUlocaleinfo_struct@@KKPBDHPADHHH@Z 10004b85 f   LIBCMT:a_map.obj
 0001:000043a2       _doexit                    100053a2 f   LIBCMT:crt0dat.obj
 0001:00004899       _parse_cmdline             10005899 f   LIBCMT:stdargv.obj
 0001:00005e4d       ?__crtGetStringTypeA_stat@@YAHPAUlocaleinfo_struct@@KPBDHPAGHHH@Z 10006e4d f   LIBCMT:a_str.obj
 0001:000069dc       _flsall                    100079dc f   LIBCMT:fflush.obj
 0001:00006c90       __unwind_handler4          10007c90 f   LIBCMT:exsup4.obj
 0001:00006f14       _siglookup                 10007f14 f   LIBCMT:winsig.obj
 0001:0000711b       __onexit_nolock            1000811b f   LIBCMT:onexit.obj
 0001:00007463       ?x_ismbbtype_l@@YAHPAUlocaleinfo_struct@@IHH@Z 10008463 f   LIBCMT:ismbbyte.obj
 0001:0000763c       __shift                    1000863c f   LIBCMT:cvt.obj
 0001:00007681       __cftoe2_l                 10008681 f   LIBCMT:cvt.obj
 0001:00007c3f       __cftof2_l                 10008c3f f   LIBCMT:cvt.obj
 0001:00007fc3       ?strtoxl@@YAKPAUlocaleinfo_struct@@PBDPAPBDHH@Z 10008fc3 f   LIBCMT:strtol.obj
 0001:00008f30       __unwind_handler           10009f30 f   LIBCMT:exsup.obj
 0001:000098ce       ?__crtCompareStringA_stat@@YAHPAUlocaleinfo_struct@@KKPBDH1HH@Z 1000a8ce f   LIBCMT:a_cmp.obj
 0001:00009c68       _findenv                   1000ac68 f   LIBCMT:setenv.obj
 0001:00009cba       _copy_environ              1000acba f   LIBCMT:setenv.obj
 0001:0000beef       __hw_cw                    1000ceef f   LIBCMT:_ieee87_.obj
 0001:0000bf7d       ___hw_cw_sse2              1000cf7d f   LIBCMT:_ieee87_.obj
 0001:0000c9b0       _sqlite3pager_get_codecarg 1000d9b0 f    CIL library: CIL module
 0001:0000cae0       _soundex                   1000dae0 f    CIL library: CIL module
 0001:0000cb90       _medianIterate             1000db90 f    CIL library: CIL module
 0001:0000cc40       _modeIterate               1000dc40 f    CIL library: CIL module
 0001:0000cd20       _rad2deg                   1000dd20 f    CIL library: CIL module
 0001:0000cd40       _deg2rad                   1000dd40 f    CIL library: CIL module
 0001:0000cd60       _coth                      1000dd60 f    CIL library: CIL module
 0001:0000cd80       _cot                       1000dd80 f    CIL library: CIL module
 0001:0000cda0       _atanh                     1000dda0 f    CIL library: CIL module
 0001:0000cdc0       _asinh                     1000ddc0 f    CIL library: CIL module
 0001:0000cde0       _acosh                     1000dde0 f    CIL library: CIL module
 0001:0000ce00       _sqlite3ReadUtf8           1000de00 f    CIL library: CIL module
 0001:0000cf00       _SortByDimension           1000df00 f    CIL library: CIL module
 0001:0000d0a0       _SortByDistance            1000e0a0 f    CIL library: CIL module
 0001:0000d180       _cellOverlap               1000e180 f    CIL library: CIL module
 0001:0000d240       _cellContains              1000e240 f    CIL library: CIL module
 0001:0000d2d0       _cellUnion                 1000e2d0 f    CIL library: CIL module
 0001:0000d3a0       _cellMargin                1000e3a0 f    CIL library: CIL module
 0001:0000d3e0       _cellArea                  1000e3e0 f    CIL library: CIL module
 0001:0000d420       _testRtreeGeom             1000e420 f    CIL library: CIL module
 0001:0000d500       _rtreeEof                  1000e500 f    CIL library: CIL module
 0001:0000d510       _rtreeReference            1000e510 f    CIL library: CIL module
 0001:0000d520       _nodeHash                  1000e520 f    CIL library: CIL module
 0001:0000d590       _nodeZero                  1000e590 f    CIL library: CIL module
 0001:0000d5b0       _nodeReference             1000e5b0 f    CIL library: CIL module
 0001:0000d5c0       _writeInt64                1000e5c0 f    CIL library: CIL module
 0001:0000d630       _writeCoord                1000e630 f    CIL library: CIL module
 0001:0000d660       _writeInt16                1000e660 f    CIL library: CIL module
 0001:0000d670       _readInt64                 1000e670 f    CIL library: CIL module
 0001:0000d6f0       _readCoord                 1000e6f0 f    CIL library: CIL module
 0001:0000d720       _readInt16                 1000e720 f    CIL library: CIL module
 0001:0000d730       _fts3MatchinfoLcsCb        1000e730 f    CIL library: CIL module
 0001:0000d750       _fts3MatchinfoSize         1000e750 f    CIL library: CIL module
 0001:0000d7a0       _fts3ColumnlistCount       1000e7a0 f    CIL library: CIL module
 0001:0000d7d0       _fts3ExprPhraseCountCb     1000e7d0 f    CIL library: CIL module
 0001:0000d7e0       _fts3ExprLoadDoclistsCb    1000e7e0 f    CIL library: CIL module
 0001:0000d800       _fts3ExprIterate2          1000e800 f    CIL library: CIL module
 0001:0000d870       _fts3ChecksumEntry         1000e870 f    CIL library: CIL module
 0001:0000d930       _fts3Getint                1000e930 f    CIL library: CIL module
 0001:0000d960       _fts3TermCmp               1000e960 f    CIL library: CIL module
 0001:0000d9f0       _sqlite3Fts3MsrIncrRestart 1000e9f0 f    CIL library: CIL module
 0001:0000da30       _fts3PrefixCompress        1000ea30 f    CIL library: CIL module
 0001:0000da50       _fts3SegReaderSort         1000ea50 f    CIL library: CIL module
 0001:0000dab0       _fts3SegReaderTermCmp      1000eab0 f    CIL library: CIL module
 0001:0000dbc0       _fts3SegReaderDoclistCmpRev 1000ebc0 f    CIL library: CIL module
 0001:0000dc20       _fts3SegReaderDoclistCmp   1000ec20 f    CIL library: CIL module
 0001:0000dc80       _fts3SegReaderCmp          1000ec80 f    CIL library: CIL module
 0001:0000dd70       _fts3CompareElemByTerm     1000ed70 f    CIL library: CIL module
 0001:0000de10       _getAbsoluteLevel          1000ee10 f    CIL library: CIL module
 0001:0000de40       _fts3tokRowidMethod        1000ee40 f    CIL library: CIL module
 0001:0000de60       _fts3tokEofMethod          1000ee60 f    CIL library: CIL module
 0001:0000de70       _fts3tokBestIndexMethod    1000ee70 f    CIL library: CIL module
 0001:0000ded0       _sqlite3Fts3SimpleTokenizerModule 1000eed0 f    CIL library: CIL module
 0001:0000dee0       _fts3_isalnum              1000eee0 f    CIL library: CIL module
 0001:0000df10       _simpleDelim               1000ef10 f    CIL library: CIL module
 0001:0000df30       _sqlite3Fts3IsIdChar       1000ef30 f    CIL library: CIL module
 0001:0000df50       _sqlite3Fts3PorterTokenizerModule 1000ef50 f    CIL library: CIL module
 0001:0000df60       _copy_stemmer              1000ef60 f    CIL library: CIL module
 0001:0000dff0       _stem                      1000eff0 f    CIL library: CIL module
 0001:0000e050       _isConsonant               1000f050 f    CIL library: CIL module
 0001:0000e090       _fts3HashInsertElement     1000f090 f    CIL library: CIL module
 0001:0000e0e0       _fts3BinCompare            1000f0e0 f    CIL library: CIL module
 0001:0000e170       _fts3BinHash               1000f170 f    CIL library: CIL module
 0001:0000e1a0       _fts3StrCompare            1000f1a0 f    CIL library: CIL module
 0001:0000e1d0       _fts3StrHash               1000f1d0 f    CIL library: CIL module
 0001:0000e210       _sqlite3Fts3HashInit       1000f210 f    CIL library: CIL module
 0001:0000e230       _fts3ExprCheckDepth        1000f230 f    CIL library: CIL module
 0001:0000e280       _opPrecedence              1000f280 f    CIL library: CIL module
 0001:0000e2a0       _sqlite3Fts3OpenTokenizer  1000f2a0 f    CIL library: CIL module
 0001:0000e310       _fts3isspace               1000f310 f    CIL library: CIL module
 0001:0000e340       _fts3auxRowidMethod        1000f340 f    CIL library: CIL module
 0001:0000e360       _fts3auxEofMethod          1000f360 f    CIL library: CIL module
 0001:0000e370       _fts3auxBestIndexMethod    1000f370 f    CIL library: CIL module
 0001:0000e480       _fts3ReleaseMethod         1000f480 f    CIL library: CIL module
 0001:0000e490       _fts3ReversePoslist        1000f490 f    CIL library: CIL module
 0001:0000e4e0       _fts3CommitMethod          1000f4e0 f    CIL library: CIL module
 0001:0000e4f0       _fts3BeginMethod           1000f4f0 f    CIL library: CIL module
 0001:0000e510       _fts3RowidMethod           1000f510 f    CIL library: CIL module
 0001:0000e530       _fts3EofMethod             1000f530 f    CIL library: CIL module
 0001:0000e540       _fts3ColumnlistCopy        1000f540 f    CIL library: CIL module
 0001:0000e5a0       _fts3PoslistCopy           1000f5a0 f    CIL library: CIL module
 0001:0000e600       _fts3BestIndexMethod       1000f600 f    CIL library: CIL module
 0001:0000e710       _fts3GobbleInt             1000f710 f    CIL library: CIL module
 0001:0000e750       _sqlite3Fts3Dequote        1000f750 f    CIL library: CIL module
 0001:0000e7b0       _sqlite3Fts3VarintLen      1000f7b0 f    CIL library: CIL module
 0001:0000e7e0       _sqlite3Fts3GetVarint      1000f7e0 f    CIL library: CIL module
 0001:0000e870       _sqlite3Fts3PutVarint      1000f870 f    CIL library: CIL module
 0001:0000e910       _sqlite3TempInMemory       1000f910 f    CIL library: CIL module
 0001:0000e940       _sqlite3InvokeBusyHandler  1000f940 f    CIL library: CIL module
 0001:0000e970       _sqlite3ErrStr             1000f970 f    CIL library: CIL module
 0001:0000e9c0       _allSpaces                 1000f9c0 f    CIL library: CIL module
 0001:0000ea30       _yy_find_reduce_action     1000fa30 f    CIL library: CIL module
 0001:0000ea50       _yy_find_shift_action      1000fa50 f    CIL library: CIL module
 0001:0000ead0       _sqlite3ParserAlloc        1000fad0 f    CIL library: CIL module
 0001:0000eaf0       _spanSet                   1000faf0 f    CIL library: CIL module
 0001:0000eb00       _disableTerm               1000fb00 f    CIL library: CIL module
 0001:0000eb40       _isOrderedColumn           1000fb40 f    CIL library: CIL module
 0001:0000ebd0       _estLog                    1000fbd0 f    CIL library: CIL module
 0001:0000ec20       _transferJoinMarkings      1000fc20 f    CIL library: CIL module
 0001:0000ec40       _operatorMask              1000fc40 f    CIL library: CIL module
 0001:0000ec70       _allowedOp                 1000fc70 f    CIL library: CIL module
 0001:0000ec90       _exprSelectTableUsage      1000fc90 f    CIL library: CIL module
 0001:0000ee60       _createMask                1000fe60 f    CIL library: CIL module
 0001:0000ee70       _getMask                   1000fe70 f    CIL library: CIL module
 0001:0000eea0       _whereClauseInit           1000fea0 f    CIL library: CIL module
 0001:0000eed0       _compareCost               1000fed0 f    CIL library: CIL module
 0001:0000ef30       _sqlite3VtabSavepoint      1000ff30 f    CIL library: CIL module
 0001:0000efc0       _sqlite3VtabArgExtend      1000ffc0 f    CIL library: CIL module
 0001:0000eff0       _vtabDisconnectAll         1000fff0 f    CIL library: CIL module
 0001:0000f040       _sqlite3GetVTable          10010040 f    CIL library: CIL module
 0001:0000f060       _sqlite3VtabLock           10010060 f    CIL library: CIL module
 0001:0000f070       _exprWalkNoop              10010070 f    CIL library: CIL module
 0001:0000f080       _isSimpleCount             10010080 f    CIL library: CIL module
 0001:0000f0e0       _substSelect               100100e0 f    CIL library: CIL module
 0001:0000f2a0       _selectOpName              100102a0 f    CIL library: CIL module
 0001:0000f2d0       _setJoinExpr               100102d0 f    CIL library: CIL module
 0001:0000f310       _sqlite3SelectDestInit     10010310 f    CIL library: CIL module
 0001:0000f330       _sqlite3SchemaToIndex      10010330 f    CIL library: CIL module
 0001:0000f360       _sqlite3ReadSchema         10010360 f    CIL library: CIL module
 0001:0000f390       _sqlite3JournalModename    10010390 f    CIL library: CIL module
 0001:0000f3a0       _actionName                100103a0 f    CIL library: CIL module
 0001:0000f3e0       _sqlite3SkipAccumulatorLoad 100103e0 f    CIL library: CIL module
 0001:0000f3f0       _sqlite3GetFuncCollSeq     100103f0 f    CIL library: CIL module
 0001:0000f400       _matchQuality              10010400 f    CIL library: CIL module
 0001:0000f450       _sqlite3MayAbort           10010450 f    CIL library: CIL module
 0001:0000f470       _sqlite3MultiWrite         10010470 f    CIL library: CIL module
 0001:0000f490       _sqlite3SrcListShiftJoinType 10010490 f    CIL library: CIL module
 0001:0000f4c0       _sqlite3SrcListAssignCursors 100104c0 f    CIL library: CIL module
 0001:0000f520       _sqlite3DefaultRowEst      10010520 f    CIL library: CIL module
 0001:0000f580       _sqlite3DeferForeignKey    10010580 f    CIL library: CIL module
 0001:0000f5a0       _sqlite3RootPageMoved      100105a0 f    CIL library: CIL module
 0001:0000f5f0       _identLength               100105f0 f    CIL library: CIL module
 0001:0000f610       _sqlite3AffinityType       10010610 f    CIL library: CIL module
 0001:0000f6d0       _sqlite3AddNotNull         100106d0 f    CIL library: CIL module
 0001:0000f700       _sqlite3CommitInternalChanges 10010700 f    CIL library: CIL module
 0001:0000f710       _sqlite3BeginParse         10010710 f    CIL library: CIL module
 0001:0000f730       _sqlite3AuthContextPop     10010730 f    CIL library: CIL module
 0001:0000f750       _sqlite3AuthContextPush    10010750 f    CIL library: CIL module
 0001:0000f770       _sqlite3FixExprList        10010770 f    CIL library: CIL module
 0001:0000f7b0       _sqlite3FixExpr            100107b0 f    CIL library: CIL module
 0001:0000f850       _sqlite3FixSelect          10010850 f    CIL library: CIL module
 0001:0000f8f0       _sqlite3FixInit            100108f0 f    CIL library: CIL module
 0001:0000f940       _sqlite3ClearTempRegCache  10010940 f    CIL library: CIL module
 0001:0000f950       _sqlite3GetTempRange       10010950 f    CIL library: CIL module
 0001:0000f980       _sqlite3ReleaseTempReg     10010980 f    CIL library: CIL module
 0001:0000f9b0       _sqlite3GetTempReg         100109b0 f    CIL library: CIL module
 0001:0000f9d0       _analyzeAggregatesInSelect 100109d0 f    CIL library: CIL module
 0001:0000f9e0       _exprSrcCount              100109e0 f    CIL library: CIL module
 0001:0000fa40       _sqlite3ExprListCompare    10010a40 f    CIL library: CIL module
 0001:0000fad0       _sqlite3ExprCompare        10010ad0 f    CIL library: CIL module
 0001:0000fc50       _sqlite3ExprCodeTemp       10010c50 f    CIL library: CIL module
 0001:0000fcd0       _sqlite3ExprCachePinRegister 10010cd0 f    CIL library: CIL module
 0001:0000fd60       _sqlite3ExprCachePush      10010d60 f    CIL library: CIL module
 0001:0000fd70       _sqlite3ExprCacheStore     10010d70 f    CIL library: CIL module
 0001:0000fe80       _cacheEntryClear           10010e80 f    CIL library: CIL module
 0001:0000feb0       _isCandidateForInOpt       10010eb0 f    CIL library: CIL module
 0001:0000ff00       _sqlite3ExprNeedsNoAffinityChange 10010f00 f    CIL library: CIL module
 0001:0000ffc0       _sqlite3ExprCanBeNull      10010fc0 f    CIL library: CIL module
 0001:0000fff0       _sqlite3ExprIsInteger      10010ff0 f    CIL library: CIL module
 0001:00010060       _selectNodeIsConstant      10011060 f    CIL library: CIL module
 0001:00010080       _exprNodeIsConstant        10011080 f    CIL library: CIL module
 0001:00010160       _dupedExprStructSize       10011160 f    CIL library: CIL module
 0001:00010180       _exprStructSize            10011180 f    CIL library: CIL module
 0001:000101b0       _exprAlwaysFalse           100111b0 f    CIL library: CIL module
 0001:000101f0       _heightOfExpr              100111f0 f    CIL library: CIL module
 0001:00010200       _sqlite3ExprSkipCollate    10011200 f    CIL library: CIL module
 0001:00010220       _sqlite3ExprAffinity       10011220 f    CIL library: CIL module
 0001:000102a0       _incrAggDepth              100112a0 f    CIL library: CIL module
 0001:000102c0       _sqlite3WalkSelectFrom     100112c0 f    CIL library: CIL module
 0001:00010300       _sqlite3WalkExprList       10011300 f    CIL library: CIL module
 0001:00010340       _sqlite3WalkExpr           10011340 f    CIL library: CIL module
 0001:000103e0       _sqlite3MemJournalSize     100113e0 f    CIL library: CIL module
 0001:000103f0       _sqlite3IsMemJournal       100113f0 f    CIL library: CIL module
 0001:00010400       _sqlite3MemJournalOpen     10011400 f    CIL library: CIL module
 0001:00010430       _memjrnlFileSize           10011430 f    CIL library: CIL module
 0001:00010450       _memjrnlSync               10011450 f    CIL library: CIL module
 0001:00010460       _memjrnlRead               10011460 f    CIL library: CIL module
 0001:00010540       _vdbeSorterRowkey          10011540 f    CIL library: CIL module
 0001:00010590       _sqlite3VdbeMemStoreType   10011590 f    CIL library: CIL module
 0001:00010650       _sqlite3VdbeParameterIndex 10011650 f    CIL library: CIL module
 0001:000107f0       _sqlite3VdbeSetVarmask     100117f0 f    CIL library: CIL module
 0001:00010810       _sqlite3VdbeDb             10011810 f    CIL library: CIL module
 0001:00010820       _sqlite3ExpirePreparedStatements 10011820 f    CIL library: CIL module
 0001:00010840       _sqlite3VdbeCountChanges   10011840 f    CIL library: CIL module
 0001:00010850       _sqlite3VdbeSetChanges     10011850 f    CIL library: CIL module
 0001:00010860       _sqlite3VdbeSerialTypeLen  10011860 f    CIL library: CIL module
 0001:00010880       _sqlite3VdbeSerialType     10011880 f    CIL library: CIL module
 0001:00010990       _sqlite3VdbeDeleteAuxData  10011990 f    CIL library: CIL module
 0001:000109e0       _sqlite3VdbeResetStepResult 100119e0 f    CIL library: CIL module
 0001:000109f0       _sqlite3VdbeFrameRestore   100119f0 f    CIL library: CIL module
 0001:00010a50       _sqlite3VdbeRewind         10011a50 f    CIL library: CIL module
 0001:00010a90       _allocSpace                10011a90 f    CIL library: CIL module
 0001:00010ac0       _sqlite3VdbeGetOp          10011ac0 f    CIL library: CIL module
 0001:00010ae0       _sqlite3VdbeLinkSubProgram 10011ae0 f    CIL library: CIL module
 0001:00010af0       _sqlite3VdbeChangeP5       10011af0 f    CIL library: CIL module
 0001:00010b10       _sqlite3VdbeChangeP3       10011b10 f    CIL library: CIL module
 0001:00010b20       _sqlite3VdbeChangeP2       10011b20 f    CIL library: CIL module
 0001:00010b30       _sqlite3VdbeChangeP1       10011b30 f    CIL library: CIL module
 0001:00010b40       _sqlite3VdbeCurrentAddr    10011b40 f    CIL library: CIL module
 0001:00010b50       _sqlite3VdbeRunOnlyOnce    10011b50 f    CIL library: CIL module
 0001:00010b60       _sqlite3VdbeResolveLabel   10011b60 f    CIL library: CIL module
 0001:00010b80       _sqlite3VdbeSwap           10011b80 f    CIL library: CIL module
 0001:00010c20       _sqlite3ValueBytes         10011c20 f    CIL library: CIL module
 0001:00010c50       _sqlite3VdbeMemTooBig      10011c50 f    CIL library: CIL module
 0001:00010c80       _doubleToInt64             10011c80 f    CIL library: CIL module
 0001:00010ce0       _sqlite3VdbeMemExpandBlob  10011ce0 f    CIL library: CIL module
 0001:00010d40       _sqlite3BackupRestart      10011d40 f    CIL library: CIL module
 0001:00010d80       _isFatalError              10011d80 f    CIL library: CIL module
 0001:00010da0       _sqlite3BtreeCursorHints   10011da0 f    CIL library: CIL module
 0001:00010db0       _sqlite3BtreeIsInBackup    10011db0 f    CIL library: CIL module
 0001:00010dc0       _sqlite3BtreeIsInReadTrans 10011dc0 f    CIL library: CIL module
 0001:00010dd0       _sqlite3BtreeIsInTrans     10011dd0 f    CIL library: CIL module
 0001:00010df0       _setPageReferenced         10011df0 f    CIL library: CIL module
 0001:00010e10       _getPageReferenced         10011e10 f    CIL library: CIL module
 0001:00010e30       _sqlite3BtreePager         10011e30 f    CIL library: CIL module
 0001:00010e40       _assemblePage              10011e40 f    CIL library: CIL module
 0001:00010ef0       _sqlite3BtreeEof           10011ef0 f    CIL library: CIL module
 0001:00010f00       _sqlite3BtreeGetCachedRowid 10011f00 f    CIL library: CIL module
 0001:00010f10       _sqlite3BtreeSetCachedRowid 10011f10 f    CIL library: CIL module
 0001:00010f40       _sqlite3BtreeCursorZero    10011f40 f    CIL library: CIL module
 0001:00010f50       _sqlite3BtreeCursorSize    10011f50 f    CIL library: CIL module
 0001:00010f60       _sqlite3BtreeGetReserveNoMutex 10011f60 f    CIL library: CIL module
 0001:00010f70       _sqlite3BtreeGetPageSize   10011f70 f    CIL library: CIL module
 0001:00010f80       _btreeInvokeBusyHandler    10011f80 f    CIL library: CIL module
 0001:00010fd0       _btreePagecount            10011fd0 f    CIL library: CIL module
 0001:00010fe0       _findOverflowCell          10011fe0 f    CIL library: CIL module
 0001:00011030       _ptrmapPageno              10012030 f    CIL library: CIL module
 0001:00011070       _invalidateIncrblobCursors 10012070 f    CIL library: CIL module
 0001:000110b0       _downgradeAllSharedCacheTableLocks 100120b0 f    CIL library: CIL module
 0001:000110e0       _querySharedCacheTableLock 100120e0 f    CIL library: CIL module
 0001:00011140       _sqlite3BtreeSharable      10012140 f    CIL library: CIL module
 0001:00011150       _sqlite3WalHeapMemory      10012150 f    CIL library: CIL module
 0001:00011170       _sqlite3WalCallback        10012170 f    CIL library: CIL module
 0001:00011190       _sqlite3WalSavepoint       10012190 f    CIL library: CIL module
 0001:000111b0       _sqlite3WalDbsize          100121b0 f    CIL library: CIL module
 0001:000111d0       _walPagesize               100121d0 f    CIL library: CIL module
 0001:000111f0       _walMerge                  100121f0 f    CIL library: CIL module
 0001:000112b0       _walIteratorNext           100122b0 f    CIL library: CIL module
 0001:00011330       _sqlite3WalLimit           10012330 f    CIL library: CIL module
 0001:00011350       _walFramePage              10012350 f    CIL library: CIL module
 0001:00011360       _walNextHash               10012360 f    CIL library: CIL module
 0001:00011370       _walHash                   10012370 f    CIL library: CIL module
 0001:00011380       _walChecksumBytes          10012380 f    CIL library: CIL module
 0001:00011440       _walIndexHdr               10012440 f    CIL library: CIL module
 0001:00011450       _walCkptInfo               10012450 f    CIL library: CIL module
 0001:00011460       _sqlite3PagerCodec         10012460 f    CIL library: CIL module
 0001:000114a0       _sqlite3PagerWalSupported  100124a0 f    CIL library: CIL module
 0001:000114c0       _sqlite3PagerWalCallback   100124c0 f    CIL library: CIL module
 0001:000114e0       _sqlite3PagerBackupPtr     100124e0 f    CIL library: CIL module
 0001:000114f0       _sqlite3PagerJournalSizeLimit 100124f0 f    CIL library: CIL module
 0001:00011540       _sqlite3PagerOkToChangeJournalMode 10012540 f    CIL library: CIL module
 0001:00011570       _sqlite3PagerGetJournalMode 10012570 f    CIL library: CIL module
 0001:00011580       _sqlite3PagerLockingMode   10012580 f    CIL library: CIL module
 0001:000115b0       _sqlite3PagerGetExtra      100125b0 f    CIL library: CIL module
 0001:000115c0       _sqlite3PagerGetData       100125c0 f    CIL library: CIL module
 0001:000115d0       _sqlite3PagerGetCodec      100125d0 f    CIL library: CIL module
 0001:000115e0       _sqlite3PagerNosync        100125e0 f    CIL library: CIL module
 0001:000115f0       _sqlite3PagerJournalname   100125f0 f    CIL library: CIL module
 0001:00011600       _sqlite3PagerFile          10012600 f    CIL library: CIL module
 0001:00011610       _sqlite3PagerVfs           10012610 f    CIL library: CIL module
 0001:00011620       _sqlite3PagerFilename      10012620 f    CIL library: CIL module
 0001:00011640       _sqlite3PagerIsMemdb       10012640 f    CIL library: CIL module
 0001:00011650       _sqlite3PagerCacheStat     10012650 f    CIL library: CIL module
 0001:00011680       _sqlite3PagerIsreadonly    10012680 f    CIL library: CIL module
 0001:00011690       _sqlite3PagerDontWrite     10012690 f    CIL library: CIL module
 0001:000116b0       _sqlite3PagerTruncateImage 100126b0 f    CIL library: CIL module
 0001:000116c0       _sqlite3PagerPagecount     100126c0 f    CIL library: CIL module
 0001:000116d0       _sqlite3PagerMaxPageCount  100126d0 f    CIL library: CIL module
 0001:000116f0       _sqlite3PagerTempSpace     100126f0 f    CIL library: CIL module
 0001:00011700       _sqlite3PagerSetSafetyLevel 10012700 f    CIL library: CIL module
 0001:00011780       _pagerReportSize           10012780 f    CIL library: CIL module
 0001:000117b0       _pager_cksum               100127b0 f    CIL library: CIL module
 0001:00011830       _pager_error               10012830 f    CIL library: CIL module
 0001:00011850       _journalHdrOffset          10012850 f    CIL library: CIL module
 0001:00011890       _pagerUseWal               10012890 f    CIL library: CIL module
 0001:000118a0       _rowSetNDeepTree           100128a0 f    CIL library: CIL module
 0001:00011900       _rowSetTreeToList          10012900 f    CIL library: CIL module
 0001:00011950       _rowSetEntryMerge          10012950 f    CIL library: CIL module
 0001:000119d0       _sqlite3RowSetInit         100129d0 f    CIL library: CIL module
 0001:00011a00       _pcache1Shutdown           10012a00 f    CIL library: CIL module
 0001:00011a20       _pcache1RemoveFromHash     10012a20 f    CIL library: CIL module
 0001:00011a50       _pcache1PinPage            10012a50 f    CIL library: CIL module
 0001:00011ab0       _sqlite3PCacheBufferSetup  10012ab0 f    CIL library: CIL module
 0001:00011b30       _sqlite3PcacheShrink       10012b30 f    CIL library: CIL module
 0001:00011b40       _sqlite3PcachePagecount    10012b40 f    CIL library: CIL module
 0001:00011b60       _sqlite3PcachePageRefcount 10012b60 f    CIL library: CIL module
 0001:00011b70       _sqlite3PcacheRefCount     10012b70 f    CIL library: CIL module
 0001:00011b80       _pcacheMergeDirtyList      10012b80 f    CIL library: CIL module
 0001:00011be0       _sqlite3PcacheClose        10012be0 f    CIL library: CIL module
 0001:00011bf0       _sqlite3PcacheClearSyncFlags 10012bf0 f    CIL library: CIL module
 0001:00011c20       _sqlite3PcacheRef          10012c20 f    CIL library: CIL module
 0001:00011c30       _numberOfCachePages        10012c30 f    CIL library: CIL module
 0001:00011c70       _sqlite3PcacheSetPageSize  10012c70 f    CIL library: CIL module
 0001:00011ca0       _sqlite3PcacheOpen         10012ca0 f    CIL library: CIL module
 0001:00011ce0       _sqlite3PcacheSize         10012ce0 f    CIL library: CIL module
 0001:00011cf0       _sqlite3PcacheShutdown     10012cf0 f    CIL library: CIL module
 0001:00011d10       _pcacheUnpin               10012d10 f    CIL library: CIL module
 0001:00011d40       _pcacheAddToDirtyList      10012d40 f    CIL library: CIL module
 0001:00011d70       _pcacheRemoveFromDirtyList 10012d70 f    CIL library: CIL module
 0001:00011dd0       _sqlite3BitvecSize         10012dd0 f    CIL library: CIL module
 0001:00011de0       _sqlite3BitvecClear        10012de0 f    CIL library: CIL module
 0001:00011eb0       _sqlite3BitvecTest         10012eb0 f    CIL library: CIL module
 0001:00011f60       _winCurrentTimeInt64       10012f60 f    CIL library: CIL module
 0001:00011fb0       _winRandomness             10012fb0 f    CIL library: CIL module
 0001:00012070       _winDlClose                10013070 f    CIL library: CIL module
 0001:00012080       _winDlSym                  10013080 f    CIL library: CIL module
 0001:000120a0       _winIsVerbatimPathname     100130a0 f    CIL library: CIL module
 0001:000120d0       _winDeviceCharacteristics  100130d0 f    CIL library: CIL module
 0001:000120f0       _winSectorSize             100130f0 f    CIL library: CIL module
 0001:00012100       _winModeBit                10013100 f    CIL library: CIL module
 0001:00012120       _winMemRoundup             10013120 f    CIL library: CIL module
 0001:00012130       _isNT                      10013130 f    CIL library: CIL module
 0001:00012220       _winNextSystemCall         10013220 f    CIL library: CIL module
 0001:000122b0       _winGetSystemCall          100132b0 f    CIL library: CIL module
 0001:00012320       _winSetSystemCall          10013320 f    CIL library: CIL module
 0001:000123f0       _sqlite3OpcodeName         100133f0 f    CIL library: CIL module
 0001:00012400       _insertElement             10013400 f    CIL library: CIL module
 0001:00012460       _strHash                   10013460 f    CIL library: CIL module
 0001:00012490       _sqlite3HashInit           10013490 f    CIL library: CIL module
 0001:000124a0       _sqlite3AbsInt32           100134a0 f    CIL library: CIL module
 0001:000124c0       _sqlite3AddInt64           100134c0 f    CIL library: CIL module
 0001:00012550       _sqlite3HexToInt           10013550 f    CIL library: CIL module
 0001:00012570       _sqlite3Put4byte           10013570 f    CIL library: CIL module
 0001:00012590       _sqlite3Get4byte           10013590 f    CIL library: CIL module
 0001:000125b0       _sqlite3VarintLen          100135b0 f    CIL library: CIL module
 0001:000125e0       _sqlite3GetVarint          100135e0 f    CIL library: CIL module
 0001:00012760       _sqlite3PutVarint          10013760 f    CIL library: CIL module
 0001:00012860       _sqlite3GetInt32           10013860 f    CIL library: CIL module
 0001:00012930       _compare2pow63             10013930 f    CIL library: CIL module
 0001:00012970       _sqlite3AtoF               10013970 f    CIL library: CIL module
 0001:00012fc0       _sqlite3Dequote            10013fc0 f    CIL library: CIL module
 0001:00013070       _sqlite3Strlen30           10014070 f    CIL library: CIL module
 0001:00013090       _sqlite3IsNaN              10014090 f    CIL library: CIL module
 0001:000130c0       _sqlite3Utf16ByteLen       100140c0 f    CIL library: CIL module
 0001:00013100       _sqlite3Utf8CharLen        10014100 f    CIL library: CIL module
 0001:00013150       _sqlite3VdbeMemHandleBom   10014150 f    CIL library: CIL module
 0001:000131d0       _sqlite3Utf8Read           100141d0 f    CIL library: CIL module
 0001:00013240       _sqlite3PrngResetState     10014240 f    CIL library: CIL module
 0001:00013250       _sqlite3PrngRestoreState   10014250 f    CIL library: CIL module
 0001:00013270       _sqlite3PrngSaveState      10014270 f    CIL library: CIL module
 0001:00013290       _sqlite3StrAccumInit       10014290 f    CIL library: CIL module
 0001:000132c0       _et_getdigit               100142c0 f    CIL library: CIL module
 0001:000132f0       _sqlite3MallocSize         100142f0 f    CIL library: CIL module
 0001:00013300       _isLookaside               10014300 f    CIL library: CIL module
 0001:00013320       _sqlite3MallocEnd          10014320 f    CIL library: CIL module
 0001:00013370       _sqlite3HeapNearlyFull     10014370 f    CIL library: CIL module
 0001:00013390       _winMutexLeave             10014390 f    CIL library: CIL module
 0001:000133a0       _winMutexTry               100143a0 f    CIL library: CIL module
 0001:000133b0       _winMutexEnter             100143b0 f    CIL library: CIL module
 0001:000133c0       _winMutexEnd               100143c0 f    CIL library: CIL module
 0001:00013410       _winMutexInit              10014410 f    CIL library: CIL module
 0001:00013470       _noopMutexLeave            10014470 f    CIL library: CIL module
 0001:00013480       _noopMutexTry              10014480 f    CIL library: CIL module
 0001:00013490       _noopMutexEnter            10014490 f    CIL library: CIL module
 0001:000134a0       _noopMutexFree             100144a0 f    CIL library: CIL module
 0001:000134b0       _noopMutexAlloc            100144b0 f    CIL library: CIL module
 0001:000134c0       _noopMutexEnd              100144c0 f    CIL library: CIL module
 0001:000134d0       _noopMutexInit             100144d0 f    CIL library: CIL module
 0001:00013560       _sqlite3MutexAlloc         10014560 f    CIL library: CIL module
 0001:000135a0       _sqlite3MutexEnd           100145a0 f    CIL library: CIL module
 0001:000135b0       _sqlite3EndBenignMalloc    100145b0 f    CIL library: CIL module
 0001:000135c0       _sqlite3BeginBenignMalloc  100145c0 f    CIL library: CIL module
 0001:000135d0       _sqlite3BenignMallocHooks  100145d0 f    CIL library: CIL module
 0001:000135e0       _vfsUnlink                 100145e0 f    CIL library: CIL module
 0001:000136e0       _sqlite3OsCurrentTimeInt64 100146e0 f    CIL library: CIL module
 0001:00013730       _sqlite3OsSleep            10014730 f    CIL library: CIL module
 0001:00013740       _sqlite3OsRandomness       10014740 f    CIL library: CIL module
 0001:00013750       _sqlite3OsDlClose          10014750 f    CIL library: CIL module
 0001:00013760       _sqlite3OsDlSym            10014760 f    CIL library: CIL module
 0001:00013770       _sqlite3OsDlError          10014770 f    CIL library: CIL module
 0001:00013780       _sqlite3OsDlOpen           10014780 f    CIL library: CIL module
 0001:00013790       _sqlite3OsFullPathname     10014790 f    CIL library: CIL module
 0001:000137b0       _sqlite3OsAccess           100147b0 f    CIL library: CIL module
 0001:000137d0       _sqlite3OsDelete           100147d0 f    CIL library: CIL module
 0001:000137e0       _sqlite3OsOpen             100147e0 f    CIL library: CIL module
 0001:00013800       _sqlite3OsUnfetch          10014800 f    CIL library: CIL module
 0001:00013820       _sqlite3OsFetch            10014820 f    CIL library: CIL module
 0001:00013840       _sqlite3OsShmMap           10014840 f    CIL library: CIL module
 0001:00013860       _sqlite3OsShmUnmap         10014860 f    CIL library: CIL module
 0001:00013870       _sqlite3OsShmBarrier       10014870 f    CIL library: CIL module
 0001:00013880       _sqlite3OsShmLock          10014880 f    CIL library: CIL module
 0001:000138a0       _sqlite3OsDeviceCharacteristics 100148a0 f    CIL library: CIL module
 0001:000138b0       _sqlite3OsSectorSize       100148b0 f    CIL library: CIL module
 0001:000138d0       _sqlite3OsFileControlHint  100148d0 f    CIL library: CIL module
 0001:000138f0       _sqlite3OsFileControl      100148f0 f    CIL library: CIL module
 0001:00013910       _sqlite3OsCheckReservedLock 10014910 f    CIL library: CIL module
 0001:00013920       _sqlite3OsUnlock           10014920 f    CIL library: CIL module
 0001:00013930       _sqlite3OsLock             10014930 f    CIL library: CIL module
 0001:00013940       _sqlite3OsFileSize         10014940 f    CIL library: CIL module
 0001:00013950       _sqlite3OsSync             10014950 f    CIL library: CIL module
 0001:00013960       _sqlite3OsTruncate         10014960 f    CIL library: CIL module
 0001:00013980       _sqlite3OsWrite            10014980 f    CIL library: CIL module
 0001:000139a0       _sqlite3OsRead             100149a0 f    CIL library: CIL module
 0001:000139c0       _sqlite3OsClose            100149c0 f    CIL library: CIL module
 0001:000139e0       _clearYMD_HMS_TZ           100149e0 f    CIL library: CIL module
 0001:000139f0       _computeYMD                100149f0 f    CIL library: CIL module
 0001:00013b10       _setDateTimeToCurrent      10014b10 f    CIL library: CIL module
 0001:00013b70       _computeJD                 10014b70 f    CIL library: CIL module
 0001:00013c90       _getDigits                 10014c90 f    CIL library: CIL module
 0001:00013d30       _localtime_s               10014d30 f    CIL library: CIL module
 0001:00013d40       _sqlite3StatusSet          10014d40 f    CIL library: CIL module
 0001:00013d60       _sqlite3StatusAdd          10014d60 f    CIL library: CIL module
 0001:00013d90       _sqlite3StatusValue        10014d90 f    CIL library: CIL module
 0001:00014050       _InitializeProvider        10015050 f    CIL library: CIL module
 0001:00014190       __substr                   10015190 f    CIL library: CIL module
 0001:00014480       _cellGrowth                10015480 f    CIL library: CIL module
 0001:00014530       _nodeGetCoord              10015530 f    CIL library: CIL module
 0001:00014570       _nodeGetRowid              10015570 f    CIL library: CIL module
 0001:00014590       _nodeDeleteCell            10015590 f    CIL library: CIL module
 0001:000145f0       _nodeOverwriteCell         100155f0 f    CIL library: CIL module
 0001:00014670       _nodeHashDelete            10015670 f    CIL library: CIL module
 0001:000146b0       _nodeHashInsert            100156b0 f    CIL library: CIL module
 0001:00014730       _nodeHashLookup            10015730 f    CIL library: CIL module
 0001:000147c0       _fts3LcsIteratorAdvance    100157c0 f    CIL library: CIL module
 0001:00014810       _fts3SnippetShift          10015810 f    CIL library: CIL module
 0001:000149d0       _fts3ExprIterate           100159d0 f    CIL library: CIL module
 0001:00014a30       _fts3StartNode             10015a30 f    CIL library: CIL module
 0001:00014a70       _fts3DecodeIntArray        10015a70 f    CIL library: CIL module
 0001:00014b30       _fts3EncodeIntArray        10015b30 f    CIL library: CIL module
 0001:00014ba0       _fts3TreeFinishNode        10015ba0 f    CIL library: CIL module
 0001:00014c00       _sqlite3Fts3NextToken      10015c00 f    CIL library: CIL module
 0001:00014d30       _doubleConsonant           10015d30 f    CIL library: CIL module
 0001:00014d70       _hasVowel                  10015d70 f    CIL library: CIL module
 0001:00014db0       _isVowel                   10015db0 f    CIL library: CIL module
 0001:00014e10       _ftsCompareFunction        10015e10 f    CIL library: CIL module
 0001:00014e30       _ftsHashFunction           10015e30 f    CIL library: CIL module
 0001:00014e50       _insertBinaryOperator      10015e50 f    CIL library: CIL module
 0001:00014ec0       _sqlite3Fts3DoclistNext    10015ec0 f    CIL library: CIL module
 0001:00014f50       _fts3DoclistCountDocids    10015f50 f    CIL library: CIL module
 0001:00014f90       _sqlite3Fts3FirstFilter    10015f90 f    CIL library: CIL module
 0001:000150f0       _fts3PutDeltaVarint3       100160f0 f    CIL library: CIL module
 0001:00015160       _fts3GetDeltaVarint3       10016160 f    CIL library: CIL module
 0001:000151a0       _fts3PutColNumber          100161a0 f    CIL library: CIL module
 0001:00015200       _fts3PutDeltaVarint        10016200 f    CIL library: CIL module
 0001:00015250       _fts3GetReverseVarint      10016250 f    CIL library: CIL module
 0001:000152f0       _fts3GetDeltaVarint        100162f0 f    CIL library: CIL module
 0001:00015320       _sqlite3Fts3GetVarint32    10016320 f    CIL library: CIL module
 0001:00015340       _sqlite3DbNameToBtree      10016340 f    CIL library: CIL module
 0001:000158a0       _sqliteDefaultBusyCallback 100168a0 f    CIL library: CIL module
 0001:00015910       _connectionIsBusy          10016910 f    CIL library: CIL module
 0001:00015950       _nocaseCollatingFunc       10016950 f    CIL library: CIL module
 0001:00015980       _binCollFunc               10016980 f    CIL library: CIL module
 0001:00015ef0       _keywordCode               10016ef0 f    CIL library: CIL module
 0001:00015fd0       _isMatchOfColumn           10016fd0 f    CIL library: CIL module
 0001:00016010       _exprTableUsage            10017010 f    CIL library: CIL module
 0001:00016130       _addToVTrans               10017130 f    CIL library: CIL module
 0001:00016150       _sqlite3TriggerList        10017150 f    CIL library: CIL module
 0001:000161d0       _minMaxQuery               100171d0 f    CIL library: CIL module
 0001:00016240       _columnType                10017240 f    CIL library: CIL module
 0001:000163f0       _columnIndex               100173f0 f    CIL library: CIL module
 0001:00016460       _getTempStore              10017460 f    CIL library: CIL module
 0001:000164b0       _getLockingMode            100174b0 f    CIL library: CIL module
 0001:00016540       _xferCompatibleCollation   10017540 f    CIL library: CIL module
 0001:00016570       _patternCompare            10017570 f    CIL library: CIL module
 0001:00016890       _functionSearch            10017890 f    CIL library: CIL module
 0001:00016920       _collationMatch            10017920 f    CIL library: CIL module
 0001:000169a0       _sqlite3IdListIndex        100179a0 f    CIL library: CIL module
 0001:00016a20       _sqlite3FindDbName         10017a20 f    CIL library: CIL module
 0001:00016af0       _sqlite3FixTriggerStep     10017af0 f    CIL library: CIL module
 0001:00016b70       _sqlite3FunctionUsesThisSrc 10017b70 f    CIL library: CIL module
 0001:00016c00       _exprCodeBetween           10017c00 f    CIL library: CIL module
 0001:00016cf0       _sqlite3ExprCacheClear     10017cf0 f    CIL library: CIL module
 0001:00016dc0       _sqlite3ExprCachePop       10017dc0 f    CIL library: CIL module
 0001:00016ec0       _sqlite3ExprCacheRemove    10017ec0 f    CIL library: CIL module
 0001:00016fc0       _sqlite3IsRowid            10017fc0 f    CIL library: CIL module
 0001:00017000       _exprIsConst               10018000 f    CIL library: CIL module
 0001:00017050       _dupedExprNodeSize         10018050 f    CIL library: CIL module
 0001:000170c0       _heightOfExprList          100180c0 f    CIL library: CIL module
 0001:000170f0       _sqlite3CompareAffinity    100180f0 f    CIL library: CIL module
 0001:00017120       _resolveAsName             10018120 f    CIL library: CIL module
 0001:000171b0       _sqlite3MatchSpanName      100181b0 f    CIL library: CIL module
 0001:00017310       _nameInUsingClause         10018310 f    CIL library: CIL module
 0001:000173a0       _incrAggFunctionDepth      100183a0 f    CIL library: CIL module
 0001:000173e0       _sqlite3WalkSelectExpr     100183e0 f    CIL library: CIL module
 0001:00017490       _fileWriterWrite           10018490 f    CIL library: CIL module
 0001:000175d0       _columnName                100185d0 f    CIL library: CIL module
 0001:00017640       _doWalCallbacks            10018640 f    CIL library: CIL module
 0001:00017780       _sqlite3VdbeSerialGet      10018780 f    CIL library: CIL module
 0001:000179b0       _sqlite3VdbeSerialPut      100189b0 f    CIL library: CIL module
 0001:00017a60       _sqlite3VdbeUsesBtree      10018a60 f    CIL library: CIL module
 0001:00017a80       _sqlite3VdbeJumpHere       10018a80 f    CIL library: CIL module
 0001:00017aa0       _sqlite3VdbeIntegerAffinity 10018aa0 f    CIL library: CIL module
 0001:00017b40       _sqlite3VdbeRealValue      10018b40 f    CIL library: CIL module
 0001:00017b90       _attachBackupObject        10018b90 f    CIL library: CIL module
 0001:00017bb0       _backupTruncateFile        10018bb0 f    CIL library: CIL module
 0001:00017bf0       _sqlite3BtreeGetJournalname 10018bf0 f    CIL library: CIL module
 0001:00017c00       _sqlite3BtreeGetFilename   10018c00 f    CIL library: CIL module
 0001:00017c20       _btreeCursor               10018c20 f    CIL library: CIL module
 0001:00017c90       _finalDbSize               10018c90 f    CIL library: CIL module
 0001:00017d40       _removeFromSharingList     10018d40 f    CIL library: CIL module
 0001:00017dd0       _sqlite3BtreeLastPage      10018dd0 f    CIL library: CIL module
 0001:00017de0       _btreePageFromDbPage       10018de0 f    CIL library: CIL module
 0001:00017e10       _btreeGetHasContent        10018e10 f    CIL library: CIL module
 0001:00017e30       _unlockBtreeMutex          10018e30 f    CIL library: CIL module
 0001:00017e50       _lockBtreeMutex            10018e50 f    CIL library: CIL module
 0001:00017e80       _walWriteToLog             10018e80 f    CIL library: CIL module
 0001:00017f20       _sqlite3WalReadFrame       10018f20 f    CIL library: CIL module
 0001:00017f70       _walMergesort              10018f70 f    CIL library: CIL module
 0001:00018230       _walFramePgno              10019230 f    CIL library: CIL module
 0001:00018260       _walUnlockExclusive        10019260 f    CIL library: CIL module
 0001:00018280       _walLockExclusive          10019280 f    CIL library: CIL module
 0001:000182b0       _walUnlockShared           100192b0 f    CIL library: CIL module
 0001:000182d0       _walLockShared             100192d0 f    CIL library: CIL module
 0001:000182f0       _walDecodeFrame            100192f0 f    CIL library: CIL module
 0001:00018410       _walEncodeFrame            10019410 f    CIL library: CIL module
 0001:000184d0       _walShmBarrier             100194d0 f    CIL library: CIL module
 0001:000184f0       _sqlite3PagerSetCodec      100194f0 f    CIL library: CIL module
 0001:00018550       _sqlite3PagerPageRefcount  10019550 f    CIL library: CIL module
 0001:00018560       _sqlite3PagerMemUsed       10019560 f    CIL library: CIL module
 0001:000185b0       _sqlite3PagerRefcount      100195b0 f    CIL library: CIL module
 0001:000185c0       _sqlite3PagerSync          100195c0 f    CIL library: CIL module
 0001:00018600       _sqlite3PagerRef           10019600 f    CIL library: CIL module
 0001:00018610       _pagerReleaseMapPage       10019610 f    CIL library: CIL module
 0001:00018660       _pagerSyncHotJournal       10019660 f    CIL library: CIL module
 0001:000186a0       _sqlite3PagerReadFileheader 100196a0 f    CIL library: CIL module
 0001:000186e0       _sqlite3PagerSetBusyhandler 100196e0 f    CIL library: CIL module
 0001:00018700       _pagerOpentemp             10019700 f    CIL library: CIL module
 0001:00018720       _sqlite3PagerShrink        10019720 f    CIL library: CIL module
 0001:00018740       _pagerFixMaplimit          10019740 f    CIL library: CIL module
 0001:000187a0       _pagerPagecount            100197a0 f    CIL library: CIL module
 0001:00018820       _pager_write_changecounter 10019820 f    CIL library: CIL module
 0001:00018890       _readDbPage                10019890 f    CIL library: CIL module
 0001:000189d0       _sqlite3SectorSize         100199d0 f    CIL library: CIL module
 0001:00018a00       _pager_truncate            10019a00 f    CIL library: CIL module
 0001:00018b00       _zeroJournalHdr            10019b00 f    CIL library: CIL module
 0001:00018bd0       _pagerLockDb               10019bd0 f    CIL library: CIL module
 0001:00018c10       _pagerUnlockDb             10019c10 f    CIL library: CIL module
 0001:00018c30       _write32bits               10019c30 f    CIL library: CIL module
 0001:00018c70       _read32bits                10019c70 f    CIL library: CIL module
 0001:00018cc0       _pageInJournal             10019cc0 f    CIL library: CIL module
 0001:00018ce0       _subjRequiresPage          10019ce0 f    CIL library: CIL module
 0001:00018df0       _rowSetListToTree          10019df0 f    CIL library: CIL module
 0001:00018eb0       _rowSetEntrySort           10019eb0 f    CIL library: CIL module
 0001:00018fc0       _pcache1Rekey              10019fc0 f    CIL library: CIL module
 0001:00019040       _pcache1Pagecount          1001a040 f    CIL library: CIL module
 0001:00019080       _pcache1Init               1001a080 f    CIL library: CIL module
 0001:000190f0       _pcache1UnderMemoryPressure 1001a0f0 f    CIL library: CIL module
 0001:00019120       _sqlite3PcacheSetCachesize 1001a120 f    CIL library: CIL module
 0001:00019170       _pcacheSortDirtyList       1001a170 f    CIL library: CIL module
 0001:000192d0       _sqlite3PcacheMove         1001a2d0 f    CIL library: CIL module
 0001:00019330       _sqlite3PcacheMakeClean    1001a330 f    CIL library: CIL module
 0001:00019380       _sqlite3PcacheMakeDirty    1001a380 f    CIL library: CIL module
 0001:000193d0       _sqlite3PcacheDrop         1001a3d0 f    CIL library: CIL module
 0001:00019410       _sqlite3PcacheRelease      1001a410 f    CIL library: CIL module
 0001:00019480       _sqlite3PcacheFetch        1001a480 f    CIL library: CIL module
 0001:00019600       _winCurrentTime            1001a600 f    CIL library: CIL module
 0001:00019650       _winSleep                  1001a650 f    CIL library: CIL module
 0001:00019680       _winShmLeaveMutex          1001a680 f    CIL library: CIL module
 0001:000196b0       _winShmEnterMutex          1001a6b0 f    CIL library: CIL module
 0001:000196e0       _winUnlockFile             1001a6e0 f    CIL library: CIL module
 0001:000197a0       _winLockFile               1001a7a0 f    CIL library: CIL module
 0001:00019860       _retryIoerr                1001a860 f    CIL library: CIL module
 0001:000198a0       _findElementGivenHash      1001a8a0 f    CIL library: CIL module
 0001:00019940       _sqlite3MulInt64           1001a940 f    CIL library: CIL module
 0001:00019a30       _sqlite3SubInt64           1001aa30 f    CIL library: CIL module
 0001:00019a80       _sqlite3GetVarint32        1001aa80 f    CIL library: CIL module
 0001:00019af0       _sqlite3PutVarint32        1001aaf0 f    CIL library: CIL module
 0001:00019b20       _sqlite3Atoi               1001ab20 f    CIL library: CIL module
 0001:00019b50       _sqlite3Atoi64             1001ab50 f    CIL library: CIL module
 0001:00019d30       _randomByte                1001ad30 f    CIL library: CIL module
 0001:00019ed0       _sqlite3DbMallocSize       1001aed0 f    CIL library: CIL module
 0001:00019f00       _sqlite3ScratchFree        1001af00 f    CIL library: CIL module
 0001:0001a010       _sqlite3MallocAlarm        1001b010 f    CIL library: CIL module
 0001:0001a090       _sqlite3MemoryAlarm        1001b090 f    CIL library: CIL module
 0001:0001a120       _softHeapLimitEnforcer     1001b120 f    CIL library: CIL module
 0001:0001a130       _winMutexFree              1001b130 f    CIL library: CIL module
 0001:0001a150       _sqlite3NoopMutex          1001b150 f    CIL library: CIL module
 0001:0001a270       _sqlite3OsCloseFree        1001b270 f    CIL library: CIL module
 0001:0001a2a0       _osLocaltime               1001b2a0 f    CIL library: CIL module
 0001:0001a2d0       _computeHMS                1001b2d0 f    CIL library: CIL module
 0001:0001a380       _parseTimezone             1001b380 f    CIL library: CIL module
 0001:0001a4d0       _DeriveKey                 1001b4d0 f    CIL library: CIL module
 0001:0001a5a0       _sqlite3CodecFree          1001b5a0 f    CIL library: CIL module
 0001:0001a640       _vtshimAuxDestructor       1001b640 f    CIL library: CIL module
 0001:0001a690       _vtshimDestroy             1001b690 f    CIL library: CIL module
 0001:0001a6e0       _vtshimDisconnect          1001b6e0 f    CIL library: CIL module
 0001:0001a730       _doSqlite3Free             1001b730 f    CIL library: CIL module
 0001:0001a740       _rtreeRowid                1001b740 f    CIL library: CIL module
 0001:0001a770       _nodeRowidIndex            1001b770 f    CIL library: CIL module
 0001:0001a860       _freeCursorConstraints     1001b860 f    CIL library: CIL module
 0001:0001a950       _nodeGetCell               1001b950 f    CIL library: CIL module
 0001:0001a9d0       _nodeInsertCell            1001b9d0 f    CIL library: CIL module
 0001:0001aa30       _fts3ExprPhraseCount       1001ba30 f    CIL library: CIL module
 0001:0001aaa0       _fts3ExprLoadDoclists      1001baa0 f    CIL library: CIL module
 0001:0001ab40       _fts3GetDeltaPosition      1001bb40 f    CIL library: CIL module
 0001:0001ab70       _fts3IncrmergeHintPop      1001bb70 f    CIL library: CIL module
 0001:0001abf0       _nodeReaderRelease         1001bbf0 f    CIL library: CIL module
 0001:0001ac00       _fts3ColumnFilter          1001bc00 f    CIL library: CIL module
 0001:0001aca0       _fts3NodeFree              1001bca0 f    CIL library: CIL module
 0001:0001ad80       _fts3PendingListDelete     1001bd80 f    CIL library: CIL module
 0001:0001ad90       _fts3tokResetCursor        1001bd90 f    CIL library: CIL module
 0001:0001add0       _fts3tokDisconnectMethod   1001bdd0 f    CIL library: CIL module
 0001:0001ae00       _simpleClose               1001be00 f    CIL library: CIL module
 0001:0001ae20       _simpleDestroy             1001be20 f    CIL library: CIL module
 0001:0001ae40       _star_oh                   1001be40 f    CIL library: CIL module
 0001:0001aeb0       _m_gt_1                    1001beb0 f    CIL library: CIL module
 0001:0001b000       _m_eq_1                    1001c000 f    CIL library: CIL module
 0001:0001b140       _m_gt_0                    1001c140 f    CIL library: CIL module
 0001:0001b1f0       _porterClose               1001c1f0 f    CIL library: CIL module
 0001:0001b210       _porterDestroy             1001c210 f    CIL library: CIL module
 0001:0001b230       _fts3FindElementByHash     1001c230 f    CIL library: CIL module
 0001:0001b290       _fts3HashFree              1001c290 f    CIL library: CIL module
 0001:0001b2a0       _fts3EvalUpdateCounts      1001c2a0 f    CIL library: CIL module
 0001:0001b360       _fts3EvalInvalidatePoslist 1001c360 f    CIL library: CIL module
 0001:0001b390       _sqlite3Fts3DoclistPrev    1001c390 f    CIL library: CIL module
 0001:0001b4c0       _fts3PoslistPhraseMerge    1001c4c0 f    CIL library: CIL module
 0001:0001b820       _fts3ReadNextPos           1001c820 f    CIL library: CIL module
 0001:0001b9e0       _sqlite3GetToken           1001c9e0 f    CIL library: CIL module
 0001:0001c050       _sqlite3KeywordCode        1001d050 f    CIL library: CIL module
 0001:0001c060       _exprListTableUsage        1001d060 f    CIL library: CIL module
 0001:0001c180       _checkColumnOverlap        1001d180 f    CIL library: CIL module
 0001:0001c350       _tableAndColumnIndex       1001d350 f    CIL library: CIL module
 0001:0001c410       _getAutoVacuum             1001d410 f    CIL library: CIL module
 0001:0001c490       _getSafetyLevel            1001d490 f    CIL library: CIL module
 0001:0001c540       _xferCompatibleIndex       1001d540 f    CIL library: CIL module
 0001:0001c610       _sqlite3FuncDefInsert      1001d610 f    CIL library: CIL module
 0001:0001c690       _identPut                  1001d690 f    CIL library: CIL module
 0001:0001c740       _sqlite3ReleaseTempRange   1001d740 f    CIL library: CIL module
 0001:0001c760       _sqlite3ExprCacheAffinityChange 1001d760 f    CIL library: CIL module
 0001:0001c770       _sqlite3ExprIsConstantOrFunction 1001d770 f    CIL library: CIL module
 0001:0001c7c0       _sqlite3ExprIsConstantNotJoin 1001d7c0 f    CIL library: CIL module
 0001:0001c810       _sqlite3ExprIsConstant     1001d810 f    CIL library: CIL module
 0001:0001c860       _dupedExprSize             1001d860 f    CIL library: CIL module
 0001:0001c8b0       _heightOfSelect            1001d8b0 f    CIL library: CIL module
 0001:0001c9a0       _binaryCompareP5           1001d9a0 f    CIL library: CIL module
 0001:0001c9e0       _comparisonAffinity        1001d9e0 f    CIL library: CIL module
 0001:0001ca40       _sqlite3WalkSelect         1001da40 f    CIL library: CIL module
 0001:0001cb10       _memjrnlTruncate           1001db10 f    CIL library: CIL module
 0001:0001cbf0       _fileWriterWriteVarint     1001dbf0 f    CIL library: CIL module
 0001:0001cc30       _applyNumericAffinity      1001dc30 f    CIL library: CIL module
 0001:0001ccb0       _findNextHostParameter     1001dcb0 f    CIL library: CIL module
 0001:0001cf90       _sqlite3VdbeRecordUnpack   1001df90 f    CIL library: CIL module
 0001:0001d0e0       _sqlite3VdbeMemNumerify    1001e0e0 f    CIL library: CIL module
 0001:0001d1a0       _sqlite3VdbeMemRealify     1001e1a0 f    CIL library: CIL module
 0001:0001d200       _sqlite3VdbeIntValue       1001e200 f    CIL library: CIL module
 0001:0001d270       _cellSizePtr               1001e270 f    CIL library: CIL module
 0001:0001d330       _btreeParseCellPtr         1001e330 f    CIL library: CIL module
 0001:0001d460       _sqlite3BtreeClearCursor   1001e460 f    CIL library: CIL module
 0001:0001d480       _invalidateOverflowCache   1001e480 f    CIL library: CIL module
 0001:0001d4a0       _clearAllSharedCacheTableLocks 1001e4a0 f    CIL library: CIL module
 0001:0001d5a0       _sqlite3BtreeLeave         1001e5a0 f    CIL library: CIL module
 0001:0001d5d0       _sqlite3BtreeEnter         1001e5d0 f    CIL library: CIL module
 0001:0001d690       _sqlite3WalExclusiveMode   1001e690 f    CIL library: CIL module
 0001:0001d700       _walWriteOneFrame          1001e700 f    CIL library: CIL module
 0001:0001d7c0       _sqlite3WalEndWriteTransaction 1001e7c0 f    CIL library: CIL module
 0001:0001d7f0       _sqlite3WalBeginWriteTransaction 1001e7f0 f    CIL library: CIL module
 0001:0001d870       _sqlite3WalEndReadTransaction 1001e870 f    CIL library: CIL module
 0001:0001d8d0       _walIndexTryHdr            1001e8d0 f    CIL library: CIL module
 0001:0001da10       _walBusyLock               1001ea10 f    CIL library: CIL module
 0001:0001da60       _walIteratorFree           1001ea60 f    CIL library: CIL module
 0001:0001da70       _walIndexClose             1001ea70 f    CIL library: CIL module
 0001:0001db50       _walIndexWriteHdr          1001eb50 f    CIL library: CIL module
 0001:0001dbd0       _pagerExclusiveLock        1001ebd0 f    CIL library: CIL module
 0001:0001dc30       _sqlite3PagerUnref         1001ec30 f    CIL library: CIL module
 0001:0001dcb0       _sqlite3PagerLookup        1001ecb0 f    CIL library: CIL module
 0001:0001dce0       _hasHotJournal             1001ece0 f    CIL library: CIL module
 0001:0001de90       _openSubJournal            1001ee90 f    CIL library: CIL module
 0001:0001dee0       _pagerFreeMapHdrs          1001eee0 f    CIL library: CIL module
 0001:0001dfa0       _pager_wait_on_lock        1001efa0 f    CIL library: CIL module
 0001:0001e000       _sqlite3PagerSetMmapLimit  1001f000 f    CIL library: CIL module
 0001:0001e060       _sqlite3PagerSetCachesize  1001f060 f    CIL library: CIL module
 0001:0001e0d0       _setSectorSize             1001f0d0 f    CIL library: CIL module
 0001:0001e140       _pager_lookup              1001f140 f    CIL library: CIL module
 0001:0001e170       _writeMasterJournal        1001f170 f    CIL library: CIL module
 0001:0001e370       _readMasterJournal         1001f370 f    CIL library: CIL module
 0001:0001e4d0       _rowSetToList              1001f4d0 f    CIL library: CIL module
 0001:0001e4f0       _pcache1Free               1001f4f0 f    CIL library: CIL module
 0001:0001e5e0       _sqlite3PcacheDirtyList    1001f5e0 f    CIL library: CIL module
 0001:0001e750       _sqlite3PcacheTruncate     1001f750 f    CIL library: CIL module
 0001:0001e800       _sqlite3PcacheCleanAll     1001f800 f    CIL library: CIL module
 0001:0001e8b0       _sqlite3BitvecDestroy      1001f8b0 f    CIL library: CIL module
 0001:0001e8f0       _winIsDir                  1001f8f0 f    CIL library: CIL module
 0001:0001e9e0       _winShmBarrier             1001f9e0 f    CIL library: CIL module
 0001:0001ea30       _winShmSystemLock          1001fa30 f    CIL library: CIL module
 0001:0001ea90       _winCheckReservedLock      1001fa90 f    CIL library: CIL module
 0001:0001eb00       _sqlite3HashFind           1001fb00 f    CIL library: CIL module
 0001:0001eb70       _sqlite3HashClear          1001fb70 f    CIL library: CIL module
 0001:0001eca0       _sqlite3DbFree             1001fca0 f    CIL library: CIL module
 0001:0001ed20       _mallocWithAlarm           1001fd20 f    CIL library: CIL module
 0001:0001ee10       _computeYMD_HMS            1001fe10 f    CIL library: CIL module
 0001:0001ee20       _parseHhMmSs               1001fe20 f    CIL library: CIL module
 0001:0001f2c0       _rtreeValueUp              100202c0 f    CIL library: CIL module
 0001:0001f360       _rtreeValueDown            10020360 f    CIL library: CIL module
 0001:0001f400       _nodeParentIndex           10020400 f    CIL library: CIL module
 0001:0001f430       _testRtreeEntry            10020430 f    CIL library: CIL module
 0001:0001f580       _testRtreeCell             10020580 f    CIL library: CIL module
 0001:0001f6d0       _fts3SnippetDetails        100206d0 f    CIL library: CIL module
 0001:0001f840       _fts3SnippetAdvance        10020840 f    CIL library: CIL module
 0001:0001f8a0       _sqlite3Fts3FreeDeferredTokens 100208a0 f    CIL library: CIL module
 0001:0001f970       _sqlite3Fts3FreeDeferredDoclists 10020970 f    CIL library: CIL module
 0001:0001f9a0       _fts3SegWriterFree         100209a0 f    CIL library: CIL module
 0001:0001f9d0       _fts3tokNextMethod         100209d0 f    CIL library: CIL module
 0001:0001fa60       _fts3tokCloseMethod        10020a60 f    CIL library: CIL module
 0001:0001fab0       _porter_stemmer            10020ab0 f    CIL library: CIL module
 0001:000204a0       _sqlite3Fts3HashFindElem   100214a0 f    CIL library: CIL module
 0001:000204e0       _sqlite3Fts3HashClear      100214e0 f    CIL library: CIL module
 0001:00020540       _hashDestroy               10021540 f    CIL library: CIL module
 0001:00020560       _fts3DoclistPhraseMerge    10021560 f    CIL library: CIL module
 0001:00020830       _fts3PoslistMerge          10021830 f    CIL library: CIL module
 0001:00020c70       _functionDestroy           10021c70 f    CIL library: CIL module
 0001:00020ca0       _sqlite3CloseSavepoints    10021ca0 f    CIL library: CIL module
 0001:00020d60       _whereAndInfoDelete        10021d60 f    CIL library: CIL module
 0001:00020d80       _whereOrInfoDelete         10021d80 f    CIL library: CIL module
 0001:00020da0       _sqlite3VtabClear          10021da0 f    CIL library: CIL module
 0001:00020df0       _sqlite3VtabUnlock         10021df0 f    CIL library: CIL module
 0001:00020e20       _sqlite3TriggerColmask     10021e20 f    CIL library: CIL module
 0001:00020ef0       _transferParseError        10021ef0 f    CIL library: CIL module
 0001:00020f10       _sqlite3TriggersExist      10021f10 f    CIL library: CIL module
 0001:00020f80       _tableOfTrigger            10021f80 f    CIL library: CIL module
 0001:00020fc0       _sqlite3GetBoolean         10021fc0 f    CIL library: CIL module
 0001:00020fe0       _sqlite3CloseExtensions    10021fe0 f    CIL library: CIL module
 0001:00021090       _sqlite3FkReferences       10022090 f    CIL library: CIL module
 0001:000210d0       _sqlite3IdListDelete       100220d0 f    CIL library: CIL module
 0001:00021180       _sqlite3CollapseDatabaseArray 10022180 f    CIL library: CIL module
 0001:00021300       _sqlite3FindIndex          10022300 f    CIL library: CIL module
 0001:00021430       _sqlite3FindTable          10022430 f    CIL library: CIL module
 0001:00021580       _sqlite3DeleteIndexSamples 10022580 f    CIL library: CIL module
 0001:00021670       _analysisLoader            10022670 f    CIL library: CIL module
 0001:00021790       _isAppropriateForFactoring 10022790 f    CIL library: CIL module
 0001:00021870       _sqlite3SelectExprHeight   10022870 f    CIL library: CIL module
 0001:00021890       _exprSetHeight             10022890 f    CIL library: CIL module
 0001:00021940       _sqlite3IndexAffinityOk    10022940 f    CIL library: CIL module
 0001:00021970       _memjrnlClose              10022970 f    CIL library: CIL module
 0001:00021990       _fileWriterFinish          10022990 f    CIL library: CIL module
 0001:00021a20       _vdbeSorterRecordFree      10022a20 f    CIL library: CIL module
 0001:00021ab0       _vdbeSorterIterZero        10022ab0 f    CIL library: CIL module
 0001:00021b60       _Cleanup                   10022b60 f    CIL library: CIL module
 0001:00021b80       _sqlite3VdbeLeave          10022b80 f    CIL library: CIL module
 0001:00021c00       _sqlite3VdbeEnter          10022c00 f    CIL library: CIL module
 0001:00021c70       _freeEphemeralFunction     10022c70 f    CIL library: CIL module
 0001:00021c80       _sqlite3VdbeMemIntegerify  10022c80 f    CIL library: CIL module
 0001:00021cb0       _sqlite3VdbeMemFinalize    10022cb0 f    CIL library: CIL module
 0001:00021d20       _sqlite3BtreeCacheOverflow 10022d20 f    CIL library: CIL module
 0001:00021d40       _sqlite3BtreeSchemaLocked  10022d40 f    CIL library: CIL module
 0001:00021db0       _sqlite3BtreeGetMeta       10022db0 f    CIL library: CIL module
 0001:00021e20       _sqlite3BtreeCursor        10022e20 f    CIL library: CIL module
 0001:00021eb0       _sqlite3BtreeGetAutoVacuum 10022eb0 f    CIL library: CIL module
 0001:00021f00       _sqlite3BtreeSetAutoVacuum 10022f00 f    CIL library: CIL module
 0001:00021f80       _sqlite3BtreeSecureDelete  10022f80 f    CIL library: CIL module
 0001:00021ff0       _sqlite3BtreeMaxPageCount  10022ff0 f    CIL library: CIL module
 0001:00022040       _sqlite3BtreeGetReserve    10023040 f    CIL library: CIL module
 0001:00022080       _sqlite3BtreeSyncDisabled  10023080 f    CIL library: CIL module
 0001:000220c0       _sqlite3BtreeSetSafetyLevel 100230c0 f    CIL library: CIL module
 0001:00022110       _sqlite3BtreeSetMmapLimit  10023110 f    CIL library: CIL module
 0001:000221a0       _sqlite3BtreeSetCacheSize  100231a0 f    CIL library: CIL module
 0001:00022240       _releasePage               10023240 f    CIL library: CIL module
 0001:00022250       _btreePageLookup           10023250 f    CIL library: CIL module
 0001:000222b0       _btreeParseCell            100232b0 f    CIL library: CIL module
 0001:000222e0       _btreeReleaseAllCursorPages 100232e0 f    CIL library: CIL module
 0001:000223d0       _btreeClearHasContent      100233d0 f    CIL library: CIL module
 0001:00022430       _invalidateAllOverflowCache 10023430 f    CIL library: CIL module
 0001:00022460       _sqlite3BtreeLeaveAll      10023460 f    CIL library: CIL module
 0001:000224c0       _sqlite3BtreeEnterAll      100234c0 f    CIL library: CIL module
 0001:000225d0       _sqlite3BtreeLeaveCursor   100235d0 f    CIL library: CIL module
 0001:00022600       _sqlite3BtreeEnterCursor   10023600 f    CIL library: CIL module
 0001:00022610       _sqlite3PagerExclusiveLock 10023610 f    CIL library: CIL module
 0001:00022630       _sqlite3PagerBegin         10023630 f    CIL library: CIL module
 0001:00022730       _releaseAllSavepoints      10023730 f    CIL library: CIL module
 0001:000227f0       _writeJournalHdr           100237f0 f    CIL library: CIL module
 0001:00022a20       _sqlite3RowSetClear        10023a20 f    CIL library: CIL module
 0001:00022ad0       _sqlite3PageFree           10023ad0 f    CIL library: CIL module
 0001:00022ae0       _pcache1FreePage           10023ae0 f    CIL library: CIL module
 0001:00022b00       _sqlite3PcacheClear        10023b00 f    CIL library: CIL module
 0001:00022b10       _winShmLock                10023b10 f    CIL library: CIL module
 0001:00022d00       _getReadLock               10023d00 f    CIL library: CIL module
 0001:00022e20       _removeElementGivenHash    10023e20 f    CIL library: CIL module
 0001:00022e70       _sqlite3StrAccumReset      10023e70 f    CIL library: CIL module
 0001:00022ea0       _sqlite3StrAccumAppend     10023ea0 f    CIL library: CIL module
 0001:00022fd0       _sqlite3AppendSpace        10023fd0 f    CIL library: CIL module
 0001:00023130       _sqlite3ScratchMalloc      10024130 f    CIL library: CIL module
 0001:00023240       _sqlite3Malloc             10024240 f    CIL library: CIL module
 0001:000232b0       _parseYyyyMmDd             100242b0 f    CIL library: CIL module
 0001:000234c0       _fixBoundingBox            100244c0 f    CIL library: CIL module
 0001:000235a0       _AdjustTree                100245a0 f    CIL library: CIL module
 0001:00023670       _fts3SnippetNextCandidate  10024670 f    CIL library: CIL module
 0001:00023800       _sqlite3Fts3PendingTermsClear 10024800 f    CIL library: CIL module
 0001:000238e0       _sqlite3Fts3HashFind       100248e0 f    CIL library: CIL module
 0001:00023920       _fts3RemoveElementByHash   10024920 f    CIL library: CIL module
 0001:000239a0       _fts3EvalPhraseMergeToken  100249a0 f    CIL library: CIL module
 0001:00023a50       _fts3RollbackToMethod      10024a50 f    CIL library: CIL module
 0001:00023a70       _fts3RollbackMethod        10024a70 f    CIL library: CIL module
 0001:00023a90       _fts3PoslistNearMerge      10024a90 f    CIL library: CIL module
 0001:00023c10       _setupLookaside            10024c10 f    CIL library: CIL module
 0001:00023d20       _explainAppendTerm         10024d20 f    CIL library: CIL module
 0001:00023d70       _termCanDriveIndex         10024d70 f    CIL library: CIL module
 0001:00023de0       _callFinaliser             10024de0 f    CIL library: CIL module
 0001:00023e80       _sqlite3VtabCallDestroy    10024e80 f    CIL library: CIL module
 0001:00023f00       _sqlite3VtabUnlockList     10024f00 f    CIL library: CIL module
 0001:00023f60       _sqlite3VtabDisconnect     10024f60 f    CIL library: CIL module
 0001:00023fb0       _sqlite3FkRequired         10024fb0 f    CIL library: CIL module
 0001:00024190       _sqlite3SrcListDelete      10025190 f    CIL library: CIL module
 0001:00024250       _freeIndex                 10025250 f    CIL library: CIL module
 0001:00024270       _stat3Push                 10025270 f    CIL library: CIL module
 0001:00024440       _sqlite3VdbeSorterClose    10025440 f    CIL library: CIL module
 0001:00024510       _sqlite3VdbeMemSetNull     10025510 f    CIL library: CIL module
 0001:00024560       _sqlite3VdbeMemReleaseExternal 10025560 f    CIL library: CIL module
 0001:000245d0       _moveToParent              100255d0 f    CIL library: CIL module
 0001:00024600       _fetchPayload              10025600 f    CIL library: CIL module
 0001:00024680       _getCellInfo               10025680 f    CIL library: CIL module
 0001:000246d0       _sqlite3BtreeTripAllCursors 100256d0 f    CIL library: CIL module
 0001:00024820       _unlockBtreeIfUnused       10025820 f    CIL library: CIL module
 0001:00024850       _freeTempSpace             10025850 f    CIL library: CIL module
 0001:00024870       _syncJournal               10025870 f    CIL library: CIL module
 0001:00024ac0       _pager_end_transaction     10025ac0 f    CIL library: CIL module
 0001:00024d00       _pager_reset               10025d00 f    CIL library: CIL module
 0001:00024d30       _sqlite3RowSetNext         10025d30 f    CIL library: CIL module
 0001:00024d80       _pcache1Unpin              10025d80 f    CIL library: CIL module
 0001:00024e30       _pcache1TruncateUnsafe     10025e30 f    CIL library: CIL module
 0001:00024f00       _pcache1EnforceMaxPage     10025f00 f    CIL library: CIL module
 0001:00024fd0       _pcache1Alloc              10025fd0 f    CIL library: CIL module
 0001:000250d0       _rehash                    100260d0 f    CIL library: CIL module
 0001:00025220       _sqlite3VXPrintf           10026220 f    CIL library: CIL module
 0001:000260a0       _sqlite3DbMallocRaw        100270a0 f    CIL library: CIL module
 0001:00026120       _sqlite3DbMallocZero       10027120 f    CIL library: CIL module
 0001:00026140       _sqlite3MallocZero         10027140 f    CIL library: CIL module
 0001:00026160       _sqlite3Realloc            10027160 f    CIL library: CIL module
 0001:000262e0       _winMutexAlloc             100272e0 f    CIL library: CIL module
 0001:00026340       _sqlite3OsOpenMalloc       10027340 f    CIL library: CIL module
 0001:000263b0       _parseDateOrTime           100273b0 f    CIL library: CIL module
 0001:00026450       _CreateCryptBlock          10027450 f    CIL library: CIL module
 0001:00026520       _sqlite3StrDup             10027520 f    CIL library: CIL module
 0001:00026560       _vtshimCopyModule          10027560 f    CIL library: CIL module
 0001:000265b0       _splitNodeStartree         100275b0 f    CIL library: CIL module
 0001:00026af0       _deserializeGeometry       10027af0 f    CIL library: CIL module
 0001:00026be0       _rtreeOpen                 10027be0 f    CIL library: CIL module
 0001:00026c30       _nodeNew                   10027c30 f    CIL library: CIL module
 0001:00026c90       _sqlite3Fts3DeferToken     10027c90 f    CIL library: CIL module
 0001:00026ce0       _sqlite3Fts3DeferredTokenList 10027ce0 f    CIL library: CIL module
 0001:00026d60       _sqlite3Fts3SegReaderNew   10027d60 f    CIL library: CIL module
 0001:00026e50       _fts3tokFilterMethod       10027e50 f    CIL library: CIL module
 0001:00026f60       _fts3tokOpenMethod         10027f60 f    CIL library: CIL module
 0001:00026fb0       _fts3tokDequoteArray       10027fb0 f    CIL library: CIL module
 0001:000270d0       _simpleOpen                100280d0 f    CIL library: CIL module
 0001:00027140       _simpleCreate              10028140 f    CIL library: CIL module
 0001:00027220       _porterOpen                10028220 f    CIL library: CIL module
 0001:00027290       _porterCreate              10028290 f    CIL library: CIL module
 0001:000272c0       _fts3HashMalloc            100282c0 f    CIL library: CIL module
 0001:000272f0       _fts3MallocZero            100282f0 f    CIL library: CIL module
 0001:00027320       _fts3auxOpenMethod         10028320 f    CIL library: CIL module
 0001:00027360       _fts3EvalNearTrim          10028360 f    CIL library: CIL module
 0001:000273e0       _fts3EvalDeferredPhrase    100283e0 f    CIL library: CIL module
 0001:00027600       _fts3DoclistOrMerge        10028600 f    CIL library: CIL module
 0001:000279c0       _fts3OpenMethod            100289c0 f    CIL library: CIL module
 0001:00027a00       _fts3PrefixParameter       10028a00 f    CIL library: CIL module
 0001:00027af0       _fts3QuoteId               10028af0 f    CIL library: CIL module
 0001:00027b50       _disconnectAllVtab         10028b50 f    CIL library: CIL module
 0001:00027d50       _bestAutomaticIndex        10028d50 f    CIL library: CIL module
 0001:00027e40       _sqlite3VtabCommit         10028e40 f    CIL library: CIL module
 0001:00027e50       _sqlite3VtabRollback       10028e50 f    CIL library: CIL module
 0001:00027e60       _triggerStepAllocate       10028e60 f    CIL library: CIL module
 0001:00027eb0       _clearSelect               10028eb0 f    CIL library: CIL module
 0001:00027f40       _autoIncBegin              10028f40 f    CIL library: CIL module
 0001:00027fb0       _sqlite3IndexAffinityStr   10028fb0 f    CIL library: CIL module
 0001:00028020       _sqlite3FindFunction       10029020 f    CIL library: CIL module
 0001:00028210       _dup8bytes                 10029210 f    CIL library: CIL module
 0001:00028230       _sqlite3ExprAlloc          10029230 f    CIL library: CIL module
 0001:00028340       _sqlite3ExprAddCollateToken 10029340 f    CIL library: CIL module
 0001:00028370       _sqlite3CreateColumnExpr   10029370 f    CIL library: CIL module
 0001:00028410       _memjrnlWrite              10029410 f    CIL library: CIL module
 0001:00028530       _fileWriterInit            10029530 f    CIL library: CIL module
 0001:000285b0       _vdbeSorterOpenTempFile    100295b0 f    CIL library: CIL module
 0001:00028750       _sqlite3VdbeAllocUnpackedRecord 10029750 f    CIL library: CIL module
 0001:000287a0       _sqlite3VdbeCreate         100297a0 f    CIL library: CIL module
 0001:00028800       _sqlite3ValueNew           10029800 f    CIL library: CIL module
 0001:00028840       _sqlite3VdbeMemCopy        10029840 f    CIL library: CIL module
 0001:000288b0       _sqlite3VdbeMemShallowCopy 100298b0 f    CIL library: CIL module
 0001:00028900       _sqlite3VdbeMemRelease     10029900 f    CIL library: CIL module
 0001:00028940       _sqlite3BtreeSchema        10029940 f    CIL library: CIL module
 0001:000289c0       _checkAppendMsg            100299c0 f    CIL library: CIL module
 0001:00028a30       _sqlite3BtreeDataFetch     10029a30 f    CIL library: CIL module
 0001:00028ac0       _sqlite3BtreeKeyFetch      10029ac0 f    CIL library: CIL module
 0001:00028b20       _sqlite3BtreeDataSize      10029b20 f    CIL library: CIL module
 0001:00028b80       _sqlite3BtreeKeySize       10029b80 f    CIL library: CIL module
 0001:00028bf0       _sqlite3BtreeCloseCursor   10029bf0 f    CIL library: CIL module
 0001:00028ce0       _btreeEndTransaction       10029ce0 f    CIL library: CIL module
 0001:00028d70       _setSharedCacheTableLock   10029d70 f    CIL library: CIL module
 0001:00028e30       _sqlite3WalOpen            10029e30 f    CIL library: CIL module
 0001:00028f50       _pagerOpenWal              10029f50 f    CIL library: CIL module
 0001:00029000       _sqlite3PagerClearCache    1002a000 f    CIL library: CIL module
 0001:00029040       _sqlite3PagerCommitPhaseTwo 1002a040 f    CIL library: CIL module
 0001:00029090       _pagerAcquireMapPage       1002a090 f    CIL library: CIL module
 0001:00029160       _pager_delmaster           1002a160 f    CIL library: CIL module
 0001:00029390       _pager_unlock              1002a390 f    CIL library: CIL module
 0001:000294c0       _rowSetEntryAlloc          1002a4c0 f    CIL library: CIL module
 0001:00029510       _pcache1Destroy            1002a510 f    CIL library: CIL module
 0001:00029580       _pcache1Truncate           1002a580 f    CIL library: CIL module
 0001:000295d0       _pcache1Shrink             1002a5d0 f    CIL library: CIL module
 0001:00029620       _pcache1Cachesize          1002a620 f    CIL library: CIL module
 0001:00029690       _pcache1Create             1002a690 f    CIL library: CIL module
 0001:00029740       _pcache1ResizeHash         1002a740 f    CIL library: CIL module
 0001:00029840       _sqlite3PageMalloc         1002a840 f    CIL library: CIL module
 0001:00029850       _pcache1AllocPage          1002a850 f    CIL library: CIL module
 0001:000298c0       _sqlite3BitvecCreate       1002a8c0 f    CIL library: CIL module
 0001:00029900       _unicodeToMbcs             1002a900 f    CIL library: CIL module
 0001:00029980       _mbcsToUnicode             1002a980 f    CIL library: CIL module
 0001:00029a00       _unicodeToUtf8             1002aa00 f    CIL library: CIL module
 0001:00029a80       _utf8ToUnicode             1002aa80 f    CIL library: CIL module
 0001:00029b00       _sqlite3HashInsert         1002ab00 f    CIL library: CIL module
 0001:00029c40       _sqlite3HexToBlob          1002ac40 f    CIL library: CIL module
 0001:00029cd0       _sqlite3XPrintf            1002acd0 f    CIL library: CIL module
 0001:00029cf0       _sqlite3StrAccumFinish     1002acf0 f    CIL library: CIL module
 0001:00029d70       _sqlite3DbStrNDup          1002ad70 f    CIL library: CIL module
 0001:00029da0       _sqlite3DbStrDup           1002ada0 f    CIL library: CIL module
 0001:00029df0       _sqlite3DefaultMutex       1002adf0 f    CIL library: CIL module
 0001:00029e00       _sqlite3MutexInit          1002ae00 f    CIL library: CIL module
 0001:00029eb0       _modeStep                  1002aeb0 f    CIL library: CIL module
 0001:0002a050       _varianceStep              1002b050 f    CIL library: CIL module
 0001:0002a150       _fts3Rehash                1002b150 f    CIL library: CIL module
 0001:0002a260       _getNextToken              1002b260 f    CIL library: CIL module
 0001:0002a430       _fts3EvalNearTest          1002b430 f    CIL library: CIL module
 0001:0002a5f0       _fts3TermSelectMerge       1002b5f0 f    CIL library: CIL module
 0001:0002a6f0       _fts3TermSelectFinishMerge 1002b6f0 f    CIL library: CIL module
 0001:0002a790       _explainIndexRange         1002b790 f    CIL library: CIL module
 0001:0002a9b0       _sqlite3VtabOverloadFunction 1002b9b0 f    CIL library: CIL module
 0001:0002aad0       _sqlite3VtabSync           1002bad0 f    CIL library: CIL module
 0001:0002abb0       _sqlite3SelectDelete       1002bbb0 f    CIL library: CIL module
 0001:0002abd0       _sqlite3IsLikeFunction     1002bbd0 f    CIL library: CIL module
 0001:0002ac50       _setLikeOptFlag            1002bc50 f    CIL library: CIL module
 0001:0002ac90       _groupConcatStep           1002bc90 f    CIL library: CIL module
 0001:0002ada0       _minmaxStep                1002bda0 f    CIL library: CIL module
 0001:0002ae90       _countStep                 1002be90 f    CIL library: CIL module
 0001:0002af00       _sumStep                   1002bf00 f    CIL library: CIL module
 0001:0002b010       _findCollSeqEntry          1002c010 f    CIL library: CIL module
 0001:0002b0d0       _sqlite3NameFromToken      1002c0d0 f    CIL library: CIL module
 0001:0002b130       _sqlite3UnlinkAndDeleteIndex 1002c130 f    CIL library: CIL module
 0001:0002b230       _sqlite3ExprListSetSpan    1002c230 f    CIL library: CIL module
 0001:0002b2b0       _sqlite3ExprListSetName    1002c2b0 f    CIL library: CIL module
 0001:0002b320       _sqlite3IdListDup          1002c320 f    CIL library: CIL module
 0001:0002b400       _sqlite3SrcListDup         1002c400 f    CIL library: CIL module
 0001:0002b680       _sqlite3ExprListDup        1002c680 f    CIL library: CIL module
 0001:0002b820       _sqlite3ExprDelete         1002c820 f    CIL library: CIL module
 0001:0002b8e0       _sqlite3ExprAttachSubtrees 1002c8e0 f    CIL library: CIL module
 0001:0002b930       _sqlite3Expr               1002c930 f    CIL library: CIL module
 0001:0002b980       _sqlite3ExprAddCollateString 1002c980 f    CIL library: CIL module
 0001:0002b9e0       _sqlite3VdbeSorterInit     1002c9e0 f    CIL library: CIL module
 0001:0002baa0       _importVtabErrMsg          1002caa0 f    CIL library: CIL module
 0001:0002bd10       _releaseMemArray           1002cd10 f    CIL library: CIL module
 0001:0002bdf0       _sqlite3VdbeSetSql         1002cdf0 f    CIL library: CIL module
 0001:0002be50       _sqlite3ValueFree          1002ce50 f    CIL library: CIL module
 0001:0002bea0       _sqlite3VdbeMemSetStr      1002cea0 f    CIL library: CIL module
 0001:0002c090       _sqlite3VdbeMemMove        1002d090 f    CIL library: CIL module
 0001:0002c0e0       _sqlite3VdbeMemSetRowSet   1002d0e0 f    CIL library: CIL module
 0001:0002c190       _sqlite3VdbeMemSetDouble   1002d190 f    CIL library: CIL module
 0001:0002c240       _sqlite3VdbeMemSetInt64    1002d240 f    CIL library: CIL module
 0001:0002c290       _sqlite3VdbeMemSetZeroBlob 1002d290 f    CIL library: CIL module
 0001:0002c2f0       _sqlite3BtreeLockTable     1002d2f0 f    CIL library: CIL module
 0001:0002c360       _checkRef                  1002d360 f    CIL library: CIL module
 0001:0002c3e0       _sqlite3BtreeCommitPhaseTwo 1002d3e0 f    CIL library: CIL module
 0001:0002c460       _allocateTempSpace         1002d460 f    CIL library: CIL module
 0001:0002c480       _sqlite3PagerOpenWal       1002d480 f    CIL library: CIL module
 0001:0002c4f0       _sqlite3PagerOpenSavepoint 1002d4f0 f    CIL library: CIL module
 0001:0002c620       _pager_open_journal        1002d620 f    CIL library: CIL module
 0001:0002c730       _sqlite3PagerSetPagesize   1002d730 f    CIL library: CIL module
 0001:0002c8b0       _pagerOpenWalIfPresent     1002d8b0 f    CIL library: CIL module
 0001:0002c940       _readJournalHdr            1002d940 f    CIL library: CIL module
 0001:0002cbf0       _sqlite3RowSetTest         1002dbf0 f    CIL library: CIL module
 0001:0002cd40       _sqlite3RowSetInsert       1002dd40 f    CIL library: CIL module
 0001:0002cdd0       _pcache1Fetch              1002ddd0 f    CIL library: CIL module
 0001:0002cfe0       _sqlite3BitvecSet          1002dfe0 f    CIL library: CIL module
 0001:0002d250       _renderLogMsg              1002e250 f    CIL library: CIL module
 0001:0002d3e0       _sqlite3VMPrintf           1002e3e0 f    CIL library: CIL module
 0001:0002d450       _sqlite3SetString          1002e450 f    CIL library: CIL module
 0001:0002d4d0       _sqlite3Fts3HashInsert     1002e4d0 f    CIL library: CIL module
 0001:0002d620       _fts3EvalTestExpr          1002e620 f    CIL library: CIL module
 0001:0002d830       _binaryToUnaryIfNull       1002e830 f    CIL library: CIL module
 0001:0002d860       _whereClauseInsert         1002e860 f    CIL library: CIL module
 0001:0002d950       _whereClauseClear          1002e950 f    CIL library: CIL module
 0001:0002d9d0       _sqlite3TriggerSelectStep  1002e9d0 f    CIL library: CIL module
 0001:0002da30       _minMaxFinalize            1002ea30 f    CIL library: CIL module
 0001:0002dab0       _nullifFunc                1002eab0 f    CIL library: CIL module
 0001:0002daf0       _minmaxFunc                1002eaf0 f    CIL library: CIL module
 0001:0002dcb0       _sqlite3FindCollSeq        1002ecb0 f    CIL library: CIL module
 0001:0002dce0       _synthCollSeq              1002ece0 f    CIL library: CIL module
 0001:0002dd80       _sqlite3SrcListIndexedBy   1002ed80 f    CIL library: CIL module
 0001:0002ddd0       _sqlite3AddColumnType      1002edd0 f    CIL library: CIL module
 0001:0002de10       _sqlite3FindDb             1002ee10 f    CIL library: CIL module
 0001:0002de80       _sqliteDeleteColumnNames   1002ee80 f    CIL library: CIL module
 0001:0002df00       _sqlite3NestedParse        1002ef00 f    CIL library: CIL module
 0001:0002e000       _sqlite3ExprListDelete     1002f000 f    CIL library: CIL module
 0001:0002e070       _sqlite3SelectDup          1002f070 f    CIL library: CIL module
 0001:0002e1a0       _exprDup                   1002f1a0 f    CIL library: CIL module
 0001:0002e410       _sqlite3ExprAnd            1002f410 f    CIL library: CIL module
 0001:0002e500       _sqlite3TransferBindings   1002f500 f    CIL library: CIL module
 0001:0002e970       _setResultStrOrError       1002f970 f    CIL library: CIL module
 0001:0002e9a0       _sqlite3VdbeCheckFk        1002f9a0 f    CIL library: CIL module
 0001:0002ea10       _sqlite3VdbeSetColName     1002fa10 f    CIL library: CIL module
 0001:0002ea50       _sqlite3VdbeSetNumCols     1002fa50 f    CIL library: CIL module
 0001:0002ead0       _freeP4                    1002fad0 f    CIL library: CIL module
 0001:0002ebd0       _sqlite3ValueSetStr        1002fbd0 f    CIL library: CIL module
 0001:0002ebf0       _sqlite3BtreeBeginStmt     1002fbf0 f    CIL library: CIL module
 0001:0002ec40       _sqlite3BtreeSetPageSize   1002fc40 f    CIL library: CIL module
 0001:0002ed20       _btreeSetHasContent        1002fd20 f    CIL library: CIL module
 0001:0002ed90       _addToSavepointBitvecs     1002fd90 f    CIL library: CIL module
 0001:0002efd0       _sqlite3BitvecBuiltinTest  1002ffd0 f    CIL library: CIL module
 0001:0002f280       _convertUtf8Filename       10030280 f    CIL library: CIL module
 0001:0002f330       _sqlite3ErrorMsg           10030330 f    CIL library: CIL module
 0001:0002f3f0       _sqlite3Error              100303f0 f    CIL library: CIL module
 0001:0002f5a0       _sqlite3MAppendf           100305a0 f    CIL library: CIL module
 0001:0002f630       _sqlite3MPrintf            10030630 f    CIL library: CIL module
 0001:0002f6b0       _sqlite3ApiExit            100306b0 f    CIL library: CIL module
 0001:0002f6f0       _localtimeOffset           100306f0 f    CIL library: CIL module
 0001:0002fa90       _lastRowsFunc              10030a90 f    CIL library: CIL module
 0001:0002faf0       _differenceFunc            10030af0 f    CIL library: CIL module
 0001:0002fd60       _varianceFinalize          10030d60 f    CIL library: CIL module
 0001:0002fde0       _stdevFinalize             10030de0 f    CIL library: CIL module
 0001:0002fe60       __medianFinalize           10030e60 f    CIL library: CIL module
 0001:0002ff70       _modeFinalize              10030f70 f    CIL library: CIL module
 0001:00030060       _charindexFunc             10031060 f    CIL library: CIL module
 0001:00030130       _floorFunc                 10031130 f    CIL library: CIL module
 0001:00030200       _ceilFunc                  10031200 f    CIL library: CIL module
 0001:000302d0       _signFunc                  100312d0 f    CIL library: CIL module
 0001:00030410       _atn2Func                  10031410 f    CIL library: CIL module
 0001:00030540       _powerFunc                 10031540 f    CIL library: CIL module
 0001:000306c0       _squareFunc                100316c0 f    CIL library: CIL module
 0001:000307b0       _piFunc                    100317b0 f    CIL library: CIL module
 0001:000307e0       _deg2radFunc               100317e0 f    CIL library: CIL module
 0001:00030900       _rad2degFunc               10031900 f    CIL library: CIL module
 0001:00030a20       _expFunc                   10031a20 f    CIL library: CIL module
 0001:00030b40       _log10Func                 10031b40 f    CIL library: CIL module
 0001:00030c60       _logFunc                   10031c60 f    CIL library: CIL module
 0001:00030d80       _cothFunc                  10031d80 f    CIL library: CIL module
 0001:00030ea0       _tanhFunc                  10031ea0 f    CIL library: CIL module
 0001:00030fc0       _coshFunc                  10031fc0 f    CIL library: CIL module
 0001:000310e0       _sinhFunc                  100320e0 f    CIL library: CIL module
 0001:00031200       _cotFunc                   10032200 f    CIL library: CIL module
 0001:00031320       _tanFunc                   10032320 f    CIL library: CIL module
 0001:00031440       _cosFunc                   10032440 f    CIL library: CIL module
 0001:00031560       _sinFunc                   10032560 f    CIL library: CIL module
 0001:00031680       _atanhFunc                 10032680 f    CIL library: CIL module
 0001:000317b0       _asinhFunc                 100327b0 f    CIL library: CIL module
 0001:000318e0       _acoshFunc                 100328e0 f    CIL library: CIL module
 0001:00031a10       _atanFunc                  10032a10 f    CIL library: CIL module
 0001:00031b30       _asinFunc                  10032b30 f    CIL library: CIL module
 0001:00031c50       _acosFunc                  10032c50 f    CIL library: CIL module
 0001:00031d70       _sqrtFunc                  10032d70 f    CIL library: CIL module
 0001:00031e90       _vtshimRollbackTo          10032e90 f    CIL library: CIL module
 0001:00031f80       _vtshimRelease             10032f80 f    CIL library: CIL module
 0001:00032070       _vtshimSavepoint           10033070 f    CIL library: CIL module
 0001:00032160       _vtshimRename              10033160 f    CIL library: CIL module
 0001:00032250       _vtshimFindFunction        10033250 f    CIL library: CIL module
 0001:00032340       _vtshimRollback            10033340 f    CIL library: CIL module
 0001:00032420       _vtshimCommit              10033420 f    CIL library: CIL module
 0001:00032500       _vtshimSync                10033500 f    CIL library: CIL module
 0001:000325e0       _vtshimBegin               100335e0 f    CIL library: CIL module
 0001:000326c0       _vtshimUpdate              100336c0 f    CIL library: CIL module
 0001:000327b0       _vtshimRowid               100337b0 f    CIL library: CIL module
 0001:000328a0       _vtshimColumn              100338a0 f    CIL library: CIL module
 0001:00032990       _vtshimEof                 10033990 f    CIL library: CIL module
 0001:00032a70       _vtshimNext                10033a70 f    CIL library: CIL module
 0001:00032b50       _vtshimFilter              10033b50 f    CIL library: CIL module
 0001:00032c40       _vtshimClose               10033c40 f    CIL library: CIL module
 0001:00032d50       _vtshimOpen                10033d50 f    CIL library: CIL module
 0001:00032e20       _vtshimBestIndex           10033e20 f    CIL library: CIL module
 0001:00032f10       _vtshimConnect             10033f10 f    CIL library: CIL module
 0001:00032fe0       _vtshimCreate              10033fe0 f    CIL library: CIL module
 0001:000330b0       _rtreedepth                100340b0 f    CIL library: CIL module
 0001:00033190       _rtreeBestIndex            10034190 f    CIL library: CIL module
 0001:00033340       _rtreeColumn               10034340 f    CIL library: CIL module
 0001:00033430       _fts3MatchinfoCheck        10034430 f    CIL library: CIL module
 0001:00033490       _fts3tokQueryTokenizer     10034490 f    CIL library: CIL module
 0001:00033510       _fts3FunctionArg           10034510 f    CIL library: CIL module
 0001:00033640       _fts3Appendf               10034640 f    CIL library: CIL module
 0001:000336b0       _fts3IsSpecialColumn       100346b0 f    CIL library: CIL module
 0001:000338c0       _sqlite3CantopenError      100348c0 f    CIL library: CIL module
 0001:000338e0       _sqlite3MisuseError        100348e0 f    CIL library: CIL module
 0001:00033900       _sqlite3CorruptError       10034900 f    CIL library: CIL module
 0001:00033920       _sqlite3ParseUri           10034920 f    CIL library: CIL module
 0001:00033ea0       _createCollation           10034ea0 f    CIL library: CIL module
 0001:00034070       _sqlite3CreateFunc         10035070 f    CIL library: CIL module
 0001:00034210       _yy_syntax_error           10035210 f    CIL library: CIL module
 0001:00034230       _whereInfoFree             10035230 f    CIL library: CIL module
 0001:000342c0       _vtabBestIndex             100352c0 f    CIL library: CIL module
 0001:000343b0       _allocateIndexInfo         100353b0 f    CIL library: CIL module
 0001:00034620       _whereSplit                10035620 f    CIL library: CIL module
 0001:00034700       _vtabCallConstructor       10035700 f    CIL library: CIL module
 0001:00034a40       _createModule              10035a40 f    CIL library: CIL module
 0001:00034b70       _sqlite3TriggerInsertStep  10035b70 f    CIL library: CIL module
 0001:00034c30       _sqlite3DeleteTriggerStep  10035c30 f    CIL library: CIL module
 0001:00034d70       _sqlite3IndexedByLookup    10035d70 f    CIL library: CIL module
 0001:00034e10       _selectColumnsFromExprList 10035e10 f    CIL library: CIL module
 0001:00035210       _generateColumnTypes       10036210 f    CIL library: CIL module
 0001:000355b0       _checkForMultiColumnSelectError 100365b0 f    CIL library: CIL module
 0001:000355e0       _sqlite3JoinType           100365e0 f    CIL library: CIL module
 0001:00035740       _corruptSchema             10036740 f    CIL library: CIL module
 0001:000357d0       _sqlite3AutoLoadExtensions 100367d0 f    CIL library: CIL module
 0001:000358a0       _sqlite3LoadExtension      100368a0 f    CIL library: CIL module
 0001:00035d00       _fkTriggerDelete           10036d00 f    CIL library: CIL module
 0001:00035d60       _sqlite3FkLocateIndex      10036d60 f    CIL library: CIL module
 0001:00035fa0       _countFinalize             10036fa0 f    CIL library: CIL module
 0001:00036030       _totalFinalize             10037030 f    CIL library: CIL module
 0001:00036090       _avgFinalize               10037090 f    CIL library: CIL module
 0001:00036100       _sumFinalize               10037100 f    CIL library: CIL module
 0001:00036200       _zeroblobFunc              10037200 f    CIL library: CIL module
 0001:00036290       _unicodeFunc               10037290 f    CIL library: CIL module
 0001:000362d0       _compileoptionusedFunc     100372d0 f    CIL library: CIL module
 0001:00036350       _errlogFunc                10037350 f    CIL library: CIL module
 0001:00036380       _likeFunc                  10037380 f    CIL library: CIL module
 0001:00036540       _total_changes             10037540 f    CIL library: CIL module
 0001:000365a0       _changes                   100375a0 f    CIL library: CIL module
 0001:00036600       _last_insert_rowid         10037600 f    CIL library: CIL module
 0001:00036660       _randomFunc                10037660 f    CIL library: CIL module
 0001:00036720       _contextMalloc             10037720 f    CIL library: CIL module
 0001:00036770       _roundFunc                 10037770 f    CIL library: CIL module
 0001:00036900       _instrFunc                 10037900 f    CIL library: CIL module
 0001:00036b80       _absFunc                   10037b80 f    CIL library: CIL module
 0001:00036ce0       _lengthFunc                10037ce0 f    CIL library: CIL module
 0001:00036e00       _sqlite3IsReadOnly         10037e00 f    CIL library: CIL module
 0001:00036e90       _sqlite3CreateForeignKey   10037e90 f    CIL library: CIL module
 0001:000371f0       _sqlite3ClearStatTables    100381f0 f    CIL library: CIL module
 0001:000373b0       _sqliteViewResetAll        100383b0 f    CIL library: CIL module
 0001:00037490       _createTableStmt           10038490 f    CIL library: CIL module
 0001:000376d0       _sqlite3CheckObjectName    100386d0 f    CIL library: CIL module
 0001:00037720       _sqlite3TwoPartName        10038720 f    CIL library: CIL module
 0001:00037780       _sqlite3LocateTable        10038780 f    CIL library: CIL module
 0001:00037810       _sqliteAuthBadReturnCode   10038810 f    CIL library: CIL module
 0001:00037830       _sqlite3FixSrcList         10038830 f    CIL library: CIL module
 0001:00037940       _stat3Get                  10038940 f    CIL library: CIL module
 0001:00037a10       _isSystemTable             10038a10 f    CIL library: CIL module
 0001:00037ab0       _whereOrName               10038ab0 f    CIL library: CIL module
 0001:00037af0       _sqlite3ExprListCheckLength 10038af0 f    CIL library: CIL module
 0001:00037b20       _sqlite3ExprDup            10038b20 f    CIL library: CIL module
 0001:00037b40       _sqlite3ExprCheckHeight    10038b40 f    CIL library: CIL module
 0001:00037b70       _resolveOutOfRangeError    10038b70 f    CIL library: CIL module
 0001:00037bf0       _columnMallocFailure       10038bf0 f    CIL library: CIL module
 0001:00037c50       _columnMem                 10038c50 f    CIL library: CIL module
 0001:00037cc0       _sqlite3InvalidFunction    10038cc0 f    CIL library: CIL module
 0001:00037ed0       _vdbeSafety                10038ed0 f    CIL library: CIL module
 0001:00037ef0       _sqlite3VdbeTransferError  10038ef0 f    CIL library: CIL module
 0001:00038020       _displayP4                 10039020 f    CIL library: CIL module
 0001:000382e0       _sqlite3VdbeChangeP4       100392e0 f    CIL library: CIL module
 0001:00038430       _sqlite3VdbeChangeToNoop   10039430 f    CIL library: CIL module
 0001:00038470       _vdbeFreeOpArray           10039470 f    CIL library: CIL module
 0001:000384c0       _setDestPgsz               100394c0 f    CIL library: CIL module
 0001:000384e0       _decodeFlags               100394e0 f    CIL library: CIL module
 0001:00038570       _freeSpace                 10039570 f    CIL library: CIL module
 0001:000387c0       _defragmentPage            100397c0 f    CIL library: CIL module
 0001:00038980       _walLimitSize              10039980 f    CIL library: CIL module
 0001:00038a00       _subjournalPage            10039a00 f    CIL library: CIL module
 0001:00038b50       _winDlOpen                 10039b50 f    CIL library: CIL module
 0001:00038bf0       _getTempname               10039bf0 f    CIL library: CIL module
 0001:00038ed0       _logIoerr                  10039ed0 f    CIL library: CIL module
 0001:00038f00       _getLastErrorMsg           10039f00 f    CIL library: CIL module
 0001:00039070       _winMemShutdown            1003a070 f    CIL library: CIL module
 0001:000390c0       _winMemInit                1003a0c0 f    CIL library: CIL module
 0001:00039120       _winMemSize                1003a120 f    CIL library: CIL module
 0001:00039160       _winMemRealloc             1003a160 f    CIL library: CIL module
 0001:000391d0       _winMemFree                1003a1d0 f    CIL library: CIL module
 0001:00039210       _winMemMalloc              1003a210 f    CIL library: CIL module
 0001:00039250       _logBadConnection          1003a250 f    CIL library: CIL module
 0001:00039270       _parseModifier             1003a270 f    CIL library: CIL module
 0001:00039c70       _upper_quartileFinalize    1003ac70 f    CIL library: CIL module
 0001:00039ce0       _lower_quartileFinalize    1003ace0 f    CIL library: CIL module
 0001:00039d30       _medianFinalize            1003ad30 f    CIL library: CIL module
 0001:00039d80       _reverseFunc               1003ad80 f    CIL library: CIL module
 0001:00039f90       _rightFunc                 1003af90 f    CIL library: CIL module
 0001:0003a1b0       _leftFunc                  1003b1b0 f    CIL library: CIL module
 0001:0003a3c0       _strfilterFunc             1003b3c0 f    CIL library: CIL module
 0001:0003a6b0       _padcFunc                  1003b6b0 f    CIL library: CIL module
 0001:0003aa20       _padrFunc                  1003ba20 f    CIL library: CIL module
 0001:0003ad50       _padlFunc                  1003bd50 f    CIL library: CIL module
 0001:0003b070       _properFunc                1003c070 f    CIL library: CIL module
 0001:0003b230       _replicateFunc             1003c230 f    CIL library: CIL module
 0001:0003b490       _geomCallback              1003c490 f    CIL library: CIL module
 0001:0003b590       _rtreenode                 1003c590 f    CIL library: CIL module
 0001:0003b7c0       _fts3tokColumnMethod       1003c7c0 f    CIL library: CIL module
 0001:0003b990       _scalarFunc                1003c990 f    CIL library: CIL module
 0001:0003bcc0       _fts3auxColumnMethod       1003ccc0 f    CIL library: CIL module
 0001:0003be40       _fts3WriteExprList         1003ce40 f    CIL library: CIL module
 0001:0003bed0       _fts3ReadExprList          1003ced0 f    CIL library: CIL module
 0001:0003c2e0       _yy_destructor             1003d2e0 f    CIL library: CIL module
 0001:0003c430       _sqlite3VtabCallConnect    1003d430 f    CIL library: CIL module
 0001:0003c540       _sqlite3DeleteTrigger      1003d540 f    CIL library: CIL module
 0001:0003c5a0       _sqlite3TriggerDeleteStep  1003d5a0 f    CIL library: CIL module
 0001:0003c630       _sqlite3TriggerUpdateStep  1003d630 f    CIL library: CIL module
 0001:0003c6d0       _substExpr                 1003d6d0 f    CIL library: CIL module
 0001:0003c7f0       _generateColumnNames       1003d7f0 f    CIL library: CIL module
 0001:0003ca00       _sqlite3TableAffinityStr   1003da00 f    CIL library: CIL module
 0001:0003cad0       _sqlite3FkDelete           1003dad0 f    CIL library: CIL module
 0001:0003cc30       _sqlite3FkOldmask          1003dc30 f    CIL library: CIL module
 0001:0003cd20       _sqlite3RegisterLikeFunctions 1003dd20 f    CIL library: CIL module
 0001:0003ceb0       _sqlite3RegisterBuiltinFunctions 1003deb0 f    CIL library: CIL module
 0001:0003ced0       _groupConcatFinalize       1003ded0 f    CIL library: CIL module
 0001:0003cf60       _loadExt                   1003df60 f    CIL library: CIL module
 0001:0003d0a0       _soundexFunc               1003e0a0 f    CIL library: CIL module
 0001:0003d290       _trimFunc                  1003e290 f    CIL library: CIL module
 0001:0003d680       _replaceFunc               1003e680 f    CIL library: CIL module
 0001:0003d960       _hexFunc                   1003e960 f    CIL library: CIL module
 0001:0003daa0       _charFunc                  1003eaa0 f    CIL library: CIL module
 0001:0003dca0       _quoteFunc                 1003eca0 f    CIL library: CIL module
 0001:0003e090       _compileoptiongetFunc      1003f090 f    CIL library: CIL module
 0001:0003e1d0       _sourceidFunc              1003f1d0 f    CIL library: CIL module
 0001:0003e2a0       _versionFunc               1003f2a0 f    CIL library: CIL module
 0001:0003e370       _randomBlob                1003f370 f    CIL library: CIL module
 0001:0003e420       _lowerFunc                 1003f420 f    CIL library: CIL module
 0001:0003e500       _upperFunc                 1003f500 f    CIL library: CIL module
 0001:0003e600       _substrFunc                1003f600 f    CIL library: CIL module
 0001:0003e970       _typeofFunc                1003f970 f    CIL library: CIL module
 0001:0003eae0       _sqlite3AddDefaultValue    1003fae0 f    CIL library: CIL module
 0001:0003ec00       _sqlite3DeleteTable        1003fc00 f    CIL library: CIL module
 0001:0003edd0       _sqlite3LocateTableItem    1003fdd0 f    CIL library: CIL module
 0001:0003ee30       _sqlite3AuthCheck          1003fe30 f    CIL library: CIL module
 0001:0003eec0       _sqlite3AuthReadCol        1003fec0 f    CIL library: CIL module
 0001:0003ef90       _stat3Init                 1003ff90 f    CIL library: CIL module
 0001:0003f0a0       _whereTempTriggers         100400a0 f    CIL library: CIL module
 0001:0003f160       _whereForeignKeys          10040160 f    CIL library: CIL module
 0001:0003f1f0       _renameTriggerFunc         100401f0 f    CIL library: CIL module
 0001:0003f2e0       _renameParentFunc          100402e0 f    CIL library: CIL module
 0001:0003f550       _renameTableFunc           10040550 f    CIL library: CIL module
 0001:0003f610       _sqlite3PExpr              10040610 f    CIL library: CIL module
 0001:0003f6d0       _sqlite3ExprSetHeight      100406d0 f    CIL library: CIL module
 0001:0003f700       _resolveAlias              10040700 f    CIL library: CIL module
 0001:0003fe10       _vdbeSafetyNotNull         10040e10 f    CIL library: CIL module
 0001:0003fe50       _sqlite3VdbeClearObject    10040e50 f    CIL library: CIL module
 0001:000402d0       _dropCell                  100412d0 f    CIL library: CIL module
 0001:000403b0       _zeroPage                  100413b0 f    CIL library: CIL module
 0001:00040480       _btreeInitPage             10041480 f    CIL library: CIL module
 0001:00040690       _allocateSpace             10041690 f    CIL library: CIL module
 0001:00040880       _pager_write               10041880 f    CIL library: CIL module
 0001:00040a80       _winGetLastError           10041a80 f    CIL library: CIL module
 0001:00040aa0       _winDlError                10041aa0 f    CIL library: CIL module
 0001:00040ac0       _winLogErrorAtLine         10041ac0 f    CIL library: CIL module
 0001:00040b70       _sqlite3MemGetWin32        10041b70 f    CIL library: CIL module
 0001:00040b80       _sqlite3SafetyCheckSickOrOk 10041b80 f    CIL library: CIL module
 0001:00040bc0       _sqlite3SafetyCheckOk      10041bc0 f    CIL library: CIL module
 0001:00040c70       _isDate                    10041c70 f    CIL library: CIL module
 0001:000416f0       _sqlite3RtreeInit          100426f0 f    CIL library: CIL module
 0001:00041810       _langidFromSelect          10042810 f    CIL library: CIL module
 0001:00041830       _sqlite3Fts3InitHashTable  10042830 f    CIL library: CIL module
 0001:00041a60       _yy_pop_parser_stack       10042a60 f    CIL library: CIL module
 0001:00041aa0       _spanUnaryPrefix           10042aa0 f    CIL library: CIL module
 0001:00041b60       _spanUnaryPostfix          10042b60 f    CIL library: CIL module
 0001:00041c20       _spanBinaryExpr            10042c20 f    CIL library: CIL module
 0001:00041c50       _spanExpr                  10042c50 f    CIL library: CIL module
 0001:00041cc0       _sqlite3UnlinkAndDeleteTrigger 10042cc0 f    CIL library: CIL module
 0001:00041e10       _substExprList             10042e10 f    CIL library: CIL module
 0001:00041f20       _addWhereTerm              10042f20 f    CIL library: CIL module
 0001:00042030       _sqlite3SrcListLookup      10043030 f    CIL library: CIL module
 0001:00042120       _sqlite3SchemaClear        10043120 f    CIL library: CIL module
 0001:00042250       _sqlite3UnlinkAndDeleteTable 10043250 f    CIL library: CIL module
 0001:00042310       _sqlite3ResetAllSchemasOfConnection 10043310 f    CIL library: CIL module
 0001:00042370       _sqlite3ResetOneSchema     10043370 f    CIL library: CIL module
 0001:000423a0       _sqlite3AuthRead           100433a0 f    CIL library: CIL module
 0001:00042480       _sqlite3AlterFunctions     10043480 f    CIL library: CIL module
 0001:00042510       _sqlite3ExprFunction       10043510 f    CIL library: CIL module
 0001:00042570       _sqlite3ResolveOrderGroupBy 10043570 f    CIL library: CIL module
 0001:00042620       _lookupName                10043620 f    CIL library: CIL module
 0001:00042d70       _vdbeUnbind                10043d70 f    CIL library: CIL module
 0001:00042ec0       _sqlite3VdbeDelete         10043ec0 f    CIL library: CIL module
 0001:00042f10       _modifyPagePointer         10043f10 f    CIL library: CIL module
 0001:00043130       _pageReinit                10044130 f    CIL library: CIL module
 0001:00043160       _sqlite3PagerWrite         10044160 f    CIL library: CIL module
 0001:000433a0       _winFullPathname           100443a0 f    CIL library: CIL module
 0001:00043680       _winAccess                 10044680 f    CIL library: CIL module
 0001:00043880       _winDelete                 10044880 f    CIL library: CIL module
 0001:00043a40       _winOpen                   10044a40 f    CIL library: CIL module
 0001:00043e00       _winUnmapfile              10044e00 f    CIL library: CIL module
 0001:00043ea0       _unlockReadLock            10044ea0 f    CIL library: CIL module
 0001:00043f70       _winFileSize               10044f70 f    CIL library: CIL module
 0001:00043fe0       _winSync                   10044fe0 f    CIL library: CIL module
 0001:00044030       _winWrite                  10045030 f    CIL library: CIL module
 0001:00044200       _winRead                   10045200 f    CIL library: CIL module
 0001:00044390       _winClose                  10045390 f    CIL library: CIL module
 0001:00044410       _seekWinFile               10045410 f    CIL library: CIL module
 0001:00044480       _sqlite3MemSetDefault      10045480 f    CIL library: CIL module
 0001:00044490       _sqlite3MallocInit         10045490 f    CIL library: CIL module
 0001:000445a0       _strftimeFunc              100455a0 f    CIL library: CIL module
 0001:00044ae0       _dateFunc                  10045ae0 f    CIL library: CIL module
 0001:00044be0       _timeFunc                  10045be0 f    CIL library: CIL module
 0001:00044cf0       _datetimeFunc              10045cf0 f    CIL library: CIL module
 0001:00044e10       _juliandayFunc             10045e10 f    CIL library: CIL module
 0001:00045250       _yy_accept                 10046250 f    CIL library: CIL module
 0001:00045290       _yyStackOverflow           10046290 f    CIL library: CIL module
 0001:000452e0       _sqlite3ParserFree         100462e0 f    CIL library: CIL module
 0001:00045320       _sqliteProcessJoin         10046320 f    CIL library: CIL module
 0001:00045540       _sqlite3SchemaGet          10046540 f    CIL library: CIL module
 0001:00045630       _resolveExprStep           10046630 f    CIL library: CIL module
 0001:00045b90       _backupOnePage             10046b90 f    CIL library: CIL module
 0001:00045da0       _sqlite3BtreeUpdateMeta    10046da0 f    CIL library: CIL module
 0001:00045e30       _copyPayload               10046e30 f    CIL library: CIL module
 0001:00045e60       _newDatabase               10046e60 f    CIL library: CIL module
 0001:00045f40       _sqlite3PCacheSetDefault   10046f40 f    CIL library: CIL module
 0001:00045f60       _sqlite3PcacheInitialize   10046f60 f    CIL library: CIL module
 0001:00046040       _winUnfetch                10047040 f    CIL library: CIL module
 0001:00046070       _winMapfile                10047070 f    CIL library: CIL module
 0001:000461e0       _winShmPurge               100471e0 f    CIL library: CIL module
 0001:000462c0       _winUnlock                 100472c0 f    CIL library: CIL module
 0001:000463a0       _winLock                   100473a0 f    CIL library: CIL module
 0001:00046550       _winTruncate               10047550 f    CIL library: CIL module
 0001:00046630       _sqlite3OsInit             10047630 f    CIL library: CIL module
 0001:00046660       _ctimestampFunc            10047660 f    CIL library: CIL module
 0001:00046680       _cdateFunc                 10047680 f    CIL library: CIL module
 0001:000466a0       _ctimeFunc                 100476a0 f    CIL library: CIL module
 0001:00046760       _yy_shift                  10047760 f    CIL library: CIL module
 0001:000467b0       _sqlite3ResolveExprNames   100477b0 f    CIL library: CIL module
 0001:000468a0       _resolveOrderGroupBy       100478a0 f    CIL library: CIL module
 0001:00046a00       _resolveOrderByTermToExprList 10047a00 f    CIL library: CIL module
 0001:00046aa0       _sqlite3BackupUpdate       10047aa0 f    CIL library: CIL module
 0001:00046b20       _sqlite3BtreeNewDb         10047b20 f    CIL library: CIL module
 0001:00046b70       _pager_write_pagelist      10047b70 f    CIL library: CIL module
 0001:00046d50       _pager_playback_one_page   10047d50 f    CIL library: CIL module
 0001:000470f0       _winFetch                  100480f0 f    CIL library: CIL module
 0001:00047160       _winShmUnmap               10048160 f    CIL library: CIL module
 0001:00047220       _winOpenSharedMemory       10048220 f    CIL library: CIL module
 0001:00047560       _winFileControl            10048560 f    CIL library: CIL module
 0001:000477b0       _sqlite3RegisterDateTimeFunctions 100487b0 f    CIL library: CIL module
 0001:00047840       _sqlite3RegisterGlobalFunctions 10048840 f    CIL library: CIL module
 0001:000478e0       _resolveAttachExpr         100488e0 f    CIL library: CIL module
 0001:00047930       _resolveCompoundOrderBy    10048930 f    CIL library: CIL module
 0001:00047c90       _pager_playback            10048c90 f    CIL library: CIL module
 0001:00048250       _resolveSelectStep         10049250 f    CIL library: CIL module
 0001:00048760       _fts3StringAppend          10049760 f    CIL library: CIL module
 0001:000487f0       _blobGrowBuffer            100497f0 f    CIL library: CIL module
 0001:00048840       _fts3MsrBufferData         10049840 f    CIL library: CIL module
 0001:000488a0       _fts3NodeAddTerm           100498a0 f    CIL library: CIL module
 0001:00048b80       _sqlite3Fts3SegReaderPending 10049b80 f    CIL library: CIL module
 0001:00048e00       _fts3PendingListAppendVarint 10049e00 f    CIL library: CIL module
 0001:00048ee0       _simpleNext                10049ee0 f    CIL library: CIL module
 0001:00049010       _sqlite3Fts3InitTokenizer  1004a010 f    CIL library: CIL module
 0001:000491b0       _porterNext                1004a1b0 f    CIL library: CIL module
 0001:000492c0       _fts3ReallocOrFree         1004a2c0 f    CIL library: CIL module
 0001:00049310       _fts3auxGrowStatArray      1004a310 f    CIL library: CIL module
 0001:00049370       _fts3ScanInteriorNode      1004a370 f    CIL library: CIL module
 0001:00049680       _sqlite3VtabMakeWritable   1004a680 f    CIL library: CIL module
 0001:00049710       _sqlite3_get_table_cb      1004a710 f    CIL library: CIL module
 0001:000499d0       _sqlite3ResolveSelectNames 1004a9d0 f    CIL library: CIL module
 0001:00049a20       _walIndexPage              1004aa20 f    CIL library: CIL module
 0001:00049b40       _winShmMap                 1004ab40 f    CIL library: CIL module
 0001:00049d80       _sqlite3DbRealloc          1004ad80 f    CIL library: CIL module
 0001:00049e60       _fts3SnippetText           1004ae60 f    CIL library: CIL module
 0001:0004a0b0       _fts3IncrmergeHintPush     1004b0b0 f    CIL library: CIL module
 0001:0004a180       _fts3AppendToNode          1004b180 f    CIL library: CIL module
 0001:0004a300       _nodeReaderNext            1004b300 f    CIL library: CIL module
 0001:0004a420       _fts3PendingListAppend     1004b420 f    CIL library: CIL module
 0001:0004a550       _getNextString             1004b550 f    CIL library: CIL module
 0001:0004a8a0       _growVTrans                1004b8a0 f    CIL library: CIL module
 0001:0004a900       _addModuleArgument         1004b900 f    CIL library: CIL module
 0001:0004a990       _sqlite3SrcListEnlarge     1004b990 f    CIL library: CIL module
 0001:0004aaa0       _sqlite3ArrayAllocate      1004baa0 f    CIL library: CIL module
 0001:0004ab10       _sqlite3AddColumn          1004bb10 f    CIL library: CIL module
 0001:0004ac50       _addAggInfoFunc            1004bc50 f    CIL library: CIL module
 0001:0004acb0       _addAggInfoColumn          1004bcb0 f    CIL library: CIL module
 0001:0004ad20       _sqlite3ExprListAppend     1004bd20 f    CIL library: CIL module
 0001:0004adc0       _sqlite3ExprAssignVarNumber 1004bdc0 f    CIL library: CIL module
 0001:0004b0b0       _growOpArray               1004c0b0 f    CIL library: CIL module
 0001:0004b130       _walHashGet                1004c130 f    CIL library: CIL module
 0001:0004b190       _sqlite3DbReallocOrFree    1004c190 f    CIL library: CIL module
 0001:0004b1b0       _sqlite3Fts3CacheDeferredDoclists 1004c1b0 f    CIL library: CIL module
 0001:0004b430       _nodeReaderInit            1004c430 f    CIL library: CIL module
 0001:0004b490       _fts3PendingTermsAddOne    1004c490 f    CIL library: CIL module
 0001:0004b580       _getNextNode               1004c580 f    CIL library: CIL module
 0001:0004b840       _exprAnalyzeOrTerm         1004c840 f    CIL library: CIL module
 0001:0004beb0       _sqlite3VtabBegin          1004ceb0 f    CIL library: CIL module
 0001:0004bfa0       _sqlite3VtabCallCreate     1004cfa0 f    CIL library: CIL module
 0001:0004c090       _addArgumentToVtab         1004d090 f    CIL library: CIL module
 0001:0004c100       _selectExpander            1004d100 f    CIL library: CIL module
 0001:0004cbd0       _sqlite3SelectNew          1004dbd0 f    CIL library: CIL module
 0001:0004cd90       _sqlite3SrcListAppend      1004dd90 f    CIL library: CIL module
 0001:0004ce50       _sqlite3IdListAppend       1004de50 f    CIL library: CIL module
 0001:0004cef0       _sqlite3AddCheckConstraint 1004def0 f    CIL library: CIL module
 0001:0004cfa0       _sqlite3TableLock          1004dfa0 f    CIL library: CIL module
 0001:0004d090       _analyzeAggregate          1004e090 f    CIL library: CIL module
 0001:0004d370       _vdbeSorterIterRead        1004e370 f    CIL library: CIL module
 0001:0004d4d0       _sqlite3VdbeAddOpList      1004e4d0 f    CIL library: CIL module
 0001:0004d590       _sqlite3VdbeMakeLabel      1004e590 f    CIL library: CIL module
 0001:0004d600       _sqlite3VdbeAddOp3         1004e600 f    CIL library: CIL module
 0001:0004d660       _sqlite3VdbeMemGrow        1004e660 f    CIL library: CIL module
 0001:0004d780       _sqlite3WalFindFrame       1004e780 f    CIL library: CIL module
 0001:0004d8c0       _walIteratorInit           1004e8c0 f    CIL library: CIL module
 0001:0004da60       _walCleanupHash            1004ea60 f    CIL library: CIL module
 0001:0004db10       _pagerUndoCallback         1004eb10 f    CIL library: CIL module
 0001:0004dbf0       _fts3TruncateNode          1004ebf0 f    CIL library: CIL module
 0001:0004de00       _fts3PendingTermsAdd       1004ee00 f    CIL library: CIL module
 0001:0004df50       _sqlite3VtabArgInit        1004ef50 f    CIL library: CIL module
 0001:0004dfe0       _targetSrcList             1004efe0 f    CIL library: CIL module
 0001:0004e110       _flattenSubquery           1004f110 f    CIL library: CIL module
 0001:0004e720       _fkActionTrigger           1004f720 f    CIL library: CIL module
 0001:0004f510       _sqlite3SrcListAppendFromTerm 10050510 f    CIL library: CIL module
 0001:0004f5e0       _sqlite3ExprAnalyzeAggregates 100505e0 f    CIL library: CIL module
 0001:0004f620       _sqlite3ExprCodeMove       10050620 f    CIL library: CIL module
 0001:0004f780       _sqlite3VdbeSorterRowkey   10050780 f    CIL library: CIL module
 0001:0004f7f0       _vdbeSorterIterVarint      100507f0 f    CIL library: CIL module
 0001:0004f8a0       _sqlite3VdbeList           100508a0 f    CIL library: CIL module
 0001:0004fd00       _sqlite3VdbeAddOp4Int      10050d00 f    CIL library: CIL module
 0001:0004fdb0       _sqlite3VdbeAddParseSchemaOp 10050db0 f    CIL library: CIL module
 0001:0004fea0       _sqlite3VdbeAddOp4         10050ea0 f    CIL library: CIL module
 0001:0004ff10       _sqlite3VdbeAddOp2         10050f10 f    CIL library: CIL module
 0001:0004ff70       _sqlite3VdbeAddOp1         10050f70 f    CIL library: CIL module
 0001:0004ffc0       _sqlite3VdbeAddOp0         10050fc0 f    CIL library: CIL module
 0001:00050010       _sqlite3VdbeMemNulTerminate 10051010 f    CIL library: CIL module
 0001:00050060       _sqlite3VdbeMemMakeWriteable 10051060 f    CIL library: CIL module
 0001:000500d0       _sqlite3WalSavepointUndo   100510d0 f    CIL library: CIL module
 0001:00050110       _sqlite3WalUndo            10051110 f    CIL library: CIL module
 0001:000501b0       _walCheckpoint             100511b0 f    CIL library: CIL module
 0001:00050510       _walIndexAppend            10051510 f    CIL library: CIL module
 0001:00050610       _pagerRollbackWal          10051610 f    CIL library: CIL module
 0001:00050660       _sqlite3VdbeMemTranslate   10051660 f    CIL library: CIL module
 0001:00050b40       _fts3InsertTerms           10051b40 f    CIL library: CIL module
 0001:00050be0       _sqlite3WhereEnd           10051be0 f    CIL library: CIL module
 0001:000511d0       _explainOneScan            100521d0 f    CIL library: CIL module
 0001:00051430       _codeApplyAffinity         10052430 f    CIL library: CIL module
 0001:000514e0       _explainSimpleCount        100524e0 f    CIL library: CIL module
 0001:000515e0       _finalizeAggFunctions      100525e0 f    CIL library: CIL module
 0001:000516f0       _convertCompoundSelectToSubquery 100526f0 f    CIL library: CIL module
 0001:00051910       _sqlite3GetVdbe            10052910 f    CIL library: CIL module
 0001:000519b0       _explainComposite          100529b0 f    CIL library: CIL module
 0001:00051ad0       _explainTempTable          10052ad0 f    CIL library: CIL module
 0001:00051bb0       _codeDistinct              10052bb0 f    CIL library: CIL module
 0001:00051cb0       _codeOffset                10052cb0 f    CIL library: CIL module
 0001:00051db0       _returnSingleInt           10052db0 f    CIL library: CIL module
 0001:00051f00       _sqlite3CompleteInsertion  10052f00 f    CIL library: CIL module
 0001:00052260       _autoIncStep               10053260 f    CIL library: CIL module
 0001:000522b0       _readsTable                100532b0 f    CIL library: CIL module
 0001:00052390       _sqlite3OpenTable          10053390 f    CIL library: CIL module
 0001:00052460       _sqlite3FkActions          10053460 f    CIL library: CIL module
 0001:000524e0       _sqlite3HaltConstraint     100534e0 f    CIL library: CIL module
 0001:00052570       _sqlite3Savepoint          10053570 f    CIL library: CIL module
 0001:00052620       _sqlite3RollbackTransaction 10053620 f    CIL library: CIL module
 0001:00052690       _sqlite3CommitTransaction  10053690 f    CIL library: CIL module
 0001:00052700       _sqlite3BeginTransaction   10053700 f    CIL library: CIL module
 0001:00052800       _destroyRootPage           10053800 f    CIL library: CIL module
 0001:000528f0       _sqlite3ChangeCookie       100538f0 f    CIL library: CIL module
 0001:000529f0       _sqlite3OpenMasterTable    100539f0 f    CIL library: CIL module
 0001:00052ac0       _codeTableLocks            10053ac0 f    CIL library: CIL module
 0001:00052be0       _loadAnalysis              10053be0 f    CIL library: CIL module
 0001:00052c30       _openStatTable             10053c30 f    CIL library: CIL module
 0001:00052e80       _sqlite3MinimumFileFormat  10053e80 f    CIL library: CIL module
 0001:000530a0       _reloadTableSchema         100540a0 f    CIL library: CIL module
 0001:00053300       _sqlite3ExprAnalyzeAggList 10054300 f    CIL library: CIL module
 0001:00053360       _sqlite3ExprCodeExprList   10054360 f    CIL library: CIL module
 0001:00053400       _sqlite3ExprCode           10054400 f    CIL library: CIL module
 0001:00053490       _codeReal                  10054490 f    CIL library: CIL module
 0001:000535a0       _sqlite3CodeOnce           100545a0 f    CIL library: CIL module
 0001:00053600       _sqlite3ExprCodeIsNullJump 10054600 f    CIL library: CIL module
 0001:00053650       _vdbeSorterIterNext        10054650 f    CIL library: CIL module
 0001:000536d0       _sqlite3VdbeChangeEncoding 100546d0 f    CIL library: CIL module
 0001:000536f0       _walIndexRecover           100546f0 f    CIL library: CIL module
 0001:00053a60       _pagerPlaybackSavepoint    10054a60 f    CIL library: CIL module
 0001:00053d20       _sqlite3Utf8to16           10054d20 f    CIL library: CIL module
 0001:00053d90       _sqlite3Utf16to8           10054d90 f    CIL library: CIL module
 0001:00053f70       _sqlite3VtabFinishParse    10054f70 f    CIL library: CIL module
 0001:00054160       _sqlite3Vacuum             10055160 f    CIL library: CIL module
 0001:000541d0       _sqlite3SelectExpand       100551d0 f    CIL library: CIL module
 0001:00054220       _generateOutputSubroutine  10055220 f    CIL library: CIL module
 0001:00054710       _computeLimitRegisters     10055710 f    CIL library: CIL module
 0001:00054890       _generateSortTail          10055890 f    CIL library: CIL module
 0001:00054fb0       _pushOntoSorter            10055fb0 f    CIL library: CIL module
 0001:00055340       _flagPragma                10056340 f    CIL library: CIL module
 0001:00055470       _sqlite3AutoincrementEnd   10056470 f    CIL library: CIL module
 0001:00055840       _sqlite3AutoincrementBegin 10056840 f    CIL library: CIL module
 0001:00055bf0       _destroyTable              10056bf0 f    CIL library: CIL module
 0001:00055c90       _codeAttach                10056c90 f    CIL library: CIL module
 0001:00055ed0       _sqlite3ExprCodeAndCache   10056ed0 f    CIL library: CIL module
 0001:00055f50       _codeInteger               10056f50 f    CIL library: CIL module
 0001:00056100       _vdbeSorterIterInit        10057100 f    CIL library: CIL module
 0001:00056210       _sqlite3VdbeExpandSql      10057210 f    CIL library: CIL module
 0001:000565d0       _bindText                  100575d0 f    CIL library: CIL module
 0001:000566c0       _sqlite3VdbeMemStringify   100576c0 f    CIL library: CIL module
 0001:00056760       _walIndexReadHdr           10057760 f    CIL library: CIL module
 0001:000568b0       _sqlite3PagerSavepoint     100578b0 f    CIL library: CIL module
 0001:000569e0       _sqlite3PagerRollback      100579e0 f    CIL library: CIL module
 0001:00056aa0       _pagerUnlockAndRollback    10057aa0 f    CIL library: CIL module
 0001:00056b00       _applyAffinity             10057b00 f    CIL library: CIL module
 0001:00056be0       _sqlite3ValueText          10057be0 f    CIL library: CIL module
 0001:00056c90       _sqlite3MemCompare         10057c90 f    CIL library: CIL module
 0001:00056f20       _sqlite3BtreeSavepoint     10057f20 f    CIL library: CIL module
 0001:00056fd0       _sqlite3WalCheckpoint      10057fd0 f    CIL library: CIL module
 0001:00057170       _walTryBeginRead           10058170 f    CIL library: CIL module
 0001:00057460       _sqlite3WalClose           10058460 f    CIL library: CIL module
 0001:00057580       _sqlite3PagerCloseWal      10058580 f    CIL library: CIL module
 0001:00057650       _sqlite3PagerCheckpoint    10058650 f    CIL library: CIL module
 0001:000576a0       _pagerUnlockIfUnused       100586a0 f    CIL library: CIL module
 0001:000576d0       _sqlite3PagerClose         100586d0 f    CIL library: CIL module
 0001:00057900       _callCollNeeded            10058900 f    CIL library: CIL module
 0001:00057a40       _sqlite3ValueApplyAffinity 10058a40 f    CIL library: CIL module
 0001:00057c80       _sqlite3VdbeGetValue       10058c80 f    CIL library: CIL module
 0001:00057d50       _sqlite3VdbeRecordCompare  10058d50 f    CIL library: CIL module
 0001:00057f30       _sqlite3VdbeCloseStatement 10058f30 f    CIL library: CIL module
 0001:00058030       _sqlite3ValueFromExpr      10059030 f    CIL library: CIL module
 0001:00058390       _sqlite3BtreeCheckpoint    10059390 f    CIL library: CIL module
 0001:00058430       _walRestartLog             10059430 f    CIL library: CIL module
 0001:000585b0       _sqlite3WalBeginReadTransaction 100595b0 f    CIL library: CIL module
 0001:000588a0       _sqlite3PagerAcquire       100598a0 f    CIL library: CIL module
 0001:00058c00       _pagerBeginReadTransaction 10059c00 f    CIL library: CIL module
 0001:00058e50       _sqlite3Checkpoint         10059e50 f    CIL library: CIL module
 0001:00059060       _valueFromExpr             1005a060 f    CIL library: CIL module
 0001:000590d0       _sqlite3ColumnDefault      1005a0d0 f    CIL library: CIL module
 0001:00059190       _sqlite3GenerateIndexKey   1005a190 f    CIL library: CIL module
 0001:00059480       _sqlite3GenerateRowIndexDelete 1005a480 f    CIL library: CIL module
 0001:00059540       _sqlite3GetCollSeq         1005a540 f    CIL library: CIL module
 0001:00059630       _sqlite3LocateCollSeq      1005a630 f    CIL library: CIL module
 0001:000596a0       _sqlite3AddCollateType     1005a6a0 f    CIL library: CIL module
 0001:00059770       _sqlite3AlterFinishAddColumn 1005a770 f    CIL library: CIL module
 0001:000599d0       _sqlite3ExprCodeGetColumnOfTable 1005a9d0 f    CIL library: CIL module
 0001:00059a70       _vdbeSorterCompare         1005aa70 f    CIL library: CIL module
 0001:00059da0       _btreeGetPage              1005ada0 f    CIL library: CIL module
 0001:00059e00       _ptrmapGet                 1005ae00 f    CIL library: CIL module
 0001:00059f00       _ptrmapPut                 1005af00 f    CIL library: CIL module
 0001:0005a050       _sqlite3WalFrames          1005b050 f    CIL library: CIL module
 0001:0005a450       _sqlite3PagerMovepage      1005b450 f    CIL library: CIL module
 0001:0005a600       _pager_incr_changecounter  1005b600 f    CIL library: CIL module
 0001:0005a6d0       _sqlite3PagerSharedLock    1005b6d0 f    CIL library: CIL module
 0001:0005a9e0       _pagerWalFrames            1005b9e0 f    CIL library: CIL module
 0001:0005aef0       _sqlite3WalDefaultHook     1005bef0 f    CIL library: CIL module
 0001:0005af30       _whereKeyStats             1005bf30 f    CIL library: CIL module
 0001:0005b2c0       _sqlite3CheckCollSeq       1005c2c0 f    CIL library: CIL module
 0001:0005b2f0       _sqlite3IndexKeyinfo       1005c2f0 f    CIL library: CIL module
 0001:0005b400       _sqlite3RefillIndex        1005c400 f    CIL library: CIL module
 0001:0005b8c0       _analyzeOneTable           1005c8c0 f    CIL library: CIL module
 0001:0005d520       _sqlite3ExprCodeGetColumn  1005e520 f    CIL library: CIL module
 0001:0005d5c0       _sqlite3ExprCollSeq        1005e5c0 f    CIL library: CIL module
 0001:0005d700       _sqlite3VdbeSorterCompare  1005e700 f    CIL library: CIL module
 0001:0005d7c0       _vdbeSorterMerge           1005e7c0 f    CIL library: CIL module
 0001:0005d870       _vdbeSorterDoCompare       1005e870 f    CIL library: CIL module
 0001:0005d930       _checkPtrmap               1005e930 f    CIL library: CIL module
 0001:0005d9b0       _freePage2                 1005e9b0 f    CIL library: CIL module
 0001:0005dd90       _allocateBtreePage         1005ed90 f    CIL library: CIL module
 0001:0005e600       _getOverflowPage           1005f600 f    CIL library: CIL module
 0001:0005e790       _lockBtree                 1005f790 f    CIL library: CIL module
 0001:0005ea50       _getAndInitPage            1005fa50 f    CIL library: CIL module
 0001:0005eaf0       _ptrmapPutOvflPtr          1005faf0 f    CIL library: CIL module
 0001:0005eb50       _sqlite3PagerSetJournalMode 1005fb50 f    CIL library: CIL module
 0001:0005ec60       _sqlite3PagerCommitPhaseOne 1005fc60 f    CIL library: CIL module
 0001:0005edd0       _pagerStress               1005fdd0 f    CIL library: CIL module
 0001:0005ef20       _whereEqualScanEst         1005ff20 f    CIL library: CIL module
 0001:0005f030       _whereRangeScanEst         10060030 f    CIL library: CIL module
 0001:0005f1d0       _findIndexCol              100601d0 f    CIL library: CIL module
 0001:0005f280       _exprCommute               10060280 f    CIL library: CIL module
 0001:0005f300       _updateAccumulator         10060300 f    CIL library: CIL module
 0001:0005f840       _multiSelectCollSeq        10060840 f    CIL library: CIL module
 0001:0005f890       _selectAddColumnTypeAndCollation 10060890 f    CIL library: CIL module
 0001:0005f9e0       _keyInfoFromExprList       100609e0 f    CIL library: CIL module
 0001:0005fa90       _selectInnerLoop           10060a90 f    CIL library: CIL module
 0001:00060170       _sqlite3OpenTableAndIndices 10061170 f    CIL library: CIL module
 0001:000602f0       _fkLookupParent            100612f0 f    CIL library: CIL module
 0001:00060e20       _sqlite3BinaryCompareCollSeq 10061e20 f    CIL library: CIL module
 0001:00060e60       _sqlite3VdbeSorterNext     10061e60 f    CIL library: CIL module
 0001:00060f10       _vdbeSorterInitMerge       10061f10 f    CIL library: CIL module
 0001:00060fa0       _vdbeSorterSort            10061fa0 f    CIL library: CIL module
 0001:00061080       _checkList                 10062080 f    CIL library: CIL module
 0001:00061290       _insertCell                10062290 f    CIL library: CIL module
 0001:00061430       _fillInCell                10062430 f    CIL library: CIL module
 0001:00061740       _clearCell                 10062740 f    CIL library: CIL module
 0001:00061900       _freePage                  10062900 f    CIL library: CIL module
 0001:00061920       _moveToChild               10062920 f    CIL library: CIL module
 0001:000619c0       _accessPayload             100629c0 f    CIL library: CIL module
 0001:00061d30       _setChildPtrmaps           10062d30 f    CIL library: CIL module
 0001:00061ea0       _sqlite3BtreeBeginTrans    10062ea0 f    CIL library: CIL module
 0001:00062160       _sqlite3PagerOpen          10063160 f    CIL library: CIL module
 0001:000625f0       _whereInScanEst            100635f0 f    CIL library: CIL module
 0001:000627f0       _constructAutomaticIndex   100637f0 f    CIL library: CIL module
 0001:00063140       _findTerm                  10064140 f    CIL library: CIL module
 0001:00063470       _resetAccumulator          10064470 f    CIL library: CIL module
 0001:000636c0       _selectAddSubqueryTypeInfo 100646c0 f    CIL library: CIL module
 0001:00063750       _multiSelectOrderBy        10064750 f    CIL library: CIL module
 0001:00065540       _multiSelect               10066540 f    CIL library: CIL module
 0001:00065ce0       _sqlite3CodeSubselect      10066ce0 f    CIL library: CIL module
 0001:00066200       _codeCompare               10067200 f    CIL library: CIL module
 0001:00066360       _vdbeSorterListToPMA       10067360 f    CIL library: CIL module
 0001:00066490       _sqlite3BtreeSetVersion    10067490 f    CIL library: CIL module
 0001:00066680       _checkTreePage             10067680 f    CIL library: CIL module
 0001:00066eb0       _clearDatabasePage         10067eb0 f    CIL library: CIL module
 0001:00067050       _copyNodeContent           10068050 f    CIL library: CIL module
 0001:00067110       _balance_quick             10068110 f    CIL library: CIL module
 0001:000672b0       _moveToRightmost           100682b0 f    CIL library: CIL module
 0001:00067340       _moveToLeftmost            10068340 f    CIL library: CIL module
 0001:000673c0       _moveToRoot                100683c0 f    CIL library: CIL module
 0001:00067570       _sqlite3BtreeKey           10068570 f    CIL library: CIL module
 0001:00067590       _relocatePage              10068590 f    CIL library: CIL module
 0001:000676f0       _sqlite3BtreeOpen          100686f0 f    CIL library: CIL module
 0001:00067d50       _saveCursorPosition        10068d50 f    CIL library: CIL module
 0001:00067de0       _isSortingIndex            10068de0 f    CIL library: CIL module
 0001:00068170       _isDistinctRedundant       10069170 f    CIL library: CIL module
 0001:00068280       _isDistinctIndex           10069280 f    CIL library: CIL module
 0001:00068410       _sqlite3SelectAddTypeInfo  10069410 f    CIL library: CIL module
 0001:00068460       _sqlite3OpenTempDatabase   10069460 f    CIL library: CIL module
 0001:000684f0       _sqlite3VdbeSorterRewind   100694f0 f    CIL library: CIL module
 0001:000687b0       _sqlite3VdbeSorterWrite    100697b0 f    CIL library: CIL module
 0001:00068860       _findBtree                 10069860 f    CIL library: CIL module
 0001:00068940       _sqlite3BtreeIntegrityCheck 10069940 f    CIL library: CIL module
 0001:00068e70       _sqlite3BtreeCount         10069e70 f    CIL library: CIL module
 0001:000690f0       _balance_deeper            1006a0f0 f    CIL library: CIL module
 0001:00069220       _balance_nonroot           1006a220 f    CIL library: CIL module
 0001:0006a3d0       _sqlite3BtreeMovetoUnpacked 1006b3d0 f    CIL library: CIL module
 0001:0006a7a0       _sqlite3BtreeLast          1006b7a0 f    CIL library: CIL module
 0001:0006a7e0       _sqlite3BtreeFirst         1006b7e0 f    CIL library: CIL module
 0001:0006a810       _incrVacuumStep            1006b810 f    CIL library: CIL module
 0001:0006aa60       _btreeMoveto               1006ba60 f    CIL library: CIL module
 0001:0006ab60       _saveAllCursors            1006bb60 f    CIL library: CIL module
 0001:0006aba0       _bestBtreeIndex            1006bba0 f    CIL library: CIL module
 0001:0006b570       _sqlite3SelectPrep         1006c570 f    CIL library: CIL module
 0001:0006b5e0       _sqlite3ResultSetOfSelect  1006c5e0 f    CIL library: CIL module
 0001:0006b710       _sqlite3CodeVerifySchema   1006c710 f    CIL library: CIL module
 0001:0006b7e0       _sqlite3ViewGetColumnNames 1006c7e0 f    CIL library: CIL module
 0001:0006b920       _sqlite3FindInIndex        1006c920 f    CIL library: CIL module
 0001:0006be00       _sqlite3BtreeClearTable    1006ce00 f    CIL library: CIL module
 0001:0006be90       _btreeCreateTable          1006ce90 f    CIL library: CIL module
 0001:0006c170       _balance                   1006d170 f    CIL library: CIL module
 0001:0006c370       _sqlite3BtreeRollback      1006d370 f    CIL library: CIL module
 0001:0006c4a0       _autoVacuumCommit          1006d4a0 f    CIL library: CIL module
 0001:0006c6a0       _sqlite3BtreeIncrVacuum    1006d6a0 f    CIL library: CIL module
 0001:0006c7e0       _sqlite3BtreeClose         1006d7e0 f    CIL library: CIL module
 0001:0006c8d0       _btreeRestoreCursorPosition 1006d8d0 f    CIL library: CIL module
 0001:0006c930       _sqlite3RollbackAll        1006d930 f    CIL library: CIL module
 0001:0006ca10       _sqlite3LeaveMutexAndCloseZombie 1006da10 f    CIL library: CIL module
 0001:0006d080       _sqlite3Close              1006e080 f    CIL library: CIL module
 0001:0006d150       _bestIndex                 1006e150 f    CIL library: CIL module
 0001:0006d1b0       _bestOrClauseIndex         1006e1b0 f    CIL library: CIL module
 0001:0006d470       _sqlite3BeginTrigger       1006e470 f    CIL library: CIL module
 0001:0006d8a0       _invalidateTempStorage     1006e8a0 f    CIL library: CIL module
 0001:0006d8f0       _xferOptimization          1006e8f0 f    CIL library: CIL module
 0001:0006ded0       _sqlite3BeginWriteOperation 1006eed0 f    CIL library: CIL module
 0001:0006df10       _sqlite3CodeVerifyNamedSchema 1006ef10 f    CIL library: CIL module
 0001:0006dfa0       _sqlite3DropIndex          1006efa0 f    CIL library: CIL module
 0001:0006e170       _sqlite3CreateIndex        1006f170 f    CIL library: CIL module
 0001:0006e9a0       _sqlite3AddPrimaryKey      1006f9a0 f    CIL library: CIL module
 0001:0006eb70       _sqlite3StartTable         1006fb70 f    CIL library: CIL module
 0001:0006f000       _detachFunc                10070000 f    CIL library: CIL module
 0001:0006f1e0       _attachFunc                100701e0 f    CIL library: CIL module
 0001:0006f8b0       _analyzeTable              100708b0 f    CIL library: CIL module
 0001:0006f9b0       _analyzeDatabase           100709b0 f    CIL library: CIL module
 0001:0006fa90       _sqlite3AlterBeginAddColumn 10070a90 f    CIL library: CIL module
 0001:0006fc70       _sqlite3AlterRenameTable   10070c70 f    CIL library: CIL module
 0001:0006ffc0       _sqlite3ExprCodeIN         10070fc0 f    CIL library: CIL module
 0001:000703d0       _sqlite3VdbeFreeCursor     100713d0 f    CIL library: CIL module
 0001:00070430       _sqlite3VdbeFrameDelete    10071430 f    CIL library: CIL module
 0001:000705e0       _sqlite3BtreePutData       100715e0 f    CIL library: CIL module
 0001:00070690       _btreeDropTable            10071690 f    CIL library: CIL module
 0001:00070930       _sqlite3BtreeCreateTable   10071930 f    CIL library: CIL module
 0001:00070980       _sqlite3BtreeInsert        10071980 f    CIL library: CIL module
 0001:00070b80       _sqlite3BtreePrevious      10071b80 f    CIL library: CIL module
 0001:00070d30       _sqlite3BtreeNext          10071d30 f    CIL library: CIL module
 0001:00070ec0       _sqlite3BtreeData          10071ec0 f    CIL library: CIL module
 0001:00070f00       _sqlite3BtreeCommitPhaseOne 10071f00 f    CIL library: CIL module
 0001:00070fb0       _sqlite3BtreeCursorHasMoved 10071fb0 f    CIL library: CIL module
 0001:000710b0       _bestVirtualIndex          100720b0 f    CIL library: CIL module
 0001:00071330       _sqlite3VtabBeginParse     10072330 f    CIL library: CIL module
 0001:000714b0       _sqlite3DropTriggerPtr     100724b0 f    CIL library: CIL module
 0001:000716f0       _sqlite3DropTrigger        100726f0 f    CIL library: CIL module
 0001:00071830       _sqlite3FinishTrigger      10072830 f    CIL library: CIL module
 0001:00071ab0       _changeTempStorage         10072ab0 f    CIL library: CIL module
 0001:00071b70       _reindexTable              10072b70 f    CIL library: CIL module
 0001:00071c30       _sqlite3CodeDropTable      10072c30 f    CIL library: CIL module
 0001:00071f00       _sqlite3Attach             10072f00 f    CIL library: CIL module
 0001:00072130       _sqlite3Detach             10073130 f    CIL library: CIL module
 0001:00072300       _sqlite3Analyze            10073300 f    CIL library: CIL module
 0001:00072470       _sqlite3ExprIfTrue         10073470 f    CIL library: CIL module
 0001:000727c0       _allocateCursor            100737c0 f    CIL library: CIL module
 0001:00072880       _sqlite3VdbeCursorMoveto   10073880 f    CIL library: CIL module
 0001:00072930       _vdbeCommit                10073930 f    CIL library: CIL module
 0001:00073140       _closeAllCursors           10074140 f    CIL library: CIL module
 0001:00073290       _resolveP2Values           10074290 f    CIL library: CIL module
 0001:00073380       _sqlite3VdbeMemFromBtree   10074380 f    CIL library: CIL module
 0001:00073f50       _sqlite3BtreeDropTable     10074f50 f    CIL library: CIL module
 0001:00073fa0       _sqlite3BtreeDelete        10074fa0 f    CIL library: CIL module
 0001:00074200       _sqlite3BtreeCommit        10075200 f    CIL library: CIL module
 0001:000745a0       _schemaIsValid             100755a0 f    CIL library: CIL module
 0001:00074850       _sqlite3GenerateConstraintChecks 10075850 f    CIL library: CIL module
 0001:00075de0       _reindexDatabases          10076de0 f    CIL library: CIL module
 0001:00075f00       _sqlite3ExprIfFalse        10076f00 f    CIL library: CIL module
 0001:00076250       _sqlite3ExprCodeTarget     10077250 f    CIL library: CIL module
 0001:00077040       _sqlite3VdbeIdxKeyCompare  10078040 f    CIL library: CIL module
 0001:00077140       _sqlite3VdbeIdxRowid       10078140 f    CIL library: CIL module
 0001:000772a0       _sqlite3VdbeHalt           100782a0 f    CIL library: CIL module
 0001:00077580       _sqlite3VdbeMakeReady      10078580 f    CIL library: CIL module
 0001:000778a0       _sqlite3VdbeTakeOpArray    100788a0 f    CIL library: CIL module
 0001:000778d0       _sqlite3BtreeCopyFile      100788d0 f    CIL library: CIL module
 0001:00077a30       _codeEqualityTerm          10078a30 f    CIL library: CIL module
 0001:00077c40       _isLikeOrGlob              10078c40 f    CIL library: CIL module
 0001:00077e30       _sqlite3Pragma             10078e30 f    CIL library: CIL module
 0001:0007a6e0       _sqlite3Reindex            1007b6e0 f    CIL library: CIL module
 0001:0007a890       _sqlite3FinishCoding       1007b890 f    CIL library: CIL module
 0001:0007ab60       _evalConstExpr             1007bb60 f    CIL library: CIL module
 0001:0007ac60       _sqlite3VdbeReset          1007bc60 f    CIL library: CIL module
 0001:0007adc0       _codeAllEqualityTerms      1007bdc0 f    CIL library: CIL module
 0001:0007b060       _exprAnalyze               1007c060 f    CIL library: CIL module
 0001:0007bb30       _exprAnalyzeAll            1007cb30 f    CIL library: CIL module
 0001:0007bb60       _sqlite3ExprCodeConstants  1007cb60 f    CIL library: CIL module
 0001:0007bc60       _sqlite3VdbeFinalize       1007cc60 f    CIL library: CIL module
 0001:0007bcf0       _codeOneLoopStart          1007ccf0 f    CIL library: CIL module
 0001:0007d210       _vacuumFinalize            1007e210 f    CIL library: CIL module
 0001:0007d240       _blobReadWrite             1007e240 f    CIL library: CIL module
 0001:0007d410       _rtreeRelease              1007e410 f    CIL library: CIL module
 0001:0007d4b0       _fts3auxDisconnectMethod   1007e4b0 f    CIL library: CIL module
 0001:0007d500       _fts3DisconnectMethod      1007e500 f    CIL library: CIL module
 0001:0007d590       _sqlite3WhereBegin         1007e590 f    CIL library: CIL module
 0001:0007e160       _sqlite3Select             1007f160 f    CIL library: CIL module
 0001:0007fc60       _sqlite3CodeCoroutine      10080c60 f    CIL library: CIL module
 0001:0007fe40       _fkScanChildren            10080e40 f    CIL library: CIL module
 0001:00080390       _sqlite3MaterializeView    10081390 f    CIL library: CIL module
 0001:000805a0       _sqlite3EndTable           100815a0 f    CIL library: CIL module
 0001:00080a80       _rtreeDisconnect           10081a80 f    CIL library: CIL module
 0001:00080aa0       _sqlite3Fts3SegReaderFree  10081aa0 f    CIL library: CIL module
 0001:00080ae0       _fts3SegReaderSetEof       10081ae0 f    CIL library: CIL module
 0001:00080b50       _fts3SegReaderIncrRead     10081b50 f    CIL library: CIL module
 0001:00080bd0       _sqlite3Fts3SegmentsClose  10081bd0 f    CIL library: CIL module
 0001:00080c40       _fts3SegReaderCursorAppend 10081c40 f    CIL library: CIL module
 0001:00080cf0       _updateVirtualTable        10081cf0 f    CIL library: CIL module
 0001:00081610       _sqlite3FkCheck            10082610 f    CIL library: CIL module
 0001:00081b00       _sqlite3CreateView         10082b00 f    CIL library: CIL module
 0001:00081ca0       _sqlite3Fts3SegReaderFinish 10082ca0 f    CIL library: CIL module
 0001:00081d20       _fts3SegReaderRequire      10082d20 f    CIL library: CIL module
 0001:00081e00       _fts3auxCloseMethod        10082e00 f    CIL library: CIL module
 0001:00081ea0       _fts3SegReaderCursorFree   10082ea0 f    CIL library: CIL module
 0001:00081ec0       _sqlite3Update             10082ec0 f    CIL library: CIL module
 0001:00084110       _sqlite3Insert             10085110 f    CIL library: CIL module
 0001:00085550       _fts3SegReaderNextDocid    10086550 f    CIL library: CIL module
 0001:00085770       _fts3SegReaderFirstDocid   10086770 f    CIL library: CIL module
 0001:000857f0       _sqlite3Fts3EvalPhraseCleanup 100867f0 f    CIL library: CIL module
 0001:00085870       _codeTriggerProgram        10086870 f    CIL library: CIL module
 0001:00085a70       _sqlite3Fts3MsrIncrNext    10086a70 f    CIL library: CIL module
 0001:00085c30       _fts3FreeExprNode          10086c30 f    CIL library: CIL module
 0001:00085c50       _fts3EvalPhraseNext        10086c50 f    CIL library: CIL module
 0001:00085d80       _codeRowTrigger            10086d80 f    CIL library: CIL module
 0001:00086080       _sqlite3Fts3ExprFree       10087080 f    CIL library: CIL module
 0001:00086110       _fts3ExprBalance           10087110 f    CIL library: CIL module
 0001:00086390       _fts3ExprParse             10087390 f    CIL library: CIL module
 0001:00086640       _fts3EvalNextRow           10087640 f    CIL library: CIL module
 0001:00086990       _fts3CloseMethod           10087990 f    CIL library: CIL module
 0001:000869d0       _getRowTrigger             100879d0 f    CIL library: CIL module
 0001:00086d20       _fts3ExprParseUnbalanced   10087d20 f    CIL library: CIL module
 0001:00086db0       _sqlite3CodeRowTriggerDirect 10087db0 f    CIL library: CIL module
 0001:00086ed0       _sqlite3Fts3ExprParse      10087ed0 f    CIL library: CIL module
 0001:00086f90       _sqlite3CodeRowTrigger     10087f90 f    CIL library: CIL module
 0001:00087000       _sqlite3GenerateRowDelete  10088000 f    CIL library: CIL module
 0001:00087390       _sqlite3DeleteFrom         10088390 f    CIL library: CIL module
 0001:00087870       _sqlite3FkDropTable        10088870 f    CIL library: CIL module
 0001:00087a80       _sqlite3DropTable          10088a80 f    CIL library: CIL module
 0001:00087cc0       _yy_reduce                 10088cc0 f    CIL library: CIL module
 0001:0008a680       _sqlite3Parser             1008b680 f    CIL library: CIL module
 0001:0008a7a0       _sqlite3RunParser          1008b7a0 f    CIL library: CIL module
 0001:0008ade0       _sqlite3Prepare            1008bde0 f    CIL library: CIL module
 0001:0008b210       _fts3tokConnectMethod      1008c210 f    CIL library: CIL module
 0001:0008b320       _fts3auxConnectMethod      1008c320 f    CIL library: CIL module
 0001:0008b490       _fts3DeclareVtab           1008c490 f    CIL library: CIL module
 0001:0008b560       _sqlite3LockAndPrepare     1008c560 f    CIL library: CIL module
 0001:0008b620       _sqlite3Fts3InitTok        1008c620 f    CIL library: CIL module
 0001:0008b640       _sqlite3Prepare16          1008c640 f    CIL library: CIL module
 0001:0008b7a0       _sqlite3Reprepare          1008c7a0 f    CIL library: CIL module
 0001:0008b820       _sqlite3InitCallback       1008c820 f    CIL library: CIL module
 0001:0008ba50       _loadStat3                 1008ca50 f    CIL library: CIL module
 0001:0008be30       _fts3SqlStmt               1008ce30 f    CIL library: CIL module
 0001:0008c0a0       _fts3CursorSeekStmt        1008d0a0 f    CIL library: CIL module
 0001:0008c100       _fts3ContentColumns        1008d100 f    CIL library: CIL module
 0001:0008c400       _execSql                   1008d400 f    CIL library: CIL module
 0001:0008c4f0       _sqlite3AnalysisLoad       1008d4f0 f    CIL library: CIL module
 0001:0008c690       _sqlite3Fts3AllSegdirs     1008d690 f    CIL library: CIL module
 0001:0008c7c0       _execExecSql               1008d7c0 f    CIL library: CIL module
 0001:0008c9c0       _sqlite3RunVacuum          1008d9c0 f    CIL library: CIL module
 0001:0008cd40       _sqlite3VdbeExec           1008dd40 f    CIL library: CIL module
 0001:00092600       _sqlite3Step               10093600 f    CIL library: CIL module
 0001:00092a70       _getIntFromStmt            10093a70 f    CIL library: CIL module
 0001:00092ad0       _newRowid                  10093ad0 f    CIL library: CIL module
 0001:00092b60       _parentWrite               10093b60 f    CIL library: CIL module
 0001:00092bc0       _rowidWrite                10093bc0 f    CIL library: CIL module
 0001:00092c20       _nodeWrite                 10093c20 f    CIL library: CIL module
 0001:00092d40       _nodeAcquire               10093d40 f    CIL library: CIL module
 0001:00092f00       _fts3IncrmergeHintLoad     10093f00 f    CIL library: CIL module
 0001:00092fe0       _fts3IncrmergeHintStore    10093fe0 f    CIL library: CIL module
 0001:000930b0       _fts3RepackSegdirLevel     100940b0 f    CIL library: CIL module
 0001:000933b0       _fts3RemoveSegdirEntry     100943b0 f    CIL library: CIL module
 0001:00093420       _fts3IncrmergeOutputIdx    10094420 f    CIL library: CIL module
 0001:00093480       _fts3IsAppendable          10094480 f    CIL library: CIL module
 0001:000934e0       _fts3IncrmergeCsr          100944e0 f    CIL library: CIL module
 0001:000935f0       _fts3UpdateDocTotals       100945f0 f    CIL library: CIL module
 0001:00093880       _fts3InsertDocsize         10094880 f    CIL library: CIL module
 0001:00093950       _fts3DeleteSegment         10094950 f    CIL library: CIL module
 0001:000939c0       _fts3SegmentMaxLevel       100949c0 f    CIL library: CIL module
 0001:00093a90       _fts3IsEmpty               10094a90 f    CIL library: CIL module
 0001:00093af0       _fts3WriteSegdir           10094af0 f    CIL library: CIL module
 0001:00093c00       _sqlite3Fts3MaxLevel       10094c00 f    CIL library: CIL module
 0001:00093c50       _fts3WriteSegment          10094c50 f    CIL library: CIL module
 0001:00093d10       _fts3AllocateSegdirIdx     10094d10 f    CIL library: CIL module
 0001:00093dc0       _fts3InsertData            10094dc0 f    CIL library: CIL module
 0001:00093ec0       _sqlite3Fts3ReadLock       10094ec0 f    CIL library: CIL module
 0001:00093f20       _fts3SqlExec               10094f20 f    CIL library: CIL module
 0001:00093f60       _sqlite3Fts3SelectDoctotal 10094f60 f    CIL library: CIL module
 0001:00093ff0       _fts3SelectDocsize         10094ff0 f    CIL library: CIL module
 0001:00094080       _fts3EvalAverageDocsize    10095080 f    CIL library: CIL module
 0001:00094180       _fts3CursorSeek            10095180 f    CIL library: CIL module
 0001:00094250       _fts3DatabasePageSize      10095250 f    CIL library: CIL module
 0001:00094850       _blobSeekToRow             10095850 f    CIL library: CIL module
 0001:000949f0       _getNodeSize               100959f0 f    CIL library: CIL module
 0001:00094ab0       _rtreeSqlInit              10095ab0 f    CIL library: CIL module
 0001:00094bf0       _rtreeRename               10095bf0 f    CIL library: CIL module
 0001:00094c50       _fixLeafParent             10095c50 f    CIL library: CIL module
 0001:00094d20       _findLeafNode              10095d20 f    CIL library: CIL module
 0001:00094da0       _rtreeDestroy              10095da0 f    CIL library: CIL module
 0001:00094e00       _nodeRelease               10095e00 f    CIL library: CIL module
 0001:00094e70       _fts3MatchinfoSelectDoctotal 10095e70 f    CIL library: CIL module
 0001:00094ee0       _fts3IncrmergeWriter       10095ee0 f    CIL library: CIL module
 0001:000950b0       _fts3IncrmergeRelease      100960b0 f    CIL library: CIL module
 0001:00095260       _fts3IncrmergePush         10096260 f    CIL library: CIL module
 0001:00095570       _fts3DeleteSegdir          10096570 f    CIL library: CIL module
 0001:00095700       _fts3SegWriterAdd          10096700 f    CIL library: CIL module
 0001:00095a90       _fts3NodeWrite             10096a90 f    CIL library: CIL module
 0001:00095b90       _fts3DeleteAll             10096b90 f    CIL library: CIL module
 0001:00095cb0       _sqlite3Fts3SelectDocsize  10096cb0 f    CIL library: CIL module
 0001:00095cd0       _fts3EvalTestDeferredAndNear 10096cd0 f    CIL library: CIL module
 0001:00095d70       _fts3ColumnMethod          10096d70 f    CIL library: CIL module
 0001:00095f00       _fts3DbExec                10096f00 f    CIL library: CIL module
 0001:00096110       _sqlite3InitOne            10097110 f    CIL library: CIL module
 0001:00097150       _rtreeInit                 10098150 f    CIL library: CIL module
 0001:000973e0       _removeNode                100983e0 f    CIL library: CIL module
 0001:00097550       _updateMapping             10098550 f    CIL library: CIL module
 0001:000975c0       _ChooseLeaf                100985c0 f    CIL library: CIL module
 0001:00097890       _descendToCell             10098890 f    CIL library: CIL module
 0001:000979c0       _rtreeClose                100989c0 f    CIL library: CIL module
 0001:00097a40       _rtreeConnect              10098a40 f    CIL library: CIL module
 0001:00097a70       _rtreeCreate               10098a70 f    CIL library: CIL module
 0001:00097aa0       _fts3IncrmergeAppend       10098aa0 f    CIL library: CIL module
 0001:00097c70       _fts3SegWriterFlush        10098c70 f    CIL library: CIL module
 0001:00097d60       _sqlite3Fts3ReadBlock      10098d60 f    CIL library: CIL module
 0001:00097ec0       _fts3EvalNext              10098ec0 f    CIL library: CIL module
 0001:00097f50       _fts3NextMethod            10098f50 f    CIL library: CIL module
 0001:00097fb0       _fts3SelectLeaf            10098fb0 f    CIL library: CIL module
 0001:000980d0       _sqlite3Fts3CreateStatTable 100990d0 f    CIL library: CIL module
 0001:00098100       _fts3DestroyMethod         10099100 f    CIL library: CIL module
 0001:000981a0       _sqlite3Init               100991a0 f    CIL library: CIL module
 0001:00098290       _Reinsert                  10099290 f    CIL library: CIL module
 0001:00098f80       _deleteCell                10099f80 f    CIL library: CIL module
 0001:00099060       _SplitNode                 1009a060 f    CIL library: CIL module
 0001:000996b0       _rtreeFilter               1009a6b0 f    CIL library: CIL module
 0001:00099980       _rtreeNext                 1009a980 f    CIL library: CIL module
 0001:00099b00       _fts3DoAutoincrmerge       1009ab00 f    CIL library: CIL module
 0001:00099bd0       _fts3TruncateSegment       1009abd0 f    CIL library: CIL module
 0001:00099ef0       _fts3IncrmergeLoad         1009aef0 f    CIL library: CIL module
 0001:0009a370       _sqlite3Fts3MsrOvfl        1009b370 f    CIL library: CIL module
 0001:0009a4d0       _fts3SegReaderNext         1009b4d0 f    CIL library: CIL module
 0001:0009a6a0       _fts3EvalTokenCosts        1009b6a0 f    CIL library: CIL module
 0001:0009a780       _fts3SegReaderCursor       1009b780 f    CIL library: CIL module
 0001:0009adb0       _fts3CreateTables          1009bdb0 f    CIL library: CIL module
 0001:0009b1c0       _rtreeInsertCell           1009c1c0 f    CIL library: CIL module
 0001:0009b300       _fts3IncrmergeChomp        1009c300 f    CIL library: CIL module
 0001:0009b610       _sqlite3Fts3SegReaderStep  1009c610 f    CIL library: CIL module
 0001:0009bc40       _fts3SegReaderStart        1009cc40 f    CIL library: CIL module
 0001:0009bd20       _fts3auxNextMethod         1009cd20 f    CIL library: CIL module
 0001:0009bfb0       _fts3SegReaderCursorAddZero 1009cfb0 f    CIL library: CIL module
 0001:0009bfe0       _sqlite3Fts3SegReaderCursor 1009cfe0 f    CIL library: CIL module
 0001:0009c020       _fts3InitVtab              1009d020 f    CIL library: CIL module
 0001:0009ca40       _reinsertNodeContent       1009da40 f    CIL library: CIL module
 0001:0009cb60       _sqlite3Fts3MsrIncrStart   1009db60 f    CIL library: CIL module
 0001:0009ccc0       _sqlite3Fts3SegReaderStart 1009dcc0 f    CIL library: CIL module
 0001:0009cce0       _fts3auxFilterMethod       1009dce0 f    CIL library: CIL module
 0001:0009ce90       _fts3TermSelect            1009de90 f    CIL library: CIL module
 0001:0009d040       _fts3TermSegReaderCursor   1009e040 f    CIL library: CIL module
 0001:0009d220       _fts3CreateMethod          1009e220 f    CIL library: CIL module
 0001:0009d250       _fts3ConnectMethod         1009e250 f    CIL library: CIL module
 0001:0009d280       _rtreeDeleteRowid          1009e280 f    CIL library: CIL module
 0001:0009d540       _fts3ChecksumIndex         1009e540 f    CIL library: CIL module
 0001:0009d700       _sqlite3Fts3Incrmerge      1009e700 f    CIL library: CIL module
 0001:0009db90       _fts3SegmentMerge          1009eb90 f    CIL library: CIL module
 0001:0009ddf0       _sqlite3Fts3InitAux        1009edf0 f    CIL library: CIL module
 0001:0009de10       _fts3EvalSelectDeferred    1009ee10 f    CIL library: CIL module
 0001:0009e050       _fts3EvalPhraseLoad        1009f050 f    CIL library: CIL module
 0001:0009e0e0       _fts3EvalAllocateReaders   1009f0e0 f    CIL library: CIL module
 0001:0009e1a0       _sqlite3Fts3Init           1009f1a0 f    CIL library: CIL module
 0001:0009e3f0       _openDatabase              1009f3f0 f    CIL library: CIL module
 0001:0009e820       _rtreeUpdate               1009f820 f    CIL library: CIL module
 0001:0009ec20       _fts3IntegrityCheck        1009fc20 f    CIL library: CIL module
 0001:0009f470       _fts3DoIncrmerge           100a0470 f    CIL library: CIL module
 0001:0009f540       _fts3DoOptimize            100a0540 f    CIL library: CIL module
 0001:0009f7e0       _sqlite3Fts3PendingTermsFlush 100a07e0 f    CIL library: CIL module
 0001:0009f8c0       _fts3PendingTermsDocid     100a08c0 f    CIL library: CIL module
 0001:0009f920       _fts3EvalPhraseStart       100a0920 f    CIL library: CIL module
 0001:0009f990       _fts3RenameMethod          100a0990 f    CIL library: CIL module
 0001:0009fa50       _fts3SyncMethod            100a0a50 f    CIL library: CIL module
 0001:0009fc70       _sqlite3Fts3Optimize       100a0c70 f    CIL library: CIL module
 0001:0009fd60       _fts3DoIntegrityCheck      100a0d60 f    CIL library: CIL module
 0001:0009fd90       _fts3DoRebuild             100a0d90 f    CIL library: CIL module
 0001:000a01d0       _fts3DeleteTerms           100a11d0 f    CIL library: CIL module
 0001:000a0330       _fts3EvalRestart           100a1330 f    CIL library: CIL module
 0001:000a03c0       _fts3EvalStartReaders      100a13c0 f    CIL library: CIL module
 0001:000a0480       _fts3SavepointMethod       100a1480 f    CIL library: CIL module
 0001:000a04a0       _fts3OptimizeFunc          100a14a0 f    CIL library: CIL module
 0001:000a06d0       _fts3DeleteByRowid         100a16d0 f    CIL library: CIL module
 0001:000a07b0       _fts3SpecialInsert         100a17b0 f    CIL library: CIL module
 0001:000a0920       _sqlite3Fts3EvalPhrasePoslist 100a1920 f    CIL library: CIL module
 0001:000a0be0       _fts3EvalGatherStats       100a1be0 f    CIL library: CIL module
 0001:000a0e50       _fts3EvalStart             100a1e50 f    CIL library: CIL module
 0001:000a0fb0       _fts3FilterMethod          100a1fb0 f    CIL library: CIL module
 0001:000a1190       _fts3ExprTermOffsetInit    100a2190 f    CIL library: CIL module
 0001:000a1220       _fts3MatchinfoLcs          100a2220 f    CIL library: CIL module
 0001:000a1440       _fts3ExprLocalHitsCb       100a2440 f    CIL library: CIL module
 0001:000a14e0       _fts3SnippetFindPositions  100a24e0 f    CIL library: CIL module
 0001:000a1550       _sqlite3Fts3UpdateMethod   100a2550 f    CIL library: CIL module
 0001:000a1870       _sqlite3Fts3EvalPhraseStats 100a2870 f    CIL library: CIL module
 0001:000a1900       _fts3UpdateMethod          100a2900 f    CIL library: CIL module
 0001:000a1920       _sqlite3Fts3Offsets        100a2920 f    CIL library: CIL module
 0001:000a1ef0       _fts3ExprGlobalHitsCb      100a2ef0 f    CIL library: CIL module
 0001:000a1f20       _fts3BestSnippet           100a2f20 f    CIL library: CIL module
 0001:000a20e0       _fts3OffsetsFunc           100a30e0 f    CIL library: CIL module
 0001:000a2130       _sqlite3Fts3Snippet        100a3130 f    CIL library: CIL module
 0001:000a2960       _fts3MatchinfoValues       100a3960 f    CIL library: CIL module
 0001:000a2de0       _fts3SnippetFunc           100a3de0 f    CIL library: CIL module
 0001:000a2f90       _fts3GetMatchinfo          100a3f90 f    CIL library: CIL module
 0001:000a31b0       _sqlite3Fts3Matchinfo      100a41b0 f    CIL library: CIL module
 0001:000a34d0       _fts3MatchinfoFunc         100a44d0 f    CIL library: CIL module
 0001:000a3530       _fts3FindFunctionMethod    100a4530 f    CIL library: CIL module
 0001:000a35f0       _versionFunc               100a45f0 f    CIL library: CIL module
 0001:000a3620       _contextRealloc            100a4620 f    CIL library: CIL module
 0001:000a3670       _contextMalloc             100a4670 f    CIL library: CIL module
 0001:000a36c0       _sqlite3Utf8Read           100a46c0 f    CIL library: CIL module
 0001:000a3720       _sqlite3Utf8CharLen        100a4720 f    CIL library: CIL module
 0001:000a3980       _sqlite3StrNICmp16         100a4980 f    CIL library: CIL module
 0001:000a3b50       _sqlite3StrNICmp           100a4b50 f    CIL library: CIL module
 0001:000a3d30       _unaccFunc                 100a4d30 f    CIL library: CIL module
 0001:000a3ef0       _caseFunc                  100a4ef0 f    CIL library: CIL module
 0001:000a3fd0       _patternCompare            100a4fd0 f    CIL library: CIL module
 0001:000a4610       _likeFunc                  100a5610 f    CIL library: CIL module

 Exports

  ordinal    name

        1    _sqlite3_activate_see
               exported name: sqlite3_activate_see
        2    _sqlite3_aggregate_context
               exported name: sqlite3_aggregate_context
        3    _sqlite3_aggregate_count
               exported name: sqlite3_aggregate_count
        4    _sqlite3_auto_extension
               exported name: sqlite3_auto_extension
        5    _sqlite3_backup_finish
               exported name: sqlite3_backup_finish
        6    _sqlite3_backup_finish_interop@4
        7    _sqlite3_backup_init
               exported name: sqlite3_backup_init
        8    _sqlite3_backup_pagecount
               exported name: sqlite3_backup_pagecount
        9    _sqlite3_backup_remaining
               exported name: sqlite3_backup_remaining
       10    _sqlite3_backup_step
               exported name: sqlite3_backup_step
       11    _sqlite3_bind_blob
               exported name: sqlite3_bind_blob
       12    _sqlite3_bind_double
               exported name: sqlite3_bind_double
       13    _sqlite3_bind_double_interop@12
       14    _sqlite3_bind_int
               exported name: sqlite3_bind_int
       15    _sqlite3_bind_int64
               exported name: sqlite3_bind_int64
       16    _sqlite3_bind_int64_interop@12
       17    _sqlite3_bind_null
               exported name: sqlite3_bind_null
       18    _sqlite3_bind_parameter_count
               exported name: sqlite3_bind_parameter_count
       19    _sqlite3_bind_parameter_index
               exported name: sqlite3_bind_parameter_index
       20    _sqlite3_bind_parameter_name
               exported name: sqlite3_bind_parameter_name
       21    _sqlite3_bind_parameter_name_interop@12
       22    _sqlite3_bind_text
               exported name: sqlite3_bind_text
       23    _sqlite3_bind_text16
               exported name: sqlite3_bind_text16
       24    _sqlite3_bind_value
               exported name: sqlite3_bind_value
       25    _sqlite3_bind_zeroblob
               exported name: sqlite3_bind_zeroblob
       26    _sqlite3_blob_bytes
               exported name: sqlite3_blob_bytes
       27    _sqlite3_blob_close
               exported name: sqlite3_blob_close
       28    _sqlite3_blob_open
               exported name: sqlite3_blob_open
       29    _sqlite3_blob_read
               exported name: sqlite3_blob_read
       30    _sqlite3_blob_reopen
               exported name: sqlite3_blob_reopen
       31    _sqlite3_blob_write
               exported name: sqlite3_blob_write
       32    _sqlite3_busy_handler
               exported name: sqlite3_busy_handler
       33    _sqlite3_busy_timeout
               exported name: sqlite3_busy_timeout
       34    _sqlite3_changes
               exported name: sqlite3_changes
       35    _sqlite3_changes_interop@4
       36    _sqlite3_clear_bindings
               exported name: sqlite3_clear_bindings
       37    _sqlite3_close
               exported name: sqlite3_close
       38    _sqlite3_close_interop@4
       39    _sqlite3_close_v2
               exported name: sqlite3_close_v2
       40    _sqlite3_collation_needed
               exported name: sqlite3_collation_needed
       41    _sqlite3_collation_needed16
               exported name: sqlite3_collation_needed16
       42    _sqlite3_column_blob
               exported name: sqlite3_column_blob
       43    _sqlite3_column_bytes
               exported name: sqlite3_column_bytes
       44    _sqlite3_column_bytes16
               exported name: sqlite3_column_bytes16
       45    _sqlite3_column_count
               exported name: sqlite3_column_count
       46    _sqlite3_column_database_name
               exported name: sqlite3_column_database_name
       47    _sqlite3_column_database_name16
               exported name: sqlite3_column_database_name16
       48    _sqlite3_column_database_name16_interop@12
       49    _sqlite3_column_database_name_interop@12
       50    _sqlite3_column_decltype
               exported name: sqlite3_column_decltype
       51    _sqlite3_column_decltype16
               exported name: sqlite3_column_decltype16
       52    _sqlite3_column_decltype16_interop@12
       53    _sqlite3_column_decltype_interop@12
       54    _sqlite3_column_double
               exported name: sqlite3_column_double
       55    _sqlite3_column_double_interop@12
       56    _sqlite3_column_int
               exported name: sqlite3_column_int
       57    _sqlite3_column_int64
               exported name: sqlite3_column_int64
       58    _sqlite3_column_int64_interop@12
       59    _sqlite3_column_name
               exported name: sqlite3_column_name
       60    _sqlite3_column_name16
               exported name: sqlite3_column_name16
       61    _sqlite3_column_name16_interop@12
       62    _sqlite3_column_name_interop@12
       63    _sqlite3_column_origin_name
               exported name: sqlite3_column_origin_name
       64    _sqlite3_column_origin_name16
               exported name: sqlite3_column_origin_name16
       65    _sqlite3_column_origin_name16_interop@12
       66    _sqlite3_column_origin_name_interop@12
       67    _sqlite3_column_table_name
               exported name: sqlite3_column_table_name
       68    _sqlite3_column_table_name16
               exported name: sqlite3_column_table_name16
       69    _sqlite3_column_table_name16_interop@12
       70    _sqlite3_column_table_name_interop@12
       71    _sqlite3_column_text
               exported name: sqlite3_column_text
       72    _sqlite3_column_text16
               exported name: sqlite3_column_text16
       73    _sqlite3_column_text16_interop@12
       74    _sqlite3_column_text_interop@12
       75    _sqlite3_column_type
               exported name: sqlite3_column_type
       76    _sqlite3_column_value
               exported name: sqlite3_column_value
       77    _sqlite3_commit_hook
               exported name: sqlite3_commit_hook
       78    _sqlite3_compileoption_get
               exported name: sqlite3_compileoption_get
       79    _sqlite3_compileoption_used
               exported name: sqlite3_compileoption_used
       80    _sqlite3_complete
               exported name: sqlite3_complete
       81    _sqlite3_complete16
               exported name: sqlite3_complete16
       82    _sqlite3_config
               exported name: sqlite3_config
       83    _sqlite3_context_collcompare_interop@20
       84    _sqlite3_context_collseq_interop@16
       85    _sqlite3_context_db_handle
               exported name: sqlite3_context_db_handle
       86    _sqlite3_create_collation
               exported name: sqlite3_create_collation
       87    _sqlite3_create_collation16
               exported name: sqlite3_create_collation16
       88    _sqlite3_create_collation_v2
               exported name: sqlite3_create_collation_v2
       89    _sqlite3_create_disposable_module
               exported name: sqlite3_create_disposable_module
       90    _sqlite3_create_disposable_module_interop@112
       91    _sqlite3_create_function
               exported name: sqlite3_create_function
       92    _sqlite3_create_function16
               exported name: sqlite3_create_function16
       93    _sqlite3_create_function_interop@36
       94    _sqlite3_create_function_v2
               exported name: sqlite3_create_function_v2
       95    _sqlite3_create_module
               exported name: sqlite3_create_module
       96    _sqlite3_create_module_v2
               exported name: sqlite3_create_module_v2
       97    _sqlite3_cursor_rowid_interop@12
       98    _sqlite3_data_count
               exported name: sqlite3_data_count
       99    _sqlite3_data_directory
               exported name: sqlite3_data_directory
      100    _sqlite3_db_config
               exported name: sqlite3_db_config
      101    _sqlite3_db_filename
               exported name: sqlite3_db_filename
      102    _sqlite3_db_handle
               exported name: sqlite3_db_handle
      103    _sqlite3_db_mutex
               exported name: sqlite3_db_mutex
      104    _sqlite3_db_readonly
               exported name: sqlite3_db_readonly
      105    _sqlite3_db_release_memory
               exported name: sqlite3_db_release_memory
      106    _sqlite3_db_status
               exported name: sqlite3_db_status
      107    _sqlite3_declare_vtab
               exported name: sqlite3_declare_vtab
      108    _sqlite3_dispose_module
               exported name: sqlite3_dispose_module
      109    _sqlite3_enable_load_extension
               exported name: sqlite3_enable_load_extension
      110    _sqlite3_enable_shared_cache
               exported name: sqlite3_enable_shared_cache
      111    _sqlite3_errcode
               exported name: sqlite3_errcode
      112    _sqlite3_errmsg
               exported name: sqlite3_errmsg
      113    _sqlite3_errmsg16
               exported name: sqlite3_errmsg16
      114    _sqlite3_errmsg_interop@8
      115    _sqlite3_errstr
               exported name: sqlite3_errstr
      116    _sqlite3_exec
               exported name: sqlite3_exec
      117    _sqlite3_expired
               exported name: sqlite3_expired
      118    _sqlite3_extended_errcode
               exported name: sqlite3_extended_errcode
      119    _sqlite3_extended_result_codes
               exported name: sqlite3_extended_result_codes
      120    _sqlite3_extension_init
               exported name: sqlite3_extension_init
      121    _sqlite3_file_control
               exported name: sqlite3_file_control
      122    _sqlite3_finalize
               exported name: sqlite3_finalize
      123    _sqlite3_finalize_interop@4
      124    _sqlite3_free
               exported name: sqlite3_free
      125    _sqlite3_free_table
               exported name: sqlite3_free_table
      126    _sqlite3_get_autocommit
               exported name: sqlite3_get_autocommit
      127    _sqlite3_get_auxdata
               exported name: sqlite3_get_auxdata
      128    _sqlite3_get_table
               exported name: sqlite3_get_table
      129    _sqlite3_global_recover
               exported name: sqlite3_global_recover
      130    _sqlite3_index_column_info_interop@32
      131    _sqlite3_initialize
               exported name: sqlite3_initialize
      132    _sqlite3_interrupt
               exported name: sqlite3_interrupt
      133    _sqlite3_key
               exported name: sqlite3_key
      134    _sqlite3_key_v2
               exported name: sqlite3_key_v2
      135    _sqlite3_last_insert_rowid
               exported name: sqlite3_last_insert_rowid
      136    _sqlite3_last_insert_rowid_interop@8
      137    _sqlite3_libversion
               exported name: sqlite3_libversion
      138    _sqlite3_libversion_number
               exported name: sqlite3_libversion_number
      139    _sqlite3_limit
               exported name: sqlite3_limit
      140    _sqlite3_load_extension
               exported name: sqlite3_load_extension
      141    _sqlite3_log
               exported name: sqlite3_log
      142    _sqlite3_malloc
               exported name: sqlite3_malloc
      143    _sqlite3_malloc_size_interop@4
      144    _sqlite3_memory_alarm
               exported name: sqlite3_memory_alarm
      145    _sqlite3_memory_highwater
               exported name: sqlite3_memory_highwater
      146    _sqlite3_memory_highwater_interop@8
      147    _sqlite3_memory_used
               exported name: sqlite3_memory_used
      148    _sqlite3_memory_used_interop@4
      149    _sqlite3_mprintf
               exported name: sqlite3_mprintf
      150    _sqlite3_mutex_alloc
               exported name: sqlite3_mutex_alloc
      151    _sqlite3_mutex_enter
               exported name: sqlite3_mutex_enter
      152    _sqlite3_mutex_free
               exported name: sqlite3_mutex_free
      153    _sqlite3_mutex_leave
               exported name: sqlite3_mutex_leave
      154    _sqlite3_mutex_try
               exported name: sqlite3_mutex_try
      155    _sqlite3_next_stmt
               exported name: sqlite3_next_stmt
      156    _sqlite3_open
               exported name: sqlite3_open
      157    _sqlite3_open16
               exported name: sqlite3_open16
      158    _sqlite3_open16_interop@12
      159    _sqlite3_open_interop@12
      160    _sqlite3_open_v2
               exported name: sqlite3_open_v2
      161    _sqlite3_os_end
               exported name: sqlite3_os_end
      162    _sqlite3_os_init
               exported name: sqlite3_os_init
      163    _sqlite3_overload_function
               exported name: sqlite3_overload_function
      164    _sqlite3_prepare
               exported name: sqlite3_prepare
      165    _sqlite3_prepare16
               exported name: sqlite3_prepare16
      166    _sqlite3_prepare16_interop@24
      167    _sqlite3_prepare16_v2
               exported name: sqlite3_prepare16_v2
      168    _sqlite3_prepare_interop@24
      169    _sqlite3_prepare_v2
               exported name: sqlite3_prepare_v2
      170    _sqlite3_profile
               exported name: sqlite3_profile
      171    _sqlite3_progress_handler
               exported name: sqlite3_progress_handler
      172    _sqlite3_randomness
               exported name: sqlite3_randomness
      173    _sqlite3_realloc
               exported name: sqlite3_realloc
      174    _sqlite3_rekey
               exported name: sqlite3_rekey
      175    _sqlite3_rekey_v2
               exported name: sqlite3_rekey_v2
      176    _sqlite3_release_memory
               exported name: sqlite3_release_memory
      177    _sqlite3_reset
               exported name: sqlite3_reset
      178    _sqlite3_reset_auto_extension
               exported name: sqlite3_reset_auto_extension
      179    _sqlite3_reset_interop@4
      180    _sqlite3_result_blob
               exported name: sqlite3_result_blob
      181    _sqlite3_result_double
               exported name: sqlite3_result_double
      182    _sqlite3_result_double_interop@8
      183    _sqlite3_result_error
               exported name: sqlite3_result_error
      184    _sqlite3_result_error16
               exported name: sqlite3_result_error16
      185    _sqlite3_result_error_code
               exported name: sqlite3_result_error_code
      186    _sqlite3_result_error_nomem
               exported name: sqlite3_result_error_nomem
      187    _sqlite3_result_error_toobig
               exported name: sqlite3_result_error_toobig
      188    _sqlite3_result_int
               exported name: sqlite3_result_int
      189    _sqlite3_result_int64
               exported name: sqlite3_result_int64
      190    _sqlite3_result_int64_interop@8
      191    _sqlite3_result_null
               exported name: sqlite3_result_null
      192    _sqlite3_result_text
               exported name: sqlite3_result_text
      193    _sqlite3_result_text16
               exported name: sqlite3_result_text16
      194    _sqlite3_result_text16be
               exported name: sqlite3_result_text16be
      195    _sqlite3_result_text16le
               exported name: sqlite3_result_text16le
      196    _sqlite3_result_value
               exported name: sqlite3_result_value
      197    _sqlite3_result_zeroblob
               exported name: sqlite3_result_zeroblob
      198    _sqlite3_rollback_hook
               exported name: sqlite3_rollback_hook
      199    _sqlite3_rtree_geometry_callback
               exported name: sqlite3_rtree_geometry_callback
      200    _sqlite3_set_authorizer
               exported name: sqlite3_set_authorizer
      201    _sqlite3_set_auxdata
               exported name: sqlite3_set_auxdata
      202    _sqlite3_shutdown
               exported name: sqlite3_shutdown
      203    _sqlite3_sleep
               exported name: sqlite3_sleep
      204    _sqlite3_snprintf
               exported name: sqlite3_snprintf
      205    _sqlite3_soft_heap_limit
               exported name: sqlite3_soft_heap_limit
      206    _sqlite3_soft_heap_limit64
               exported name: sqlite3_soft_heap_limit64
      207    _sqlite3_sourceid
               exported name: sqlite3_sourceid
      208    _sqlite3_sql
               exported name: sqlite3_sql
      209    _sqlite3_status
               exported name: sqlite3_status
      210    _sqlite3_step
               exported name: sqlite3_step
      211    _sqlite3_stmt_busy
               exported name: sqlite3_stmt_busy
      212    _sqlite3_stmt_readonly
               exported name: sqlite3_stmt_readonly
      213    _sqlite3_stmt_status
               exported name: sqlite3_stmt_status
      214    _sqlite3_strglob
               exported name: sqlite3_strglob
      215    _sqlite3_stricmp
               exported name: sqlite3_stricmp
      216    _sqlite3_strnicmp
               exported name: sqlite3_strnicmp
      217    _sqlite3_table_column_metadata
               exported name: sqlite3_table_column_metadata
      218    _sqlite3_table_column_metadata_interop@44
      219    _sqlite3_table_cursor_interop@12
      220    _sqlite3_temp_directory
               exported name: sqlite3_temp_directory
      221    _sqlite3_test_control
               exported name: sqlite3_test_control
      222    _sqlite3_thread_cleanup
               exported name: sqlite3_thread_cleanup
      223    _sqlite3_threadsafe
               exported name: sqlite3_threadsafe
      224    _sqlite3_total_changes
               exported name: sqlite3_total_changes
      225    _sqlite3_trace
               exported name: sqlite3_trace
      226    _sqlite3_transfer_bindings
               exported name: sqlite3_transfer_bindings
      227    _sqlite3_unicode_collate
               exported name: sqlite3_unicode_collate
      228    _sqlite3_unicode_fold
               exported name: sqlite3_unicode_fold
      229    _sqlite3_unicode_free
               exported name: sqlite3_unicode_free
      230    _sqlite3_unicode_init
               exported name: sqlite3_unicode_init
      231    _sqlite3_unicode_load
               exported name: sqlite3_unicode_load
      232    _sqlite3_unicode_lower
               exported name: sqlite3_unicode_lower
      233    _sqlite3_unicode_title
               exported name: sqlite3_unicode_title
      234    _sqlite3_unicode_unacc
               exported name: sqlite3_unicode_unacc
      235    _sqlite3_unicode_upper
               exported name: sqlite3_unicode_upper
      236    _sqlite3_update_hook
               exported name: sqlite3_update_hook
      237    _sqlite3_uri_boolean
               exported name: sqlite3_uri_boolean
      238    _sqlite3_uri_int64
               exported name: sqlite3_uri_int64
      239    _sqlite3_uri_parameter
               exported name: sqlite3_uri_parameter
      240    _sqlite3_user_data
               exported name: sqlite3_user_data
      241    _sqlite3_value_blob
               exported name: sqlite3_value_blob
      242    _sqlite3_value_bytes
               exported name: sqlite3_value_bytes
      243    _sqlite3_value_bytes16
               exported name: sqlite3_value_bytes16
      244    _sqlite3_value_double
               exported name: sqlite3_value_double
      245    _sqlite3_value_double_interop@8
      246    _sqlite3_value_int
               exported name: sqlite3_value_int
      247    _sqlite3_value_int64
               exported name: sqlite3_value_int64
      248    _sqlite3_value_int64_interop@8
      249    _sqlite3_value_numeric_type
               exported name: sqlite3_value_numeric_type
      250    _sqlite3_value_text
               exported name: sqlite3_value_text
      251    _sqlite3_value_text16
               exported name: sqlite3_value_text16
      252    _sqlite3_value_text16_interop@8
      253    _sqlite3_value_text16be
               exported name: sqlite3_value_text16be
      254    _sqlite3_value_text16le
               exported name: sqlite3_value_text16le
      255    _sqlite3_value_text_interop@8
      256    _sqlite3_value_type
               exported name: sqlite3_value_type
      257    _sqlite3_version
               exported name: sqlite3_version
      258    _sqlite3_vfs_find
               exported name: sqlite3_vfs_find
      259    _sqlite3_vfs_register
               exported name: sqlite3_vfs_register
      260    _sqlite3_vfs_unregister
               exported name: sqlite3_vfs_unregister
      261    _sqlite3_vmprintf
               exported name: sqlite3_vmprintf
      262    _sqlite3_vsnprintf
               exported name: sqlite3_vsnprintf
      263    _sqlite3_vtab_config
               exported name: sqlite3_vtab_config
      264    _sqlite3_vtab_on_conflict
               exported name: sqlite3_vtab_on_conflict
      265    _sqlite3_vtshim_init
               exported name: sqlite3_vtshim_init
      266    _sqlite3_wal_autocheckpoint
               exported name: sqlite3_wal_autocheckpoint
      267    _sqlite3_wal_checkpoint
               exported name: sqlite3_wal_checkpoint
      268    _sqlite3_wal_checkpoint_v2
               exported name: sqlite3_wal_checkpoint_v2
      269    _sqlite3_wal_hook
               exported name: sqlite3_wal_hook
      270    _sqlite3_win32_mbcs_to_utf8
               exported name: sqlite3_win32_mbcs_to_utf8
      271    _sqlite3_win32_set_directory
               exported name: sqlite3_win32_set_directory
      272    _sqlite3_win32_sleep
               exported name: sqlite3_win32_sleep
      273    _sqlite3_win32_utf8_to_mbcs
               exported name: sqlite3_win32_utf8_to_mbcs
      274    _sqlite3_win32_write_debug
               exported name: sqlite3_win32_write_debug
